 chroma_view

 Timestamp is 5dee365b (Mon Dec 09 18:56:11 2019)

 Preferred load address is 10000000

 Start         Length     Name                   Class
 0001:00000000 00000ca4H .text$di                CODE
 0001:00000cb0 0000c9e8H .text$mn                CODE
 0001:0000d6a0 00001224H .text$x                 CODE
 0001:0000e8d0 0000048aH .text$yd                CODE
 0002:00000000 000007b8H .idata$5                DATA
 0002:000007b8 00000004H .CRT$XCA                DATA
 0002:000007bc 00000108H .CRT$XCU                DATA
 0002:000008c4 00000004H .CRT$XCZ                DATA
 0002:000008c8 00000004H .CRT$XIA                DATA
 0002:000008cc 00000004H .CRT$XIAA               DATA
 0002:000008d0 00000004H .CRT$XIC                DATA
 0002:000008d4 00000004H .CRT$XIZ                DATA
 0002:000008e0 00001cf0H .rdata                  DATA
 0002:000025d0 00000074H .rdata$debug            DATA
 0002:00002644 00000a34H .rdata$r                DATA
 0002:00003080 00000118H .rdata$sxdata           DATA
 0002:00003198 00000004H .rtc$IAA                DATA
 0002:0000319c 00000004H .rtc$IZZ                DATA
 0002:000031a0 00000004H .rtc$TAA                DATA
 0002:000031a4 00000004H .rtc$TZZ                DATA
 0002:000031a8 00001584H .xdata$x                DATA
 0002:00004730 00000054H .edata                  DATA
 0002:00004784 000000b4H .idata$2                DATA
 0002:00004838 00000014H .idata$3                DATA
 0002:0000484c 000007b8H .idata$4                DATA
 0002:00005004 000057d6H .idata$6                DATA
 0003:00000000 000001d4H .data                   DATA
 0003:000001d4 00000488H .data$r                 DATA
 0003:00000660 000004dcH .bss                    DATA
 0004:00000000 00000058H .rsrc$01                DATA
 0004:00000060 00000180H .rsrc$02                DATA

  Address         Publics by Value              Rva+Base       Lib:Object

 0000:00000000       ___guard_flags             00000000     <absolute>
 0000:00000000       ___guard_fids_table        00000000     <absolute>
 0000:00000000       __except_list              00000000     <absolute>
 0000:00000000       ___guard_fids_count        00000000     <absolute>
 0000:00000046       ___safe_se_handler_count   00000046     <absolute>
 0000:00009876       __fltused                  00009876     <absolute>
 0000:00009876       __ldused                   00009876     <absolute>
 0000:00000000       ___ImageBase               10000000     <linker-defined>
 0001:00000cb0       ??$_Allocate@D@std@@YAPADIPAD@Z 10001cb0 f i ChromaViewPlugin.obj
 0001:00000ce0       ??$addressof@D@std@@YAPADAAD@Z 10001ce0 f i ChromaViewPlugin.obj
 0001:00000cf0       ??$atomic@H@?$QAtomicOpsBySize@$03@@CAPAJPAH@Z 10001cf0 f i ChromaViewPlugin.obj
 0001:00000d00       ??$construct@PADAAPAD@?$_Wrap_alloc@V?$allocator@D@std@@@std@@QAEXPAPADAAPAD@Z 10001d00 f i ChromaViewPlugin.obj
 0001:00000d20       ??$construct@PADAAPAD@?$allocator@D@std@@QAEXPAPADAAPAD@Z 10001d20 f i ChromaViewPlugin.obj
 0001:00000d40       ??$construct@PADAAPAD@?$allocator_traits@V?$allocator@D@std@@@std@@SAXAAV?$allocator@D@1@PAPADAAPAD@Z 10001d40 f i ChromaViewPlugin.obj
 0001:00000d60       ??$deref@H@?$QAtomicOpsBySize@$03@@SA_NAAH@Z 10001d60 f i ChromaViewPlugin.obj
 0001:00000d80       ??$destroy@PAD@?$_Wrap_alloc@V?$allocator@D@std@@@std@@QAEXPAPAD@Z 10001d80 f i ChromaViewPlugin.obj
 0001:00000d90       ??$destroy@PAD@?$allocator@D@std@@QAEXPAPAD@Z 10001d90 f i ChromaViewPlugin.obj
 0001:00000da0       ??$destroy@PAD@?$allocator_traits@V?$allocator@D@std@@@std@@SAXAAV?$allocator@D@1@PAPAD@Z 10001da0 f i ChromaViewPlugin.obj
 0001:00000db0       ??$forward@AAPAD@std@@YAAAPADAAPAD@Z 10001db0 f i ChromaViewPlugin.obj
 0001:00000dc0       ??$load@H@?$QGenericAtomicOps@U?$QAtomicOpsBySize@$03@@@@SAHABH@Z 10001dc0 f i ChromaViewPlugin.obj
 0001:00000dd0       ??$qobject_cast@PAVADVSingleSequenceWidget@U2@@@@YAPAVADVSingleSequenceWidget@U2@@PAVQObject@@@Z 10001dd0 f i ChromaViewPlugin.obj
 0001:00000df0       ??$qobject_cast@PAVAnnotatedDNAView@U2@@@@YAPAVAnnotatedDNAView@U2@@PAVQObject@@@Z 10001df0 f i ChromaViewPlugin.obj
 0001:00000e10       ??$qobject_cast@PAVChromaViewAction@U2@@@@YAPAVChromaViewAction@U2@@PAVQObject@@@Z 10001e10 f i ChromaViewPlugin.obj
 0001:00000e30       ??$qobject_cast@PAVDNAChromatogramObject@U2@@@@YAPAVDNAChromatogramObject@U2@@PAVQObject@@@Z 10001e30 f i ChromaViewPlugin.obj
 0001:00000e50       ??$ref@H@?$QAtomicOpsBySize@$03@@SA_NAAH@Z 10001e50 f i ChromaViewPlugin.obj
 0001:00000e70       ??0?$AbstractId@H@U2@@IAE@ABH@Z 10001e70 f i ChromaViewPlugin.obj
 0001:00000e90       ??0?$QForeachContainer@$$CBV?$QList@PAVADVSequenceWidget@U2@@@@@@QAE@ABV?$QList@PAVADVSequenceWidget@U2@@@@@Z 10001e90 f i ChromaViewPlugin.obj
 0001:00000ed0       ??0?$QList@PAVADVSequenceWidget@U2@@@@QAE@ABV0@@Z 10001ed0 f i ChromaViewPlugin.obj
 0001:00000f90       ??0?$_String_alloc@$0A@U?$_String_base_types@DV?$allocator@D@std@@@std@@@std@@QAE@ABV?$allocator@D@1@@Z 10001f90 f i ChromaViewPlugin.obj
 0001:00000fb0       ??0?$_String_val@U?$_Simple_types@D@std@@@std@@QAE@XZ 10001fb0 f i ChromaViewPlugin.obj
 0001:00000fd0       ??0?$_Wrap_alloc@V?$allocator@D@std@@@std@@QAE@XZ 10001fd0 f i ChromaViewPlugin.obj
 0001:00000fe0       ??0?$allocator@D@std@@QAE@XZ 10001fe0 f i ChromaViewPlugin.obj
 0001:00000ff0       ??0?$basic_string@DU?$char_traits@D@std@@V?$allocator@D@2@@std@@QAE@PBD@Z 10001ff0 f i ChromaViewPlugin.obj
 0001:00001050       ??0AbstractInt32Id@U2@@IAE@H@Z 10002050 f i ChromaViewPlugin.obj
 0001:00001070       ??0ChromaViewAction@U2@@QAE@XZ 10002070 f   ChromaViewPlugin.obj
 0001:00001120       ??0ChromaViewContext@U2@@QAE@PAVQObject@@@Z 10002120 f   ChromaViewPlugin.obj
 0001:000011b0       ??0ChromaViewPlugin@U2@@QAE@XZ 100021b0 f   ChromaViewPlugin.obj
 0001:000012c0       ??0GObjectViewFactoryId@U2@@QAE@PBD@Z 100022c0 f i ChromaViewPlugin.obj
 0001:00001300       ??0ServiceType@U2@@QAE@H@Z 10002300 f i ChromaViewPlugin.obj
 0001:00001320       ??0_Generic_error_category@std@@QAE@XZ 10002320 f i ChromaViewPlugin.obj
 0001:00001330       ??0_Ignore@std@@QAE@XZ     10002330 f i ChromaViewPlugin.obj
 0001:00001340       ??0_Iostream_error_category@std@@QAE@XZ 10002340 f i ChromaViewPlugin.obj
 0001:00001350       ??0_System_error_category@std@@QAE@XZ 10002350 f i ChromaViewPlugin.obj
 0001:00001360       ??0const_iterator@?$QList@PAVADVSequenceWidget@U2@@@@QAE@PAUNode@1@@Z 10002360 f i ChromaViewPlugin.obj
 0001:00001370       ??0error_category@std@@QAE@XZ 10002370 f i ChromaViewPlugin.obj
 0001:00001380       ??0error_condition@std@@QAE@HABVerror_category@1@@Z 10002380 f i ChromaViewPlugin.obj
 0001:000013a0       ??0iterator@?$QList@PAVGObject@U2@@@@QAE@PAUNode@1@@Z 100023a0 f i ChromaViewPlugin.obj
 0001:000013b0       ??1?$AbstractId@H@U2@@MAE@XZ 100023b0 f i ChromaViewPlugin.obj
 0001:000013c0       ??1?$QForeachContainer@$$CBV?$QList@PAVADVSequenceWidget@U2@@@@@@QAE@XZ 100023c0 f i ChromaViewPlugin.obj
 0001:000013f0       ??1?$QList@PAVADVSequenceWidget@U2@@@@QAE@XZ 100023f0 f i ChromaViewPlugin.obj
 0001:00001420       ??1?$QList@PAVGObject@U2@@@@QAE@XZ 10002420 f i ChromaViewPlugin.obj
 0001:00001450       ??1?$basic_string@DU?$char_traits@D@std@@V?$allocator@D@2@@std@@QAE@XZ 10002450 f i ChromaViewPlugin.obj
 0001:00001480       ??1AbstractInt32Id@U2@@UAE@XZ 10002480 f i ChromaViewPlugin.obj
 0001:00001490       ??1ChromaViewAction@U2@@UAE@XZ 10002490 f i ChromaViewPlugin.obj
 0001:000014a0       ??1ChromaViewContext@U2@@UAE@XZ 100024a0 f i ChromaViewPlugin.obj
 0001:000014b0       ??1ChromaViewPlugin@U2@@UAE@XZ 100024b0 f   ChromaViewPlugin.obj
 0001:000014c0       ??1GObjectViewFactoryId@U2@@QAE@XZ 100024c0 f i ChromaViewPlugin.obj
 0001:000014d0       ??1ServiceType@U2@@UAE@XZ  100024d0 f i ChromaViewPlugin.obj
 0001:000014e0       ??1_Generic_error_category@std@@UAE@XZ 100024e0 f i ChromaViewPlugin.obj
 0001:000014f0       ??1_Iostream_error_category@std@@UAE@XZ 100024f0 f i ChromaViewPlugin.obj
 0001:00001500       ??1_System_error_category@std@@UAE@XZ 10002500 f i ChromaViewPlugin.obj
 0001:00001510       ??1error_category@std@@UAE@XZ 10002510 f i ChromaViewPlugin.obj
 0001:00001520       ??2@YAPAXIPAX@Z            10002520 f i ChromaViewPlugin.obj
 0001:00001530       ??3@YAXPAX0@Z              10002530 f i ChromaViewPlugin.obj
 0001:00001540       ??8error_category@std@@QBE_NABV01@@Z 10002540 f i ChromaViewPlugin.obj
 0001:00001550       ??8error_condition@std@@QBE_NABV01@@Z 10002550 f i ChromaViewPlugin.obj
 0001:00001570       ??9const_iterator@?$QList@PAVADVSequenceWidget@U2@@@@QBE_NABV01@@Z 10002570 f i ChromaViewPlugin.obj
 0001:00001590       ??Dconst_iterator@?$QList@PAVADVSequenceWidget@U2@@@@QBEABQAVADVSequenceWidget@U2@@XZ 10002590 f i ChromaViewPlugin.obj
 0001:000015a0       ??Diterator@?$QList@PAVGObject@U2@@@@QBEAAPAVGObject@U2@@XZ 100025a0 f i ChromaViewPlugin.obj
 0001:000015b0       ??Econst_iterator@?$QList@PAVADVSequenceWidget@U2@@@@QAEAAV01@XZ 100025b0 f i ChromaViewPlugin.obj
 0001:000015b6       ??_EChromaViewContext@U2@@W7AEPAXI@Z 100025b6 f i ChromaViewPlugin.obj
 0001:000015c0       ??_E?$AbstractId@H@U2@@MAEPAXI@Z 100025c0 f i ChromaViewPlugin.obj
 0001:000015c0       ??_G?$AbstractId@H@U2@@MAEPAXI@Z 100025c0 f i ChromaViewPlugin.obj
 0001:000015f0       ??_EAbstractInt32Id@U2@@UAEPAXI@Z 100025f0 f i ChromaViewPlugin.obj
 0001:000015f0       ??_GAbstractInt32Id@U2@@UAEPAXI@Z 100025f0 f i ChromaViewPlugin.obj
 0001:00001620       ??_GChromaViewAction@U2@@UAEPAXI@Z 10002620 f i ChromaViewPlugin.obj
 0001:00001620       ??_EChromaViewAction@U2@@UAEPAXI@Z 10002620 f i ChromaViewPlugin.obj
 0001:00001650       ??_GChromaViewContext@U2@@UAEPAXI@Z 10002650 f i ChromaViewPlugin.obj
 0001:00001650       ??_EChromaViewContext@U2@@UAEPAXI@Z 10002650 f i ChromaViewPlugin.obj
 0001:00001680       ??_GChromaViewPlugin@U2@@UAEPAXI@Z 10002680 f i ChromaViewPlugin.obj
 0001:00001680       ??_EChromaViewPlugin@U2@@UAEPAXI@Z 10002680 f i ChromaViewPlugin.obj
 0001:000016b0       ??_EServiceType@U2@@UAEPAXI@Z 100026b0 f i ChromaViewPlugin.obj
 0001:000016b0       ??_GServiceType@U2@@UAEPAXI@Z 100026b0 f i ChromaViewPlugin.obj
 0001:000016e0       ??_G_Generic_error_category@std@@UAEPAXI@Z 100026e0 f i ChromaViewPlugin.obj
 0001:000016e0       ??_E_Generic_error_category@std@@UAEPAXI@Z 100026e0 f i ChromaViewPlugin.obj
 0001:00001710       ??_E_Iostream_error_category@std@@UAEPAXI@Z 10002710 f i ChromaViewPlugin.obj
 0001:00001710       ??_G_Iostream_error_category@std@@UAEPAXI@Z 10002710 f i ChromaViewPlugin.obj
 0001:00001740       ??_G_System_error_category@std@@UAEPAXI@Z 10002740 f i ChromaViewPlugin.obj
 0001:00001740       ??_E_System_error_category@std@@UAEPAXI@Z 10002740 f i ChromaViewPlugin.obj
 0001:00001770       ??_Eerror_category@std@@UAEPAXI@Z 10002770 f i ChromaViewPlugin.obj
 0001:00001770       ??_Gerror_category@std@@UAEPAXI@Z 10002770 f i ChromaViewPlugin.obj
 0001:000017a0       ?_Copy@?$basic_string@DU?$char_traits@D@std@@V?$allocator@D@2@@std@@QAEXII@Z 100027a0 f i ChromaViewPlugin.obj
 0001:000018f0       ?_Eos@?$basic_string@DU?$char_traits@D@std@@V?$allocator@D@2@@std@@QAEXI@Z 100028f0 f i ChromaViewPlugin.obj
 0001:00001920       ?_Getal@?$_String_alloc@$0A@U?$_String_base_types@DV?$allocator@D@std@@@std@@@std@@QBE?AU?$_Wrap_alloc@V?$allocator@D@std@@@2@XZ 10002920 f i ChromaViewPlugin.obj
 0001:00001930       ?_Grow@?$basic_string@DU?$char_traits@D@std@@V?$allocator@D@2@@std@@QAE_NI_N@Z 10002930 f i ChromaViewPlugin.obj
 0001:000019e0       ?_Inside@?$basic_string@DU?$char_traits@D@std@@V?$allocator@D@2@@std@@QAE_NPBD@Z 100029e0 f i ChromaViewPlugin.obj
 0001:00001a20       ?_Myptr@?$_String_val@U?$_Simple_types@D@std@@@std@@QAEPADXZ 10002a20 f i ChromaViewPlugin.obj
 0001:00001a30       ?_Myptr@?$_String_val@U?$_Simple_types@D@std@@@std@@QBEPBDXZ 10002a30 f i ChromaViewPlugin.obj
 0001:00001a40       ?_Tidy@?$basic_string@DU?$char_traits@D@std@@V?$allocator@D@2@@std@@QAEX_NI@Z 10002a40 f i ChromaViewPlugin.obj
 0001:00001a90       ?_Xlen@?$basic_string@DU?$char_traits@D@std@@V?$allocator@D@2@@std@@QBEXXZ 10002a90 f i ChromaViewPlugin.obj
 0001:00001aa0       ?_Xran@?$basic_string@DU?$char_traits@D@std@@V?$allocator@D@2@@std@@QBEXXZ 10002aa0 f i ChromaViewPlugin.obj
 0001:00001ab0       ?allocate@?$_Wrap_alloc@V?$allocator@D@std@@@std@@QAEPADI@Z 10002ab0 f i ChromaViewPlugin.obj
 0001:00001ae0       ?allocate@?$allocator@D@std@@QAEPADI@Z 10002ae0 f i ChromaViewPlugin.obj
 0001:00001b10       ?assign@?$basic_string@DU?$char_traits@D@std@@V?$allocator@D@2@@std@@QAEAAV12@ABV12@II@Z 10002b10 f i ChromaViewPlugin.obj
 0001:00001c30       ?assign@?$basic_string@DU?$char_traits@D@std@@V?$allocator@D@2@@std@@QAEAAV12@PBD@Z 10002c30 f i ChromaViewPlugin.obj
 0001:00001c70       ?assign@?$basic_string@DU?$char_traits@D@std@@V?$allocator@D@2@@std@@QAEAAV12@PBDI@Z 10002c70 f i ChromaViewPlugin.obj
 0001:00001d70       ?assign@?$char_traits@D@std@@SAXAADABD@Z 10002d70 f i ChromaViewPlugin.obj
 0001:00001d80       ?begin@?$QList@PAVADVSequenceWidget@U2@@@@QBE?AVconst_iterator@1@XZ 10002d80 f i ChromaViewPlugin.obj
 0001:00001da0       ?begin@?$QList@PAVGObject@U2@@@@QAE?AViterator@1@XZ 10002da0 f i ChromaViewPlugin.obj
 0001:00001de0       ?canHandle@ChromaViewContext@U2@@UAE_NPAVGObjectView@2@PAVGObject@2@@Z 10002de0 f   ChromaViewPlugin.obj
 0001:00001e00       ?category@error_code@std@@QBEABVerror_category@2@XZ 10002e00 f i ChromaViewPlugin.obj
 0001:00001e10       ?category@error_condition@std@@QBEABVerror_category@2@XZ 10002e10 f i ChromaViewPlugin.obj
 0001:00001e20       ?copy@?$char_traits@D@std@@SAPADPADPBDI@Z 10002e20 f i ChromaViewPlugin.obj
 0001:00001e40       ?dealloc@?$QList@PAVADVSequenceWidget@U2@@@@AAEXPAUData@QListData@@@Z 10002e40 f i ChromaViewPlugin.obj
 0001:00001e60       ?dealloc@?$QList@PAVGObject@U2@@@@AAEXPAUData@QListData@@@Z 10002e60 f i ChromaViewPlugin.obj
 0001:00001e80       ?deallocate@?$_Wrap_alloc@V?$allocator@D@std@@@std@@QAEXPADI@Z 10002e80 f i ChromaViewPlugin.obj
 0001:00001ea0       ?deallocate@?$allocator@D@std@@QAEXPADI@Z 10002ea0 f i ChromaViewPlugin.obj
 0001:00001ec0       ?default_error_condition@_System_error_category@std@@UBE?AVerror_condition@2@H@Z 10002ec0 f i ChromaViewPlugin.obj
 0001:00001f00       ?default_error_condition@error_category@std@@UBE?AVerror_condition@2@H@Z 10002f00 f i ChromaViewPlugin.obj
 0001:00001f20       ?deref@?$QBasicAtomicInteger@H@@QAE_NXZ 10002f20 f i ChromaViewPlugin.obj
 0001:00001f30       ?deref@RefCount@QtPrivate@@QAE_NXZ 10002f30 f i ChromaViewPlugin.obj
 0001:00001f50       ?detach@?$QList@PAVGObject@U2@@@@QAEXXZ 10002f50 f i ChromaViewPlugin.obj
 0001:00001f70       ?detach_helper@?$QList@PAVGObject@U2@@@@AAEXH@Z 10002f70 f i ChromaViewPlugin.obj
 0001:00002040       ?detach_helper@?$QList@PAVGObject@U2@@@@AAEXXZ 10003040 f i ChromaViewPlugin.obj
 0001:00002050       ?end@?$QList@PAVADVSequenceWidget@U2@@@@QBE?AVconst_iterator@1@XZ 10003050 f i ChromaViewPlugin.obj
 0001:00002070       ?equivalent@error_category@std@@UBE_NABVerror_code@2@H@Z 10003070 f i ChromaViewPlugin.obj
 0001:00002090       ?equivalent@error_category@std@@UBE_NHABVerror_condition@2@@Z 10003090 f i ChromaViewPlugin.obj
 0001:000020d0       ?erase@?$basic_string@DU?$char_traits@D@std@@V?$allocator@D@2@@std@@QAEAAV12@I@Z 100030d0 f i ChromaViewPlugin.obj
 0001:00002110       ?erase@?$basic_string@DU?$char_traits@D@std@@V?$allocator@D@2@@std@@QAEAAV12@II@Z 10003110 f i ChromaViewPlugin.obj
 0001:000022e0       ?first@?$QList@PAVGObject@U2@@@@QAEAAPAVGObject@U2@@XZ 100032e0 f i ChromaViewPlugin.obj
 0001:00002310       ?generic_category@std@@YAABVerror_category@1@XZ 10003310 f i ChromaViewPlugin.obj
 0001:00002320       ?getEditedSequence@ChromatogramView@U2@@QBEPAVU2SequenceObject@2@XZ 10003320 f i ChromaViewPlugin.obj
 0001:00002330       ?initViewContext@ChromaViewContext@U2@@MAEXPAVGObjectView@2@@Z 10003330 f   ChromaViewPlugin.obj
 0001:00002470       ?isEmpty@?$QList@PAVGObject@U2@@@@QBE_NXZ 10003470 f i ChromaViewPlugin.obj
 0001:00002480       ?isShared@RefCount@QtPrivate@@QBE_NXZ 10003480 f i ChromaViewPlugin.obj
 0001:000024a0       ?isValid@AbstractInt32Id@U2@@UBE_NXZ 100034a0 f i ChromaViewPlugin.obj
 0001:000024b0       ?length@?$char_traits@D@std@@SAIPBD@Z 100034b0 f i ChromaViewPlugin.obj
 0001:000024d0       ?load@?$QBasicAtomicInteger@H@@QBEHXZ 100034d0 f i ChromaViewPlugin.obj
 0001:000024e0       ?max_size@?$_Wrap_alloc@V?$allocator@D@std@@@std@@QBEIXZ 100034e0 f i ChromaViewPlugin.obj
 0001:000024f0       ?max_size@?$allocator@D@std@@QBEIXZ 100034f0 f i ChromaViewPlugin.obj
 0001:00002500       ?max_size@?$allocator_traits@V?$allocator@D@std@@@std@@SAIABV?$allocator@D@2@@Z 10003500 f i ChromaViewPlugin.obj
 0001:00002510       ?max_size@?$basic_string@DU?$char_traits@D@std@@V?$allocator@D@2@@std@@QBEIXZ 10003510 f i ChromaViewPlugin.obj
 0001:00002520       ?message@_Generic_error_category@std@@UBE?AV?$basic_string@DU?$char_traits@D@std@@V?$allocator@D@2@@2@H@Z 10003520 f i ChromaViewPlugin.obj
 0001:000025a0       ?message@_Iostream_error_category@std@@UBE?AV?$basic_string@DU?$char_traits@D@std@@V?$allocator@D@2@@2@H@Z 100035a0 f i ChromaViewPlugin.obj
 0001:000025f0       ?message@_System_error_category@std@@UBE?AV?$basic_string@DU?$char_traits@D@std@@V?$allocator@D@2@@2@H@Z 100035f0 f i ChromaViewPlugin.obj
 0001:00002670       ?move@?$char_traits@D@std@@SAPADPADPBDI@Z 10003670 f i ChromaViewPlugin.obj
 0001:00002690       ?name@_Generic_error_category@std@@UBEPBDXZ 10003690 f i ChromaViewPlugin.obj
 0001:000026a0       ?name@_Iostream_error_category@std@@UBEPBDXZ 100036a0 f i ChromaViewPlugin.obj
 0001:000026b0       ?name@_System_error_category@std@@UBEPBDXZ 100036b0 f i ChromaViewPlugin.obj
 0001:000026c0       ?node_copy@?$QList@PAVADVSequenceWidget@U2@@@@AAEXPAUNode@1@00@Z 100036c0 f i ChromaViewPlugin.obj
 0001:000026f0       ?node_copy@?$QList@PAVGObject@U2@@@@AAEXPAUNode@1@00@Z 100036f0 f i ChromaViewPlugin.obj
 0001:00002720       ?node_destruct@?$QList@PAVADVSequenceWidget@U2@@@@AAEXPAUNode@1@0@Z 10003720 f i ChromaViewPlugin.obj
 0001:00002730       ?node_destruct@?$QList@PAVGObject@U2@@@@AAEXPAUNode@1@0@Z 10003730 f i ChromaViewPlugin.obj
 0001:00002740       ?qt_noop@@YAXXZ            10003740 f i ChromaViewPlugin.obj
 0001:00002750       ?ref@?$QBasicAtomicInteger@H@@QAE_NXZ 10003750 f i ChromaViewPlugin.obj
 0001:00002770       ?ref@RefCount@QtPrivate@@QAE_NXZ 10003770 f i ChromaViewPlugin.obj
 0001:00002790       ?size@?$basic_string@DU?$char_traits@D@std@@V?$allocator@D@2@@std@@QBEIXZ 10003790 f i ChromaViewPlugin.obj
 0001:000027a0       ?sl_sequenceWidgetAdded@ChromaViewContext@U2@@IAEXPAVADVSequenceWidget@2@@Z 100037a0 f   ChromaViewPlugin.obj
 0001:000028f0       ?sl_showChromatogram@ChromaViewContext@U2@@IAEXXZ 100038f0 f   ChromaViewPlugin.obj
 0001:00002a70       ?system_category@std@@YAABVerror_category@1@XZ 10003a70 f i ChromaViewPlugin.obj
 0001:00002a80       ?t@Node@?$QList@PAVADVSequenceWidget@U2@@@@QAEAAPAVADVSequenceWidget@U2@@XZ 10003a80 f i ChromaViewPlugin.obj
 0001:00002a90       ?t@Node@?$QList@PAVGObject@U2@@@@QAEAAPAVGObject@U2@@XZ 10003a90 f i ChromaViewPlugin.obj
 0001:00002aa0       ?tr@ChromaViewAction@U2@@SA?AVQString@@PBD0H@Z 10003aa0 f i ChromaViewPlugin.obj
 0001:00002ad0       ?tr@ChromaViewPlugin@U2@@SA?AVQString@@PBD0H@Z 10003ad0 f i ChromaViewPlugin.obj
 0001:00002b00       ?value@error_code@std@@QBEHXZ 10003b00 f i ChromaViewPlugin.obj
 0001:00002b10       ?value@error_condition@std@@QBEHXZ 10003b10 f i ChromaViewPlugin.obj
 0001:00002b20       _hypot                     10003b20 f i ChromaViewPlugin.obj
 0001:00002b50       _ugene_plugin_init         10003b50 f   ChromaViewPlugin.obj
 0001:00002b80       ??$?0VGObject@U2@@@?$QWeakPointer@VQObject@@@@AAE@PAVGObject@U2@@_N@Z 10003b80 f i ChromatogramView.obj
 0001:00002bc0       ??$_Move@AAPAUQHashData@@@std@@YA$$QAPAUQHashData@@AAPAU1@@Z 10003bc0 f i ChromatogramView.obj
 0001:00002bd0       ??$qAbs@N@@YANABN@Z        10003bd0 f i ChromatogramView.obj
 0001:00002c00       ??$qHash@PAVGObjectConstraints@U2@@@@YAIABQAVGObjectConstraints@U2@@I@Z 10003c00 f i ChromatogramView.obj
 0001:00002c10       ??$qHash@VGObjectConstraints@U2@@@@YAIPBVGObjectConstraints@U2@@I@Z 10003c10 f i ChromatogramView.obj
 0001:00002c20       ??$qMax@H@@YAABHABH0@Z     10003c20 f i ChromatogramView.obj
 0001:00002c40       ??$qMin@H@@YAABHABH0@Z     10003c40 f i ChromatogramView.obj
 0001:00002c60       ??$qMin@N@@YAABNABN0@Z     10003c60 f i ChromatogramView.obj
 0001:00002c80       ??$qSwap@PAUQHashData@@@@YAXAAPAUQHashData@@0@Z 10003c80 f i ChromatogramView.obj
 0001:00002ca0       ??$qobject_cast@PAVChromatogramView@U2@@@@YAPAVChromatogramView@U2@@PAVQObject@@@Z 10003ca0 f i ChromatogramView.obj
 0001:00002cc0       ??$qobject_cast@PAVLoadUnloadedDocumentTask@U2@@@@YAPAVLoadUnloadedDocumentTask@U2@@PAVQObject@@@Z 10003cc0 f i ChromatogramView.obj
 0001:00002ce0       ??$qobject_cast@PAVQAction@@@@YAPAVQAction@@PAVQObject@@@Z 10003ce0 f i ChromatogramView.obj
 0001:00002d00       ??$qobject_cast@PAVU2SequenceObject@U2@@@@YAPAVU2SequenceObject@U2@@PAVQObject@@@Z 10003d00 f i ChromatogramView.obj
 0001:00002d20       ??$swap@PAUQHashData@@@std@@YAXAAPAUQHashData@@0@Z 10003d20 f i ChromatogramView.obj
 0001:00002d40       ??0?$QFlags@W4AlignmentFlag@Qt@@@@QAE@PQPrivate@0@H@Z 10003d40 f i ChromatogramView.obj
 0001:00002d50       ??0?$QFlags@W4AllocationOption@QArrayData@@@@QAE@W4AllocationOption@QArrayData@@@Z 10003d50 f i ChromatogramView.obj
 0001:00002d60       ??0?$QFlags@W4DocumentFormatFlag@U2@@@@QAE@PQPrivate@0@H@Z 10003d60 f i ChromatogramView.obj
 0001:00002d70       ??0?$QFlags@W4StandardButton@QMessageBox@@@@QAE@W4StandardButton@QMessageBox@@@Z 10003d70 f i ChromatogramView.obj
 0001:00002d80       ??0?$QForeachContainer@$$CBV?$QList@PAVGObject@U2@@@@@@QAE@ABV?$QList@PAVGObject@U2@@@@@Z 10003d80 f i ChromatogramView.obj
 0001:00002dc0       ??0?$QForeachContainer@V?$QList@H@@@@QAE@ABV?$QList@H@@@Z 10003dc0 f i ChromatogramView.obj
 0001:00002e00       ??0?$QForeachContainer@V?$QList@PAVQAction@@@@@@QAE@ABV?$QList@PAVQAction@@@@@Z 10003e00 f i ChromatogramView.obj
 0001:00002e40       ??0?$QHash@HUQHashDummyValue@@@@QAE@XZ 10003e40 f i ChromatogramView.obj
 0001:00002e50       ??0?$QHash@VQString@@UQHashDummyValue@@@@QAE@XZ 10003e50 f i ChromatogramView.obj
 0001:00002e60       ??0?$QHashNode@HUQHashDummyValue@@@@QAE@ABHABUQHashDummyValue@@IPAU0@@Z 10003e60 f i ChromatogramView.obj
 0001:00002e80       ??0?$QHashNode@PAVGObjectConstraints@U2@@UQHashDummyValue@@@@QAE@ABQAVGObjectConstraints@U2@@ABUQHashDummyValue@@IPAU0@@Z 10003e80 f i ChromatogramView.obj
 0001:00002ea0       ??0?$QHashNode@VQString@@UQHashDummyValue@@@@QAE@ABVQString@@ABUQHashDummyValue@@IPAU0@@Z 10003ea0 f i ChromatogramView.obj
 0001:00002ed0       ??0?$QList@H@@QAE@ABV0@@Z  10003ed0 f i ChromatogramView.obj
 0001:00002f90       ??0?$QList@H@@QAE@XZ       10003f90 f i ChromatogramView.obj
 0001:00002fa0       ??0?$QList@PAVGObject@U2@@@@QAE@ABV0@@Z 10003fa0 f i ChromatogramView.obj
 0001:00003060       ??0?$QList@PAVQAction@@@@QAE@ABV0@@Z 10004060 f i ChromatogramView.obj
 0001:00003120       ??0?$QMap@VQString@@VQVariant@@@@QAE@XZ 10004120 f i ChromatogramView.obj
 0001:00003130       ??0?$QPointer@VGObject@U2@@@@QAE@ABV0@@Z 10004130 f i ChromatogramView.obj
 0001:00003160       ??0?$QPointer@VGObject@U2@@@@QAE@PAVGObject@U2@@@Z 10004160 f i ChromatogramView.obj
 0001:000031a0       ??0?$QSet@H@@QAE@XZ        100041a0 f i ChromatogramView.obj
 0001:000031b0       ??0?$QSet@VQString@@@@QAE@XZ 100041b0 f i ChromatogramView.obj
 0001:000031c0       ??0?$QWeakPointer@VQObject@@@@QAE@ABV0@@Z 100041c0 f i ChromatogramView.obj
 0001:000031f0       ??0ChromatogramView@U2@@QAE@PAVQWidget@@PAVADVSequenceObjectContext@1@PAVGSequenceLineView@1@ABVDNAChromatogram@1@@Z 100041f0 f   ChromatogramView.obj
 0001:00003b40       ??0ChromatogramViewRenderArea@U2@@QAE@PAVChromatogramView@1@ABVDNAChromatogram@1@@Z 10004b40 f   ChromatogramView.obj
 0001:00004150       ??0ChromatogramViewSettings@U2@@QAE@XZ 10005150 f i ChromatogramView.obj
 0001:00004160       ??0DocumentFormatConstraints@U2@@QAE@XZ 10005160 f i ChromatogramView.obj
 0001:000041e0       ??0QLatin1Char@@QAE@D@Z    100051e0 f i ChromatogramView.obj
 0001:000041f0       ??0const_iterator@?$QHash@HUQHashDummyValue@@@@QAE@PAX@Z 100051f0 f i ChromatogramView.obj
 0001:00004200       ??0const_iterator@?$QList@H@@QAE@PAUNode@1@@Z 10005200 f i ChromatogramView.obj
 0001:00004210       ??0const_iterator@?$QList@PAVGObject@U2@@@@QAE@PAUNode@1@@Z 10005210 f i ChromatogramView.obj
 0001:00004220       ??0const_iterator@?$QList@PAVQAction@@@@QAE@PAUNode@1@@Z 10005220 f i ChromatogramView.obj
 0001:00004230       ??0const_iterator@?$QSet@H@@QAE@V0?$QHash@HUQHashDummyValue@@@@@Z 10005230 f i ChromatogramView.obj
 0001:00004240       ??0iterator@?$QHash@HUQHashDummyValue@@@@QAE@PAX@Z 10005240 f i ChromatogramView.obj
 0001:00004250       ??0iterator@?$QHash@PAVGObjectConstraints@U2@@UQHashDummyValue@@@@QAE@PAX@Z 10005250 f i ChromatogramView.obj
 0001:00004260       ??0iterator@?$QHash@VQString@@UQHashDummyValue@@@@QAE@PAX@Z 10005260 f i ChromatogramView.obj
 0001:00004270       ??0iterator@?$QSet@H@@QAE@V0?$QHash@HUQHashDummyValue@@@@@Z 10005270 f i ChromatogramView.obj
 0001:00004280       ??0iterator@?$QSet@PAVGObjectConstraints@U2@@@@QAE@V0?$QHash@PAVGObjectConstraints@U2@@UQHashDummyValue@@@@@Z 10005280 f i ChromatogramView.obj
 0001:00004290       ??0iterator@?$QSet@VQString@@@@QAE@V0?$QHash@VQString@@UQHashDummyValue@@@@@Z 10005290 f i ChromatogramView.obj
 0001:000042a0       ??1?$QForeachContainer@$$CBV?$QList@PAVGObject@U2@@@@@@QAE@XZ 100052a0 f i ChromatogramView.obj
 0001:000042d0       ??1?$QForeachContainer@V?$QList@H@@@@QAE@XZ 100052d0 f i ChromatogramView.obj
 0001:00004300       ??1?$QForeachContainer@V?$QList@PAVQAction@@@@@@QAE@XZ 10005300 f i ChromatogramView.obj
 0001:00004330       ??1?$QHash@HUQHashDummyValue@@@@QAE@XZ 10005330 f i ChromatogramView.obj
 0001:00004360       ??1?$QHash@VQString@@UQHashDummyValue@@@@QAE@XZ 10005360 f i ChromatogramView.obj
 0001:00004390       ??1?$QHashNode@VQString@@UQHashDummyValue@@@@QAE@XZ 10005390 f i ChromatogramView.obj
 0001:000043a0       ??1?$QList@H@@QAE@XZ       100053a0 f i ChromatogramView.obj
 0001:000043d0       ??1?$QList@PAVQAction@@@@QAE@XZ 100053d0 f i ChromatogramView.obj
 0001:00004400       ??1?$QMap@VQString@@VQVariant@@@@QAE@XZ 10005400 f i ChromatogramView.obj
 0001:00004450       ??1?$QPointer@VGObject@U2@@@@QAE@XZ 10005450 f i ChromatogramView.obj
 0001:00004470       ??1?$QSet@H@@QAE@XZ        10005470 f i ChromatogramView.obj
 0001:000044a0       ??1?$QSet@VQString@@@@QAE@XZ 100054a0 f i ChromatogramView.obj
 0001:000044d0       ??1?$QWeakPointer@VQObject@@@@QAE@XZ 100054d0 f i ChromatogramView.obj
 0001:000044f0       ??1ChromatogramView@U2@@UAE@XZ 100054f0 f i ChromatogramView.obj
 0001:000045c0       ??1ChromatogramViewRenderArea@U2@@UAE@XZ 100055c0 f   ChromatogramView.obj
 0001:00004660       ??1DocumentFormatConstraints@U2@@QAE@XZ 10005660 f i ChromatogramView.obj
 0001:00004710       ??1ExternalRefCountData@QtSharedPointer@@QAE@XZ 10005710 f i ChromatogramView.obj
 0001:00004720       ??3ExternalRefCountData@QtSharedPointer@@SAXPAX@Z 10005720 f i ChromatogramView.obj
 0001:00004730       ??4?$QHash@HUQHashDummyValue@@@@QAEAAV0@$$QAV0@@Z 10005730 f i ChromatogramView.obj
 0001:00004750       ??9const_iterator@?$QHash@HUQHashDummyValue@@@@QBE_NABV01@@Z 10005750 f i ChromatogramView.obj
 0001:00004770       ??9const_iterator@?$QList@H@@QBE_NABV01@@Z 10005770 f i ChromatogramView.obj
 0001:00004790       ??9const_iterator@?$QList@PAVGObject@U2@@@@QBE_NABV01@@Z 10005790 f i ChromatogramView.obj
 0001:000047b0       ??9const_iterator@?$QList@PAVQAction@@@@QBE_NABV01@@Z 100057b0 f i ChromatogramView.obj
 0001:000047d0       ??9const_iterator@?$QSet@H@@QBE_NABV01@@Z 100057d0 f i ChromatogramView.obj
 0001:000047f0       ??A?$QVector@D@@QAEAADH@Z  100057f0 f i ChromatogramView.obj
 0001:00004860       ??A?$QVector@G@@QAEAAGH@Z  10005860 f i ChromatogramView.obj
 0001:000048e0       ??A?$QVector@G@@QBEABGH@Z  100058e0 f i ChromatogramView.obj
 0001:00004900       ??Dconst_iterator@?$QList@H@@QBEABHXZ 10005900 f i ChromatogramView.obj
 0001:00004910       ??Dconst_iterator@?$QList@PAVGObject@U2@@@@QBEABQAVGObject@U2@@XZ 10005910 f i ChromatogramView.obj
 0001:00004920       ??Dconst_iterator@?$QList@PAVQAction@@@@QBEABQAVQAction@@XZ 10005920 f i ChromatogramView.obj
 0001:00004930       ??Dconst_iterator@?$QSet@H@@QBEABHXZ 10005930 f i ChromatogramView.obj
 0001:00004940       ??Econst_iterator@?$QHash@HUQHashDummyValue@@@@QAEAAV01@XZ 10005940 f i ChromatogramView.obj
 0001:00004960       ??Econst_iterator@?$QList@H@@QAEAAV01@XZ 10005960 f i ChromatogramView.obj
 0001:00004970       ??Econst_iterator@?$QList@PAVGObject@U2@@@@QAEAAV01@XZ 10005970 f i ChromatogramView.obj
 0001:00004980       ??Econst_iterator@?$QList@PAVQAction@@@@QAEAAV01@XZ 10005980 f i ChromatogramView.obj
 0001:00004990       ??Econst_iterator@?$QSet@H@@QAEAAV01@XZ 10005990 f i ChromatogramView.obj
 0001:000049b0       ??H@YA?BVQString@@ABV0@0@Z 100059b0 f i ChromatogramView.obj
 0001:00004a20       ??H@YA?BVQString@@ABV0@PBD@Z 10005a20 f i ChromatogramView.obj
 0001:00004ac0       ??H@YA?BVQString@@PBDABV0@@Z 10005ac0 f i ChromatogramView.obj
 0001:00004b30       ??Y?$QSet@VQString@@@@QAEAAV0@ABVQString@@@Z 10005b30 f i ChromatogramView.obj
 0001:00004b50       ??_5?$QFlags@W4DocumentFormatFlag@U2@@@@QAEAAV0@W4DocumentFormatFlag@U2@@@Z 10005b50 f i ChromatogramView.obj
 0001:00004b5e       ??_EChromatogramView@U2@@W7AEPAXI@Z 10005b5e f i ChromatogramView.obj
 0001:00004b66       ??_EChromatogramViewRenderArea@U2@@W7AEPAXI@Z 10005b66 f i ChromatogramView.obj
 0001:00004b6e       ??_EQHBoxLayout@@W7AEPAXI@Z 10005b6e f i ChromatogramView.obj
 0001:00004b76       ??_EQMenu@@W7AEPAXI@Z      10005b76 f i ChromatogramView.obj
 0001:00004b7e       ??_EScaleBar@U2@@W7AEPAXI@Z 10005b7e f i ChromatogramView.obj
 0001:00004b90       ??_G?$QHashNode@VQString@@UQHashDummyValue@@@@QAEPAXI@Z 10005b90 f i ChromatogramView.obj
 0001:00004bc0       ??_G?$QPointer@VGObject@U2@@@@QAEPAXI@Z 10005bc0 f i ChromatogramView.obj
 0001:00004c00       ??_EChromatogramView@U2@@UAEPAXI@Z 10005c00 f i ChromatogramView.obj
 0001:00004c00       ??_GChromatogramView@U2@@UAEPAXI@Z 10005c00 f i ChromatogramView.obj
 0001:00004c30       ??_GChromatogramViewRenderArea@U2@@UAEPAXI@Z 10005c30 f i ChromatogramView.obj
 0001:00004c30       ??_EChromatogramViewRenderArea@U2@@UAEPAXI@Z 10005c30 f i ChromatogramView.obj
 0001:00004c60       ??_GExternalRefCountData@QtSharedPointer@@QAEPAXI@Z 10005c60 f i ChromatogramView.obj
 0001:00004c80       ??_ELoadUnloadedDocumentTask@U2@@UAEPAXI@Z 10005c80 f i ChromatogramView.obj
 0001:00004c80       ??_GLoadUnloadedDocumentTask@U2@@UAEPAXI@Z 10005c80 f i ChromatogramView.obj
 0001:00004cb0       ??_EQAction@@UAEPAXI@Z     10005cb0 f i ChromatogramView.obj
 0001:00004cb0       ??_GQAction@@UAEPAXI@Z     10005cb0 f i ChromatogramView.obj
 0001:00004ce0       ??_GQHBoxLayout@@UAEPAXI@Z 10005ce0 f i ChromatogramView.obj
 0001:00004ce0       ??_EQHBoxLayout@@UAEPAXI@Z 10005ce0 f i ChromatogramView.obj
 0001:00004d10       ??_EQMenu@@UAEPAXI@Z       10005d10 f i ChromatogramView.obj
 0001:00004d10       ??_GQMenu@@UAEPAXI@Z       10005d10 f i ChromatogramView.obj
 0001:00004d40       ??_GQString@@QAEPAXI@Z     10005d40 f i ChromatogramView.obj
 0001:00004d70       ??_GQVariant@@QAEPAXI@Z    10005d70 f i ChromatogramView.obj
 0001:00004da0       ??_EScaleBar@U2@@UAEPAXI@Z 10005da0 f i ChromatogramView.obj
 0001:00004da0       ??_GScaleBar@U2@@UAEPAXI@Z 10005da0 f i ChromatogramView.obj
 0001:00004dd0       ??_GTaskSignalMapper@U2@@UAEPAXI@Z 10005dd0 f i ChromatogramView.obj
 0001:00004dd0       ??_ETaskSignalMapper@U2@@UAEPAXI@Z 10005dd0 f i ChromatogramView.obj
 0001:00004e00       ?addFlagToExclude@DocumentFormatConstraints@U2@@QAEXW4DocumentFormatFlag@2@@Z 10005e00 f i ChromatogramView.obj
 0001:00004e10       ?addFlagToSupport@DocumentFormatConstraints@U2@@QAEXW4DocumentFormatFlag@2@@Z 10005e10 f i ChromatogramView.obj
 0001:00004e20       ?alignOfNode@?$QHash@HUQHashDummyValue@@@@CAHXZ 10005e20 f i ChromatogramView.obj
 0001:00004e30       ?alignOfNode@?$QHash@PAVGObjectConstraints@U2@@UQHashDummyValue@@@@CAHXZ 10005e30 f i ChromatogramView.obj
 0001:00004e40       ?alignOfNode@?$QHash@VQString@@UQHashDummyValue@@@@CAHXZ 10005e40 f i ChromatogramView.obj
 0001:00004e50       ?allocate@?$QTypedArrayData@D@@SAPAU1@IV?$QFlags@W4AllocationOption@QArrayData@@@@@Z 10005e50 f i ChromatogramView.obj
 0001:00004e70       ?allocate@?$QTypedArrayData@G@@SAPAU1@IV?$QFlags@W4AllocationOption@QArrayData@@@@@Z 10005e70 f i ChromatogramView.obj
 0001:00004e90       ?append@?$QList@H@@QAEXABH@Z 10005e90 f i ChromatogramView.obj
 0001:00004f20       ?append@?$QList@V?$QPointer@VGObject@U2@@@@@@QAEXABV?$QPointer@VGObject@U2@@@@@Z 10005f20 f i ChromatogramView.obj
 0001:00005000       ?begin@?$QList@H@@QBE?AVconst_iterator@1@XZ 10006000 f i ChromatogramView.obj
 0001:00005020       ?begin@?$QList@PAVGObject@U2@@@@QBE?AVconst_iterator@1@XZ 10006020 f i ChromatogramView.obj
 0001:00005040       ?begin@?$QList@PAVQAction@@@@QBE?AVconst_iterator@1@XZ 10006040 f i ChromatogramView.obj
 0001:00005060       ?begin@?$QTypedArrayData@D@@QAEPADPAD@Z 10006060 f i ChromatogramView.obj
 0001:00005070       ?begin@?$QTypedArrayData@G@@QAEPAGPAG@Z 10006070 f i ChromatogramView.obj
 0001:00005080       ?begin@?$QVector@VU2Region@U2@@@@QBEPBVU2Region@U2@@XZ 10006080 f i ChromatogramView.obj
 0001:00005090       ?buildPopupMenu@ChromatogramView@U2@@UAEXAAVQMenu@@@Z 10006090 f   ChromatogramView.obj
 0001:00005200       ?clear@?$QHash@HUQHashDummyValue@@@@QAEXXZ 10006200 f i ChromatogramView.obj
 0001:00005240       ?clear@?$QSet@H@@QAEXXZ    10006240 f i ChromatogramView.obj
 0001:00005280       ?concrete@?$QHash@HUQHashDummyValue@@@@CAPAU?$QHashNode@HUQHashDummyValue@@@@PAUNode@QHashData@@@Z 10006280 f i ChromatogramView.obj
 0001:00005290       ?concrete@?$QHash@PAVGObjectConstraints@U2@@UQHashDummyValue@@@@CAPAU?$QHashNode@PAVGObjectConstraints@U2@@UQHashDummyValue@@@@PAUNode@QHashData@@@Z 10006290 f i ChromatogramView.obj
 0001:000052a0       ?concrete@?$QHash@VQString@@UQHashDummyValue@@@@CAPAU?$QHashNode@VQString@@UQHashDummyValue@@@@PAUNode@QHashData@@@Z 100062a0 f i ChromatogramView.obj
 0001:000052b0       ?constBegin@?$QHash@HUQHashDummyValue@@@@QBE?AVconst_iterator@1@XZ 100062b0 f i ChromatogramView.obj
 0001:000052e0       ?constBegin@?$QSet@H@@QBE?AVconst_iterator@1@XZ 100062e0 f i ChromatogramView.obj
 0001:00005310       ?constBegin@?$QTypedArrayData@VU2Region@U2@@@@QBEPBVU2Region@U2@@PBV23@@Z 10006310 f i ChromatogramView.obj
 0001:00005320       ?constEnd@?$QHash@HUQHashDummyValue@@@@QBE?AVconst_iterator@1@XZ 10006320 f i ChromatogramView.obj
 0001:00005330       ?constEnd@?$QSet@H@@QBE?AVconst_iterator@1@XZ 10006330 f i ChromatogramView.obj
 0001:00005340       ?contains@?$QHash@HUQHashDummyValue@@@@QBE_NABH@Z 10006340 f i ChromatogramView.obj
 0001:000053a0       ?contains@?$QSet@H@@QBE_NABH@Z 100063a0 f i ChromatogramView.obj
 0001:000053b0       ?coordToPos@ChromatogramViewRenderArea@U2@@UBE_JH@Z 100063b0 f   ChromatogramView.obj
 0001:00005560       ?createNode@?$QHash@HUQHashDummyValue@@@@AAEPAU?$QHashNode@HUQHashDummyValue@@@@IABHABUQHashDummyValue@@PAPAU2@@Z 10006560 f i ChromatogramView.obj
 0001:000055b0       ?createNode@?$QHash@PAVGObjectConstraints@U2@@UQHashDummyValue@@@@AAEPAU?$QHashNode@PAVGObjectConstraints@U2@@UQHashDummyValue@@@@IABQAVGObjectConstraints@U2@@ABUQHashDummyValue@@PAPAU2@@Z 100065b0 f i ChromatogramView.obj
 0001:00005600       ?createNode@?$QHash@VQString@@UQHashDummyValue@@@@AAEPAU?$QHashNode@VQString@@UQHashDummyValue@@@@IABVQString@@ABUQHashDummyValue@@PAPAU2@@Z 10006600 f i ChromatogramView.obj
 0001:00005690       ?createToggleTraceAction@ChromatogramView@U2@@AAEPAVQAction@@ABVQString@@@Z 10006690 f   ChromatogramView.obj
 0001:00005750       ?data@?$QTypedArrayData@D@@QAEPADXZ 10006750 f i ChromatogramView.obj
 0001:00005760       ?data@?$QTypedArrayData@G@@QAEPAGXZ 10006760 f i ChromatogramView.obj
 0001:00005770       ?data@?$QTypedArrayData@VU2Region@U2@@@@QBEPBVU2Region@U2@@XZ 10006770 f i ChromatogramView.obj
 0001:00005780       ?data@?$QVector@D@@QAEPADXZ 10006780 f i ChromatogramView.obj
 0001:000057e0       ?data@?$QVector@G@@QAEPAGXZ 100067e0 f i ChromatogramView.obj
 0001:00005840       ?dealloc@?$QList@H@@AAEXPAUData@QListData@@@Z 10006840 f i ChromatogramView.obj
 0001:00005860       ?dealloc@?$QList@PAVQAction@@@@AAEXPAUData@QListData@@@Z 10006860 f i ChromatogramView.obj
 0001:00005880       ?dealloc@?$QList@V?$QPointer@VGObject@U2@@@@@@AAEXPAUData@QListData@@@Z 10006880 f i ChromatogramView.obj
 0001:000058b0       ?deallocate@?$QTypedArrayData@D@@SAXPAUQArrayData@@@Z 100068b0 f i ChromatogramView.obj
 0001:000058d0       ?deallocate@?$QTypedArrayData@G@@SAXPAUQArrayData@@@Z 100068d0 f i ChromatogramView.obj
 0001:000058f0       ?defaultConstruct@?$QVector@D@@AAEXPAD0@Z 100068f0 f i ChromatogramView.obj
 0001:00005910       ?defaultConstruct@?$QVector@G@@AAEXPAG0@Z 10006910 f i ChromatogramView.obj
 0001:00005930       ?deleteNode2@?$QHash@HUQHashDummyValue@@@@CAXPAUNode@QHashData@@@Z 10006930 f i ChromatogramView.obj
 0001:00005940       ?deleteNode2@?$QHash@PAVGObjectConstraints@U2@@UQHashDummyValue@@@@CAXPAUNode@QHashData@@@Z 10006940 f i ChromatogramView.obj
 0001:00005950       ?deleteNode2@?$QHash@VQString@@UQHashDummyValue@@@@CAXPAUNode@QHashData@@@Z 10006950 f i ChromatogramView.obj
 0001:00005960       ?deleteNode@?$QHash@HUQHashDummyValue@@@@AAEXPAU?$QHashNode@HUQHashDummyValue@@@@@Z 10006960 f i ChromatogramView.obj
 0001:00005970       ?destroy@?$QMapData@VQString@@VQVariant@@@@QAEXXZ 10006970 f i ChromatogramView.obj
 0001:000059a0       ?destroySubTree@?$QMapNode@VQString@@VQVariant@@@@QAEXXZ 100069a0 f i ChromatogramView.obj
 0001:000059e0       ?destruct@?$QVector@D@@AAEXPAD0@Z 100069e0 f i ChromatogramView.obj
 0001:000059f0       ?destruct@?$QVector@G@@AAEXPAG0@Z 100069f0 f i ChromatogramView.obj
 0001:00005a00       ?detach@?$QHash@HUQHashDummyValue@@@@QAEXXZ 10006a00 f i ChromatogramView.obj
 0001:00005a60       ?detach@?$QHash@PAVGObjectConstraints@U2@@UQHashDummyValue@@@@QAEXXZ 10006a60 f i ChromatogramView.obj
 0001:00005ac0       ?detach@?$QHash@VQString@@UQHashDummyValue@@@@QAEXXZ 10006ac0 f i ChromatogramView.obj
 0001:00005b20       ?detach@?$QList@H@@QAEXXZ  10006b20 f i ChromatogramView.obj
 0001:00005b40       ?detach@?$QVector@D@@QAEXXZ 10006b40 f i ChromatogramView.obj
 0001:00005b90       ?detach@?$QVector@G@@QAEXXZ 10006b90 f i ChromatogramView.obj
 0001:00005be0       ?detach_helper@?$QHash@HUQHashDummyValue@@@@AAEXXZ 10006be0 f i ChromatogramView.obj
 0001:00005c30       ?detach_helper@?$QHash@PAVGObjectConstraints@U2@@UQHashDummyValue@@@@AAEXXZ 10006c30 f i ChromatogramView.obj
 0001:00005c80       ?detach_helper@?$QHash@VQString@@UQHashDummyValue@@@@AAEXXZ 10006c80 f i ChromatogramView.obj
 0001:00005cd0       ?detach_helper@?$QList@H@@AAEXH@Z 10006cd0 f i ChromatogramView.obj
 0001:00005da0       ?detach_helper@?$QList@H@@AAEXXZ 10006da0 f i ChromatogramView.obj
 0001:00005db0       ?detach_helper_grow@?$QList@H@@AAEPAUNode@1@HH@Z 10006db0 f i ChromatogramView.obj
 0001:00005ec0       ?detach_helper_grow@?$QList@V?$QPointer@VGObject@U2@@@@@@AAEPAUNode@1@HH@Z 10006ec0 f i ChromatogramView.obj
 0001:00006030       ?drawAll@ChromatogramViewRenderArea@U2@@MAEXPAVQPaintDevice@@@Z 10007030 f   ChromatogramView.obj
 0001:00006ae0       ?drawChromatogramBaseCallsLines@ChromatogramViewRenderArea@U2@@AAEXNNNNAAVQPainter@@ABVU2Region@2@ABVQByteArray@@ABUChromatogramViewSettings@2@@Z 10007ae0 f   ChromatogramView.obj
 0001:00006fa0       ?drawChromatogramTrace@ChromatogramViewRenderArea@U2@@AAEXNNNNAAVQPainter@@ABVU2Region@2@ABUChromatogramViewSettings@2@@Z 10007fa0 f   ChromatogramView.obj
 0001:00007610       ?drawOriginalBaseCalls@ChromatogramViewRenderArea@U2@@AAEXNNNNAAVQPainter@@ABVU2Region@2@ABVQByteArray@@_N@Z 10008610 f   ChromatogramView.obj
 0001:00007af0       ?drawQualityValues@ChromatogramViewRenderArea@U2@@AAEXNNNNAAVQPainter@@ABVU2Region@2@ABVQByteArray@@@Z 10008af0 f   ChromatogramView.obj
 0001:00008180       ?duplicateNode@?$QHash@HUQHashDummyValue@@@@CAXPAUNode@QHashData@@PAX@Z 10009180 f i ChromatogramView.obj
 0001:000081b0       ?duplicateNode@?$QHash@PAVGObjectConstraints@U2@@UQHashDummyValue@@@@CAXPAUNode@QHashData@@PAX@Z 100091b0 f i ChromatogramView.obj
 0001:000081e0       ?duplicateNode@?$QHash@VQString@@UQHashDummyValue@@@@CAXPAUNode@QHashData@@PAX@Z 100091e0 f i ChromatogramView.obj
 0001:00008240       ?end@?$QList@H@@QBE?AVconst_iterator@1@XZ 10009240 f i ChromatogramView.obj
 0001:00008260       ?end@?$QList@PAVGObject@U2@@@@QBE?AVconst_iterator@1@XZ 10009260 f i ChromatogramView.obj
 0001:00008280       ?end@?$QList@PAVQAction@@@@QBE?AVconst_iterator@1@XZ 10009280 f i ChromatogramView.obj
 0001:000082a0       ?end@?$QTypedArrayData@D@@QAEPADPAD@Z 100092a0 f i ChromatogramView.obj
 0001:000082b0       ?end@?$QTypedArrayData@G@@QAEPAGPAG@Z 100092b0 f i ChromatogramView.obj
 0001:000082d0       ?findNode@?$QHash@HUQHashDummyValue@@@@ABEPAPAU?$QHashNode@HUQHashDummyValue@@@@ABHPAI@Z 100092d0 f i ChromatogramView.obj
 0001:00008340       ?findNode@?$QHash@PAVGObjectConstraints@U2@@UQHashDummyValue@@@@ABEPAPAU?$QHashNode@PAVGObjectConstraints@U2@@UQHashDummyValue@@@@ABQAVGObjectConstraints@U2@@PAI@Z 10009340 f i ChromatogramView.obj
 0001:000083b0       ?findNode@?$QHash@VQString@@UQHashDummyValue@@@@ABEPAPAU?$QHashNode@VQString@@UQHashDummyValue@@@@ABVQString@@PAI@Z 100093b0 f i ChromatogramView.obj
 0001:00008440       ?first@?$QVector@VU2Region@U2@@@@QBEABVU2Region@U2@@XZ 10009440 f i ChromatogramView.obj
 0001:00008450       ?freeData@?$QHash@HUQHashDummyValue@@@@AAEXPAUQHashData@@@Z 10009450 f i ChromatogramView.obj
 0001:00008470       ?freeData@?$QHash@PAVGObjectConstraints@U2@@UQHashDummyValue@@@@AAEXPAUQHashData@@@Z 10009470 f i ChromatogramView.obj
 0001:00008490       ?freeData@?$QHash@VQString@@UQHashDummyValue@@@@AAEXPAUQHashData@@@Z 10009490 f i ChromatogramView.obj
 0001:000084b0       ?freeData@?$QVector@D@@AAEXPAU?$QTypedArrayData@D@@@Z 100094b0 f i ChromatogramView.obj
 0001:000084e0       ?freeData@?$QVector@G@@AAEXPAU?$QTypedArrayData@G@@@Z 100094e0 f i ChromatogramView.obj
 0001:00008510       ?getBaseColor@ChromatogramViewRenderArea@U2@@AAE?AVQColor@@D@Z 10009510 f   ChromatogramView.obj
 0001:000085b0       ?getEditSeqIndex@ChromatogramView@U2@@AAEHH@Z 100095b0 f   ChromatogramView.obj
 0001:00008640       ?getHeightAreaBC@ChromatogramViewRenderArea@U2@@QBEHXZ 10009640 f i ChromatogramView.obj
 0001:00008650       ?getSettings@ChromatogramView@U2@@QBEABUChromatogramViewSettings@2@XZ 10009650 f i ChromatogramView.obj
 0001:00008660       ?indexOf@?$QList@H@@QBEHABHH@Z 10009660 f i ChromatogramView.obj
 0001:000086f0       ?insert@?$QHash@HUQHashDummyValue@@@@QAE?AViterator@1@ABHABUQHashDummyValue@@@Z 100096f0 f i ChromatogramView.obj
 0001:000087c0       ?insert@?$QHash@PAVGObjectConstraints@U2@@UQHashDummyValue@@@@QAE?AViterator@1@ABQAVGObjectConstraints@U2@@ABUQHashDummyValue@@@Z 100097c0 f i ChromatogramView.obj
 0001:00008890       ?insert@?$QHash@VQString@@UQHashDummyValue@@@@QAE?AViterator@1@ABVQString@@ABUQHashDummyValue@@@Z 10009890 f i ChromatogramView.obj
 0001:000089e0       ?insert@?$QSet@H@@QAE?AViterator@1@ABH@Z 100099e0 f i ChromatogramView.obj
 0001:00008a10       ?insert@?$QSet@PAVGObjectConstraints@U2@@@@QAE?AViterator@1@ABQAVGObjectConstraints@U2@@@Z 10009a10 f i ChromatogramView.obj
 0001:00008a40       ?insert@?$QSet@VQString@@@@QAE?AViterator@1@ABVQString@@@Z 10009a40 f i ChromatogramView.obj
 0001:00008a70       ?isDetached@?$QVector@D@@QBE_NXZ 10009a70 f i ChromatogramView.obj
 0001:00008aa0       ?isDetached@?$QVector@G@@QBE_NXZ 10009aa0 f i ChromatogramView.obj
 0001:00008ad0       ?isEmpty@?$QHash@HUQHashDummyValue@@@@QBE_NXZ 10009ad0 f i ChromatogramView.obj
 0001:00008ae0       ?isEmpty@?$QVector@VU2Region@U2@@@@QBE_NXZ 10009ae0 f i ChromatogramView.obj
 0001:00008af0       ?isWidgetOnlyObject@ChromatogramView@U2@@UBE_NPAVGObject@2@@Z 10009af0 f   ChromatogramView.obj
 0001:00008b10       ?key@const_iterator@?$QHash@HUQHashDummyValue@@@@QBEABHXZ 10009b10 f i ChromatogramView.obj
 0001:00008b20       ?leftNode@?$QMapNode@VQString@@VQVariant@@@@QBEPAU1@XZ 10009b20 f i ChromatogramView.obj
 0001:00008b30       ?mousePressEvent@ChromatogramView@U2@@MAEXPAVQMouseEvent@@@Z 10009b30 f   ChromatogramView.obj
 0001:00008d30       ?node_construct@?$QList@H@@AAEXPAUNode@1@ABH@Z 10009d30 f i ChromatogramView.obj
 0001:00008d50       ?node_construct@?$QList@V?$QPointer@VGObject@U2@@@@@@AAEXPAUNode@1@ABV?$QPointer@VGObject@U2@@@@@Z 10009d50 f i ChromatogramView.obj
 0001:00008da0       ?node_copy@?$QList@H@@AAEXPAUNode@1@00@Z 10009da0 f i ChromatogramView.obj
 0001:00008dd0       ?node_copy@?$QList@PAVQAction@@@@AAEXPAUNode@1@00@Z 10009dd0 f i ChromatogramView.obj
 0001:00008e00       ?node_copy@?$QList@V?$QPointer@VGObject@U2@@@@@@AAEXPAUNode@1@00@Z 10009e00 f i ChromatogramView.obj
 0001:00008ef0       ?node_destruct@?$QList@H@@AAEXPAUNode@1@0@Z 10009ef0 f i ChromatogramView.obj
 0001:00008f00       ?node_destruct@?$QList@H@@AAEXPAUNode@1@@Z 10009f00 f i ChromatogramView.obj
 0001:00008f10       ?node_destruct@?$QList@PAVQAction@@@@AAEXPAUNode@1@0@Z 10009f10 f i ChromatogramView.obj
 0001:00008f20       ?node_destruct@?$QList@V?$QPointer@VGObject@U2@@@@@@AAEXPAUNode@1@0@Z 10009f20 f i ChromatogramView.obj
 0001:00008f70       ?node_destruct@?$QList@V?$QPointer@VGObject@U2@@@@@@AAEXPAUNode@1@@Z 10009f70 f i ChromatogramView.obj
 0001:00008fc0       ?pack@ChromatogramView@U2@@MAEXXZ 10009fc0 f   ChromatogramView.obj
 0001:000090a0       ?posToCoord@ChromatogramViewRenderArea@U2@@UBEH_J_N@Z 1000a0a0 f   ChromatogramView.obj
 0001:00009140       ?posToRect@ChromatogramViewRenderArea@U2@@QBE?AVQRectF@@H@Z 1000a140 f   ChromatogramView.obj
 0001:000091c0       ?qHash@@YAIHI@Z            1000a1c0 f i ChromatogramView.obj
 0001:000091d0       ?qHash@@YAIII@Z            1000a1d0 f i ChromatogramView.obj
 0001:000091e0       ?reallocData@?$QVector@D@@AAEXHHV?$QFlags@W4AllocationOption@QArrayData@@@@@Z 1000a1e0 f i ChromatogramView.obj
 0001:00009410       ?reallocData@?$QVector@G@@AAEXHHV?$QFlags@W4AllocationOption@QArrayData@@@@@Z 1000a410 f i ChromatogramView.obj
 0001:00009650       ?remove@?$QHash@HUQHashDummyValue@@@@QAEHABH@Z 1000a650 f i ChromatogramView.obj
 0001:00009710       ?remove@?$QSet@H@@QAE_NABH@Z 1000a710 f i ChromatogramView.obj
 0001:00009730       ?removeAt@?$QList@H@@QAEXH@Z 1000a730 f i ChromatogramView.obj
 0001:00009770       ?removeOne@?$QList@H@@QAE_NABH@Z 1000a770 f i ChromatogramView.obj
 0001:00009800       ?rightNode@?$QMapNode@VQString@@VQVariant@@@@QBEPAU1@XZ 1000a800 f i ChromatogramView.obj
 0001:00009810       ?root@?$QMapData@VQString@@VQVariant@@@@QBEPAU?$QMapNode@VQString@@VQVariant@@@@XZ 1000a810 f i ChromatogramView.obj
 0001:00009820       ?same_key@?$QHashNode@HUQHashDummyValue@@@@QBE_NIABH@Z 1000a820 f i ChromatogramView.obj
 0001:00009850       ?same_key@?$QHashNode@PAVGObjectConstraints@U2@@UQHashDummyValue@@@@QBE_NIABQAVGObjectConstraints@U2@@@Z 1000a850 f i ChromatogramView.obj
 0001:00009880       ?same_key@?$QHashNode@VQString@@UQHashDummyValue@@@@QBE_NIABVQString@@@Z 1000a880 f i ChromatogramView.obj
 0001:000098b0       ?setAreaHeight@ChromatogramViewRenderArea@U2@@QAEXH@Z 1000a8b0 f   ChromatogramView.obj
 0001:000098c0       ?setRenderAreaHeight@ChromatogramView@U2@@AAEXH@Z 1000a8c0 f   ChromatogramView.obj
 0001:000098e0       ?sharedNull@?$QTypedArrayData@D@@SAPAU1@XZ 1000a8e0 f i ChromatogramView.obj
 0001:000098f0       ?sharedNull@?$QTypedArrayData@G@@SAPAU1@XZ 1000a8f0 f i ChromatogramView.obj
 0001:00009900       ?showQV@ChromatogramView@U2@@QBE_NXZ 1000a900 f i ChromatogramView.obj
 0001:00009910       ?size@?$QList@PAVGObject@U2@@@@QBEHXZ 1000a910 f i ChromatogramView.obj
 0001:00009920       ?sl_addNewSequenceObject@ChromatogramView@U2@@AAEXXZ 1000a920 f   ChromatogramView.obj
 0001:00009e80       ?sl_clearEditableSequence@ChromatogramView@U2@@AAEXXZ 1000ae80 f   ChromatogramView.obj
 0001:00009ea0       ?sl_onAddExistingSequenceObject@ChromatogramView@U2@@AAEXXZ 1000aea0 f   ChromatogramView.obj
 0001:0000a2e0       ?sl_onObjectRemoved@ChromatogramView@U2@@AAEXPAVGObjectView@2@PAVGObject@2@@Z 1000b2e0 f   ChromatogramView.obj
 0001:0000a340       ?sl_onPopupMenuCkicked@ChromatogramView@U2@@AAEXPAVQAction@@@Z 1000b340 f   ChromatogramView.obj
 0001:0000a7b0       ?sl_onSequenceObjectLoaded@ChromatogramView@U2@@AAEXPAVTask@2@@Z 1000b7b0 f   ChromatogramView.obj
 0001:0000a8e0       ?sl_removeChanges@ChromatogramView@U2@@AAEXXZ 1000b8e0 f   ChromatogramView.obj
 0001:0000aac0       ?sl_showAllTraces@ChromatogramView@U2@@AAEXXZ 1000bac0 f   ChromatogramView.obj
 0001:0000abe0       ?sl_showHideTrace@ChromatogramView@U2@@AAEXXZ 1000bbe0 f   ChromatogramView.obj
 0001:0000ad60       ?t@Node@?$QList@H@@QAEAAHXZ 1000bd60 f i ChromatogramView.obj
 0001:0000ad70       ?t@Node@?$QList@PAVQAction@@@@QAEAAPAVQAction@@XZ 1000bd70 f i ChromatogramView.obj
 0001:0000ad80       ?testFlag@?$QFlags@W4GSLV_UpdateFlag@U2@@@@QBE_NW4GSLV_UpdateFlag@U2@@@Z 1000bd80 f i ChromatogramView.obj
 0001:0000adb0       ?tr@ChromatogramView@U2@@SA?AVQString@@PBD0H@Z 1000bdb0 f i ChromatogramView.obj
 0001:0000ade0       ?tr@ChromatogramViewRenderArea@U2@@SA?AVQString@@PBD0H@Z 1000bde0 f i ChromatogramView.obj
 0001:0000ae10       ?unsharableEmpty@?$QTypedArrayData@D@@SAPAU1@XZ 1000be10 f i ChromatogramView.obj
 0001:0000ae30       ?unsharableEmpty@?$QTypedArrayData@G@@SAPAU1@XZ 1000be30 f i ChromatogramView.obj
 0001:0000ae50       ??$acquireMemoryFence@H@?$QGenericAtomicOps@U?$QAtomicOpsBySize@$03@@@@SAXABH@Z 1000be50 f i moc_ChromaViewPlugin.obj
 0001:0000ae60       ??$loadAcquire@H@?$QGenericAtomicOps@U?$QAtomicOpsBySize@$03@@@@SAHABH@Z 1000be60 f i moc_ChromaViewPlugin.obj
 0001:0000ae70       ??$orderedMemoryFence@H@?$QGenericAtomicOps@U?$QAtomicOpsBySize@$03@@@@SAXABH@Z 1000be70 f i moc_ChromaViewPlugin.obj
 0001:0000ae80       ??$qMetaTypeId@PAVADVSequenceWidget@U2@@@@YAHXZ 1000be80 f i moc_ChromaViewPlugin.obj
 0001:0000ae90       ??$qRegisterMetaType@PAVADVSequenceWidget@U2@@@@YAHXZ 1000be90 f i moc_ChromaViewPlugin.obj
 0001:0000aea0       ??$qRegisterNormalizedMetaType@PAVADVSequenceWidget@U2@@@@YAHABVQByteArray@@PAPAVADVSequenceWidget@U2@@W4DefinedType@?$MetaTypeDefinedHelper@PAVADVSequenceWidget@U2@@$00@QtPrivate@@@Z 1000bea0 f i moc_ChromaViewPlugin.obj
 0001:0000af00       ??$releaseMemoryFence@H@?$QGenericAtomicOps@U?$QAtomicOpsBySize@$03@@@@SAXABH@Z 1000bf00 f i moc_ChromaViewPlugin.obj
 0001:0000af10       ??$storeRelease@HH@?$QGenericAtomicOps@U?$QAtomicOpsBySize@$03@@@@SAXAAHH@Z 1000bf10 f i moc_ChromaViewPlugin.obj
 0001:0000af20       ??0?$QFlags@W4TypeFlag@QMetaType@@@@QAE@VQFlag@@@Z 1000bf20 f i moc_ChromaViewPlugin.obj
 0001:0000af30       ??0QFlag@@QAE@H@Z          1000bf30 f i moc_ChromaViewPlugin.obj
 0001:0000af40       ??BQFlag@@QBEHXZ           1000bf40 f i moc_ChromaViewPlugin.obj
 0001:0000af50       ??C?$QScopedPointer@VQObjectData@@U?$QScopedPointerDeleter@VQObjectData@@@@@@QBEPAVQObjectData@@XZ 1000bf50 f i moc_ChromaViewPlugin.obj
 0001:0000af60       ??_5?$QFlags@W4TypeFlag@QMetaType@@@@QAEAAV0@W4TypeFlag@QMetaType@@@Z 1000bf60 f i moc_ChromaViewPlugin.obj
 0001:0000af70       ?Construct@?$QMetaTypeFunctionHelper@PAVADVSequenceWidget@U2@@$00@QtMetaTypePrivate@@SAPAXPAXPBX@Z 1000bf70 f i moc_ChromaViewPlugin.obj
 0001:0000afa0       ?Create@?$QMetaTypeFunctionHelper@PAVADVSequenceWidget@U2@@$00@QtMetaTypePrivate@@SAPAXPBX@Z 1000bfa0 f i moc_ChromaViewPlugin.obj
 0001:0000afe0       ?Delete@?$QMetaTypeFunctionHelper@PAVADVSequenceWidget@U2@@$00@QtMetaTypePrivate@@SAXPAX@Z 1000bfe0 f i moc_ChromaViewPlugin.obj
 0001:0000aff0       ?Destruct@?$QMetaTypeFunctionHelper@PAVADVSequenceWidget@U2@@$00@QtMetaTypePrivate@@SAXPAX@Z 1000bff0 f i moc_ChromaViewPlugin.obj
 0001:0000b000       ?loadAcquire@?$QBasicAtomicInteger@H@@QBEHXZ 1000c000 f i moc_ChromaViewPlugin.obj
 0001:0000b010       ?metaObject@ChromaViewAction@U2@@UBEPBUQMetaObject@@XZ 1000c010 f   moc_ChromaViewPlugin.obj
 0001:0000b030       ?metaObject@ChromaViewContext@U2@@UBEPBUQMetaObject@@XZ 1000c030 f   moc_ChromaViewPlugin.obj
 0001:0000b050       ?metaObject@ChromaViewPlugin@U2@@UBEPBUQMetaObject@@XZ 1000c050 f   moc_ChromaViewPlugin.obj
 0001:0000b070       ?qt_metacall@ChromaViewAction@U2@@UAEHW4Call@QMetaObject@@HPAPAX@Z 1000c070 f   moc_ChromaViewPlugin.obj
 0001:0000b080       ?qt_metacall@ChromaViewContext@U2@@UAEHW4Call@QMetaObject@@HPAPAX@Z 1000c080 f   moc_ChromaViewPlugin.obj
 0001:0000b0e0       ?qt_metacall@ChromaViewPlugin@U2@@UAEHW4Call@QMetaObject@@HPAPAX@Z 1000c0e0 f   moc_ChromaViewPlugin.obj
 0001:0000b0f0       ?qt_metacast@ChromaViewAction@U2@@UAEPAXPBD@Z 1000c0f0 f   moc_ChromaViewPlugin.obj
 0001:0000b150       ?qt_metacast@ChromaViewContext@U2@@UAEPAXPBD@Z 1000c150 f   moc_ChromaViewPlugin.obj
 0001:0000b1b0       ?qt_metacast@ChromaViewPlugin@U2@@UAEPAXPBD@Z 1000c1b0 f   moc_ChromaViewPlugin.obj
 0001:0000b210       ?qt_metatype_id@?$QMetaTypeId2@PAVADVSequenceWidget@U2@@@@SAHXZ 1000c210 f i moc_ChromaViewPlugin.obj
 0001:0000b220       ?qt_metatype_id@?$QMetaTypeIdHelper@PAVADVSequenceWidget@U2@@$00@QtPrivate@@SAHXZ 1000c220 f i moc_ChromaViewPlugin.obj
 0001:0000b230       ?qt_metatype_id@?$QMetaTypeIdQObject@PAVADVSequenceWidget@U2@@$00@@SAHXZ 1000c230 f i moc_ChromaViewPlugin.obj
 0001:0000b310       ?qt_static_metacall@ChromaViewAction@U2@@CAXPAVQObject@@W4Call@QMetaObject@@HPAPAX@Z 1000c310 f   moc_ChromaViewPlugin.obj
 0001:0000b320       ?qt_static_metacall@ChromaViewContext@U2@@CAXPAVQObject@@W4Call@QMetaObject@@HPAPAX@Z 1000c320 f   moc_ChromaViewPlugin.obj
 0001:0000b390       ?qt_static_metacall@ChromaViewPlugin@U2@@CAXPAVQObject@@W4Call@QMetaObject@@HPAPAX@Z 1000c390 f   moc_ChromaViewPlugin.obj
 0001:0000b3a0       ?registerConverter@?$AssociativeContainerConverterHelper@PAVADVSequenceWidget@U2@@$0A@@QtPrivate@@SA_NH@Z 1000c3a0 f i moc_ChromaViewPlugin.obj
 0001:0000b3b0       ?registerConverter@?$IsPair@PAVADVSequenceWidget@U2@@@QtPrivate@@SA_NH@Z 1000c3b0 f i moc_ChromaViewPlugin.obj
 0001:0000b3c0       ?registerConverter@?$MetaTypeSmartPointerHelper@PAVADVSequenceWidget@U2@@X@QtPrivate@@SA_NH@Z 1000c3c0 f i moc_ChromaViewPlugin.obj
 0001:0000b3d0       ?registerConverter@?$SequentialContainerConverterHelper@PAVADVSequenceWidget@U2@@$0A@@QtPrivate@@SA_NH@Z 1000c3d0 f i moc_ChromaViewPlugin.obj
 0001:0000b3e0       ?storeRelease@?$QBasicAtomicInteger@H@@QAEXH@Z 1000c3e0 f i moc_ChromaViewPlugin.obj
 0001:0000b3f0       ?value@?$MetaObjectForType@PAVADVSequenceWidget@U2@@$00@QtPrivate@@SAPBUQMetaObject@@XZ 1000c3f0 f i moc_ChromaViewPlugin.obj
 0001:0000b400       ??$qMetaTypeId@PAVGObject@U2@@@@YAHXZ 1000c400 f i moc_ChromatogramView.obj
 0001:0000b410       ??$qMetaTypeId@PAVQAction@@@@YAHXZ 1000c410 f i moc_ChromatogramView.obj
 0001:0000b420       ??$qRegisterMetaType@PAVGObject@U2@@@@YAHXZ 1000c420 f i moc_ChromatogramView.obj
 0001:0000b430       ??$qRegisterMetaType@PAVQAction@@@@YAHXZ 1000c430 f i moc_ChromatogramView.obj
 0001:0000b440       ??$qRegisterNormalizedMetaType@PAVGObject@U2@@@@YAHABVQByteArray@@PAPAVGObject@U2@@W4DefinedType@?$MetaTypeDefinedHelper@PAVGObject@U2@@$00@QtPrivate@@@Z 1000c440 f i moc_ChromatogramView.obj
 0001:0000b4a0       ??$qRegisterNormalizedMetaType@PAVQAction@@@@YAHABVQByteArray@@PAPAVQAction@@W4DefinedType@?$MetaTypeDefinedHelper@PAVQAction@@$00@QtPrivate@@@Z 1000c4a0 f i moc_ChromatogramView.obj
 0001:0000b500       ?Construct@?$QMetaTypeFunctionHelper@PAVGObject@U2@@$00@QtMetaTypePrivate@@SAPAXPAXPBX@Z 1000c500 f i moc_ChromatogramView.obj
 0001:0000b530       ?Construct@?$QMetaTypeFunctionHelper@PAVQAction@@$00@QtMetaTypePrivate@@SAPAXPAXPBX@Z 1000c530 f i moc_ChromatogramView.obj
 0001:0000b560       ?Create@?$QMetaTypeFunctionHelper@PAVGObject@U2@@$00@QtMetaTypePrivate@@SAPAXPBX@Z 1000c560 f i moc_ChromatogramView.obj
 0001:0000b5a0       ?Create@?$QMetaTypeFunctionHelper@PAVQAction@@$00@QtMetaTypePrivate@@SAPAXPBX@Z 1000c5a0 f i moc_ChromatogramView.obj
 0001:0000b5e0       ?Delete@?$QMetaTypeFunctionHelper@PAVGObject@U2@@$00@QtMetaTypePrivate@@SAXPAX@Z 1000c5e0 f i moc_ChromatogramView.obj
 0001:0000b5f0       ?Delete@?$QMetaTypeFunctionHelper@PAVQAction@@$00@QtMetaTypePrivate@@SAXPAX@Z 1000c5f0 f i moc_ChromatogramView.obj
 0001:0000b600       ?Destruct@?$QMetaTypeFunctionHelper@PAVGObject@U2@@$00@QtMetaTypePrivate@@SAXPAX@Z 1000c600 f i moc_ChromatogramView.obj
 0001:0000b610       ?Destruct@?$QMetaTypeFunctionHelper@PAVQAction@@$00@QtMetaTypePrivate@@SAXPAX@Z 1000c610 f i moc_ChromatogramView.obj
 0001:0000b620       ?metaObject@ChromatogramView@U2@@UBEPBUQMetaObject@@XZ 1000c620 f   moc_ChromatogramView.obj
 0001:0000b640       ?metaObject@ChromatogramViewRenderArea@U2@@UBEPBUQMetaObject@@XZ 1000c640 f   moc_ChromatogramView.obj
 0001:0000b660       ?qt_metacall@ChromatogramView@U2@@UAEHW4Call@QMetaObject@@HPAPAX@Z 1000c660 f   moc_ChromatogramView.obj
 0001:0000b6c0       ?qt_metacall@ChromatogramViewRenderArea@U2@@UAEHW4Call@QMetaObject@@HPAPAX@Z 1000c6c0 f   moc_ChromatogramView.obj
 0001:0000b6d0       ?qt_metacast@ChromatogramView@U2@@UAEPAXPBD@Z 1000c6d0 f   moc_ChromatogramView.obj
 0001:0000b730       ?qt_metacast@ChromatogramViewRenderArea@U2@@UAEPAXPBD@Z 1000c730 f   moc_ChromatogramView.obj
 0001:0000b790       ?qt_metatype_id@?$QMetaTypeId2@PAVGObject@U2@@@@SAHXZ 1000c790 f i moc_ChromatogramView.obj
 0001:0000b7a0       ?qt_metatype_id@?$QMetaTypeId2@PAVQAction@@@@SAHXZ 1000c7a0 f i moc_ChromatogramView.obj
 0001:0000b7b0       ?qt_metatype_id@?$QMetaTypeIdHelper@PAVGObject@U2@@$00@QtPrivate@@SAHXZ 1000c7b0 f i moc_ChromatogramView.obj
 0001:0000b7c0       ?qt_metatype_id@?$QMetaTypeIdHelper@PAVQAction@@$00@QtPrivate@@SAHXZ 1000c7c0 f i moc_ChromatogramView.obj
 0001:0000b7d0       ?qt_metatype_id@?$QMetaTypeIdQObject@PAVGObject@U2@@$00@@SAHXZ 1000c7d0 f i moc_ChromatogramView.obj
 0001:0000b8b0       ?qt_metatype_id@?$QMetaTypeIdQObject@PAVQAction@@$00@@SAHXZ 1000c8b0 f i moc_ChromatogramView.obj
 0001:0000b990       ?qt_static_metacall@ChromatogramView@U2@@CAXPAVQObject@@W4Call@QMetaObject@@HPAPAX@Z 1000c990 f   moc_ChromatogramView.obj
 0001:0000bac0       ?qt_static_metacall@ChromatogramViewRenderArea@U2@@CAXPAVQObject@@W4Call@QMetaObject@@HPAPAX@Z 1000cac0 f   moc_ChromatogramView.obj
 0001:0000bad0       ?registerConverter@?$AssociativeContainerConverterHelper@PAVGObject@U2@@$0A@@QtPrivate@@SA_NH@Z 1000cad0 f i moc_ChromatogramView.obj
 0001:0000bae0       ?registerConverter@?$AssociativeContainerConverterHelper@PAVQAction@@$0A@@QtPrivate@@SA_NH@Z 1000cae0 f i moc_ChromatogramView.obj
 0001:0000baf0       ?registerConverter@?$IsPair@PAVGObject@U2@@@QtPrivate@@SA_NH@Z 1000caf0 f i moc_ChromatogramView.obj
 0001:0000bb00       ?registerConverter@?$IsPair@PAVQAction@@@QtPrivate@@SA_NH@Z 1000cb00 f i moc_ChromatogramView.obj
 0001:0000bb10       ?registerConverter@?$MetaTypeSmartPointerHelper@PAVGObject@U2@@X@QtPrivate@@SA_NH@Z 1000cb10 f i moc_ChromatogramView.obj
 0001:0000bb20       ?registerConverter@?$MetaTypeSmartPointerHelper@PAVQAction@@X@QtPrivate@@SA_NH@Z 1000cb20 f i moc_ChromatogramView.obj
 0001:0000bb30       ?registerConverter@?$SequentialContainerConverterHelper@PAVGObject@U2@@$0A@@QtPrivate@@SA_NH@Z 1000cb30 f i moc_ChromatogramView.obj
 0001:0000bb40       ?registerConverter@?$SequentialContainerConverterHelper@PAVQAction@@$0A@@QtPrivate@@SA_NH@Z 1000cb40 f i moc_ChromatogramView.obj
 0001:0000bb50       ?value@?$MetaObjectForType@PAVGObject@U2@@$00@QtPrivate@@SAPBUQMetaObject@@XZ 1000cb50 f i moc_ChromatogramView.obj
 0001:0000bb60       ?value@?$MetaObjectForType@PAVQAction@@$00@QtPrivate@@SAPBUQMetaObject@@XZ 1000cb60 f i moc_ChromatogramView.obj
 0001:0000bb70       ??0initializer@?A0xc45d533f@@QAE@XZ 1000cb70 f i qrc_chroma_view.obj
 0001:0000bb90       ??1initializer@?A0xc45d533f@@QAE@XZ 1000cb90 f i qrc_chroma_view.obj
 0001:0000bbb0       ?qCleanupResources_chroma_view@@YAHXZ 1000cbb0 f   qrc_chroma_view.obj
 0001:0000bbd0       ?qInitResources_chroma_view@@YAHXZ 1000cbd0 f   qrc_chroma_view.obj
 0001:0000bbf0       ?getMainWindow@AppContext@U2@@SAPAVMainWindow@2@XZ 1000cbf0 f   U2Core:U2Core.dll
 0001:0000bbf6       ??0Plugin@U2@@QAE@ABVQString@@0_NW4PluginState@1@@Z 1000cbf6 f   U2Core:U2Core.dll
 0001:0000bbfc       ??1Plugin@U2@@UAE@XZ       1000cbfc f   U2Core:U2Core.dll
 0001:0000bc02       ?getChromatogram@DNAChromatogramObject@U2@@QBEABVDNAChromatogram@2@XZ 1000cc02 f   U2Core:U2Core.dll
 0001:0000bc08       ?findAllObjects@GObjectUtils@U2@@SA?AV?$QList@PAVGObject@U2@@@@W4UnloadedObjectFilter@2@VQString@@@Z 1000cc08 f   U2Core:U2Core.dll
 0001:0000bc0e       ?findObjectsRelatedToObjectByRole@GObjectUtils@U2@@SA?AV?$QList@PAVGObject@U2@@@@PBVGObject@2@VQString@@W4GObjectRelationRole@2@ABV3@W4UnloadedObjectFilter@2@@Z 1000cc0e f   U2Core:U2Core.dll
 0001:0000bc14       ??0Logger@U2@@QAE@ABVQString@@@Z 1000cc14 f   U2Core:U2Core.dll
 0001:0000bc1a       ??1Logger@U2@@UAE@XZ       1000cc1a f   U2Core:U2Core.dll
 0001:0000bc20       ??0GObjectReference@U2@@QAE@PBVGObject@1@_N@Z 1000cc20 f   U2Core:U2Core.dll
 0001:0000bc26       ??1GObjectReference@U2@@QAE@XZ 1000cc26 f   U2Core:U2Core.dll
 0001:0000bc2c       ?getGObjectType@GObject@U2@@QBE?AVQString@@XZ 1000cc2c f   U2Core:U2Core.dll
 0001:0000bc32       ??0DNAChromatogram@U2@@QAE@XZ 1000cc32 f   U2Core:U2Core.dll
 0001:0000bc38       ??1DNAChromatogram@U2@@QAE@XZ 1000cc38 f   U2Core:U2Core.dll
 0001:0000bc3e       ??4DNAChromatogram@U2@@QAEAAV01@ABV01@@Z 1000cc3e f   U2Core:U2Core.dll
 0001:0000bc44       ??0DNASequence@U2@@QAE@ABVQByteArray@@PBVDNAAlphabet@1@@Z 1000cc44 f   U2Core:U2Core.dll
 0001:0000bc4a       ??1DNASequence@U2@@QAE@XZ  1000cc4a f   U2Core:U2Core.dll
 0001:0000bc50       ?getSequenceLength@U2SequenceObject@U2@@QBE_JXZ 1000cc50 f   U2Core:U2Core.dll
 0001:0000bc56       ?getWholeSequenceData@U2SequenceObject@U2@@QBE?AVQByteArray@@AAVU2OpStatus@2@@Z 1000cc56 f   U2Core:U2Core.dll
 0001:0000bc5c       ?setWholeSequence@U2SequenceObject@U2@@QAEXABVDNASequence@2@@Z 1000cc5c f   U2Core:U2Core.dll
 0001:0000bc62       ?getAlphabet@U2SequenceObject@U2@@QBEPBVDNAAlphabet@2@XZ 1000cc62 f   U2Core:U2Core.dll
 0001:0000bc68       ?replaceRegion@U2SequenceObject@U2@@QAEXABVU2Region@2@ABVDNASequence@2@AAVU2OpStatus@2@@Z 1000cc68 f   U2Core:U2Core.dll
 0001:0000bc6e       ??0U2SequenceObjectConstraints@U2@@QAE@PAVQObject@@@Z 1000cc6e f   U2Core:U2Core.dll
 0001:0000bc74       ??1U2SequenceObjectConstraints@U2@@UAE@XZ 1000cc74 f   U2Core:U2Core.dll
 0001:0000bc7a       ??0GUrl@U2@@QAE@ABVQString@@@Z 1000cc7a f   U2Core:U2Core.dll
 0001:0000bc80       ??0GUrl@U2@@QAE@ABV01@@Z   1000cc80 f   U2Core:U2Core.dll
 0001:0000bc86       ?dirPath@GUrl@U2@@QBE?AVQString@@XZ 1000cc86 f   U2Core:U2Core.dll
 0001:0000bc8c       ?baseFileName@GUrl@U2@@QBE?AVQString@@XZ 1000cc8c f   U2Core:U2Core.dll
 0001:0000bc92       ??1GUrl@U2@@QAE@XZ         1000cc92 f   U2Core:U2Core.dll
 0001:0000bc98       ?addObject@Document@U2@@QAEXPAVGObject@2@@Z 1000cc98 f   U2Core:U2Core.dll
 0001:0000bc9e       ?getDbiRef@Document@U2@@QBEABVU2DbiRef@2@XZ 1000cc9e f   U2Core:U2Core.dll
 0001:0000bca4       ?getNewDocFileNameExcludesHint@DocumentUtils@U2@@SA?AV?$QSet@VQString@@@@XZ 1000cca4 f   U2Core:U2Core.dll
 0001:0000bcaa       ?selectObjectByReference@GObjectUtils@U2@@SAPAVGObject@2@ABVGObjectReference@2@ABV?$QList@PAVGObject@U2@@@@W4UnloadedObjectFilter@2@@Z 1000ccaa f   U2Core:U2Core.dll
 0001:0000bcb0       ?rollFileName@GUrlUtils@U2@@SA?AVQString@@ABV3@ABV?$QSet@VQString@@@@@Z 1000ccb0 f   U2Core:U2Core.dll
 0001:0000bcb6       ?errorTitle@L10N@U2@@SA?AVQString@@XZ 1000ccb6 f   U2Core:U2Core.dll
 0001:0000bcbc       ?error@Logger@U2@@QAEXABVQString@@@Z 1000ccbc f   U2Core:U2Core.dll
 0001:0000bcc2       ?isCoR@U2OpStatus@U2@@UBE_NXZ 1000ccc2 f   U2Core:U2Core.dll
 0001:0000bcc8       ??0LoadDocumentTaskConfig@U2@@QAE@_NABVGObjectReference@1@PAVLDTObjectFactory@1@@Z 1000ccc8 f   U2Core:U2Core.dll
 0001:0000bcce       ??1LoadDocumentTaskConfig@U2@@QAE@XZ 1000ccce f   U2Core:U2Core.dll
 0001:0000bcd4       ??0LoadUnloadedDocumentTask@U2@@QAE@PAVDocument@1@ABVLoadDocumentTaskConfig@1@@Z 1000ccd4 f   U2Core:U2Core.dll
 0001:0000bcda       ??1LoadUnloadedDocumentTask@U2@@UAE@XZ 1000ccda f   U2Core:U2Core.dll
 0001:0000bce0       ??0TaskSignalMapper@U2@@QAE@PAVTask@1@@Z 1000cce0 f   U2Core:U2Core.dll
 0001:0000bce6       ??0U2OpStatusImpl@U2@@QAE@XZ 1000cce6 f   U2Core:U2Core.dll
 0001:0000bcec       ?getError@U2OpStatusImpl@U2@@UBE?AVQString@@XZ 1000ccec f   U2Core:U2Core.dll
 0001:0000bcf2       ??1U2OpStatusImpl@U2@@UAE@XZ 1000ccf2 f   U2Core:U2Core.dll
 0001:0000bcf8       ??0U2OpStatus2Log@U2@@QAE@W4LogLevel@1@@Z 1000ccf8 f   U2Core:U2Core.dll
 0001:0000bcfe       ??1U2OpStatus2Log@U2@@UAE@XZ 1000ccfe f   U2Core:U2Core.dll
 0001:0000bd04       ??0ProjectTreeControllerModeSettings@U2@@QAE@XZ 1000cd04 f   U2Core:U2Core.dll
 0001:0000bd0a       ??1ProjectTreeControllerModeSettings@U2@@QAE@XZ 1000cd0a f   U2Core:U2Core.dll
 0001:0000bd10       ?getProject@AppContext@U2@@SAPAVProject@2@XZ 1000cd10 f   U2Core:U2Core.dll
 0001:0000bd16       ?getDocumentFormatRegistry@AppContext@U2@@SAPAVDocumentFormatRegistry@2@XZ 1000cd16 f   U2Core:U2Core.dll
 0001:0000bd1c       ?getIOAdapterRegistry@AppContext@U2@@SAPAVIOAdapterRegistry@2@XZ 1000cd1c f   U2Core:U2Core.dll
 0001:0000bd22       ?getTaskScheduler@AppContext@U2@@SAPAVTaskScheduler@2@XZ 1000cd22 f   U2Core:U2Core.dll
 0001:0000bd28       ?cleanup@DocumentProviderTask@U2@@UAEXXZ 1000cd28 f   U2Core:U2Core.dll
 0001:0000bd2e       ?generateReport@Task@U2@@UBE?AVQString@@XZ 1000cd2e f   U2Core:U2Core.dll
 0001:0000bd34       ?getDocument@LoadUnloadedDocumentTask@U2@@UAEPAVDocument@2@_N@Z 1000cd34 f   U2Core:U2Core.dll
 0001:0000bd3a       ?getDocumentDescription@DocumentProviderTask@U2@@UBE?AVQString@@XZ 1000cd3a f   U2Core:U2Core.dll
 0001:0000bd40       ?getNumParallelSubtasks@Task@U2@@UBEHXZ 1000cd40 f   U2Core:U2Core.dll
 0001:0000bd46       ?getParentTask@Task@U2@@UBEPAV12@XZ 1000cd46 f   U2Core:U2Core.dll
 0001:0000bd4c       ?getSubtaskWithErrors@Task@U2@@UBEPAV12@XZ 1000cd4c f   U2Core:U2Core.dll
 0001:0000bd52       ?getTaskId@Task@U2@@UBE_JXZ 1000cd52 f   U2Core:U2Core.dll
 0001:0000bd58       ?getTopLevelParentTask@Task@U2@@UAEPAV12@XZ 1000cd58 f   U2Core:U2Core.dll
 0001:0000bd5e       ?getWarnings@Task@U2@@UBE?AVQStringList@@XZ 1000cd5e f   U2Core:U2Core.dll
 0001:0000bd64       ?hasSubtasksWithErrors@Task@U2@@UBE_NXZ 1000cd64 f   U2Core:U2Core.dll
 0001:0000bd6a       ?hasWarning@Task@U2@@UBE_NXZ 1000cd6a f   U2Core:U2Core.dll
 0001:0000bd70       ?isNotificationReport@Task@U2@@UBE_NXZ 1000cd70 f   U2Core:U2Core.dll
 0001:0000bd76       ?isReportingEnabled@Task@U2@@UBE_NXZ 1000cd76 f   U2Core:U2Core.dll
 0001:0000bd7c       ?isReportingSupported@Task@U2@@UBE_NXZ 1000cd7c f   U2Core:U2Core.dll
 0001:0000bd82       ?isTopLevelTask@Task@U2@@UBE_NXZ 1000cd82 f   U2Core:U2Core.dll
 0001:0000bd88       ?metaObject@LoadUnloadedDocumentTask@U2@@UBEPBUQMetaObject@@XZ 1000cd88 f   U2Core:U2Core.dll
 0001:0000bd8e       ?metaObject@TaskSignalMapper@U2@@UBEPBUQMetaObject@@XZ 1000cd8e f   U2Core:U2Core.dll
 0001:0000bd94       ?onSubTaskFinished@Task@U2@@MAE?AV?$QList@PAVTask@U2@@@@PAV12@@Z 1000cd94 f   U2Core:U2Core.dll
 0001:0000bd9a       ?prepare@LoadUnloadedDocumentTask@U2@@UAEXXZ 1000cd9a f   U2Core:U2Core.dll
 0001:0000bda0       ?propagateSubtaskError@Task@U2@@UAE_NXZ 1000cda0 f   U2Core:U2Core.dll
 0001:0000bda6       ?qt_metacall@LoadUnloadedDocumentTask@U2@@UAEHW4Call@QMetaObject@@HPAPAX@Z 1000cda6 f   U2Core:U2Core.dll
 0001:0000bdac       ?qt_metacall@TaskSignalMapper@U2@@UAEHW4Call@QMetaObject@@HPAPAX@Z 1000cdac f   U2Core:U2Core.dll
 0001:0000bdb2       ?qt_metacast@LoadUnloadedDocumentTask@U2@@UAEPAXPBD@Z 1000cdb2 f   U2Core:U2Core.dll
 0001:0000bdb8       ?qt_metacast@TaskSignalMapper@U2@@UAEPAXPBD@Z 1000cdb8 f   U2Core:U2Core.dll
 0001:0000bdbe       ?report@LoadUnloadedDocumentTask@U2@@UAE?AW4ReportResult@Task@2@XZ 1000cdbe f   U2Core:U2Core.dll
 0001:0000bdc4       ?run@Task@U2@@UAEXXZ       1000cdc4 f   U2Core:U2Core.dll
 0001:0000bdca       ?setCollectChildrensWarningsFlag@Task@U2@@UAEX_N@Z 1000cdca f   U2Core:U2Core.dll
 0001:0000bdd0       ?setNoAutoDelete@Task@U2@@UAEX_N@Z 1000cdd0 f   U2Core:U2Core.dll
 0001:0000bdd6       ?setNotificationReport@Task@U2@@UAEX_N@Z 1000cdd6 f   U2Core:U2Core.dll
 0001:0000bddc       ?setReportingEnabled@Task@U2@@UAEX_N@Z 1000cddc f   U2Core:U2Core.dll
 0001:0000bde2       ?setReportingSupported@Task@U2@@UAEX_N@Z 1000cde2 f   U2Core:U2Core.dll
 0001:0000bde8       ?takeDocument@DocumentProviderTask@U2@@UAEPAVDocument@2@_N@Z 1000cde8 f   U2Core:U2Core.dll
 0001:0000bdee       ?qt_metacast@Plugin@U2@@UAEPAXPBD@Z 1000cdee f   U2Core:U2Core.dll
 0001:0000bdf4       ?qt_metacall@Plugin@U2@@UAEHW4Call@QMetaObject@@HPAPAX@Z 1000cdf4 f   U2Core:U2Core.dll
 0001:0000bdfa       ??0GObjectViewWindowContext@U2@@QAE@PAVQObject@@ABVGObjectViewFactoryId@1@@Z 1000cdfa f   U2Gui:U2Gui.dll
 0001:0000be00       ??1GObjectViewWindowContext@U2@@UAE@XZ 1000ce00 f   U2Gui:U2Gui.dll
 0001:0000be06       ?buildMenu@GObjectViewWindowContext@U2@@MAEXPAVGObjectView@2@PAVQMenu@@@Z 1000ce06 f   U2Gui:U2Gui.dll
 0001:0000be0c       ?disconnectView@GObjectViewWindowContext@U2@@MAEXPAVGObjectView@2@@Z 1000ce0c f   U2Gui:U2Gui.dll
 0001:0000be12       ?init@GObjectViewWindowContext@U2@@UAEXXZ 1000ce12 f   U2Gui:U2Gui.dll
 0001:0000be18       ?onObjectAdded@GObjectViewObjectHandler@U2@@UAEXPAVGObjectView@2@PAVGObject@2@@Z 1000ce18 f   U2Gui:U2Gui.dll
 0001:0000be1e       ?onObjectRemoved@GObjectViewWindowContext@U2@@UAEXPAVGObjectView@2@PAVGObject@2@@Z 1000ce1e f   U2Gui:U2Gui.dll
 0001:0000be24       ?sl_buildContextMenu@GObjectViewWindowContext@U2@@MAEXPAVGObjectView@2@PAVQMenu@@@Z 1000ce24 f   U2Gui:U2Gui.dll
 0001:0000be2a       ?sl_buildStaticMenu@GObjectViewWindowContext@U2@@MAEXPAVGObjectView@2@PAVQMenu@@@Z 1000ce2a f   U2Gui:U2Gui.dll
 0001:0000be30       ?sl_windowAdded@GObjectViewWindowContext@U2@@MAEXPAVMWMDIWindow@2@@Z 1000ce30 f   U2Gui:U2Gui.dll
 0001:0000be36       ?sl_windowClosing@GObjectViewWindowContext@U2@@MAEXPAVMWMDIWindow@2@@Z 1000ce36 f   U2Gui:U2Gui.dll
 0001:0000be3c       ??0AddNewDocumentDialogModel@U2@@QAE@ABVQString@@V2@@Z 1000ce3c f   U2Gui:U2Gui.dll
 0001:0000be42       ??1AddNewDocumentDialogModel@U2@@QAE@XZ 1000ce42 f   U2Gui:U2Gui.dll
 0001:0000be48       ?run@AddNewDocumentDialogController@U2@@SAXPAVQWidget@@AAVAddNewDocumentDialogModel@2@ABVDocumentFormatConstraints@2@@Z 1000ce48 f   U2Gui:U2Gui.dll
 0001:0000be4e       ?findActionAfter@GUIUtils@U2@@SAPAVQAction@@ABV?$QList@PAVQAction@@@@ABVQString@@@Z 1000ce4e f   U2Gui:U2Gui.dll
 0001:0000be54       ?selectObjects@ProjectTreeItemSelectorDialog@U2@@SA?AV?$QList@PAVGObject@U2@@@@ABVProjectTreeControllerModeSettings@2@PAVQWidget@@@Z 1000ce54 f   U2Gui:U2Gui.dll
 0001:0000be5a       ?setContentLayout@WidgetWithLocalToolbar@U2@@QAEXPAVQLayout@@@Z 1000ce5a f   U2Gui:U2Gui.dll
 0001:0000be60       ?addActionToLocalToolbar@WidgetWithLocalToolbar@U2@@QAEPAVQToolButton@@PAVQAction@@@Z 1000ce60 f   U2Gui:U2Gui.dll
 0001:0000be66       ??0ScaleBar@U2@@QAE@W4Orientation@Qt@@PAVQWidget@@@Z 1000ce66 f   U2Gui:U2Gui.dll
 0001:0000be6c       ?setValue@ScaleBar@U2@@QAEXH@Z 1000ce6c f   U2Gui:U2Gui.dll
 0001:0000be72       ?setRange@ScaleBar@U2@@QAEXHH@Z 1000ce72 f   U2Gui:U2Gui.dll
 0001:0000be78       ?setTickInterval@ScaleBar@U2@@QAEXH@Z 1000ce78 f   U2Gui:U2Gui.dll
 0001:0000be7e       ?metaObject@ScaleBar@U2@@UBEPBUQMetaObject@@XZ 1000ce7e f   U2Gui:U2Gui.dll
 0001:0000be84       ?qt_metacall@ScaleBar@U2@@UAEHW4Call@QMetaObject@@HPAPAX@Z 1000ce84 f   U2Gui:U2Gui.dll
 0001:0000be8a       ?qt_metacast@ScaleBar@U2@@UAEPAXPBD@Z 1000ce8a f   U2Gui:U2Gui.dll
 0001:0000be90       ?qt_metacast@GObjectViewWindowContext@U2@@UAEPAXPBD@Z 1000ce90 f   U2Gui:U2Gui.dll
 0001:0000be96       ?qt_metacall@GObjectViewWindowContext@U2@@UAEHW4Call@QMetaObject@@HPAPAX@Z 1000ce96 f   U2Gui:U2Gui.dll
 0001:0000be9c       ??0ADVSequenceWidgetAction@U2@@QAE@ABVQString@@0@Z 1000ce9c f   U2View:U2View.dll
 0001:0000bea2       ??1ADVSequenceWidgetAction@U2@@UAE@XZ 1000cea2 f   U2View:U2View.dll
 0001:0000bea8       ?getSequenceWidgets@AnnotatedDNAView@U2@@QBE?BV?$QList@PAVADVSequenceWidget@U2@@@@XZ 1000cea8 f   U2View:U2View.dll
 0001:0000beae       ?getPanGSLView@ADVSingleSequenceWidget@U2@@QBEPAVGSequenceLineView@2@XZ 1000ceae f   U2View:U2View.dll
 0001:0000beb4       ?getSequenceContext@ADVSingleSequenceWidget@U2@@QBEPAVADVSequenceObjectContext@2@XZ 1000ceb4 f   U2View:U2View.dll
 0001:0000beba       ?getSequenceObject@ADVSingleSequenceWidget@U2@@QBEPAVU2SequenceObject@2@XZ 1000ceba f   U2View:U2View.dll
 0001:0000bec0       ?addADVSequenceWidgetActionToViewsToolbar@ADVSingleSequenceWidget@U2@@QAEXPAVADVSequenceWidgetAction@2@@Z 1000cec0 f   U2View:U2View.dll
 0001:0000bec6       ?getSequenceGObject@SequenceObjectContext@U2@@QBEPAVGObject@2@XZ 1000cec6 f   U2View:U2View.dll
 0001:0000becc       ?getSequenceLength@SequenceObjectContext@U2@@QBE_JXZ 1000cecc f   U2View:U2View.dll
 0001:0000bed2       ?getSequenceData@SequenceObjectContext@U2@@QBE?AVQByteArray@@ABVU2Region@2@AAVU2OpStatus@2@@Z 1000ced2 f   U2View:U2View.dll
 0001:0000bed8       ??0GSequenceLineView@U2@@QAE@PAVQWidget@@PAVSequenceObjectContext@1@@Z 1000ced8 f   U2View:U2View.dll
 0001:0000bede       ?setCoherentRangeView@GSequenceLineView@U2@@UAEXPAV12@@Z 1000cede f   U2View:U2View.dll
 0001:0000bee4       ?mousePressEvent@GSequenceLineView@U2@@MAEXPAVQMouseEvent@@@Z 1000cee4 f   U2View:U2View.dll
 0001:0000beea       ?completeUpdate@GSequenceLineView@U2@@IAEXXZ 1000ceea f   U2View:U2View.dll
 0001:0000bef0       ?toRenderAreaPoint@GSequenceLineView@U2@@IBE?AVQPoint@@ABV3@@Z 1000cef0 f   U2View:U2View.dll
 0001:0000bef6       ??1GSequenceLineView@U2@@UAE@XZ 1000cef6 f   U2View:U2View.dll
 0001:0000befc       ??0GSequenceLineViewRenderArea@U2@@QAE@PAVGSequenceLineView@1@@Z 1000cefc f   U2View:U2View.dll
 0001:0000bf02       ??1GSequenceLineViewRenderArea@U2@@UAE@XZ 1000cf02 f   U2View:U2View.dll
 0001:0000bf08       ?addUpdateFlags@GSequenceLineView@U2@@UAEXV?$QFlags@W4GSLV_UpdateFlag@U2@@@@@Z 1000cf08 f   U2View:U2View.dll
 0001:0000bf0e       ?clearUpdateFlags@GSequenceLineView@U2@@UAEXXZ 1000cf0e f   U2View:U2View.dll
 0001:0000bf14       ?coordToPos@GSequenceLineViewRenderArea@U2@@UBE_JABVQPoint@@@Z 1000cf14 f   U2View:U2View.dll
 0001:0000bf1a       ?drawFocus@GSequenceLineViewRenderArea@U2@@MAEXAAVQPainter@@@Z 1000cf1a f   U2View:U2View.dll
 0001:0000bf20       ?eventFilter@GSequenceLineView@U2@@UAE_NPAVQObject@@PAVQEvent@@@Z 1000cf20 f   U2View:U2View.dll
 0001:0000bf26       ?focusInEvent@GSequenceLineView@U2@@MAEXPAVQFocusEvent@@@Z 1000cf26 f   U2View:U2View.dll
 0001:0000bf2c       ?focusOutEvent@GSequenceLineView@U2@@MAEXPAVQFocusEvent@@@Z 1000cf2c f   U2View:U2View.dll
 0001:0000bf32       ?getConherentRangeView@GSequenceLineView@U2@@UBEPAV12@XZ 1000cf32 f   U2View:U2View.dll
 0001:0000bf38       ?getCurrentScale@GSequenceLineViewRenderArea@U2@@UBENXZ 1000cf38 f   U2View:U2View.dll
 0001:0000bf3e       ?getFrameView@GSequenceLineView@U2@@UBEPAV12@XZ 1000cf3e f   U2View:U2View.dll
 0001:0000bf44       ?getPageStep@GSequenceLineView@U2@@MBEHXZ 1000cf44 f   U2View:U2View.dll
 0001:0000bf4a       ?getSequenceObject@GSequenceLineView@U2@@UBEPAVU2SequenceObject@2@XZ 1000cf4a f   U2View:U2View.dll
 0001:0000bf50       ?getSingleStep@GSequenceLineView@U2@@MBEHXZ 1000cf50 f   U2View:U2View.dll
 0001:0000bf56       ?getZoomInAction@GSequenceLineView@U2@@UBEPAVQAction@@XZ 1000cf56 f   U2View:U2View.dll
 0001:0000bf5c       ?getZoomOutAction@GSequenceLineView@U2@@UBEPAVQAction@@XZ 1000cf5c f   U2View:U2View.dll
 0001:0000bf62       ?getZoomToSelectionAction@GSequenceLineView@U2@@UBEPAVQAction@@XZ 1000cf62 f   U2View:U2View.dll
 0001:0000bf68       ?getZoomToSequenceAction@GSequenceLineView@U2@@UBEPAVQAction@@XZ 1000cf68 f   U2View:U2View.dll
 0001:0000bf6e       ?keyPressEvent@GSequenceLineView@U2@@MAEXPAVQKeyEvent@@@Z 1000cf6e f   U2View:U2View.dll
 0001:0000bf74       ?mouseDoubleClickEvent@GSequenceLineView@U2@@MAEXPAVQMouseEvent@@@Z 1000cf74 f   U2View:U2View.dll
 0001:0000bf7a       ?mouseMoveEvent@GSequenceLineView@U2@@MAEXPAVQMouseEvent@@@Z 1000cf7a f   U2View:U2View.dll
 0001:0000bf80       ?mouseReleaseEvent@GSequenceLineView@U2@@MAEXPAVQMouseEvent@@@Z 1000cf80 f   U2View:U2View.dll
 0001:0000bf86       ?moveBorder@GSequenceLineView@U2@@MAEXABVQPoint@@@Z 1000cf86 f   U2View:U2View.dll
 0001:0000bf8c       ?onVisibleRangeChanged@GSequenceLineView@U2@@MAEX_N@Z 1000cf8c f   U2View:U2View.dll
 0001:0000bf92       ?paintEvent@GSequenceLineViewRenderArea@U2@@MAEXPAVQPaintEvent@@@Z 1000cf92 f   U2View:U2View.dll
 0001:0000bf98       ?posToCoordF@GSequenceLineViewRenderArea@U2@@UBEM_J_N@Z 1000cf98 f   U2View:U2View.dll
 0001:0000bf9e       ?resizeEvent@GSequenceLineView@U2@@MAEXPAVQResizeEvent@@@Z 1000cf9e f   U2View:U2View.dll
 0001:0000bfa4       ?resizeSelection@GSequenceLineView@U2@@MAEXABVQPoint@@@Z 1000cfa4 f   U2View:U2View.dll
 0001:0000bfaa       ?setBorderCursor@GSequenceLineView@U2@@MAEXABVQPoint@@@Z 1000cfaa f   U2View:U2View.dll
 0001:0000bfb0       ?setCenterPos@GSequenceLineView@U2@@UAEX_J@Z 1000cfb0 f   U2View:U2View.dll
 0001:0000bfb6       ?setFrameView@GSequenceLineView@U2@@UAEXPAV12@@Z 1000cfb6 f   U2View:U2View.dll
 0001:0000bfbc       ?setStartPos@GSequenceLineView@U2@@UAEX_J@Z 1000cfbc f   U2View:U2View.dll
 0001:0000bfc2       ?setVisibleRange@GSequenceLineView@U2@@UAEXABVU2Region@2@_N@Z 1000cfc2 f   U2View:U2View.dll
 0001:0000bfc8       ?sl_onDNASelectionChanged@GSequenceLineView@U2@@MAEXPAVLRegionsSelection@2@ABV?$QVector@VU2Region@U2@@@@1@Z 1000cfc8 f   U2View:U2View.dll
 0001:0000bfce       ?sl_onScrollBarMoved@GSequenceLineView@U2@@MAEXH@Z 1000cfce f   U2View:U2View.dll
 0001:0000bfd4       ?sl_sequenceChanged@GSequenceLineView@U2@@MAEXXZ 1000cfd4 f   U2View:U2View.dll
 0001:0000bfda       ?updateScrollBar@GSequenceLineView@U2@@MAEXXZ 1000cfda f   U2View:U2View.dll
 0001:0000bfe0       ?wheelEvent@GSequenceLineView@U2@@MAEXPAVQWheelEvent@@@Z 1000cfe0 f   U2View:U2View.dll
 0001:0000bfe6       ?qt_metacast@ADVSequenceWidgetAction@U2@@UAEPAXPBD@Z 1000cfe6 f   U2View:U2View.dll
 0001:0000bfec       ?qt_metacall@ADVSequenceWidgetAction@U2@@UAEHW4Call@QMetaObject@@HPAPAX@Z 1000cfec f   U2View:U2View.dll
 0001:0000bff2       ?qt_metacast@GSequenceLineView@U2@@UAEPAXPBD@Z 1000cff2 f   U2View:U2View.dll
 0001:0000bff8       ?qt_metacall@GSequenceLineView@U2@@UAEHW4Call@QMetaObject@@HPAPAX@Z 1000cff8 f   U2View:U2View.dll
 0001:0000bffe       ?setIcon@QAction@@QAEXABVQIcon@@@Z 1000cffe f   Qt5Widgets:Qt5Widgets.dll
 0001:0000c004       ?setCheckable@QAction@@QAEX_N@Z 1000d004 f   Qt5Widgets:Qt5Widgets.dll
 0001:0000c00a       ?isChecked@QAction@@QBE_NXZ 1000d00a f   Qt5Widgets:Qt5Widgets.dll
 0001:0000c010       ?activate@QAction@@QAEXW4ActionEvent@1@@Z 1000d010 f   Qt5Widgets:Qt5Widgets.dll
 0001:0000c016       ?setChecked@QAction@@QAEX_N@Z 1000d016 f   Qt5Widgets:Qt5Widgets.dll
 0001:0000c01c       ?event@QAction@@MAE_NPAVQEvent@@@Z 1000d01c f   Qt5Widgets:Qt5Widgets.dll
 0001:0000c022       ??1QWidget@@UAE@XZ         1000d022 f   Qt5Widgets:Qt5Widgets.dll
 0001:0000c028       ?rect@QWidget@@QBE?AVQRect@@XZ 1000d028 f   Qt5Widgets:Qt5Widgets.dll
 0001:0000c02e       ?minimumSize@QWidget@@QBE?AVQSize@@XZ 1000d02e f   Qt5Widgets:Qt5Widgets.dll
 0001:0000c034       ?setMinimumHeight@QWidget@@QAEXH@Z 1000d034 f   Qt5Widgets:Qt5Widgets.dll
 0001:0000c03a       ?mapToGlobal@QWidget@@QBE?AVQPoint@@ABV2@@Z 1000d03a f   Qt5Widgets:Qt5Widgets.dll
 0001:0000c040       ?mapFromGlobal@QWidget@@QBE?AVQPoint@@ABV2@@Z 1000d040 f   Qt5Widgets:Qt5Widgets.dll
 0001:0000c046       ?setFocus@QWidget@@QAEXW4FocusReason@Qt@@@Z 1000d046 f   Qt5Widgets:Qt5Widgets.dll
 0001:0000c04c       ?update@QWidget@@QAEXXZ    1000d04c f   Qt5Widgets:Qt5Widgets.dll
 0001:0000c052       ?setHidden@QWidget@@QAEX_N@Z 1000d052 f   Qt5Widgets:Qt5Widgets.dll
 0001:0000c058       ?addAction@QWidget@@QAEXPAVQAction@@@Z 1000d058 f   Qt5Widgets:Qt5Widgets.dll
 0001:0000c05e       ?insertAction@QWidget@@QAEXPAVQAction@@0@Z 1000d05e f   Qt5Widgets:Qt5Widgets.dll
 0001:0000c064       ?actions@QWidget@@QBE?AV?$QList@PAVQAction@@@@XZ 1000d064 f   Qt5Widgets:Qt5Widgets.dll
 0001:0000c06a       ?critical@QMessageBox@@SA?AW4StandardButton@1@PAVQWidget@@ABVQString@@1V?$QFlags@W4StandardButton@QMessageBox@@@@W421@@Z 1000d06a f   Qt5Widgets:Qt5Widgets.dll
 0001:0000c070       ??0QAction@@QAE@ABVQString@@PAVQObject@@@Z 1000d070 f   Qt5Widgets:Qt5Widgets.dll
 0001:0000c076       ??1QAction@@UAE@XZ         1000d076 f   Qt5Widgets:Qt5Widgets.dll
 0001:0000c07c       ?text@QAction@@QBE?AVQString@@XZ 1000d07c f   Qt5Widgets:Qt5Widgets.dll
 0001:0000c082       ?setEnabled@QAction@@QAEX_N@Z 1000d082 f   Qt5Widgets:Qt5Widgets.dll
 0001:0000c088       ??0QMenu@@QAE@PAVQWidget@@@Z 1000d088 f   Qt5Widgets:Qt5Widgets.dll
 0001:0000c08e       ??0QMenu@@QAE@ABVQString@@PAVQWidget@@@Z 1000d08e f   Qt5Widgets:Qt5Widgets.dll
 0001:0000c094       ??1QMenu@@UAE@XZ           1000d094 f   Qt5Widgets:Qt5Widgets.dll
 0001:0000c09a       ?addAction@QMenu@@QAEPAVQAction@@ABVQString@@@Z 1000d09a f   Qt5Widgets:Qt5Widgets.dll
 0001:0000c0a0       ?addSeparator@QMenu@@QAEPAVQAction@@XZ 1000d0a0 f   Qt5Widgets:Qt5Widgets.dll
 0001:0000c0a6       ?insertMenu@QMenu@@QAEPAVQAction@@PAV2@PAV1@@Z 1000d0a6 f   Qt5Widgets:Qt5Widgets.dll
 0001:0000c0ac       ?insertSeparator@QMenu@@QAEPAVQAction@@PAV2@@Z 1000d0ac f   Qt5Widgets:Qt5Widgets.dll
 0001:0000c0b2       ?popup@QMenu@@QAEXABVQPoint@@PAVQAction@@@Z 1000d0b2 f   Qt5Widgets:Qt5Widgets.dll
 0001:0000c0b8       ?menuAction@QMenu@@QBEPAVQAction@@XZ 1000d0b8 f   Qt5Widgets:Qt5Widgets.dll
 0001:0000c0be       ?setIcon@QAbstractButton@@QAEXABVQIcon@@@Z 1000d0be f   Qt5Widgets:Qt5Widgets.dll
 0001:0000c0c4       ?setPopupMode@QToolButton@@QAEXW4ToolButtonPopupMode@1@@Z 1000d0c4 f   Qt5Widgets:Qt5Widgets.dll
 0001:0000c0ca       ?setMargin@QLayout@@QAEXH@Z 1000d0ca f   Qt5Widgets:Qt5Widgets.dll
 0001:0000c0d0       ?addWidget@QBoxLayout@@QAEXPAVQWidget@@HV?$QFlags@W4AlignmentFlag@Qt@@@@@Z 1000d0d0 f   Qt5Widgets:Qt5Widgets.dll
 0001:0000c0d6       ??0QHBoxLayout@@QAE@XZ     1000d0d6 f   Qt5Widgets:Qt5Widgets.dll
 0001:0000c0dc       ??1QHBoxLayout@@UAE@XZ     1000d0dc f   Qt5Widgets:Qt5Widgets.dll
 0001:0000c0e2       ?actionEvent@QMenu@@MAEXPAVQActionEvent@@@Z 1000d0e2 f   Qt5Widgets:Qt5Widgets.dll
 0001:0000c0e8       ?actionEvent@QWidget@@MAEXPAVQActionEvent@@@Z 1000d0e8 f   Qt5Widgets:Qt5Widgets.dll
 0001:0000c0ee       ?addItem@QBoxLayout@@UAEXPAVQLayoutItem@@@Z 1000d0ee f   Qt5Widgets:Qt5Widgets.dll
 0001:0000c0f4       ?changeEvent@QMenu@@MAEXPAVQEvent@@@Z 1000d0f4 f   Qt5Widgets:Qt5Widgets.dll
 0001:0000c0fa       ?changeEvent@QWidget@@MAEXPAVQEvent@@@Z 1000d0fa f   Qt5Widgets:Qt5Widgets.dll
 0001:0000c100       ?childEvent@QLayout@@MAEXPAVQChildEvent@@@Z 1000d100 f   Qt5Widgets:Qt5Widgets.dll
 0001:0000c106       ?closeEvent@QWidget@@MAEXPAVQCloseEvent@@@Z 1000d106 f   Qt5Widgets:Qt5Widgets.dll
 0001:0000c10c       ?contextMenuEvent@QWidget@@MAEXPAVQContextMenuEvent@@@Z 1000d10c f   Qt5Widgets:Qt5Widgets.dll
 0001:0000c112       ?controlTypes@QLayout@@UBE?AV?$QFlags@W4ControlType@QSizePolicy@@@@XZ 1000d112 f   Qt5Widgets:Qt5Widgets.dll
 0001:0000c118       ?count@QBoxLayout@@UBEHXZ  1000d118 f   Qt5Widgets:Qt5Widgets.dll
 0001:0000c11e       ?devType@QWidget@@UBEHXZ   1000d11e f   Qt5Widgets:Qt5Widgets.dll
 0001:0000c124       ?dragEnterEvent@QWidget@@MAEXPAVQDragEnterEvent@@@Z 1000d124 f   Qt5Widgets:Qt5Widgets.dll
 0001:0000c12a       ?dragLeaveEvent@QWidget@@MAEXPAVQDragLeaveEvent@@@Z 1000d12a f   Qt5Widgets:Qt5Widgets.dll
 0001:0000c130       ?dragMoveEvent@QWidget@@MAEXPAVQDragMoveEvent@@@Z 1000d130 f   Qt5Widgets:Qt5Widgets.dll
 0001:0000c136       ?dropEvent@QWidget@@MAEXPAVQDropEvent@@@Z 1000d136 f   Qt5Widgets:Qt5Widgets.dll
 0001:0000c13c       ?enterEvent@QMenu@@MAEXPAVQEvent@@@Z 1000d13c f   Qt5Widgets:Qt5Widgets.dll
 0001:0000c142       ?enterEvent@QWidget@@MAEXPAVQEvent@@@Z 1000d142 f   Qt5Widgets:Qt5Widgets.dll
 0001:0000c148       ?event@QMenu@@MAE_NPAVQEvent@@@Z 1000d148 f   Qt5Widgets:Qt5Widgets.dll
 0001:0000c14e       ?event@QWidget@@MAE_NPAVQEvent@@@Z 1000d14e f   Qt5Widgets:Qt5Widgets.dll
 0001:0000c154       ?expandingDirections@QBoxLayout@@UBE?AV?$QFlags@W4Orientation@Qt@@@@XZ 1000d154 f   Qt5Widgets:Qt5Widgets.dll
 0001:0000c15a       ?focusInEvent@QWidget@@MAEXPAVQFocusEvent@@@Z 1000d15a f   Qt5Widgets:Qt5Widgets.dll
 0001:0000c160       ?focusNextPrevChild@QMenu@@MAE_N_N@Z 1000d160 f   Qt5Widgets:Qt5Widgets.dll
 0001:0000c166       ?focusNextPrevChild@QWidget@@MAE_N_N@Z 1000d166 f   Qt5Widgets:Qt5Widgets.dll
 0001:0000c16c       ?focusOutEvent@QWidget@@MAEXPAVQFocusEvent@@@Z 1000d16c f   Qt5Widgets:Qt5Widgets.dll
 0001:0000c172       ?geometry@QLayout@@UBE?AVQRect@@XZ 1000d172 f   Qt5Widgets:Qt5Widgets.dll
 0001:0000c178       ?hasHeightForWidth@QBoxLayout@@UBE_NXZ 1000d178 f   Qt5Widgets:Qt5Widgets.dll
 0001:0000c17e       ?hasHeightForWidth@QWidget@@UBE_NXZ 1000d17e f   Qt5Widgets:Qt5Widgets.dll
 0001:0000c184       ?heightForWidth@QBoxLayout@@UBEHH@Z 1000d184 f   Qt5Widgets:Qt5Widgets.dll
 0001:0000c18a       ?heightForWidth@QWidget@@UBEHH@Z 1000d18a f   Qt5Widgets:Qt5Widgets.dll
 0001:0000c190       ?hideEvent@QMenu@@MAEXPAVQHideEvent@@@Z 1000d190 f   Qt5Widgets:Qt5Widgets.dll
 0001:0000c196       ?hideEvent@QWidget@@MAEXPAVQHideEvent@@@Z 1000d196 f   Qt5Widgets:Qt5Widgets.dll
 0001:0000c19c       ?indexOf@QLayout@@UBEHPAVQWidget@@@Z 1000d19c f   Qt5Widgets:Qt5Widgets.dll
 0001:0000c1a2       ?initPainter@QWidget@@MBEXPAVQPainter@@@Z 1000d1a2 f   Qt5Widgets:Qt5Widgets.dll
 0001:0000c1a8       ?inputMethodEvent@QWidget@@MAEXPAVQInputMethodEvent@@@Z 1000d1a8 f   Qt5Widgets:Qt5Widgets.dll
 0001:0000c1ae       ?inputMethodQuery@QWidget@@UBE?AVQVariant@@W4InputMethodQuery@Qt@@@Z 1000d1ae f   Qt5Widgets:Qt5Widgets.dll
 0001:0000c1b4       ?invalidate@QBoxLayout@@UAEXXZ 1000d1b4 f   Qt5Widgets:Qt5Widgets.dll
 0001:0000c1ba       ?isEmpty@QLayout@@UBE_NXZ  1000d1ba f   Qt5Widgets:Qt5Widgets.dll
 0001:0000c1c0       ?itemAt@QBoxLayout@@UBEPAVQLayoutItem@@H@Z 1000d1c0 f   Qt5Widgets:Qt5Widgets.dll
 0001:0000c1c6       ?keyPressEvent@QMenu@@MAEXPAVQKeyEvent@@@Z 1000d1c6 f   Qt5Widgets:Qt5Widgets.dll
 0001:0000c1cc       ?keyPressEvent@QWidget@@MAEXPAVQKeyEvent@@@Z 1000d1cc f   Qt5Widgets:Qt5Widgets.dll
 0001:0000c1d2       ?keyReleaseEvent@QWidget@@MAEXPAVQKeyEvent@@@Z 1000d1d2 f   Qt5Widgets:Qt5Widgets.dll
 0001:0000c1d8       ?layout@QLayout@@UAEPAV1@XZ 1000d1d8 f   Qt5Widgets:Qt5Widgets.dll
 0001:0000c1de       ?leaveEvent@QMenu@@MAEXPAVQEvent@@@Z 1000d1de f   Qt5Widgets:Qt5Widgets.dll
 0001:0000c1e4       ?leaveEvent@QWidget@@MAEXPAVQEvent@@@Z 1000d1e4 f   Qt5Widgets:Qt5Widgets.dll
 0001:0000c1ea       ?maximumSize@QBoxLayout@@UBE?AVQSize@@XZ 1000d1ea f   Qt5Widgets:Qt5Widgets.dll
 0001:0000c1f0       ?metaObject@QAction@@UBEPBUQMetaObject@@XZ 1000d1f0 f   Qt5Widgets:Qt5Widgets.dll
 0001:0000c1f6       ?metaObject@QHBoxLayout@@UBEPBUQMetaObject@@XZ 1000d1f6 f   Qt5Widgets:Qt5Widgets.dll
 0001:0000c1fc       ?metaObject@QMenu@@UBEPBUQMetaObject@@XZ 1000d1fc f   Qt5Widgets:Qt5Widgets.dll
 0001:0000c202       ?metric@QWidget@@MBEHW4PaintDeviceMetric@QPaintDevice@@@Z 1000d202 f   Qt5Widgets:Qt5Widgets.dll
 0001:0000c208       ?minimumHeightForWidth@QBoxLayout@@UBEHH@Z 1000d208 f   Qt5Widgets:Qt5Widgets.dll
 0001:0000c20e       ?minimumSize@QBoxLayout@@UBE?AVQSize@@XZ 1000d20e f   Qt5Widgets:Qt5Widgets.dll
 0001:0000c214       ?minimumSizeHint@QWidget@@UBE?AVQSize@@XZ 1000d214 f   Qt5Widgets:Qt5Widgets.dll
 0001:0000c21a       ?mouseDoubleClickEvent@QWidget@@MAEXPAVQMouseEvent@@@Z 1000d21a f   Qt5Widgets:Qt5Widgets.dll
 0001:0000c220       ?mouseMoveEvent@QMenu@@MAEXPAVQMouseEvent@@@Z 1000d220 f   Qt5Widgets:Qt5Widgets.dll
 0001:0000c226       ?mouseMoveEvent@QWidget@@MAEXPAVQMouseEvent@@@Z 1000d226 f   Qt5Widgets:Qt5Widgets.dll
 0001:0000c22c       ?mousePressEvent@QMenu@@MAEXPAVQMouseEvent@@@Z 1000d22c f   Qt5Widgets:Qt5Widgets.dll
 0001:0000c232       ?mousePressEvent@QWidget@@MAEXPAVQMouseEvent@@@Z 1000d232 f   Qt5Widgets:Qt5Widgets.dll
 0001:0000c238       ?mouseReleaseEvent@QMenu@@MAEXPAVQMouseEvent@@@Z 1000d238 f   Qt5Widgets:Qt5Widgets.dll
 0001:0000c23e       ?mouseReleaseEvent@QWidget@@MAEXPAVQMouseEvent@@@Z 1000d23e f   Qt5Widgets:Qt5Widgets.dll
 0001:0000c244       ?moveEvent@QWidget@@MAEXPAVQMoveEvent@@@Z 1000d244 f   Qt5Widgets:Qt5Widgets.dll
 0001:0000c24a       ?nativeEvent@QWidget@@MAE_NABVQByteArray@@PAXPAJ@Z 1000d24a f   Qt5Widgets:Qt5Widgets.dll
 0001:0000c250       ?paintEngine@QWidget@@UBEPAVQPaintEngine@@XZ 1000d250 f   Qt5Widgets:Qt5Widgets.dll
 0001:0000c256       ?paintEvent@QMenu@@MAEXPAVQPaintEvent@@@Z 1000d256 f   Qt5Widgets:Qt5Widgets.dll
 0001:0000c25c       ?paintEvent@QWidget@@MAEXPAVQPaintEvent@@@Z 1000d25c f   Qt5Widgets:Qt5Widgets.dll
 0001:0000c262       ?qt_metacall@QAction@@UAEHW4Call@QMetaObject@@HPAPAX@Z 1000d262 f   Qt5Widgets:Qt5Widgets.dll
 0001:0000c268       ?qt_metacall@QHBoxLayout@@UAEHW4Call@QMetaObject@@HPAPAX@Z 1000d268 f   Qt5Widgets:Qt5Widgets.dll
 0001:0000c26e       ?qt_metacall@QMenu@@UAEHW4Call@QMetaObject@@HPAPAX@Z 1000d26e f   Qt5Widgets:Qt5Widgets.dll
 0001:0000c274       ?qt_metacast@QAction@@UAEPAXPBD@Z 1000d274 f   Qt5Widgets:Qt5Widgets.dll
 0001:0000c27a       ?qt_metacast@QHBoxLayout@@UAEPAXPBD@Z 1000d27a f   Qt5Widgets:Qt5Widgets.dll
 0001:0000c280       ?qt_metacast@QMenu@@UAEPAXPBD@Z 1000d280 f   Qt5Widgets:Qt5Widgets.dll
 0001:0000c286       ?redirected@QWidget@@MBEPAVQPaintDevice@@PAVQPoint@@@Z 1000d286 f   Qt5Widgets:Qt5Widgets.dll
 0001:0000c28c       ?resizeEvent@QWidget@@MAEXPAVQResizeEvent@@@Z 1000d28c f   Qt5Widgets:Qt5Widgets.dll
 0001:0000c292       ?setGeometry@QBoxLayout@@UAEXABVQRect@@@Z 1000d292 f   Qt5Widgets:Qt5Widgets.dll
 0001:0000c298       ?setVisible@QWidget@@UAEX_N@Z 1000d298 f   Qt5Widgets:Qt5Widgets.dll
 0001:0000c29e       ?sharedPainter@QWidget@@MBEPAVQPainter@@XZ 1000d29e f   Qt5Widgets:Qt5Widgets.dll
 0001:0000c2a4       ?showEvent@QWidget@@MAEXPAVQShowEvent@@@Z 1000d2a4 f   Qt5Widgets:Qt5Widgets.dll
 0001:0000c2aa       ?sizeHint@QBoxLayout@@UBE?AVQSize@@XZ 1000d2aa f   Qt5Widgets:Qt5Widgets.dll
 0001:0000c2b0       ?sizeHint@QMenu@@UBE?AVQSize@@XZ 1000d2b0 f   Qt5Widgets:Qt5Widgets.dll
 0001:0000c2b6       ?sizeHint@QWidget@@UBE?AVQSize@@XZ 1000d2b6 f   Qt5Widgets:Qt5Widgets.dll
 0001:0000c2bc       ?spacerItem@QLayoutItem@@UAEPAVQSpacerItem@@XZ 1000d2bc f   Qt5Widgets:Qt5Widgets.dll
 0001:0000c2c2       ?tabletEvent@QWidget@@MAEXPAVQTabletEvent@@@Z 1000d2c2 f   Qt5Widgets:Qt5Widgets.dll
 0001:0000c2c8       ?takeAt@QBoxLayout@@UAEPAVQLayoutItem@@H@Z 1000d2c8 f   Qt5Widgets:Qt5Widgets.dll
 0001:0000c2ce       ?timerEvent@QMenu@@MAEXPAVQTimerEvent@@@Z 1000d2ce f   Qt5Widgets:Qt5Widgets.dll
 0001:0000c2d4       ?wheelEvent@QMenu@@MAEXPAVQWheelEvent@@@Z 1000d2d4 f   Qt5Widgets:Qt5Widgets.dll
 0001:0000c2da       ?wheelEvent@QWidget@@MAEXPAVQWheelEvent@@@Z 1000d2da f   Qt5Widgets:Qt5Widgets.dll
 0001:0000c2e0       ?widget@QLayoutItem@@UAEPAVQWidget@@XZ 1000d2e0 f   Qt5Widgets:Qt5Widgets.dll
 0001:0000c2e6       ?qt_metacast@QWidget@@UAEPAXPBD@Z 1000d2e6 f   Qt5Widgets:Qt5Widgets.dll
 0001:0000c2ec       ?qt_metacall@QWidget@@UAEHW4Call@QMetaObject@@HPAPAX@Z 1000d2ec f   Qt5Widgets:Qt5Widgets.dll
 0001:0000c2f2       ??0QIcon@@QAE@ABVQString@@@Z 1000d2f2 f   Qt5Gui:Qt5Gui.dll
 0001:0000c2f8       ??1QIcon@@QAE@XZ           1000d2f8 f   Qt5Gui:Qt5Gui.dll
 0001:0000c2fe       ?width@QPaintDevice@@QBEHXZ 1000d2fe f   Qt5Gui:Qt5Gui.dll
 0001:0000c304       ?height@QPaintDevice@@QBEHXZ 1000d304 f   Qt5Gui:Qt5Gui.dll
 0001:0000c30a       ??0QColor@@QAE@W4GlobalColor@Qt@@@Z 1000d30a f   Qt5Gui:Qt5Gui.dll
 0001:0000c310       ??1QPolygonF@@QAE@XZ       1000d310 f   Qt5Gui:Qt5Gui.dll
 0001:0000c316       ??0QPolygonF@@QAE@H@Z      1000d316 f   Qt5Gui:Qt5Gui.dll
 0001:0000c31c       ??0QBrush@@QAE@W4GlobalColor@Qt@@W4BrushStyle@2@@Z 1000d31c f   Qt5Gui:Qt5Gui.dll
 0001:0000c322       ??0QBrush@@QAE@ABVQGradient@@@Z 1000d322 f   Qt5Gui:Qt5Gui.dll
 0001:0000c328       ??1QBrush@@QAE@XZ          1000d328 f   Qt5Gui:Qt5Gui.dll
 0001:0000c32e       ?setColorAt@QGradient@@QAEXNABVQColor@@@Z 1000d32e f   Qt5Gui:Qt5Gui.dll
 0001:0000c334       ??0QLinearGradient@@QAE@NNNN@Z 1000d334 f   Qt5Gui:Qt5Gui.dll
 0001:0000c33a       ??1QLinearGradient@@QAE@XZ 1000d33a f   Qt5Gui:Qt5Gui.dll
 0001:0000c340       ??0QFont@@QAE@XZ           1000d340 f   Qt5Gui:Qt5Gui.dll
 0001:0000c346       ??0QFont@@QAE@ABVQString@@HH_N@Z 1000d346 f   Qt5Gui:Qt5Gui.dll
 0001:0000c34c       ??1QFont@@QAE@XZ           1000d34c f   Qt5Gui:Qt5Gui.dll
 0001:0000c352       ?setFamily@QFont@@QAEXABVQString@@@Z 1000d352 f   Qt5Gui:Qt5Gui.dll
 0001:0000c358       ?setPointSize@QFont@@QAEXH@Z 1000d358 f   Qt5Gui:Qt5Gui.dll
 0001:0000c35e       ?setWeight@QFont@@QAEXH@Z  1000d35e f   Qt5Gui:Qt5Gui.dll
 0001:0000c364       ??4QFont@@QAEAAV0@ABV0@@Z  1000d364 f   Qt5Gui:Qt5Gui.dll
 0001:0000c36a       ??0QFontMetricsF@@QAE@ABVQFont@@@Z 1000d36a f   Qt5Gui:Qt5Gui.dll
 0001:0000c370       ??1QFontMetricsF@@QAE@XZ   1000d370 f   Qt5Gui:Qt5Gui.dll
 0001:0000c376       ?ascent@QFontMetricsF@@QBENXZ 1000d376 f   Qt5Gui:Qt5Gui.dll
 0001:0000c37c       ?width@QFontMetricsF@@QBENVQChar@@@Z 1000d37c f   Qt5Gui:Qt5Gui.dll
 0001:0000c382       ?pos@QCursor@@SA?AVQPoint@@XZ 1000d382 f   Qt5Gui:Qt5Gui.dll
 0001:0000c388       ??0QPen@@QAE@ABVQBrush@@NW4PenStyle@Qt@@W4PenCapStyle@3@W4PenJoinStyle@3@@Z 1000d388 f   Qt5Gui:Qt5Gui.dll
 0001:0000c38e       ??1QPen@@QAE@XZ            1000d38e f   Qt5Gui:Qt5Gui.dll
 0001:0000c394       ?width@QPen@@QBEHXZ        1000d394 f   Qt5Gui:Qt5Gui.dll
 0001:0000c39a       ?pos@QMouseEvent@@QBE?AVQPoint@@XZ 1000d39a f   Qt5Gui:Qt5Gui.dll
 0001:0000c3a0       ??0QPainter@@QAE@PAVQPaintDevice@@@Z 1000d3a0 f   Qt5Gui:Qt5Gui.dll
 0001:0000c3a6       ??1QPainter@@QAE@XZ        1000d3a6 f   Qt5Gui:Qt5Gui.dll
 0001:0000c3ac       ?setFont@QPainter@@QAEXABVQFont@@@Z 1000d3ac f   Qt5Gui:Qt5Gui.dll
 0001:0000c3b2       ?setPen@QPainter@@QAEXABVQColor@@@Z 1000d3b2 f   Qt5Gui:Qt5Gui.dll
 0001:0000c3b8       ?setPen@QPainter@@QAEXABVQPen@@@Z 1000d3b8 f   Qt5Gui:Qt5Gui.dll
 0001:0000c3be       ?setBrush@QPainter@@QAEXABVQBrush@@@Z 1000d3be f   Qt5Gui:Qt5Gui.dll
 0001:0000c3c4       ?resetTransform@QPainter@@QAEXXZ 1000d3c4 f   Qt5Gui:Qt5Gui.dll
 0001:0000c3ca       ?translate@QPainter@@QAEXABVQPointF@@@Z 1000d3ca f   Qt5Gui:Qt5Gui.dll
 0001:0000c3d0       ?drawLines@QPainter@@QAEXPBVQLine@@H@Z 1000d3d0 f   Qt5Gui:Qt5Gui.dll
 0001:0000c3d6       ?drawRects@QPainter@@QAEXPBVQRectF@@H@Z 1000d3d6 f   Qt5Gui:Qt5Gui.dll
 0001:0000c3dc       ?drawRects@QPainter@@QAEXPBVQRect@@H@Z 1000d3dc f   Qt5Gui:Qt5Gui.dll
 0001:0000c3e2       ?drawPolyline@QPainter@@QAEXABVQPolygonF@@@Z 1000d3e2 f   Qt5Gui:Qt5Gui.dll
 0001:0000c3e8       ?drawRoundedRect@QPainter@@QAEXABVQRectF@@NNW4SizeMode@Qt@@@Z 1000d3e8 f   Qt5Gui:Qt5Gui.dll
 0001:0000c3ee       ?drawPixmap@QPainter@@QAEXABVQPointF@@ABVQPixmap@@@Z 1000d3ee f   Qt5Gui:Qt5Gui.dll
 0001:0000c3f4       ?drawText@QPainter@@QAEXABVQPointF@@ABVQString@@@Z 1000d3f4 f   Qt5Gui:Qt5Gui.dll
 0001:0000c3fa       ?drawText@QPainter@@QAEXABVQRectF@@HABVQString@@PAV2@@Z 1000d3fa f   Qt5Gui:Qt5Gui.dll
 0001:0000c400       ?fillRect@QPainter@@QAEXABVQRect@@ABVQColor@@@Z 1000d400 f   Qt5Gui:Qt5Gui.dll
 0001:0000c406       ?setRenderHint@QPainter@@QAEXW4RenderHint@1@_N@Z 1000d406 f   Qt5Gui:Qt5Gui.dll
 0001:0000c40c       ?cast@QMetaObject@@QBEPAVQObject@@PAV2@@Z 1000d40c f   Qt5Core:Qt5Core.dll
 0001:0000c412       ?tr@QMetaObject@@QBE?AVQString@@PBD0H@Z 1000d412 f   Qt5Core:Qt5Core.dll
 0001:0000c418       ??1Connection@QMetaObject@@QAE@XZ 1000d418 f   Qt5Core:Qt5Core.dll
 0001:0000c41e       ??0QString@@QAE@ABV0@@Z    1000d41e f   Qt5Core:Qt5Core.dll
 0001:0000c424       ??1QString@@QAE@XZ         1000d424 f   Qt5Core:Qt5Core.dll
 0001:0000c42a       ?fromAscii_helper@QString@@CAPAU?$QTypedArrayData@G@@PBDH@Z 1000d42a f   Qt5Core:Qt5Core.dll
 0001:0000c430       ?detach@QListData@@QAEPAUData@1@H@Z 1000d430 f   Qt5Core:Qt5Core.dll
 0001:0000c436       ?dispose@QListData@@SAXPAUData@1@@Z 1000d436 f   Qt5Core:Qt5Core.dll
 0001:0000c43c       ?connect@QObject@@QBE?AVConnection@QMetaObject@@PBV1@PBD1W4ConnectionType@Qt@@@Z 1000d43c f   Qt5Core:Qt5Core.dll
 0001:0000c442       ?sender@QObject@@IBEPAV1@XZ 1000d442 f   Qt5Core:Qt5Core.dll
 0001:0000c448       ?childEvent@QObject@@MAEXPAVQChildEvent@@@Z 1000d448 f   Qt5Core:Qt5Core.dll
 0001:0000c44e       ?connectNotify@QObject@@MAEXABVQMetaMethod@@@Z 1000d44e f   Qt5Core:Qt5Core.dll
 0001:0000c454       ?customEvent@QObject@@MAEXPAVQEvent@@@Z 1000d454 f   Qt5Core:Qt5Core.dll
 0001:0000c45a       ?disconnectNotify@QObject@@MAEXABVQMetaMethod@@@Z 1000d45a f   Qt5Core:Qt5Core.dll
 0001:0000c460       ?event@QObject@@UAE_NPAVQEvent@@@Z 1000d460 f   Qt5Core:Qt5Core.dll
 0001:0000c466       ?eventFilter@QObject@@UAE_NPAV1@PAVQEvent@@@Z 1000d466 f   Qt5Core:Qt5Core.dll
 0001:0000c46c       ?timerEvent@QObject@@MAEXPAVQTimerEvent@@@Z 1000d46c f   Qt5Core:Qt5Core.dll
 0001:0000c472       ?qBadAlloc@@YAXXZ          1000d472 f   Qt5Core:Qt5Core.dll
 0001:0000c478       ??0QMessageLogger@@QAE@PBDH0@Z 1000d478 f   Qt5Core:Qt5Core.dll
 0001:0000c47e       ?critical@QMessageLogger@@QBAXPBDZZ 1000d47e f   Qt5Core:Qt5Core.dll
 0001:0000c484       ??0QChar@@QAE@UQLatin1Char@@@Z 1000d484 f   Qt5Core:Qt5Core.dll
 0001:0000c48a       ?data@QArrayData@@QAEPAXXZ 1000d48a f   Qt5Core:Qt5Core.dll
 0001:0000c490       ?data@QArrayData@@QBEPBXXZ 1000d490 f   Qt5Core:Qt5Core.dll
 0001:0000c496       ?allocate@QArrayData@@SAPAU1@IIIV?$QFlags@W4AllocationOption@QArrayData@@@@@Z 1000d496 f   Qt5Core:Qt5Core.dll
 0001:0000c49c       ?deallocate@QArrayData@@SAXPAU1@II@Z 1000d49c f   Qt5Core:Qt5Core.dll
 0001:0000c4a2       ??0QByteArray@@QAE@XZ      1000d4a2 f   Qt5Core:Qt5Core.dll
 0001:0000c4a8       ??0QByteArray@@QAE@PBDH@Z  1000d4a8 f   Qt5Core:Qt5Core.dll
 0001:0000c4ae       ??1QByteArray@@QAE@XZ      1000d4ae f   Qt5Core:Qt5Core.dll
 0001:0000c4b4       ??4QByteArray@@QAEAAV0@$$QAV0@@Z 1000d4b4 f   Qt5Core:Qt5Core.dll
 0001:0000c4ba       ?at@QByteArray@@QBEDH@Z    1000d4ba f   Qt5Core:Qt5Core.dll
 0001:0000c4c0       ??AQByteArray@@QBEDH@Z     1000d4c0 f   Qt5Core:Qt5Core.dll
 0001:0000c4c6       ??AQByteArray@@QAE?AVQByteRef@@H@Z 1000d4c6 f   Qt5Core:Qt5Core.dll
 0001:0000c4cc       ??4QByteRef@@QAEAAV0@D@Z   1000d4cc f   Qt5Core:Qt5Core.dll
 0001:0000c4d2       ??4QByteRef@@QAEAAV0@ABV0@@Z 1000d4d2 f   Qt5Core:Qt5Core.dll
 0001:0000c4d8       ??0QString@@QAE@VQChar@@@Z 1000d4d8 f   Qt5Core:Qt5Core.dll
 0001:0000c4de       ??4QString@@QAEAAV0@$$QAV0@@Z 1000d4de f   Qt5Core:Qt5Core.dll
 0001:0000c4e4       ?at@QString@@QBE?BVQChar@@H@Z 1000d4e4 f   Qt5Core:Qt5Core.dll
 0001:0000c4ea       ?arg@QString@@QBE?AV1@HHHVQChar@@@Z 1000d4ea f   Qt5Core:Qt5Core.dll
 0001:0000c4f0       ?arg@QString@@QBE?AV1@ABV1@HVQChar@@@Z 1000d4f0 f   Qt5Core:Qt5Core.dll
 0001:0000c4f6       ?append@QString@@QAEAAV1@ABV1@@Z 1000d4f6 f   Qt5Core:Qt5Core.dll
 0001:0000c4fc       ?fromUtf8@QString@@SA?AV1@PBDH@Z 1000d4fc f   Qt5Core:Qt5Core.dll
 0001:0000c502       ??8@YA_NABVQString@@0@Z    1000d502 f   Qt5Core:Qt5Core.dll
 0001:0000c508       ??8QString@@QBE_NPBD@Z     1000d508 f   Qt5Core:Qt5Core.dll
 0001:0000c50e       ??0QString@@QAE@ABUNull@0@@Z 1000d50e f   Qt5Core:Qt5Core.dll
 0001:0000c514       ?detach_grow@QListData@@QAEPAUData@1@PAHH@Z 1000d514 f   Qt5Core:Qt5Core.dll
 0001:0000c51a       ?append@QListData@@QAEPAPAXXZ 1000d51a f   Qt5Core:Qt5Core.dll
 0001:0000c520       ?remove@QListData@@QAEXH@Z 1000d520 f   Qt5Core:Qt5Core.dll
 0001:0000c526       ??1QObject@@UAE@XZ         1000d526 f   Qt5Core:Qt5Core.dll
 0001:0000c52c       ?setObjectName@QObject@@QAEXABVQString@@@Z 1000d52c f   Qt5Core:Qt5Core.dll
 0001:0000c532       ?toPoint@QPointF@@QBE?AVQPoint@@XZ 1000d532 f   Qt5Core:Qt5Core.dll
 0001:0000c538       ?contains@QRect@@QBE_NABVQPoint@@_N@Z 1000d538 f   Qt5Core:Qt5Core.dll
 0001:0000c53e       ?setCoords@QRectF@@QAEXNNNN@Z 1000d53e f   Qt5Core:Qt5Core.dll
 0001:0000c544       ?contains@QRectF@@QBE_NABVQPointF@@@Z 1000d544 f   Qt5Core:Qt5Core.dll
 0001:0000c54a       ??A?$QVector@VQPointF@@@@QAEAAVQPointF@@H@Z 1000d54a f   Qt5Core:Qt5Core.dll
 0001:0000c550       ?qHash@@YAIABVQString@@I@Z 1000d550 f   Qt5Core:Qt5Core.dll
 0001:0000c556       ?allocateNode@QHashData@@QAEPAXH@Z 1000d556 f   Qt5Core:Qt5Core.dll
 0001:0000c55c       ?freeNode@QHashData@@QAEXPAX@Z 1000d55c f   Qt5Core:Qt5Core.dll
 0001:0000c562       ?detach_helper@QHashData@@QAEPAU1@P6AXPAUNode@1@PAX@ZP6AX0@ZHH@Z 1000d562 f   Qt5Core:Qt5Core.dll
 0001:0000c568       ?hasShrunk@QHashData@@QAEXXZ 1000d568 f   Qt5Core:Qt5Core.dll
 0001:0000c56e       ?rehash@QHashData@@QAEXH@Z 1000d56e f   Qt5Core:Qt5Core.dll
 0001:0000c574       ?free_helper@QHashData@@QAEXP6AXPAUNode@1@@Z@Z 1000d574 f   Qt5Core:Qt5Core.dll
 0001:0000c57a       ?firstNode@QHashData@@QAEPAUNode@1@XZ 1000d57a f   Qt5Core:Qt5Core.dll
 0001:0000c580       ?nextNode@QHashData@@SAPAUNode@1@PAU21@@Z 1000d580 f   Qt5Core:Qt5Core.dll
 0001:0000c586       ?getAndRef@ExternalRefCountData@QtSharedPointer@@SAPAU12@PBVQObject@@@Z 1000d586 f   Qt5Core:Qt5Core.dll
 0001:0000c58c       ?freeTree@QMapDataBase@@QAEXPAUQMapNodeBase@@H@Z 1000d58c f   Qt5Core:Qt5Core.dll
 0001:0000c592       ?freeData@QMapDataBase@@SAXPAU1@@Z 1000d592 f   Qt5Core:Qt5Core.dll
 0001:0000c598       ??1QVariant@@QAE@XZ        1000d598 f   Qt5Core:Qt5Core.dll
 0001:0000c59e       ?className@QMetaObject@@QBEPBDXZ 1000d59e f   Qt5Core:Qt5Core.dll
 0001:0000c5a4       ?reserve@QByteArray@@QAEXH@Z 1000d5a4 f   Qt5Core:Qt5Core.dll
 0001:0000c5aa       ?append@QByteArray@@QAEAAV1@D@Z 1000d5aa f   Qt5Core:Qt5Core.dll
 0001:0000c5b0       ?append@QByteArray@@QAEAAV1@PBD@Z 1000d5b0 f   Qt5Core:Qt5Core.dll
 0001:0000c5b6       ?registerNormalizedType@QMetaType@@SAHABVQByteArray@@P6AXPAX@ZP6APAXPBX@Z2P6APAX13@ZHV?$QFlags@W4TypeFlag@QMetaType@@@@PBUQMetaObject@@@Z 1000d5b6 f   Qt5Core:Qt5Core.dll
 0001:0000c5bc       ?registerNormalizedTypedef@QMetaType@@SAHABVQByteArray@@H@Z 1000d5bc f   Qt5Core:Qt5Core.dll
 0001:0000c5c2       ?dynamicMetaObject@QObjectData@@QBEPAUQMetaObject@@XZ 1000d5c2 f   Qt5Core:Qt5Core.dll
 0001:0000c5c8       ?qRegisterResourceData@@YA_NHPBE00@Z 1000d5c8 f   Qt5Core:Qt5Core.dll
 0001:0000c5ce       ?qUnregisterResourceData@@YA_NHPBE00@Z 1000d5ce f   Qt5Core:Qt5Core.dll
 0001:0000c5d4       ?_Xbad_alloc@std@@YAXXZ    1000d5d4 f   msvcprt:MSVCP120.dll
 0001:0000c5da       ?_Xlength_error@std@@YAXPBD@Z 1000d5da f   msvcprt:MSVCP120.dll
 0001:0000c5e0       ?_Xout_of_range@std@@YAXPBD@Z 1000d5e0 f   msvcprt:MSVCP120.dll
 0001:0000c5e6       ?_Syserror_map@std@@YAPBDH@Z 1000d5e6 f   msvcprt:MSVCP120.dll
 0001:0000c5ec       ?_Winerror_map@std@@YAPBDH@Z 1000d5ec f   msvcprt:MSVCP120.dll
 0001:0000c5f2       __purecall                 1000d5f2 f   MSVCRT:MSVCR120.dll
 0001:0000c5f8       ??2@YAPAXI@Z               1000d5f8 f   MSVCRT:MSVCR120.dll
 0001:0000c5fe       ??3@YAXPAX@Z               1000d5fe f   MSVCRT:MSVCR120.dll
 0001:0000c604       ___atonexitinit            1000d604 f   MSVCRT:atonexit.obj
 0001:0000c640       __onexit                   1000d640 f   MSVCRT:atonexit.obj
 0001:0000c6e9       _atexit                    1000d6e9 f   MSVCRT:atonexit.obj
 0001:0000c6fe       _memmove                   1000d6fe f   MSVCRT:MSVCR120.dll
 0001:0000c704       __hypot                    1000d704 f   MSVCRT:MSVCR120.dll
 0001:0000c70a       @__security_check_cookie@4 1000d70a f   MSVCRT:secchk.obj
 0001:0000c71a       __CxxThrowException@8      1000d71a f   MSVCRT:MSVCR120.dll
 0001:0000c720       ___CxxFrameHandler3        1000d720 f   MSVCRT:MSVCR120.dll
 0001:0000c726       _memcpy                    1000d726 f   MSVCRT:MSVCR120.dll
 0001:0000c72c       ??0type_info@@AAE@ABV0@@Z  1000d72c f   MSVCRT:ti_inst.obj
 0001:0000c737       ??4type_info@@AAEAAV0@ABV0@@Z 1000d737 f   MSVCRT:ti_inst.obj
 0001:0000c73c       ??_Etype_info@@UAEPAXI@Z   1000d73c f i MSVCRT:ti_inst.obj
 0001:0000c790       ??_M@YGXPAXIHP6EX0@Z@Z     1000d790 f   MSVCRT:ehvecdtr.obj
 0001:0000c818       ?__ArrayUnwind@@YGXPAXIHP6EX0@Z@Z 1000d818 f   MSVCRT:ehvecdtr.obj
 0001:0000c880       __ftoui3                   1000d880 f   MSVCRT:ftol3.obj
 0001:0000c88f       __ftoul3                   1000d88f f   MSVCRT:ftol3.obj
 0001:0000c89e       __ftol3                    1000d89e f   MSVCRT:ftol3.obj
 0001:0000c8ab       __ftol3_NaN                1000d8ab f   MSVCRT:ftol3.obj
 0001:0000c8c3       __ftol3_work               1000d8c3 f   MSVCRT:ftol3.obj
 0001:0000c949       __ftol3_common             1000d949 f   MSVCRT:ftol3.obj
 0001:0000ca0b       __ftol3_arg_error          1000da0b f   MSVCRT:ftol3.obj
 0001:0000ca1d       __ftol3_except             1000da1d f   MSVCRT:ftol3.obj
 0001:0000ca61       __dtoui3                   1000da61 f   MSVCRT:ftol3.obj
 0001:0000ca70       __dtoul3                   1000da70 f   MSVCRT:ftol3.obj
 0001:0000ca7f       __dtol3                    1000da7f f   MSVCRT:ftol3.obj
 0001:0000ca8c       __dtol3_NaN                1000da8c f   MSVCRT:ftol3.obj
 0001:0000caa9       __dtol3_work               1000daa9 f   MSVCRT:ftol3.obj
 0001:0000cb8e       __ultod3                   1000db8e f   MSVCRT:ftol3.obj
 0001:0000cc1f       __ltod3                    1000dc1f f   MSVCRT:ftol3.obj
 0001:0000cc4e       _memset                    1000dc4e f   MSVCRT:MSVCR120.dll
 0001:0000cca0       _NtCurrentTeb              1000dca0 f i MSVCRT:crtdll.obj
 0001:0000cca7       __CRT_INIT@12              1000dca7 f   MSVCRT:crtdll.obj
 0001:0000ce9e       __DllMainCRTStartup@12     1000de9e f   MSVCRT:crtdll.obj
 0001:0000cff4       __lock                     1000dff4 f   MSVCRT:MSVCR120.dll
 0001:0000cffa       __unlock                   1000dffa f   MSVCRT:MSVCR120.dll
 0001:0000d000       __calloc_crt               1000e000 f   MSVCRT:MSVCR120.dll
 0001:0000d006       ___dllonexit               1000e006 f   MSVCRT:MSVCR120.dll
 0001:0000d010       __SEH_prolog4              1000e010 f   MSVCRT:sehprolg4.obj
 0001:0000d055       __SEH_epilog4              1000e055 f   MSVCRT:sehprolg4.obj
 0001:0000d069       __except_handler4          1000e069 f   MSVCRT:chandler4gs.obj
 0001:0000d08c       ___raise_securityfailure   1000e08c f   MSVCRT:gs_report.obj
 0001:0000d0c9       ___report_gsfailure        1000e0c9 f   MSVCRT:gs_report.obj
 0001:0000d1c4       ___report_rangecheckfailure 1000e1c4 f   MSVCRT:gs_report.obj
 0001:0000d1d0       ___report_securityfailure  1000e1d0 f   MSVCRT:gs_report.obj
 0001:0000d2a0       ___report_securityfailureEx 1000e2a0 f   MSVCRT:gs_report.obj
 0001:0000d3b6       ??1type_info@@UAE@XZ       1000e3b6 f   MSVCRT:MSVCR120.dll
 0001:0000d3bc       ?terminate@@YAXXZ          1000e3bc f   MSVCRT:MSVCR120.dll
 0001:0000d3c2       __except1                  1000e3c2 f   MSVCRT:MSVCR120.dll
 0001:0000d3c8       ___CppXcptFilter           1000e3c8 f   MSVCRT:MSVCR120.dll
 0001:0000d3ce       __amsg_exit                1000e3ce f   MSVCRT:MSVCR120.dll
 0001:0000d3e0       __FindPESection            1000e3e0 f   MSVCRT:pesect.obj
 0001:0000d430       __IsNonwritableInCurrentImage 1000e430 f   MSVCRT:pesect.obj
 0001:0000d4f0       __ValidateImageBase        1000e4f0 f   MSVCRT:pesect.obj
 0001:0000d522       _free                      1000e522 f   MSVCRT:MSVCR120.dll
 0001:0000d528       ___security_init_cookie    1000e528 f   MSVCRT:gs_support.obj
 0001:0000d5c4       _DllMain@12                1000e5c4 f   MSVCRT:dllmain.obj
 0001:0000d5e6       __malloc_crt               1000e5e6 f   MSVCRT:MSVCR120.dll
 0001:0000d5ec       __RTC_Initialize           1000e5ec f   MSVCRT:initsect.obj
 0001:0000d60c       __RTC_Terminate            1000e60c f   MSVCRT:initsect.obj
 0001:0000d62c       __initterm                 1000e62c f   MSVCRT:MSVCR120.dll
 0001:0000d632       __initterm_e               1000e632 f   MSVCRT:MSVCR120.dll
 0001:0000d638       ___clean_type_info_names   1000e638 f   MSVCRT:tncleanup.obj
 0001:0000d644       __except_handler4_common   1000e644 f   MSVCRT:MSVCR120.dll
 0001:0000d64a       __crt_debugger_hook        1000e64a f   MSVCRT:MSVCR120.dll
 0001:0000d650       ___crtUnhandledException   1000e650 f   MSVCRT:MSVCR120.dll
 0001:0000d656       ___crtTerminateProcess     1000e656 f   MSVCRT:MSVCR120.dll
 0001:0000d65c       ___clean_type_info_names_internal 1000e65c f   MSVCRT:MSVCR120.dll
 0001:0000d662       _EncodePointer@4           1000e662 f   kernel32:KERNEL32.dll
 0001:0000d668       _DecodePointer@4           1000e668 f   kernel32:KERNEL32.dll
 0001:0000d66e       _IsDebuggerPresent@0       1000e66e f   kernel32:KERNEL32.dll
 0001:0000d674       _IsProcessorFeaturePresent@4 1000e674 f   kernel32:KERNEL32.dll
 0001:0000d67a       _QueryPerformanceCounter@4 1000e67a f   kernel32:KERNEL32.dll
 0001:0000d680       _GetCurrentProcessId@0     1000e680 f   kernel32:KERNEL32.dll
 0001:0000d686       _GetCurrentThreadId@0      1000e686 f   kernel32:KERNEL32.dll
 0001:0000d68c       _GetSystemTimeAsFileTime@4 1000e68c f   kernel32:KERNEL32.dll
 0001:0000d692       _DisableThreadLibraryCalls@4 1000e692 f   kernel32:KERNEL32.dll
 0002:00000000       __imp__DisableThreadLibraryCalls@4 10010000     kernel32:KERNEL32.dll
 0002:00000004       __imp__GetSystemTimeAsFileTime@4 10010004     kernel32:KERNEL32.dll
 0002:00000008       __imp__GetCurrentThreadId@0 10010008     kernel32:KERNEL32.dll
 0002:0000000c       __imp__GetCurrentProcessId@0 1001000c     kernel32:KERNEL32.dll
 0002:00000010       __imp__QueryPerformanceCounter@4 10010010     kernel32:KERNEL32.dll
 0002:00000014       __imp__IsProcessorFeaturePresent@4 10010014     kernel32:KERNEL32.dll
 0002:00000018       __imp__IsDebuggerPresent@0 10010018     kernel32:KERNEL32.dll
 0002:0000001c       __imp__DecodePointer@4     1001001c     kernel32:KERNEL32.dll
 0002:00000020       __imp__EncodePointer@4     10010020     kernel32:KERNEL32.dll
 0002:00000024       \177KERNEL32_NULL_THUNK_DATA 10010024     kernel32:KERNEL32.dll
 0002:00000028       __imp_?_Xlength_error@std@@YAXPBD@Z 10010028     msvcprt:MSVCP120.dll
 0002:0000002c       __imp_?_Xout_of_range@std@@YAXPBD@Z 1001002c     msvcprt:MSVCP120.dll
 0002:00000030       __imp_?_Syserror_map@std@@YAPBDH@Z 10010030     msvcprt:MSVCP120.dll
 0002:00000034       __imp_?_Winerror_map@std@@YAPBDH@Z 10010034     msvcprt:MSVCP120.dll
 0002:00000038       __imp_?_Xbad_alloc@std@@YAXXZ 10010038     msvcprt:MSVCP120.dll
 0002:0000003c       \177MSVCP120_NULL_THUNK_DATA 1001003c     msvcprt:MSVCP120.dll
 0002:00000040       __imp___initterm_e         10010040     MSVCRT:MSVCR120.dll
 0002:00000044       __imp___initterm           10010044     MSVCRT:MSVCR120.dll
 0002:00000048       __imp___malloc_crt         10010048     MSVCRT:MSVCR120.dll
 0002:0000004c       __imp__free                1001004c     MSVCRT:MSVCR120.dll
 0002:00000050       __imp___amsg_exit          10010050     MSVCRT:MSVCR120.dll
 0002:00000054       __imp____CppXcptFilter     10010054     MSVCRT:MSVCR120.dll
 0002:00000058       __imp_?terminate@@YAXXZ    10010058     MSVCRT:MSVCR120.dll
 0002:0000005c       __imp_??1type_info@@UAE@XZ 1001005c     MSVCRT:MSVCR120.dll
 0002:00000060       __imp___onexit             10010060     MSVCRT:MSVCR120.dll
 0002:00000064       __imp____dllonexit         10010064     MSVCRT:MSVCR120.dll
 0002:00000068       __imp___calloc_crt         10010068     MSVCRT:MSVCR120.dll
 0002:0000006c       __imp___unlock             1001006c     MSVCRT:MSVCR120.dll
 0002:00000070       __imp___lock               10010070     MSVCRT:MSVCR120.dll
 0002:00000074       __imp__memset              10010074     MSVCRT:MSVCR120.dll
 0002:00000078       __imp__memcpy              10010078     MSVCRT:MSVCR120.dll
 0002:0000007c       __imp____CxxFrameHandler3  1001007c     MSVCRT:MSVCR120.dll
 0002:00000080       __imp___CxxThrowException@8 10010080     MSVCRT:MSVCR120.dll
 0002:00000084       __imp___hypot              10010084     MSVCRT:MSVCR120.dll
 0002:00000088       __imp__memmove             10010088     MSVCRT:MSVCR120.dll
 0002:0000008c       __imp_??3@YAXPAX@Z         1001008c     MSVCRT:MSVCR120.dll
 0002:00000090       __imp_??2@YAPAXI@Z         10010090     MSVCRT:MSVCR120.dll
 0002:00000094       __imp___purecall           10010094     MSVCRT:MSVCR120.dll
 0002:00000098       __imp___except_handler4_common 10010098     MSVCRT:MSVCR120.dll
 0002:0000009c       __imp___crt_debugger_hook  1001009c     MSVCRT:MSVCR120.dll
 0002:000000a0       __imp____crtUnhandledException 100100a0     MSVCRT:MSVCR120.dll
 0002:000000a4       __imp____crtTerminateProcess 100100a4     MSVCRT:MSVCR120.dll
 0002:000000a8       __imp____clean_type_info_names_internal 100100a8     MSVCRT:MSVCR120.dll
 0002:000000ac       __imp___except1            100100ac     MSVCRT:MSVCR120.dll
 0002:000000b0       \177MSVCR120_NULL_THUNK_DATA 100100b0     MSVCRT:MSVCR120.dll
 0002:000000b4       __imp_?qUnregisterResourceData@@YA_NHPBE00@Z 100100b4     Qt5Core:Qt5Core.dll
 0002:000000b8       __imp_?qRegisterResourceData@@YA_NHPBE00@Z 100100b8     Qt5Core:Qt5Core.dll
 0002:000000bc       __imp_?dynamicMetaObject@QObjectData@@QBEPAUQMetaObject@@XZ 100100bc     Qt5Core:Qt5Core.dll
 0002:000000c0       __imp_?registerNormalizedTypedef@QMetaType@@SAHABVQByteArray@@H@Z 100100c0     Qt5Core:Qt5Core.dll
 0002:000000c4       __imp_?registerNormalizedType@QMetaType@@SAHABVQByteArray@@P6AXPAX@ZP6APAXPBX@Z2P6APAX13@ZHV?$QFlags@W4TypeFlag@QMetaType@@@@PBUQMetaObject@@@Z 100100c4     Qt5Core:Qt5Core.dll
 0002:000000c8       __imp_?append@QByteArray@@QAEAAV1@PBD@Z 100100c8     Qt5Core:Qt5Core.dll
 0002:000000cc       __imp_?append@QByteArray@@QAEAAV1@D@Z 100100cc     Qt5Core:Qt5Core.dll
 0002:000000d0       __imp_?reserve@QByteArray@@QAEXH@Z 100100d0     Qt5Core:Qt5Core.dll
 0002:000000d4       __imp_?className@QMetaObject@@QBEPBDXZ 100100d4     Qt5Core:Qt5Core.dll
 0002:000000d8       __imp_?shared_null@QMapDataBase@@2U1@B 100100d8     Qt5Core:Qt5Core.dll
 0002:000000dc       __imp_?shared_null@QHashData@@2U1@B 100100dc     Qt5Core:Qt5Core.dll
 0002:000000e0       __imp_?shared_null@QListData@@2UData@1@B 100100e0     Qt5Core:Qt5Core.dll
 0002:000000e4       __imp_?null@QString@@2UNull@1@B 100100e4     Qt5Core:Qt5Core.dll
 0002:000000e8       __imp_?shared_null@QArrayData@@2QBU1@B 100100e8     Qt5Core:Qt5Core.dll
 0002:000000ec       __imp_??1QVariant@@QAE@XZ  100100ec     Qt5Core:Qt5Core.dll
 0002:000000f0       __imp_?freeData@QMapDataBase@@SAXPAU1@@Z 100100f0     Qt5Core:Qt5Core.dll
 0002:000000f4       __imp_?freeTree@QMapDataBase@@QAEXPAUQMapNodeBase@@H@Z 100100f4     Qt5Core:Qt5Core.dll
 0002:000000f8       __imp_?getAndRef@ExternalRefCountData@QtSharedPointer@@SAPAU12@PBVQObject@@@Z 100100f8     Qt5Core:Qt5Core.dll
 0002:000000fc       __imp_?nextNode@QHashData@@SAPAUNode@1@PAU21@@Z 100100fc     Qt5Core:Qt5Core.dll
 0002:00000100       __imp_?firstNode@QHashData@@QAEPAUNode@1@XZ 10010100     Qt5Core:Qt5Core.dll
 0002:00000104       __imp_?free_helper@QHashData@@QAEXP6AXPAUNode@1@@Z@Z 10010104     Qt5Core:Qt5Core.dll
 0002:00000108       __imp_?rehash@QHashData@@QAEXH@Z 10010108     Qt5Core:Qt5Core.dll
 0002:0000010c       __imp_?hasShrunk@QHashData@@QAEXXZ 1001010c     Qt5Core:Qt5Core.dll
 0002:00000110       __imp_?detach_helper@QHashData@@QAEPAU1@P6AXPAUNode@1@PAX@ZP6AX0@ZHH@Z 10010110     Qt5Core:Qt5Core.dll
 0002:00000114       __imp_?freeNode@QHashData@@QAEXPAX@Z 10010114     Qt5Core:Qt5Core.dll
 0002:00000118       __imp_?allocateNode@QHashData@@QAEPAXH@Z 10010118     Qt5Core:Qt5Core.dll
 0002:0000011c       __imp_?qHash@@YAIABVQString@@I@Z 1001011c     Qt5Core:Qt5Core.dll
 0002:00000120       __imp_??A?$QVector@VQPointF@@@@QAEAAVQPointF@@H@Z 10010120     Qt5Core:Qt5Core.dll
 0002:00000124       __imp_?contains@QRectF@@QBE_NABVQPointF@@@Z 10010124     Qt5Core:Qt5Core.dll
 0002:00000128       __imp_?setCoords@QRectF@@QAEXNNNN@Z 10010128     Qt5Core:Qt5Core.dll
 0002:0000012c       __imp_?contains@QRect@@QBE_NABVQPoint@@_N@Z 1001012c     Qt5Core:Qt5Core.dll
 0002:00000130       __imp_?toPoint@QPointF@@QBE?AVQPoint@@XZ 10010130     Qt5Core:Qt5Core.dll
 0002:00000134       __imp_?setObjectName@QObject@@QAEXABVQString@@@Z 10010134     Qt5Core:Qt5Core.dll
 0002:00000138       __imp_??1QObject@@UAE@XZ   10010138     Qt5Core:Qt5Core.dll
 0002:0000013c       __imp_?remove@QListData@@QAEXH@Z 1001013c     Qt5Core:Qt5Core.dll
 0002:00000140       __imp_?append@QListData@@QAEPAPAXXZ 10010140     Qt5Core:Qt5Core.dll
 0002:00000144       __imp_?detach_grow@QListData@@QAEPAUData@1@PAHH@Z 10010144     Qt5Core:Qt5Core.dll
 0002:00000148       __imp_??0QString@@QAE@ABUNull@0@@Z 10010148     Qt5Core:Qt5Core.dll
 0002:0000014c       __imp_??8QString@@QBE_NPBD@Z 1001014c     Qt5Core:Qt5Core.dll
 0002:00000150       __imp_??8@YA_NABVQString@@0@Z 10010150     Qt5Core:Qt5Core.dll
 0002:00000154       __imp_?fromUtf8@QString@@SA?AV1@PBDH@Z 10010154     Qt5Core:Qt5Core.dll
 0002:00000158       __imp_?append@QString@@QAEAAV1@ABV1@@Z 10010158     Qt5Core:Qt5Core.dll
 0002:0000015c       __imp_?arg@QString@@QBE?AV1@ABV1@HVQChar@@@Z 1001015c     Qt5Core:Qt5Core.dll
 0002:00000160       __imp_?arg@QString@@QBE?AV1@HHHVQChar@@@Z 10010160     Qt5Core:Qt5Core.dll
 0002:00000164       __imp_?at@QString@@QBE?BVQChar@@H@Z 10010164     Qt5Core:Qt5Core.dll
 0002:00000168       __imp_??4QString@@QAEAAV0@$$QAV0@@Z 10010168     Qt5Core:Qt5Core.dll
 0002:0000016c       __imp_??0QString@@QAE@VQChar@@@Z 1001016c     Qt5Core:Qt5Core.dll
 0002:00000170       __imp_??4QByteRef@@QAEAAV0@ABV0@@Z 10010170     Qt5Core:Qt5Core.dll
 0002:00000174       __imp_??4QByteRef@@QAEAAV0@D@Z 10010174     Qt5Core:Qt5Core.dll
 0002:00000178       __imp_??AQByteArray@@QAE?AVQByteRef@@H@Z 10010178     Qt5Core:Qt5Core.dll
 0002:0000017c       __imp_??AQByteArray@@QBEDH@Z 1001017c     Qt5Core:Qt5Core.dll
 0002:00000180       __imp_?at@QByteArray@@QBEDH@Z 10010180     Qt5Core:Qt5Core.dll
 0002:00000184       __imp_??4QByteArray@@QAEAAV0@$$QAV0@@Z 10010184     Qt5Core:Qt5Core.dll
 0002:00000188       __imp_??1QByteArray@@QAE@XZ 10010188     Qt5Core:Qt5Core.dll
 0002:0000018c       __imp_??0QByteArray@@QAE@PBDH@Z 1001018c     Qt5Core:Qt5Core.dll
 0002:00000190       __imp_??0QByteArray@@QAE@XZ 10010190     Qt5Core:Qt5Core.dll
 0002:00000194       __imp_?deallocate@QArrayData@@SAXPAU1@II@Z 10010194     Qt5Core:Qt5Core.dll
 0002:00000198       __imp_?allocate@QArrayData@@SAPAU1@IIIV?$QFlags@W4AllocationOption@QArrayData@@@@@Z 10010198     Qt5Core:Qt5Core.dll
 0002:0000019c       __imp_?data@QArrayData@@QBEPBXXZ 1001019c     Qt5Core:Qt5Core.dll
 0002:000001a0       __imp_?data@QArrayData@@QAEPAXXZ 100101a0     Qt5Core:Qt5Core.dll
 0002:000001a4       __imp_??0QChar@@QAE@UQLatin1Char@@@Z 100101a4     Qt5Core:Qt5Core.dll
 0002:000001a8       __imp_?critical@QMessageLogger@@QBAXPBDZZ 100101a8     Qt5Core:Qt5Core.dll
 0002:000001ac       __imp_??0QMessageLogger@@QAE@PBDH0@Z 100101ac     Qt5Core:Qt5Core.dll
 0002:000001b0       __imp_?qBadAlloc@@YAXXZ    100101b0     Qt5Core:Qt5Core.dll
 0002:000001b4       __imp_?timerEvent@QObject@@MAEXPAVQTimerEvent@@@Z 100101b4     Qt5Core:Qt5Core.dll
 0002:000001b8       __imp_?eventFilter@QObject@@UAE_NPAV1@PAVQEvent@@@Z 100101b8     Qt5Core:Qt5Core.dll
 0002:000001bc       __imp_?event@QObject@@UAE_NPAVQEvent@@@Z 100101bc     Qt5Core:Qt5Core.dll
 0002:000001c0       __imp_?disconnectNotify@QObject@@MAEXABVQMetaMethod@@@Z 100101c0     Qt5Core:Qt5Core.dll
 0002:000001c4       __imp_?customEvent@QObject@@MAEXPAVQEvent@@@Z 100101c4     Qt5Core:Qt5Core.dll
 0002:000001c8       __imp_?connectNotify@QObject@@MAEXABVQMetaMethod@@@Z 100101c8     Qt5Core:Qt5Core.dll
 0002:000001cc       __imp_?childEvent@QObject@@MAEXPAVQChildEvent@@@Z 100101cc     Qt5Core:Qt5Core.dll
 0002:000001d0       __imp_?sender@QObject@@IBEPAV1@XZ 100101d0     Qt5Core:Qt5Core.dll
 0002:000001d4       __imp_?connect@QObject@@QBE?AVConnection@QMetaObject@@PBV1@PBD1W4ConnectionType@Qt@@@Z 100101d4     Qt5Core:Qt5Core.dll
 0002:000001d8       __imp_?dispose@QListData@@SAXPAUData@1@@Z 100101d8     Qt5Core:Qt5Core.dll
 0002:000001dc       __imp_?detach@QListData@@QAEPAUData@1@H@Z 100101dc     Qt5Core:Qt5Core.dll
 0002:000001e0       __imp_?fromAscii_helper@QString@@CAPAU?$QTypedArrayData@G@@PBDH@Z 100101e0     Qt5Core:Qt5Core.dll
 0002:000001e4       __imp_??1QString@@QAE@XZ   100101e4     Qt5Core:Qt5Core.dll
 0002:000001e8       __imp_??0QString@@QAE@ABV0@@Z 100101e8     Qt5Core:Qt5Core.dll
 0002:000001ec       __imp_??1Connection@QMetaObject@@QAE@XZ 100101ec     Qt5Core:Qt5Core.dll
 0002:000001f0       __imp_?tr@QMetaObject@@QBE?AVQString@@PBD0H@Z 100101f0     Qt5Core:Qt5Core.dll
 0002:000001f4       __imp_?cast@QMetaObject@@QBEPAVQObject@@PAV2@@Z 100101f4     Qt5Core:Qt5Core.dll
 0002:000001f8       \177Qt5Core_NULL_THUNK_DATA 100101f8     Qt5Core:Qt5Core.dll
 0002:000001fc       __imp_?setRenderHint@QPainter@@QAEXW4RenderHint@1@_N@Z 100101fc     Qt5Gui:Qt5Gui.dll
 0002:00000200       __imp_?fillRect@QPainter@@QAEXABVQRect@@ABVQColor@@@Z 10010200     Qt5Gui:Qt5Gui.dll
 0002:00000204       __imp_?drawText@QPainter@@QAEXABVQRectF@@HABVQString@@PAV2@@Z 10010204     Qt5Gui:Qt5Gui.dll
 0002:00000208       __imp_?drawText@QPainter@@QAEXABVQPointF@@ABVQString@@@Z 10010208     Qt5Gui:Qt5Gui.dll
 0002:0000020c       __imp_?drawPixmap@QPainter@@QAEXABVQPointF@@ABVQPixmap@@@Z 1001020c     Qt5Gui:Qt5Gui.dll
 0002:00000210       __imp_?drawRoundedRect@QPainter@@QAEXABVQRectF@@NNW4SizeMode@Qt@@@Z 10010210     Qt5Gui:Qt5Gui.dll
 0002:00000214       __imp_?drawPolyline@QPainter@@QAEXABVQPolygonF@@@Z 10010214     Qt5Gui:Qt5Gui.dll
 0002:00000218       __imp_?drawRects@QPainter@@QAEXPBVQRect@@H@Z 10010218     Qt5Gui:Qt5Gui.dll
 0002:0000021c       __imp_?drawRects@QPainter@@QAEXPBVQRectF@@H@Z 1001021c     Qt5Gui:Qt5Gui.dll
 0002:00000220       __imp_?drawLines@QPainter@@QAEXPBVQLine@@H@Z 10010220     Qt5Gui:Qt5Gui.dll
 0002:00000224       __imp_?translate@QPainter@@QAEXABVQPointF@@@Z 10010224     Qt5Gui:Qt5Gui.dll
 0002:00000228       __imp_?resetTransform@QPainter@@QAEXXZ 10010228     Qt5Gui:Qt5Gui.dll
 0002:0000022c       __imp_?setBrush@QPainter@@QAEXABVQBrush@@@Z 1001022c     Qt5Gui:Qt5Gui.dll
 0002:00000230       __imp_?setPen@QPainter@@QAEXABVQPen@@@Z 10010230     Qt5Gui:Qt5Gui.dll
 0002:00000234       __imp_?setPen@QPainter@@QAEXABVQColor@@@Z 10010234     Qt5Gui:Qt5Gui.dll
 0002:00000238       __imp_?setFont@QPainter@@QAEXABVQFont@@@Z 10010238     Qt5Gui:Qt5Gui.dll
 0002:0000023c       __imp_??1QPainter@@QAE@XZ  1001023c     Qt5Gui:Qt5Gui.dll
 0002:00000240       __imp_??0QPainter@@QAE@PAVQPaintDevice@@@Z 10010240     Qt5Gui:Qt5Gui.dll
 0002:00000244       __imp_?pos@QMouseEvent@@QBE?AVQPoint@@XZ 10010244     Qt5Gui:Qt5Gui.dll
 0002:00000248       __imp_?width@QPen@@QBEHXZ  10010248     Qt5Gui:Qt5Gui.dll
 0002:0000024c       __imp_??1QPen@@QAE@XZ      1001024c     Qt5Gui:Qt5Gui.dll
 0002:00000250       __imp_??0QPen@@QAE@ABVQBrush@@NW4PenStyle@Qt@@W4PenCapStyle@3@W4PenJoinStyle@3@@Z 10010250     Qt5Gui:Qt5Gui.dll
 0002:00000254       __imp_?pos@QCursor@@SA?AVQPoint@@XZ 10010254     Qt5Gui:Qt5Gui.dll
 0002:00000258       __imp_?width@QFontMetricsF@@QBENVQChar@@@Z 10010258     Qt5Gui:Qt5Gui.dll
 0002:0000025c       __imp_?ascent@QFontMetricsF@@QBENXZ 1001025c     Qt5Gui:Qt5Gui.dll
 0002:00000260       __imp_??1QFontMetricsF@@QAE@XZ 10010260     Qt5Gui:Qt5Gui.dll
 0002:00000264       __imp_??0QFontMetricsF@@QAE@ABVQFont@@@Z 10010264     Qt5Gui:Qt5Gui.dll
 0002:00000268       __imp_??4QFont@@QAEAAV0@ABV0@@Z 10010268     Qt5Gui:Qt5Gui.dll
 0002:0000026c       __imp_?setWeight@QFont@@QAEXH@Z 1001026c     Qt5Gui:Qt5Gui.dll
 0002:00000270       __imp_?setPointSize@QFont@@QAEXH@Z 10010270     Qt5Gui:Qt5Gui.dll
 0002:00000274       __imp_?setFamily@QFont@@QAEXABVQString@@@Z 10010274     Qt5Gui:Qt5Gui.dll
 0002:00000278       __imp_??1QFont@@QAE@XZ     10010278     Qt5Gui:Qt5Gui.dll
 0002:0000027c       __imp_??0QFont@@QAE@ABVQString@@HH_N@Z 1001027c     Qt5Gui:Qt5Gui.dll
 0002:00000280       __imp_??0QFont@@QAE@XZ     10010280     Qt5Gui:Qt5Gui.dll
 0002:00000284       __imp_??1QLinearGradient@@QAE@XZ 10010284     Qt5Gui:Qt5Gui.dll
 0002:00000288       __imp_??0QLinearGradient@@QAE@NNNN@Z 10010288     Qt5Gui:Qt5Gui.dll
 0002:0000028c       __imp_?setColorAt@QGradient@@QAEXNABVQColor@@@Z 1001028c     Qt5Gui:Qt5Gui.dll
 0002:00000290       __imp_??1QBrush@@QAE@XZ    10010290     Qt5Gui:Qt5Gui.dll
 0002:00000294       __imp_??0QBrush@@QAE@ABVQGradient@@@Z 10010294     Qt5Gui:Qt5Gui.dll
 0002:00000298       __imp_??0QBrush@@QAE@W4GlobalColor@Qt@@W4BrushStyle@2@@Z 10010298     Qt5Gui:Qt5Gui.dll
 0002:0000029c       __imp_??0QPolygonF@@QAE@H@Z 1001029c     Qt5Gui:Qt5Gui.dll
 0002:000002a0       __imp_??1QPolygonF@@QAE@XZ 100102a0     Qt5Gui:Qt5Gui.dll
 0002:000002a4       __imp_??0QColor@@QAE@W4GlobalColor@Qt@@@Z 100102a4     Qt5Gui:Qt5Gui.dll
 0002:000002a8       __imp_?height@QPaintDevice@@QBEHXZ 100102a8     Qt5Gui:Qt5Gui.dll
 0002:000002ac       __imp_?width@QPaintDevice@@QBEHXZ 100102ac     Qt5Gui:Qt5Gui.dll
 0002:000002b0       __imp_??1QIcon@@QAE@XZ     100102b0     Qt5Gui:Qt5Gui.dll
 0002:000002b4       __imp_??0QIcon@@QAE@ABVQString@@@Z 100102b4     Qt5Gui:Qt5Gui.dll
 0002:000002b8       \177Qt5Gui_NULL_THUNK_DATA 100102b8     Qt5Gui:Qt5Gui.dll
 0002:000002bc       __imp_?staticMetaObject@QWidget@@2UQMetaObject@@B 100102bc     Qt5Widgets:Qt5Widgets.dll
 0002:000002c0       __imp_?qt_metacall@QWidget@@UAEHW4Call@QMetaObject@@HPAPAX@Z 100102c0     Qt5Widgets:Qt5Widgets.dll
 0002:000002c4       __imp_?qt_metacast@QWidget@@UAEPAXPBD@Z 100102c4     Qt5Widgets:Qt5Widgets.dll
 0002:000002c8       __imp_?staticMetaObject@QAction@@2UQMetaObject@@B 100102c8     Qt5Widgets:Qt5Widgets.dll
 0002:000002cc       __imp_?widget@QLayoutItem@@UAEPAVQWidget@@XZ 100102cc     Qt5Widgets:Qt5Widgets.dll
 0002:000002d0       __imp_?wheelEvent@QWidget@@MAEXPAVQWheelEvent@@@Z 100102d0     Qt5Widgets:Qt5Widgets.dll
 0002:000002d4       __imp_?wheelEvent@QMenu@@MAEXPAVQWheelEvent@@@Z 100102d4     Qt5Widgets:Qt5Widgets.dll
 0002:000002d8       __imp_?timerEvent@QMenu@@MAEXPAVQTimerEvent@@@Z 100102d8     Qt5Widgets:Qt5Widgets.dll
 0002:000002dc       __imp_?takeAt@QBoxLayout@@UAEPAVQLayoutItem@@H@Z 100102dc     Qt5Widgets:Qt5Widgets.dll
 0002:000002e0       __imp_?tabletEvent@QWidget@@MAEXPAVQTabletEvent@@@Z 100102e0     Qt5Widgets:Qt5Widgets.dll
 0002:000002e4       __imp_?spacerItem@QLayoutItem@@UAEPAVQSpacerItem@@XZ 100102e4     Qt5Widgets:Qt5Widgets.dll
 0002:000002e8       __imp_?sizeHint@QWidget@@UBE?AVQSize@@XZ 100102e8     Qt5Widgets:Qt5Widgets.dll
 0002:000002ec       __imp_?sizeHint@QMenu@@UBE?AVQSize@@XZ 100102ec     Qt5Widgets:Qt5Widgets.dll
 0002:000002f0       __imp_?sizeHint@QBoxLayout@@UBE?AVQSize@@XZ 100102f0     Qt5Widgets:Qt5Widgets.dll
 0002:000002f4       __imp_?setIcon@QAction@@QAEXABVQIcon@@@Z 100102f4     Qt5Widgets:Qt5Widgets.dll
 0002:000002f8       __imp_?setCheckable@QAction@@QAEX_N@Z 100102f8     Qt5Widgets:Qt5Widgets.dll
 0002:000002fc       __imp_?isChecked@QAction@@QBE_NXZ 100102fc     Qt5Widgets:Qt5Widgets.dll
 0002:00000300       __imp_?activate@QAction@@QAEXW4ActionEvent@1@@Z 10010300     Qt5Widgets:Qt5Widgets.dll
 0002:00000304       __imp_?setChecked@QAction@@QAEX_N@Z 10010304     Qt5Widgets:Qt5Widgets.dll
 0002:00000308       __imp_?event@QAction@@MAE_NPAVQEvent@@@Z 10010308     Qt5Widgets:Qt5Widgets.dll
 0002:0000030c       __imp_??1QWidget@@UAE@XZ   1001030c     Qt5Widgets:Qt5Widgets.dll
 0002:00000310       __imp_?rect@QWidget@@QBE?AVQRect@@XZ 10010310     Qt5Widgets:Qt5Widgets.dll
 0002:00000314       __imp_?minimumSize@QWidget@@QBE?AVQSize@@XZ 10010314     Qt5Widgets:Qt5Widgets.dll
 0002:00000318       __imp_?setMinimumHeight@QWidget@@QAEXH@Z 10010318     Qt5Widgets:Qt5Widgets.dll
 0002:0000031c       __imp_?mapToGlobal@QWidget@@QBE?AVQPoint@@ABV2@@Z 1001031c     Qt5Widgets:Qt5Widgets.dll
 0002:00000320       __imp_?mapFromGlobal@QWidget@@QBE?AVQPoint@@ABV2@@Z 10010320     Qt5Widgets:Qt5Widgets.dll
 0002:00000324       __imp_?setFocus@QWidget@@QAEXW4FocusReason@Qt@@@Z 10010324     Qt5Widgets:Qt5Widgets.dll
 0002:00000328       __imp_?update@QWidget@@QAEXXZ 10010328     Qt5Widgets:Qt5Widgets.dll
 0002:0000032c       __imp_?setHidden@QWidget@@QAEX_N@Z 1001032c     Qt5Widgets:Qt5Widgets.dll
 0002:00000330       __imp_?addAction@QWidget@@QAEXPAVQAction@@@Z 10010330     Qt5Widgets:Qt5Widgets.dll
 0002:00000334       __imp_?insertAction@QWidget@@QAEXPAVQAction@@0@Z 10010334     Qt5Widgets:Qt5Widgets.dll
 0002:00000338       __imp_?actions@QWidget@@QBE?AV?$QList@PAVQAction@@@@XZ 10010338     Qt5Widgets:Qt5Widgets.dll
 0002:0000033c       __imp_?critical@QMessageBox@@SA?AW4StandardButton@1@PAVQWidget@@ABVQString@@1V?$QFlags@W4StandardButton@QMessageBox@@@@W421@@Z 1001033c     Qt5Widgets:Qt5Widgets.dll
 0002:00000340       __imp_??0QAction@@QAE@ABVQString@@PAVQObject@@@Z 10010340     Qt5Widgets:Qt5Widgets.dll
 0002:00000344       __imp_??1QAction@@UAE@XZ   10010344     Qt5Widgets:Qt5Widgets.dll
 0002:00000348       __imp_?text@QAction@@QBE?AVQString@@XZ 10010348     Qt5Widgets:Qt5Widgets.dll
 0002:0000034c       __imp_?setEnabled@QAction@@QAEX_N@Z 1001034c     Qt5Widgets:Qt5Widgets.dll
 0002:00000350       __imp_??0QMenu@@QAE@PAVQWidget@@@Z 10010350     Qt5Widgets:Qt5Widgets.dll
 0002:00000354       __imp_??0QMenu@@QAE@ABVQString@@PAVQWidget@@@Z 10010354     Qt5Widgets:Qt5Widgets.dll
 0002:00000358       __imp_??1QMenu@@UAE@XZ     10010358     Qt5Widgets:Qt5Widgets.dll
 0002:0000035c       __imp_?addAction@QMenu@@QAEPAVQAction@@ABVQString@@@Z 1001035c     Qt5Widgets:Qt5Widgets.dll
 0002:00000360       __imp_?addSeparator@QMenu@@QAEPAVQAction@@XZ 10010360     Qt5Widgets:Qt5Widgets.dll
 0002:00000364       __imp_?insertMenu@QMenu@@QAEPAVQAction@@PAV2@PAV1@@Z 10010364     Qt5Widgets:Qt5Widgets.dll
 0002:00000368       __imp_?insertSeparator@QMenu@@QAEPAVQAction@@PAV2@@Z 10010368     Qt5Widgets:Qt5Widgets.dll
 0002:0000036c       __imp_?popup@QMenu@@QAEXABVQPoint@@PAVQAction@@@Z 1001036c     Qt5Widgets:Qt5Widgets.dll
 0002:00000370       __imp_?menuAction@QMenu@@QBEPAVQAction@@XZ 10010370     Qt5Widgets:Qt5Widgets.dll
 0002:00000374       __imp_?setIcon@QAbstractButton@@QAEXABVQIcon@@@Z 10010374     Qt5Widgets:Qt5Widgets.dll
 0002:00000378       __imp_?setPopupMode@QToolButton@@QAEXW4ToolButtonPopupMode@1@@Z 10010378     Qt5Widgets:Qt5Widgets.dll
 0002:0000037c       __imp_?setMargin@QLayout@@QAEXH@Z 1001037c     Qt5Widgets:Qt5Widgets.dll
 0002:00000380       __imp_?addWidget@QBoxLayout@@QAEXPAVQWidget@@HV?$QFlags@W4AlignmentFlag@Qt@@@@@Z 10010380     Qt5Widgets:Qt5Widgets.dll
 0002:00000384       __imp_??0QHBoxLayout@@QAE@XZ 10010384     Qt5Widgets:Qt5Widgets.dll
 0002:00000388       __imp_??1QHBoxLayout@@UAE@XZ 10010388     Qt5Widgets:Qt5Widgets.dll
 0002:0000038c       __imp_?actionEvent@QMenu@@MAEXPAVQActionEvent@@@Z 1001038c     Qt5Widgets:Qt5Widgets.dll
 0002:00000390       __imp_?actionEvent@QWidget@@MAEXPAVQActionEvent@@@Z 10010390     Qt5Widgets:Qt5Widgets.dll
 0002:00000394       __imp_?addItem@QBoxLayout@@UAEXPAVQLayoutItem@@@Z 10010394     Qt5Widgets:Qt5Widgets.dll
 0002:00000398       __imp_?changeEvent@QMenu@@MAEXPAVQEvent@@@Z 10010398     Qt5Widgets:Qt5Widgets.dll
 0002:0000039c       __imp_?changeEvent@QWidget@@MAEXPAVQEvent@@@Z 1001039c     Qt5Widgets:Qt5Widgets.dll
 0002:000003a0       __imp_?childEvent@QLayout@@MAEXPAVQChildEvent@@@Z 100103a0     Qt5Widgets:Qt5Widgets.dll
 0002:000003a4       __imp_?closeEvent@QWidget@@MAEXPAVQCloseEvent@@@Z 100103a4     Qt5Widgets:Qt5Widgets.dll
 0002:000003a8       __imp_?contextMenuEvent@QWidget@@MAEXPAVQContextMenuEvent@@@Z 100103a8     Qt5Widgets:Qt5Widgets.dll
 0002:000003ac       __imp_?controlTypes@QLayout@@UBE?AV?$QFlags@W4ControlType@QSizePolicy@@@@XZ 100103ac     Qt5Widgets:Qt5Widgets.dll
 0002:000003b0       __imp_?count@QBoxLayout@@UBEHXZ 100103b0     Qt5Widgets:Qt5Widgets.dll
 0002:000003b4       __imp_?devType@QWidget@@UBEHXZ 100103b4     Qt5Widgets:Qt5Widgets.dll
 0002:000003b8       __imp_?dragEnterEvent@QWidget@@MAEXPAVQDragEnterEvent@@@Z 100103b8     Qt5Widgets:Qt5Widgets.dll
 0002:000003bc       __imp_?dragLeaveEvent@QWidget@@MAEXPAVQDragLeaveEvent@@@Z 100103bc     Qt5Widgets:Qt5Widgets.dll
 0002:000003c0       __imp_?dragMoveEvent@QWidget@@MAEXPAVQDragMoveEvent@@@Z 100103c0     Qt5Widgets:Qt5Widgets.dll
 0002:000003c4       __imp_?dropEvent@QWidget@@MAEXPAVQDropEvent@@@Z 100103c4     Qt5Widgets:Qt5Widgets.dll
 0002:000003c8       __imp_?enterEvent@QMenu@@MAEXPAVQEvent@@@Z 100103c8     Qt5Widgets:Qt5Widgets.dll
 0002:000003cc       __imp_?enterEvent@QWidget@@MAEXPAVQEvent@@@Z 100103cc     Qt5Widgets:Qt5Widgets.dll
 0002:000003d0       __imp_?event@QMenu@@MAE_NPAVQEvent@@@Z 100103d0     Qt5Widgets:Qt5Widgets.dll
 0002:000003d4       __imp_?event@QWidget@@MAE_NPAVQEvent@@@Z 100103d4     Qt5Widgets:Qt5Widgets.dll
 0002:000003d8       __imp_?expandingDirections@QBoxLayout@@UBE?AV?$QFlags@W4Orientation@Qt@@@@XZ 100103d8     Qt5Widgets:Qt5Widgets.dll
 0002:000003dc       __imp_?focusInEvent@QWidget@@MAEXPAVQFocusEvent@@@Z 100103dc     Qt5Widgets:Qt5Widgets.dll
 0002:000003e0       __imp_?focusNextPrevChild@QMenu@@MAE_N_N@Z 100103e0     Qt5Widgets:Qt5Widgets.dll
 0002:000003e4       __imp_?focusNextPrevChild@QWidget@@MAE_N_N@Z 100103e4     Qt5Widgets:Qt5Widgets.dll
 0002:000003e8       __imp_?focusOutEvent@QWidget@@MAEXPAVQFocusEvent@@@Z 100103e8     Qt5Widgets:Qt5Widgets.dll
 0002:000003ec       __imp_?geometry@QLayout@@UBE?AVQRect@@XZ 100103ec     Qt5Widgets:Qt5Widgets.dll
 0002:000003f0       __imp_?hasHeightForWidth@QBoxLayout@@UBE_NXZ 100103f0     Qt5Widgets:Qt5Widgets.dll
 0002:000003f4       __imp_?hasHeightForWidth@QWidget@@UBE_NXZ 100103f4     Qt5Widgets:Qt5Widgets.dll
 0002:000003f8       __imp_?heightForWidth@QBoxLayout@@UBEHH@Z 100103f8     Qt5Widgets:Qt5Widgets.dll
 0002:000003fc       __imp_?heightForWidth@QWidget@@UBEHH@Z 100103fc     Qt5Widgets:Qt5Widgets.dll
 0002:00000400       __imp_?hideEvent@QMenu@@MAEXPAVQHideEvent@@@Z 10010400     Qt5Widgets:Qt5Widgets.dll
 0002:00000404       __imp_?hideEvent@QWidget@@MAEXPAVQHideEvent@@@Z 10010404     Qt5Widgets:Qt5Widgets.dll
 0002:00000408       __imp_?indexOf@QLayout@@UBEHPAVQWidget@@@Z 10010408     Qt5Widgets:Qt5Widgets.dll
 0002:0000040c       __imp_?initPainter@QWidget@@MBEXPAVQPainter@@@Z 1001040c     Qt5Widgets:Qt5Widgets.dll
 0002:00000410       __imp_?inputMethodEvent@QWidget@@MAEXPAVQInputMethodEvent@@@Z 10010410     Qt5Widgets:Qt5Widgets.dll
 0002:00000414       __imp_?inputMethodQuery@QWidget@@UBE?AVQVariant@@W4InputMethodQuery@Qt@@@Z 10010414     Qt5Widgets:Qt5Widgets.dll
 0002:00000418       __imp_?invalidate@QBoxLayout@@UAEXXZ 10010418     Qt5Widgets:Qt5Widgets.dll
 0002:0000041c       __imp_?isEmpty@QLayout@@UBE_NXZ 1001041c     Qt5Widgets:Qt5Widgets.dll
 0002:00000420       __imp_?itemAt@QBoxLayout@@UBEPAVQLayoutItem@@H@Z 10010420     Qt5Widgets:Qt5Widgets.dll
 0002:00000424       __imp_?keyPressEvent@QMenu@@MAEXPAVQKeyEvent@@@Z 10010424     Qt5Widgets:Qt5Widgets.dll
 0002:00000428       __imp_?keyPressEvent@QWidget@@MAEXPAVQKeyEvent@@@Z 10010428     Qt5Widgets:Qt5Widgets.dll
 0002:0000042c       __imp_?keyReleaseEvent@QWidget@@MAEXPAVQKeyEvent@@@Z 1001042c     Qt5Widgets:Qt5Widgets.dll
 0002:00000430       __imp_?layout@QLayout@@UAEPAV1@XZ 10010430     Qt5Widgets:Qt5Widgets.dll
 0002:00000434       __imp_?leaveEvent@QMenu@@MAEXPAVQEvent@@@Z 10010434     Qt5Widgets:Qt5Widgets.dll
 0002:00000438       __imp_?leaveEvent@QWidget@@MAEXPAVQEvent@@@Z 10010438     Qt5Widgets:Qt5Widgets.dll
 0002:0000043c       __imp_?maximumSize@QBoxLayout@@UBE?AVQSize@@XZ 1001043c     Qt5Widgets:Qt5Widgets.dll
 0002:00000440       __imp_?metaObject@QAction@@UBEPBUQMetaObject@@XZ 10010440     Qt5Widgets:Qt5Widgets.dll
 0002:00000444       __imp_?metaObject@QHBoxLayout@@UBEPBUQMetaObject@@XZ 10010444     Qt5Widgets:Qt5Widgets.dll
 0002:00000448       __imp_?metaObject@QMenu@@UBEPBUQMetaObject@@XZ 10010448     Qt5Widgets:Qt5Widgets.dll
 0002:0000044c       __imp_?metric@QWidget@@MBEHW4PaintDeviceMetric@QPaintDevice@@@Z 1001044c     Qt5Widgets:Qt5Widgets.dll
 0002:00000450       __imp_?minimumHeightForWidth@QBoxLayout@@UBEHH@Z 10010450     Qt5Widgets:Qt5Widgets.dll
 0002:00000454       __imp_?minimumSize@QBoxLayout@@UBE?AVQSize@@XZ 10010454     Qt5Widgets:Qt5Widgets.dll
 0002:00000458       __imp_?minimumSizeHint@QWidget@@UBE?AVQSize@@XZ 10010458     Qt5Widgets:Qt5Widgets.dll
 0002:0000045c       __imp_?mouseDoubleClickEvent@QWidget@@MAEXPAVQMouseEvent@@@Z 1001045c     Qt5Widgets:Qt5Widgets.dll
 0002:00000460       __imp_?mouseMoveEvent@QMenu@@MAEXPAVQMouseEvent@@@Z 10010460     Qt5Widgets:Qt5Widgets.dll
 0002:00000464       __imp_?mouseMoveEvent@QWidget@@MAEXPAVQMouseEvent@@@Z 10010464     Qt5Widgets:Qt5Widgets.dll
 0002:00000468       __imp_?mousePressEvent@QMenu@@MAEXPAVQMouseEvent@@@Z 10010468     Qt5Widgets:Qt5Widgets.dll
 0002:0000046c       __imp_?mousePressEvent@QWidget@@MAEXPAVQMouseEvent@@@Z 1001046c     Qt5Widgets:Qt5Widgets.dll
 0002:00000470       __imp_?mouseReleaseEvent@QMenu@@MAEXPAVQMouseEvent@@@Z 10010470     Qt5Widgets:Qt5Widgets.dll
 0002:00000474       __imp_?mouseReleaseEvent@QWidget@@MAEXPAVQMouseEvent@@@Z 10010474     Qt5Widgets:Qt5Widgets.dll
 0002:00000478       __imp_?moveEvent@QWidget@@MAEXPAVQMoveEvent@@@Z 10010478     Qt5Widgets:Qt5Widgets.dll
 0002:0000047c       __imp_?nativeEvent@QWidget@@MAE_NABVQByteArray@@PAXPAJ@Z 1001047c     Qt5Widgets:Qt5Widgets.dll
 0002:00000480       __imp_?paintEngine@QWidget@@UBEPAVQPaintEngine@@XZ 10010480     Qt5Widgets:Qt5Widgets.dll
 0002:00000484       __imp_?paintEvent@QMenu@@MAEXPAVQPaintEvent@@@Z 10010484     Qt5Widgets:Qt5Widgets.dll
 0002:00000488       __imp_?paintEvent@QWidget@@MAEXPAVQPaintEvent@@@Z 10010488     Qt5Widgets:Qt5Widgets.dll
 0002:0000048c       __imp_?qt_metacall@QAction@@UAEHW4Call@QMetaObject@@HPAPAX@Z 1001048c     Qt5Widgets:Qt5Widgets.dll
 0002:00000490       __imp_?qt_metacall@QHBoxLayout@@UAEHW4Call@QMetaObject@@HPAPAX@Z 10010490     Qt5Widgets:Qt5Widgets.dll
 0002:00000494       __imp_?qt_metacall@QMenu@@UAEHW4Call@QMetaObject@@HPAPAX@Z 10010494     Qt5Widgets:Qt5Widgets.dll
 0002:00000498       __imp_?qt_metacast@QAction@@UAEPAXPBD@Z 10010498     Qt5Widgets:Qt5Widgets.dll
 0002:0000049c       __imp_?qt_metacast@QHBoxLayout@@UAEPAXPBD@Z 1001049c     Qt5Widgets:Qt5Widgets.dll
 0002:000004a0       __imp_?qt_metacast@QMenu@@UAEPAXPBD@Z 100104a0     Qt5Widgets:Qt5Widgets.dll
 0002:000004a4       __imp_?redirected@QWidget@@MBEPAVQPaintDevice@@PAVQPoint@@@Z 100104a4     Qt5Widgets:Qt5Widgets.dll
 0002:000004a8       __imp_?resizeEvent@QWidget@@MAEXPAVQResizeEvent@@@Z 100104a8     Qt5Widgets:Qt5Widgets.dll
 0002:000004ac       __imp_?setGeometry@QBoxLayout@@UAEXABVQRect@@@Z 100104ac     Qt5Widgets:Qt5Widgets.dll
 0002:000004b0       __imp_?setVisible@QWidget@@UAEX_N@Z 100104b0     Qt5Widgets:Qt5Widgets.dll
 0002:000004b4       __imp_?sharedPainter@QWidget@@MBEPAVQPainter@@XZ 100104b4     Qt5Widgets:Qt5Widgets.dll
 0002:000004b8       __imp_?showEvent@QWidget@@MAEXPAVQShowEvent@@@Z 100104b8     Qt5Widgets:Qt5Widgets.dll
 0002:000004bc       \177Qt5Widgets_NULL_THUNK_DATA 100104bc     Qt5Widgets:Qt5Widgets.dll
 0002:000004c0       __imp_?staticMetaObject@GObject@U2@@2UQMetaObject@@B 100104c0     U2Core:U2Core.dll
 0002:000004c4       __imp_??0Plugin@U2@@QAE@ABVQString@@0_NW4PluginState@1@@Z 100104c4     U2Core:U2Core.dll
 0002:000004c8       __imp_??1Plugin@U2@@UAE@XZ 100104c8     U2Core:U2Core.dll
 0002:000004cc       __imp_?getChromatogram@DNAChromatogramObject@U2@@QBEABVDNAChromatogram@2@XZ 100104cc     U2Core:U2Core.dll
 0002:000004d0       __imp_?findAllObjects@GObjectUtils@U2@@SA?AV?$QList@PAVGObject@U2@@@@W4UnloadedObjectFilter@2@VQString@@@Z 100104d0     U2Core:U2Core.dll
 0002:000004d4       __imp_?findObjectsRelatedToObjectByRole@GObjectUtils@U2@@SA?AV?$QList@PAVGObject@U2@@@@PBVGObject@2@VQString@@W4GObjectRelationRole@2@ABV3@W4UnloadedObjectFilter@2@@Z 100104d4     U2Core:U2Core.dll
 0002:000004d8       __imp_??0Logger@U2@@QAE@ABVQString@@@Z 100104d8     U2Core:U2Core.dll
 0002:000004dc       __imp_??1Logger@U2@@UAE@XZ 100104dc     U2Core:U2Core.dll
 0002:000004e0       __imp_?staticMetaObject@DNAChromatogramObject@U2@@2UQMetaObject@@B 100104e0     U2Core:U2Core.dll
 0002:000004e4       __imp_?CHROMATOGRAM@GObjectTypes@U2@@2VQString@@B 100104e4     U2Core:U2Core.dll
 0002:000004e8       __imp_??0GObjectReference@U2@@QAE@PBVGObject@1@_N@Z 100104e8     U2Core:U2Core.dll
 0002:000004ec       __imp_??1GObjectReference@U2@@QAE@XZ 100104ec     U2Core:U2Core.dll
 0002:000004f0       __imp_?getGObjectType@GObject@U2@@QBE?AVQString@@XZ 100104f0     U2Core:U2Core.dll
 0002:000004f4       __imp_??0DNAChromatogram@U2@@QAE@XZ 100104f4     U2Core:U2Core.dll
 0002:000004f8       __imp_??1DNAChromatogram@U2@@QAE@XZ 100104f8     U2Core:U2Core.dll
 0002:000004fc       __imp_??4DNAChromatogram@U2@@QAEAAV01@ABV01@@Z 100104fc     U2Core:U2Core.dll
 0002:00000500       __imp_??0DNASequence@U2@@QAE@ABVQByteArray@@PBVDNAAlphabet@1@@Z 10010500     U2Core:U2Core.dll
 0002:00000504       __imp_??1DNASequence@U2@@QAE@XZ 10010504     U2Core:U2Core.dll
 0002:00000508       __imp_?getSequenceLength@U2SequenceObject@U2@@QBE_JXZ 10010508     U2Core:U2Core.dll
 0002:0000050c       __imp_?getWholeSequenceData@U2SequenceObject@U2@@QBE?AVQByteArray@@AAVU2OpStatus@2@@Z 1001050c     U2Core:U2Core.dll
 0002:00000510       __imp_?setWholeSequence@U2SequenceObject@U2@@QAEXABVDNASequence@2@@Z 10010510     U2Core:U2Core.dll
 0002:00000514       __imp_?getAlphabet@U2SequenceObject@U2@@QBEPBVDNAAlphabet@2@XZ 10010514     U2Core:U2Core.dll
 0002:00000518       __imp_?replaceRegion@U2SequenceObject@U2@@QAEXABVU2Region@2@ABVDNASequence@2@AAVU2OpStatus@2@@Z 10010518     U2Core:U2Core.dll
 0002:0000051c       __imp_??0U2SequenceObjectConstraints@U2@@QAE@PAVQObject@@@Z 1001051c     U2Core:U2Core.dll
 0002:00000520       __imp_??1U2SequenceObjectConstraints@U2@@UAE@XZ 10010520     U2Core:U2Core.dll
 0002:00000524       __imp_??0GUrl@U2@@QAE@ABVQString@@@Z 10010524     U2Core:U2Core.dll
 0002:00000528       __imp_??0GUrl@U2@@QAE@ABV01@@Z 10010528     U2Core:U2Core.dll
 0002:0000052c       __imp_?dirPath@GUrl@U2@@QBE?AVQString@@XZ 1001052c     U2Core:U2Core.dll
 0002:00000530       __imp_?baseFileName@GUrl@U2@@QBE?AVQString@@XZ 10010530     U2Core:U2Core.dll
 0002:00000534       __imp_??1GUrl@U2@@QAE@XZ   10010534     U2Core:U2Core.dll
 0002:00000538       __imp_?addObject@Document@U2@@QAEXPAVGObject@2@@Z 10010538     U2Core:U2Core.dll
 0002:0000053c       __imp_?getDbiRef@Document@U2@@QBEABVU2DbiRef@2@XZ 1001053c     U2Core:U2Core.dll
 0002:00000540       __imp_?getNewDocFileNameExcludesHint@DocumentUtils@U2@@SA?AV?$QSet@VQString@@@@XZ 10010540     U2Core:U2Core.dll
 0002:00000544       __imp_?selectObjectByReference@GObjectUtils@U2@@SAPAVGObject@2@ABVGObjectReference@2@ABV?$QList@PAVGObject@U2@@@@W4UnloadedObjectFilter@2@@Z 10010544     U2Core:U2Core.dll
 0002:00000548       __imp_?rollFileName@GUrlUtils@U2@@SA?AVQString@@ABV3@ABV?$QSet@VQString@@@@@Z 10010548     U2Core:U2Core.dll
 0002:0000054c       __imp_?errorTitle@L10N@U2@@SA?AVQString@@XZ 1001054c     U2Core:U2Core.dll
 0002:00000550       __imp_?error@Logger@U2@@QAEXABVQString@@@Z 10010550     U2Core:U2Core.dll
 0002:00000554       __imp_?isCoR@U2OpStatus@U2@@UBE_NXZ 10010554     U2Core:U2Core.dll
 0002:00000558       __imp_??0LoadDocumentTaskConfig@U2@@QAE@_NABVGObjectReference@1@PAVLDTObjectFactory@1@@Z 10010558     U2Core:U2Core.dll
 0002:0000055c       __imp_??1LoadDocumentTaskConfig@U2@@QAE@XZ 1001055c     U2Core:U2Core.dll
 0002:00000560       __imp_??0LoadUnloadedDocumentTask@U2@@QAE@PAVDocument@1@ABVLoadDocumentTaskConfig@1@@Z 10010560     U2Core:U2Core.dll
 0002:00000564       __imp_??1LoadUnloadedDocumentTask@U2@@UAE@XZ 10010564     U2Core:U2Core.dll
 0002:00000568       __imp_??0TaskSignalMapper@U2@@QAE@PAVTask@1@@Z 10010568     U2Core:U2Core.dll
 0002:0000056c       __imp_??0U2OpStatusImpl@U2@@QAE@XZ 1001056c     U2Core:U2Core.dll
 0002:00000570       __imp_?getError@U2OpStatusImpl@U2@@UBE?AVQString@@XZ 10010570     U2Core:U2Core.dll
 0002:00000574       __imp_??1U2OpStatusImpl@U2@@UAE@XZ 10010574     U2Core:U2Core.dll
 0002:00000578       __imp_??0U2OpStatus2Log@U2@@QAE@W4LogLevel@1@@Z 10010578     U2Core:U2Core.dll
 0002:0000057c       __imp_??1U2OpStatus2Log@U2@@UAE@XZ 1001057c     U2Core:U2Core.dll
 0002:00000580       __imp_??0ProjectTreeControllerModeSettings@U2@@QAE@XZ 10010580     U2Core:U2Core.dll
 0002:00000584       __imp_??1ProjectTreeControllerModeSettings@U2@@QAE@XZ 10010584     U2Core:U2Core.dll
 0002:00000588       __imp_?getProject@AppContext@U2@@SAPAVProject@2@XZ 10010588     U2Core:U2Core.dll
 0002:0000058c       __imp_?getDocumentFormatRegistry@AppContext@U2@@SAPAVDocumentFormatRegistry@2@XZ 1001058c     U2Core:U2Core.dll
 0002:00000590       __imp_?getIOAdapterRegistry@AppContext@U2@@SAPAVIOAdapterRegistry@2@XZ 10010590     U2Core:U2Core.dll
 0002:00000594       __imp_?getTaskScheduler@AppContext@U2@@SAPAVTaskScheduler@2@XZ 10010594     U2Core:U2Core.dll
 0002:00000598       __imp_?cleanup@DocumentProviderTask@U2@@UAEXXZ 10010598     U2Core:U2Core.dll
 0002:0000059c       __imp_?generateReport@Task@U2@@UBE?AVQString@@XZ 1001059c     U2Core:U2Core.dll
 0002:000005a0       __imp_?getDocument@LoadUnloadedDocumentTask@U2@@UAEPAVDocument@2@_N@Z 100105a0     U2Core:U2Core.dll
 0002:000005a4       __imp_?getDocumentDescription@DocumentProviderTask@U2@@UBE?AVQString@@XZ 100105a4     U2Core:U2Core.dll
 0002:000005a8       __imp_?getNumParallelSubtasks@Task@U2@@UBEHXZ 100105a8     U2Core:U2Core.dll
 0002:000005ac       __imp_?getParentTask@Task@U2@@UBEPAV12@XZ 100105ac     U2Core:U2Core.dll
 0002:000005b0       __imp_?getSubtaskWithErrors@Task@U2@@UBEPAV12@XZ 100105b0     U2Core:U2Core.dll
 0002:000005b4       __imp_?getTaskId@Task@U2@@UBE_JXZ 100105b4     U2Core:U2Core.dll
 0002:000005b8       __imp_?getTopLevelParentTask@Task@U2@@UAEPAV12@XZ 100105b8     U2Core:U2Core.dll
 0002:000005bc       __imp_?getWarnings@Task@U2@@UBE?AVQStringList@@XZ 100105bc     U2Core:U2Core.dll
 0002:000005c0       __imp_?hasSubtasksWithErrors@Task@U2@@UBE_NXZ 100105c0     U2Core:U2Core.dll
 0002:000005c4       __imp_?hasWarning@Task@U2@@UBE_NXZ 100105c4     U2Core:U2Core.dll
 0002:000005c8       __imp_?isNotificationReport@Task@U2@@UBE_NXZ 100105c8     U2Core:U2Core.dll
 0002:000005cc       __imp_?isReportingEnabled@Task@U2@@UBE_NXZ 100105cc     U2Core:U2Core.dll
 0002:000005d0       __imp_?isReportingSupported@Task@U2@@UBE_NXZ 100105d0     U2Core:U2Core.dll
 0002:000005d4       __imp_?isTopLevelTask@Task@U2@@UBE_NXZ 100105d4     U2Core:U2Core.dll
 0002:000005d8       __imp_?metaObject@LoadUnloadedDocumentTask@U2@@UBEPBUQMetaObject@@XZ 100105d8     U2Core:U2Core.dll
 0002:000005dc       __imp_?metaObject@TaskSignalMapper@U2@@UBEPBUQMetaObject@@XZ 100105dc     U2Core:U2Core.dll
 0002:000005e0       __imp_?onSubTaskFinished@Task@U2@@MAE?AV?$QList@PAVTask@U2@@@@PAV12@@Z 100105e0     U2Core:U2Core.dll
 0002:000005e4       __imp_?prepare@LoadUnloadedDocumentTask@U2@@UAEXXZ 100105e4     U2Core:U2Core.dll
 0002:000005e8       __imp_?propagateSubtaskError@Task@U2@@UAE_NXZ 100105e8     U2Core:U2Core.dll
 0002:000005ec       __imp_?qt_metacall@LoadUnloadedDocumentTask@U2@@UAEHW4Call@QMetaObject@@HPAPAX@Z 100105ec     U2Core:U2Core.dll
 0002:000005f0       __imp_?qt_metacall@TaskSignalMapper@U2@@UAEHW4Call@QMetaObject@@HPAPAX@Z 100105f0     U2Core:U2Core.dll
 0002:000005f4       __imp_?qt_metacast@LoadUnloadedDocumentTask@U2@@UAEPAXPBD@Z 100105f4     U2Core:U2Core.dll
 0002:000005f8       __imp_?qt_metacast@TaskSignalMapper@U2@@UAEPAXPBD@Z 100105f8     U2Core:U2Core.dll
 0002:000005fc       __imp_?report@LoadUnloadedDocumentTask@U2@@UAE?AW4ReportResult@Task@2@XZ 100105fc     U2Core:U2Core.dll
 0002:00000600       __imp_?run@Task@U2@@UAEXXZ 10010600     U2Core:U2Core.dll
 0002:00000604       __imp_?setCollectChildrensWarningsFlag@Task@U2@@UAEX_N@Z 10010604     U2Core:U2Core.dll
 0002:00000608       __imp_?setNoAutoDelete@Task@U2@@UAEX_N@Z 10010608     U2Core:U2Core.dll
 0002:0000060c       __imp_?setNotificationReport@Task@U2@@UAEX_N@Z 1001060c     U2Core:U2Core.dll
 0002:00000610       __imp_?setReportingEnabled@Task@U2@@UAEX_N@Z 10010610     U2Core:U2Core.dll
 0002:00000614       __imp_?setReportingSupported@Task@U2@@UAEX_N@Z 10010614     U2Core:U2Core.dll
 0002:00000618       __imp_?takeDocument@DocumentProviderTask@U2@@UAEPAVDocument@2@_N@Z 10010618     U2Core:U2Core.dll
 0002:0000061c       __imp_?staticMetaObject@U2SequenceObject@U2@@2UQMetaObject@@B 1001061c     U2Core:U2Core.dll
 0002:00000620       __imp_?UNLOADED@GObjectTypes@U2@@2VQString@@B 10010620     U2Core:U2Core.dll
 0002:00000624       __imp_?SEQUENCE@GObjectTypes@U2@@2VQString@@B 10010624     U2Core:U2Core.dll
 0002:00000628       __imp_?staticMetaObject@LoadUnloadedDocumentTask@U2@@2UQMetaObject@@B 10010628     U2Core:U2Core.dll
 0002:0000062c       __imp_?qt_metacast@Plugin@U2@@UAEPAXPBD@Z 1001062c     U2Core:U2Core.dll
 0002:00000630       __imp_?qt_metacall@Plugin@U2@@UAEHW4Call@QMetaObject@@HPAPAX@Z 10010630     U2Core:U2Core.dll
 0002:00000634       __imp_?staticMetaObject@Plugin@U2@@2UQMetaObject@@B 10010634     U2Core:U2Core.dll
 0002:00000638       __imp_?getMainWindow@AppContext@U2@@SAPAVMainWindow@2@XZ 10010638     U2Core:U2Core.dll
 0002:0000063c       \177U2Core_NULL_THUNK_DATA 1001063c     U2Core:U2Core.dll
 0002:00000640       __imp_??0GObjectViewWindowContext@U2@@QAE@PAVQObject@@ABVGObjectViewFactoryId@1@@Z 10010640     U2Gui:U2Gui.dll
 0002:00000644       __imp_??1GObjectViewWindowContext@U2@@UAE@XZ 10010644     U2Gui:U2Gui.dll
 0002:00000648       __imp_?buildMenu@GObjectViewWindowContext@U2@@MAEXPAVGObjectView@2@PAVQMenu@@@Z 10010648     U2Gui:U2Gui.dll
 0002:0000064c       __imp_?disconnectView@GObjectViewWindowContext@U2@@MAEXPAVGObjectView@2@@Z 1001064c     U2Gui:U2Gui.dll
 0002:00000650       __imp_?init@GObjectViewWindowContext@U2@@UAEXXZ 10010650     U2Gui:U2Gui.dll
 0002:00000654       __imp_?onObjectAdded@GObjectViewObjectHandler@U2@@UAEXPAVGObjectView@2@PAVGObject@2@@Z 10010654     U2Gui:U2Gui.dll
 0002:00000658       __imp_?onObjectRemoved@GObjectViewWindowContext@U2@@UAEXPAVGObjectView@2@PAVGObject@2@@Z 10010658     U2Gui:U2Gui.dll
 0002:0000065c       __imp_?sl_buildContextMenu@GObjectViewWindowContext@U2@@MAEXPAVGObjectView@2@PAVQMenu@@@Z 1001065c     U2Gui:U2Gui.dll
 0002:00000660       __imp_?sl_buildStaticMenu@GObjectViewWindowContext@U2@@MAEXPAVGObjectView@2@PAVQMenu@@@Z 10010660     U2Gui:U2Gui.dll
 0002:00000664       __imp_?sl_windowAdded@GObjectViewWindowContext@U2@@MAEXPAVMWMDIWindow@2@@Z 10010664     U2Gui:U2Gui.dll
 0002:00000668       __imp_?sl_windowClosing@GObjectViewWindowContext@U2@@MAEXPAVMWMDIWindow@2@@Z 10010668     U2Gui:U2Gui.dll
 0002:0000066c       __imp_??0AddNewDocumentDialogModel@U2@@QAE@ABVQString@@V2@@Z 1001066c     U2Gui:U2Gui.dll
 0002:00000670       __imp_??1AddNewDocumentDialogModel@U2@@QAE@XZ 10010670     U2Gui:U2Gui.dll
 0002:00000674       __imp_?run@AddNewDocumentDialogController@U2@@SAXPAVQWidget@@AAVAddNewDocumentDialogModel@2@ABVDocumentFormatConstraints@2@@Z 10010674     U2Gui:U2Gui.dll
 0002:00000678       __imp_?findActionAfter@GUIUtils@U2@@SAPAVQAction@@ABV?$QList@PAVQAction@@@@ABVQString@@@Z 10010678     U2Gui:U2Gui.dll
 0002:0000067c       __imp_?selectObjects@ProjectTreeItemSelectorDialog@U2@@SA?AV?$QList@PAVGObject@U2@@@@ABVProjectTreeControllerModeSettings@2@PAVQWidget@@@Z 1001067c     U2Gui:U2Gui.dll
 0002:00000680       __imp_?setContentLayout@WidgetWithLocalToolbar@U2@@QAEXPAVQLayout@@@Z 10010680     U2Gui:U2Gui.dll
 0002:00000684       __imp_?addActionToLocalToolbar@WidgetWithLocalToolbar@U2@@QAEPAVQToolButton@@PAVQAction@@@Z 10010684     U2Gui:U2Gui.dll
 0002:00000688       __imp_??0ScaleBar@U2@@QAE@W4Orientation@Qt@@PAVQWidget@@@Z 10010688     U2Gui:U2Gui.dll
 0002:0000068c       __imp_?setValue@ScaleBar@U2@@QAEXH@Z 1001068c     U2Gui:U2Gui.dll
 0002:00000690       __imp_?setRange@ScaleBar@U2@@QAEXHH@Z 10010690     U2Gui:U2Gui.dll
 0002:00000694       __imp_?setTickInterval@ScaleBar@U2@@QAEXH@Z 10010694     U2Gui:U2Gui.dll
 0002:00000698       __imp_?metaObject@ScaleBar@U2@@UBEPBUQMetaObject@@XZ 10010698     U2Gui:U2Gui.dll
 0002:0000069c       __imp_?qt_metacall@ScaleBar@U2@@UAEHW4Call@QMetaObject@@HPAPAX@Z 1001069c     U2Gui:U2Gui.dll
 0002:000006a0       __imp_?qt_metacast@ScaleBar@U2@@UAEPAXPBD@Z 100106a0     U2Gui:U2Gui.dll
 0002:000006a4       __imp_?qt_metacast@GObjectViewWindowContext@U2@@UAEPAXPBD@Z 100106a4     U2Gui:U2Gui.dll
 0002:000006a8       __imp_?qt_metacall@GObjectViewWindowContext@U2@@UAEHW4Call@QMetaObject@@HPAPAX@Z 100106a8     U2Gui:U2Gui.dll
 0002:000006ac       __imp_?staticMetaObject@GObjectViewWindowContext@U2@@2UQMetaObject@@B 100106ac     U2Gui:U2Gui.dll
 0002:000006b0       \177U2Gui_NULL_THUNK_DATA  100106b0     U2Gui:U2Gui.dll
 0002:000006b4       __imp_??0ADVSequenceWidgetAction@U2@@QAE@ABVQString@@0@Z 100106b4     U2View:U2View.dll
 0002:000006b8       __imp_??1ADVSequenceWidgetAction@U2@@UAE@XZ 100106b8     U2View:U2View.dll
 0002:000006bc       __imp_?getSequenceWidgets@AnnotatedDNAView@U2@@QBE?BV?$QList@PAVADVSequenceWidget@U2@@@@XZ 100106bc     U2View:U2View.dll
 0002:000006c0       __imp_?getPanGSLView@ADVSingleSequenceWidget@U2@@QBEPAVGSequenceLineView@2@XZ 100106c0     U2View:U2View.dll
 0002:000006c4       __imp_?getSequenceContext@ADVSingleSequenceWidget@U2@@QBEPAVADVSequenceObjectContext@2@XZ 100106c4     U2View:U2View.dll
 0002:000006c8       __imp_?getSequenceObject@ADVSingleSequenceWidget@U2@@QBEPAVU2SequenceObject@2@XZ 100106c8     U2View:U2View.dll
 0002:000006cc       __imp_?addADVSequenceWidgetActionToViewsToolbar@ADVSingleSequenceWidget@U2@@QAEXPAVADVSequenceWidgetAction@2@@Z 100106cc     U2View:U2View.dll
 0002:000006d0       __imp_?staticMetaObject@AnnotatedDNAView@U2@@2UQMetaObject@@B 100106d0     U2View:U2View.dll
 0002:000006d4       __imp_?staticMetaObject@ADVSingleSequenceWidget@U2@@2UQMetaObject@@B 100106d4     U2View:U2View.dll
 0002:000006d8       __imp_?getSequenceGObject@SequenceObjectContext@U2@@QBEPAVGObject@2@XZ 100106d8     U2View:U2View.dll
 0002:000006dc       __imp_?getSequenceLength@SequenceObjectContext@U2@@QBE_JXZ 100106dc     U2View:U2View.dll
 0002:000006e0       __imp_?getSequenceData@SequenceObjectContext@U2@@QBE?AVQByteArray@@ABVU2Region@2@AAVU2OpStatus@2@@Z 100106e0     U2View:U2View.dll
 0002:000006e4       __imp_??0GSequenceLineView@U2@@QAE@PAVQWidget@@PAVSequenceObjectContext@1@@Z 100106e4     U2View:U2View.dll
 0002:000006e8       __imp_?setCoherentRangeView@GSequenceLineView@U2@@UAEXPAV12@@Z 100106e8     U2View:U2View.dll
 0002:000006ec       __imp_?mousePressEvent@GSequenceLineView@U2@@MAEXPAVQMouseEvent@@@Z 100106ec     U2View:U2View.dll
 0002:000006f0       __imp_?completeUpdate@GSequenceLineView@U2@@IAEXXZ 100106f0     U2View:U2View.dll
 0002:000006f4       __imp_?toRenderAreaPoint@GSequenceLineView@U2@@IBE?AVQPoint@@ABV3@@Z 100106f4     U2View:U2View.dll
 0002:000006f8       __imp_??1GSequenceLineView@U2@@UAE@XZ 100106f8     U2View:U2View.dll
 0002:000006fc       __imp_??0GSequenceLineViewRenderArea@U2@@QAE@PAVGSequenceLineView@1@@Z 100106fc     U2View:U2View.dll
 0002:00000700       __imp_??1GSequenceLineViewRenderArea@U2@@UAE@XZ 10010700     U2View:U2View.dll
 0002:00000704       __imp_?addUpdateFlags@GSequenceLineView@U2@@UAEXV?$QFlags@W4GSLV_UpdateFlag@U2@@@@@Z 10010704     U2View:U2View.dll
 0002:00000708       __imp_?clearUpdateFlags@GSequenceLineView@U2@@UAEXXZ 10010708     U2View:U2View.dll
 0002:0000070c       __imp_?coordToPos@GSequenceLineViewRenderArea@U2@@UBE_JABVQPoint@@@Z 1001070c     U2View:U2View.dll
 0002:00000710       __imp_?drawFocus@GSequenceLineViewRenderArea@U2@@MAEXAAVQPainter@@@Z 10010710     U2View:U2View.dll
 0002:00000714       __imp_?eventFilter@GSequenceLineView@U2@@UAE_NPAVQObject@@PAVQEvent@@@Z 10010714     U2View:U2View.dll
 0002:00000718       __imp_?focusInEvent@GSequenceLineView@U2@@MAEXPAVQFocusEvent@@@Z 10010718     U2View:U2View.dll
 0002:0000071c       __imp_?focusOutEvent@GSequenceLineView@U2@@MAEXPAVQFocusEvent@@@Z 1001071c     U2View:U2View.dll
 0002:00000720       __imp_?getConherentRangeView@GSequenceLineView@U2@@UBEPAV12@XZ 10010720     U2View:U2View.dll
 0002:00000724       __imp_?getCurrentScale@GSequenceLineViewRenderArea@U2@@UBENXZ 10010724     U2View:U2View.dll
 0002:00000728       __imp_?getFrameView@GSequenceLineView@U2@@UBEPAV12@XZ 10010728     U2View:U2View.dll
 0002:0000072c       __imp_?getPageStep@GSequenceLineView@U2@@MBEHXZ 1001072c     U2View:U2View.dll
 0002:00000730       __imp_?getSequenceObject@GSequenceLineView@U2@@UBEPAVU2SequenceObject@2@XZ 10010730     U2View:U2View.dll
 0002:00000734       __imp_?getSingleStep@GSequenceLineView@U2@@MBEHXZ 10010734     U2View:U2View.dll
 0002:00000738       __imp_?getZoomInAction@GSequenceLineView@U2@@UBEPAVQAction@@XZ 10010738     U2View:U2View.dll
 0002:0000073c       __imp_?getZoomOutAction@GSequenceLineView@U2@@UBEPAVQAction@@XZ 1001073c     U2View:U2View.dll
 0002:00000740       __imp_?getZoomToSelectionAction@GSequenceLineView@U2@@UBEPAVQAction@@XZ 10010740     U2View:U2View.dll
 0002:00000744       __imp_?getZoomToSequenceAction@GSequenceLineView@U2@@UBEPAVQAction@@XZ 10010744     U2View:U2View.dll
 0002:00000748       __imp_?keyPressEvent@GSequenceLineView@U2@@MAEXPAVQKeyEvent@@@Z 10010748     U2View:U2View.dll
 0002:0000074c       __imp_?mouseDoubleClickEvent@GSequenceLineView@U2@@MAEXPAVQMouseEvent@@@Z 1001074c     U2View:U2View.dll
 0002:00000750       __imp_?mouseMoveEvent@GSequenceLineView@U2@@MAEXPAVQMouseEvent@@@Z 10010750     U2View:U2View.dll
 0002:00000754       __imp_?mouseReleaseEvent@GSequenceLineView@U2@@MAEXPAVQMouseEvent@@@Z 10010754     U2View:U2View.dll
 0002:00000758       __imp_?moveBorder@GSequenceLineView@U2@@MAEXABVQPoint@@@Z 10010758     U2View:U2View.dll
 0002:0000075c       __imp_?onVisibleRangeChanged@GSequenceLineView@U2@@MAEX_N@Z 1001075c     U2View:U2View.dll
 0002:00000760       __imp_?paintEvent@GSequenceLineViewRenderArea@U2@@MAEXPAVQPaintEvent@@@Z 10010760     U2View:U2View.dll
 0002:00000764       __imp_?posToCoordF@GSequenceLineViewRenderArea@U2@@UBEM_J_N@Z 10010764     U2View:U2View.dll
 0002:00000768       __imp_?resizeEvent@GSequenceLineView@U2@@MAEXPAVQResizeEvent@@@Z 10010768     U2View:U2View.dll
 0002:0000076c       __imp_?resizeSelection@GSequenceLineView@U2@@MAEXABVQPoint@@@Z 1001076c     U2View:U2View.dll
 0002:00000770       __imp_?setBorderCursor@GSequenceLineView@U2@@MAEXABVQPoint@@@Z 10010770     U2View:U2View.dll
 0002:00000774       __imp_?setCenterPos@GSequenceLineView@U2@@UAEX_J@Z 10010774     U2View:U2View.dll
 0002:00000778       __imp_?setFrameView@GSequenceLineView@U2@@UAEXPAV12@@Z 10010778     U2View:U2View.dll
 0002:0000077c       __imp_?setStartPos@GSequenceLineView@U2@@UAEX_J@Z 1001077c     U2View:U2View.dll
 0002:00000780       __imp_?setVisibleRange@GSequenceLineView@U2@@UAEXABVU2Region@2@_N@Z 10010780     U2View:U2View.dll
 0002:00000784       __imp_?sl_onDNASelectionChanged@GSequenceLineView@U2@@MAEXPAVLRegionsSelection@2@ABV?$QVector@VU2Region@U2@@@@1@Z 10010784     U2View:U2View.dll
 0002:00000788       __imp_?sl_onScrollBarMoved@GSequenceLineView@U2@@MAEXH@Z 10010788     U2View:U2View.dll
 0002:0000078c       __imp_?sl_sequenceChanged@GSequenceLineView@U2@@MAEXXZ 1001078c     U2View:U2View.dll
 0002:00000790       __imp_?updateScrollBar@GSequenceLineView@U2@@MAEXXZ 10010790     U2View:U2View.dll
 0002:00000794       __imp_?wheelEvent@GSequenceLineView@U2@@MAEXPAVQWheelEvent@@@Z 10010794     U2View:U2View.dll
 0002:00000798       __imp_?qt_metacast@ADVSequenceWidgetAction@U2@@UAEPAXPBD@Z 10010798     U2View:U2View.dll
 0002:0000079c       __imp_?qt_metacall@ADVSequenceWidgetAction@U2@@UAEHW4Call@QMetaObject@@HPAPAX@Z 1001079c     U2View:U2View.dll
 0002:000007a0       __imp_?staticMetaObject@ADVSequenceWidget@U2@@2UQMetaObject@@B 100107a0     U2View:U2View.dll
 0002:000007a4       __imp_?staticMetaObject@ADVSequenceWidgetAction@U2@@2UQMetaObject@@B 100107a4     U2View:U2View.dll
 0002:000007a8       __imp_?qt_metacast@GSequenceLineView@U2@@UAEPAXPBD@Z 100107a8     U2View:U2View.dll
 0002:000007ac       __imp_?qt_metacall@GSequenceLineView@U2@@UAEHW4Call@QMetaObject@@HPAPAX@Z 100107ac     U2View:U2View.dll
 0002:000007b0       __imp_?staticMetaObject@GSequenceLineView@U2@@2UQMetaObject@@B 100107b0     U2View:U2View.dll
 0002:000007b4       \177U2View_NULL_THUNK_DATA 100107b4     U2View:U2View.dll
 0002:000007b8       ___xc_a                    100107b8     MSVCRT:cinitexe.obj
 0002:000008c4       ___xc_z                    100108c4     MSVCRT:cinitexe.obj
 0002:000008c8       ___xi_a                    100108c8     MSVCRT:cinitexe.obj
 0002:000008d4       ___xi_z                    100108d4     MSVCRT:cinitexe.obj
 0002:0000091c       ??_7error_category@std@@6B@ 1001091c     ChromaViewPlugin.obj
 0002:00000938       ??_7_Generic_error_category@std@@6B@ 10010938     ChromaViewPlugin.obj
 0002:00000950       ??_C@_07DCLBNMLN@generic?$AA@ 10010950     ChromaViewPlugin.obj
 0002:00000958       ??_C@_0O@BFJCFAAK@unknown?5error?$AA@ 10010958     ChromaViewPlugin.obj
 0002:0000096c       ??_7_Iostream_error_category@std@@6B@ 1001096c     ChromaViewPlugin.obj
 0002:00000984       ??_C@_08LLGCOLLL@iostream?$AA@ 10010984     ChromaViewPlugin.obj
 0002:00000990       ??_C@_0BG@PADBLCHM@iostream?5stream?5error?$AA@ 10010990     ChromaViewPlugin.obj
 0002:000009ac       ??_7_System_error_category@std@@6B@ 100109ac     ChromaViewPlugin.obj
 0002:000009c4       ??_C@_06FHFOAHML@system?$AA@ 100109c4     ChromaViewPlugin.obj
 0002:000009d0       ??_7?$AbstractId@H@U2@@6B@ 100109d0     ChromaViewPlugin.obj
 0002:000009dc       ??_7AbstractInt32Id@U2@@6B@ 100109dc     ChromaViewPlugin.obj
 0002:000009e8       ??_7ServiceType@U2@@6B@    100109e8     ChromaViewPlugin.obj
 0002:000009f4       ??_7ChromaViewPlugin@U2@@6B@ 100109f4     ChromaViewPlugin.obj
 0002:00000a24       ??_7ChromaViewContext@U2@@6BQObject@@@ 10010a24     ChromaViewPlugin.obj
 0002:00000a74       ??_7ChromaViewContext@U2@@6BGObjectViewObjectHandler@1@@ 10010a74     ChromaViewPlugin.obj
 0002:00000a88       ??_7ChromaViewAction@U2@@6B@ 10010a88     ChromaViewPlugin.obj
 0002:00000ab4       ??_C@_0L@JLHNEGIN@Algorithms?$AA@ 10010ab4     ChromaViewPlugin.obj
 0002:00000ac0       ??_C@_07PGLPGHFC@Console?$AA@ 10010ac0     ChromaViewPlugin.obj
 0002:00000ac8       ??_C@_0O@BOFHOPCF@Core?5Services?$AA@ 10010ac8     ChromaViewPlugin.obj
 0002:00000ad8       ??_C@_0N@PPADAKBM@Input?1Output?$AA@ 10010ad8     ChromaViewPlugin.obj
 0002:00000ae8       ??_C@_0M@KPPBKPKK@Performance?$AA@ 10010ae8     ChromaViewPlugin.obj
 0002:00000af4       ??_C@_07BFDHHBBI@Scripts?$AA@ 10010af4     ChromaViewPlugin.obj
 0002:00000afc       ??_C@_05EEGKELMG@Tasks?$AA@ 10010afc     ChromaViewPlugin.obj
 0002:00000b04       ??_C@_0P@NIIOBHGA@User?5Interface?$AA@ 10010b04     ChromaViewPlugin.obj
 0002:00000b14       ??_C@_0N@JINCGGMN@User?5Actions?$AA@ 10010b14     ChromaViewPlugin.obj
 0002:00000b24       ??_C@_0BM@JHHMCLOL@Chromatograms?5visualization?$AA@ 10010b24     ChromaViewPlugin.obj
 0002:00000b40       ??_C@_0BC@NMLFKJIM@Chromatogram?5View?$AA@ 10010b40     ChromaViewPlugin.obj
 0002:00000b54       ??_C@_0BB@JDMPMKOK@AnnotatedDNAView?$AA@ 10010b54     ChromaViewPlugin.obj
 0002:00000b68       ??_C@_0CM@JOICIJIL@1sl_sequenceWidgetAdded?$CIADVSeque@ 10010b68     ChromaViewPlugin.obj
 0002:00000b94       ??_C@_0CM@KILGFMLI@2si_sequenceWidgetAdded?$CIADVSeque@ 10010b94     ChromaViewPlugin.obj
 0002:00000bc0       ??_C@_0BL@IKEJIJNG@?3chroma_view?1images?1cv?4png?$AA@ 10010bc0     ChromaViewPlugin.obj
 0002:00000bdc       ??_C@_0BH@HEOMJEBP@1sl_showChromatogram?$CI?$CJ?$AA@ 10010bdc     ChromaViewPlugin.obj
 0002:00000bf4       ??_C@_0N@NBJIAFIH@2triggered?$CI?$CJ?$AA@ 10010bf4     ChromaViewPlugin.obj
 0002:00000c04       ??_C@_0BC@KMGEHOJE@Show?5chromatogram?$AA@ 10010c04     ChromaViewPlugin.obj
 0002:00000c18       ??_C@_0O@BKEKJFJF@CHROMA_ACTION?$AA@ 10010c18     ChromaViewPlugin.obj
 0002:00000c28       ??_C@_0BA@JFNIOLAK@string?5too?5long?$AA@ 10010c28     ChromaViewPlugin.obj
 0002:00000c38       ??_C@_0BI@CFPLBAOH@invalid?5string?5position?$AA@ 10010c38     ChromaViewPlugin.obj
 0002:00000c50       ??_C@_01GFHCPBMG@C?$AA@    10010c50     ChromatogramView.obj
 0002:00000c5c       ??_SLoadUnloadedDocumentTask@U2@@6B@ 10010c5c     ChromatogramView.obj
 0002:00000cf8       ??_SQAction@@6B@           10010cf8     ChromatogramView.obj
 0002:00000d28       ??_STaskSignalMapper@U2@@6B@ 10010d28     ChromatogramView.obj
 0002:00000d5c       ??_SQMenu@@6BQObject@@@    10010d5c     ChromatogramView.obj
 0002:00000e14       ??_SQMenu@@6BQPaintDevice@@@ 10010e14     ChromatogramView.obj
 0002:00000e34       ??_SQHBoxLayout@@6BQObject@@@ 10010e34     ChromatogramView.obj
 0002:00000e7c       ??_SQHBoxLayout@@6BQLayoutItem@@@ 10010e7c     ChromatogramView.obj
 0002:00000ec4       ??_SScaleBar@U2@@6BQObject@@@ 10010ec4     ChromatogramView.obj
 0002:00000f7c       ??_SScaleBar@U2@@6BQPaintDevice@@@ 10010f7c     ChromatogramView.obj
 0002:00000f9c       ??_7ChromatogramView@U2@@6BQObject@@@ 10010f9c     ChromatogramView.obj
 0002:000010c0       ??_7ChromatogramView@U2@@6BQPaintDevice@@@ 100110c0     ChromatogramView.obj
 0002:000010e0       ??_7ChromatogramViewRenderArea@U2@@6BQObject@@@ 100110e0     ChromatogramView.obj
 0002:000011b4       ??_7ChromatogramViewRenderArea@U2@@6BQPaintDevice@@@ 100111b4     ChromatogramView.obj
 0002:000011d0       ??_C@_0BD@OCPJOINJ@chromatogram_view_?$AA@ 100111d0     ChromatogramView.obj
 0002:000011e4       ??_C@_0BC@IAKIHKBD@Show?5quality?5bars?$AA@ 100111e4     ChromatogramView.obj
 0002:000011f8       ??_C@_0BN@LNCKCCGN@?3chroma_view?1images?1bars?4png?$AA@ 100111f8     ChromatogramView.obj
 0002:00001218       ??_C@_0BC@MACDHODD@1completeUpdate?$CI?$CJ?$AA@ 10011218     ChromatogramView.obj
 0002:0000122c       ??_C@_0P@POCECEMJ@2toggled?$CIbool?$CJ?$AA@ 1001122c     ChromatogramView.obj
 0002:0000123c       ??_C@_08PACAIFBE@Show?5all?$AA@ 1001123c     ChromatogramView.obj
 0002:00001248       ??_C@_0BE@KHGGOKFP@1sl_showAllTraces?$CI?$CJ?$AA@ 10011248     ChromatogramView.obj
 0002:0000125c       ??_C@_0BA@FLPFNNHL@Show?1hide?5trace?$AA@ 1001125c     ChromatogramView.obj
 0002:0000126c       ??_C@_01FHEEJDEE@A?$AA@    1001126c     ChromatogramView.obj
 0002:00001270       ??_C@_01BBODEMC@G?$AA@     10011270     ChromatogramView.obj
 0002:00001274       ??_C@_01GAPBHFFA@T?$AA@    10011274     ChromatogramView.obj
 0002:00001278       ??_C@_0BK@DJGCMFIK@1setRenderAreaHeight?$CIint?$CJ?$AA@ 10011278     ChromatogramView.obj
 0002:00001294       ??_C@_0BD@OIBDOPAP@2valueChanged?$CIint?$CJ?$AA@ 10011294     ChromatogramView.obj
 0002:000012a8       ??_C@_01NANMIPIL@N?$AA@    100112a8     ChromatogramView.obj
 0002:000012ac       ??_C@_0CB@LABJIAHG@1sl_onPopupMenuCkicked?$CIQAction?$CK?$CJ@ 100112ac     ChromatogramView.obj
 0002:000012d0       ??_C@_0BF@LKKOICAI@2triggered?$CIQAction?$CK?$CJ?$AA@ 100112d0     ChromatogramView.obj
 0002:000012e8       ??_C@_0BC@CHEFBIFI@Edit?5new?5sequence?$AA@ 100112e8     ChromatogramView.obj
 0002:000012fc       ??_C@_0BL@LFEBONOI@1sl_addNewSequenceObject?$CI?$CJ?$AA@ 100112fc     ChromatogramView.obj
 0002:00001318       ??_C@_0BH@BEHPMDIL@Edit?5existing?5sequence?$AA@ 10011318     ChromatogramView.obj
 0002:00001330       ??_C@_0CC@PEFPEMJE@1sl_onAddExistingSequenceObject?$CI@ 10011330     ChromatogramView.obj
 0002:00001354       ??_C@_0BH@GJBCOJGI@Remove?5edited?5sequence?$AA@ 10011354     ChromatogramView.obj
 0002:0000136c       ??_C@_0BM@EIAJFFKI@1sl_clearEditableSequence?$CI?$CJ?$AA@ 1001136c     ChromatogramView.obj
 0002:00001388       ??_C@_0N@IIDFOGKA@Undo?5changes?$AA@ 10011388     ChromatogramView.obj
 0002:00001398       ??_C@_0BE@ICIDGHK@1sl_removeChanges?$CI?$CJ?$AA@ 10011398     ChromatogramView.obj
 0002:000013ac       ??_C@_0CM@DLIEHMPD@1sl_onObjectRemoved?$CIGObjectView?$CK@ 100113ac     ChromatogramView.obj
 0002:000013d8       ??_C@_0CK@ICCFNPLK@2si_objectRemoved?$CIGObjectView?$CK?0?5@ 100113d8     ChromatogramView.obj
 0002:00001404       ??_C@_0BP@FLEPONNA@?3chroma_view?1images?1traces?4png?$AA@ 10011404     ChromatogramView.obj
 0002:00001424       ??_C@_0O@HHGALPIN@ADV_MENU_ZOOM?$AA@ 10011424     ChromatogramView.obj
 0002:00001434       ??_C@_0BH@HONGNIML@The?5sequence?5is?5locked?$AA@ 10011434     ChromatogramView.obj
 0002:0000144c       ??_C@_0CK@IGBIANDN@Trying?5to?5recover?5from?5error?3?5?$CF1@ 1001144c     ChromatogramView.obj
 0002:00001478       ??_C@_0BJ@FKKMLMPC@src?2ChromatogramView?4cpp?$AA@ 10011478     ChromatogramView.obj
 0002:00001494       ??_C@_0N@ODPIHDKM@_sequence?4fa?$AA@ 10011494     ChromatogramView.obj
 0002:000014a4       ??_C@_01KMDKNFGN@?1?$AA@   100114a4     ChromatogramView.obj
 0002:000014a8       ??_C@_0BP@IEDDOKEF@Format?5is?5not?5registered?3?5?8?$CF1?8?$AA@ 100114a8     ChromatogramView.obj
 0002:000014c8       ??_C@_0CC@OEAHFBCP@1sl_onSequenceObjectLoaded?$CITask?$CK@ 100114c8     ChromatogramView.obj
 0002:000014ec       ??_C@_0BJ@HEEBJCDM@2si_taskSucceeded?$CITask?$CK?$CJ?$AA@ 100114ec     ChromatogramView.obj
 0002:00001508       ??_C@_0BC@EODLHPBE@object?5not?5found?$CB?$AA@ 10011508     ChromatogramView.obj
 0002:0000151c       ??_C@_0BE@LPNAFJID@1sl_showHideTrace?$CI?$CJ?$AA@ 1001151c     ChromatogramView.obj
 0002:00001530       ??_C@_0BB@CGDKPOPA@2triggered?$CIbool?$CJ?$AA@ 10011530     ChromatogramView.obj
 0002:00001544       ??_C@_07INPHFMHP@Courier?$AA@ 10011544     ChromatogramView.obj
 0002:0000154c       ??_C@_0CO@FMAJFLDH@Chromatogram?5view?5?$CIzoom?5in?5to?5se@ 1001154c     ChromatogramView.obj
 0002:0000157c       ??_C@_0M@KGGAJAJ@Courier?5New?$AA@ 1001157c     ChromatogramView.obj
 0002:00001588       ??_C@_0BC@OMMCMOOF@original?5sequence?$AA@ 10011588     ChromatogramView.obj
 0002:000015a0       __real@0000000000000000    100115a0     ChromatogramView.obj
 0002:000015a8       __real@3fd51eb851eb851f    100115a8     ChromatogramView.obj
 0002:000015b0       __real@3fe0000000000000    100115b0     ChromatogramView.obj
 0002:000015b8       __real@3fe51eb851eb851f    100115b8     ChromatogramView.obj
 0002:000015c0       __real@3ff0000000000000    100115c0     ChromatogramView.obj
 0002:000015c8       __real@3ff4cccccccccccd    100115c8     ChromatogramView.obj
 0002:000015d0       __real@3ff8000000000000    100115d0     ChromatogramView.obj
 0002:000015d8       __real@4000000000000000    100115d8     ChromatogramView.obj
 0002:000015e0       __real@4018000000000000    100115e0     ChromatogramView.obj
 0002:000015e8       __real@4024000000000000    100115e8     ChromatogramView.obj
 0002:000015f0       __real@4059000000000000    100115f0     ChromatogramView.obj
 0002:000015f8       __real@bfd0000000000000    100115f8     ChromatogramView.obj
 0002:00001600       __real@bfe0000000000000    10011600     ChromatogramView.obj
 0002:00001608       __real@c059000000000000    10011608     ChromatogramView.obj
 0002:00001610       __xmm@3ff00000000000003ff0000000000000 10011610     ChromatogramView.obj
 0002:00001620       __xmm@80000000000000008000000000000000 10011620     ChromatogramView.obj
 0002:000024cc       ?value@?$integral_constant@_N$0A@@std@@2_NB 100124cc     MSVCRT:ti_inst.obj
 0002:000024cd       ?value@?$integral_constant@_N$00@std@@2_NB 100124cd     MSVCRT:ti_inst.obj
 0002:000024d4       ??_7type_info@@6B@         100124d4     MSVCRT:ti_inst.obj
 0002:00002564       __pDefaultRawDllMain       10012564     MSVCRT:crtdll.obj
 0002:00002564       __pRawDllMain              10012564     MSVCRT:crtdll.obj
 0002:00002570       ?ProcessDetach@NativeDll@<CrtImplementationDetails>@@0IB 10012570     MSVCRT:initsect.obj
 0002:00002574       ?ProcessAttach@NativeDll@<CrtImplementationDetails>@@0IB 10012574     MSVCRT:initsect.obj
 0002:00002578       ?ThreadAttach@NativeDll@<CrtImplementationDetails>@@0IB 10012578     MSVCRT:initsect.obj
 0002:0000257c       ?ThreadDetach@NativeDll@<CrtImplementationDetails>@@0IB 1001257c     MSVCRT:initsect.obj
 0002:00002580       ?ProcessVerifier@NativeDll@<CrtImplementationDetails>@@0IB 10012580     MSVCRT:initsect.obj
 0002:00002588       __load_config_used         10012588     MSVCRT:loadcfg.obj
 0002:00002644       ??_R4error_category@std@@6B@ 10012644     ChromaViewPlugin.obj
 0002:00002658       ??_R3error_category@std@@8 10012658     ChromaViewPlugin.obj
 0002:00002668       ??_R2error_category@std@@8 10012668     ChromaViewPlugin.obj
 0002:00002670       ??_R1A@?0A@EA@error_category@std@@8 10012670     ChromaViewPlugin.obj
 0002:0000268c       ??_R4_Generic_error_category@std@@6B@ 1001268c     ChromaViewPlugin.obj
 0002:000026a0       ??_R3_Generic_error_category@std@@8 100126a0     ChromaViewPlugin.obj
 0002:000026b0       ??_R2_Generic_error_category@std@@8 100126b0     ChromaViewPlugin.obj
 0002:000026bc       ??_R1A@?0A@EA@_Generic_error_category@std@@8 100126bc     ChromaViewPlugin.obj
 0002:000026d8       ??_R4_Iostream_error_category@std@@6B@ 100126d8     ChromaViewPlugin.obj
 0002:000026ec       ??_R3_Iostream_error_category@std@@8 100126ec     ChromaViewPlugin.obj
 0002:000026fc       ??_R2_Iostream_error_category@std@@8 100126fc     ChromaViewPlugin.obj
 0002:0000270c       ??_R1A@?0A@EA@_Iostream_error_category@std@@8 1001270c     ChromaViewPlugin.obj
 0002:00002728       ??_R4_System_error_category@std@@6B@ 10012728     ChromaViewPlugin.obj
 0002:0000273c       ??_R3_System_error_category@std@@8 1001273c     ChromaViewPlugin.obj
 0002:0000274c       ??_R2_System_error_category@std@@8 1001274c     ChromaViewPlugin.obj
 0002:0000275c       ??_R1A@?0A@EA@_System_error_category@std@@8 1001275c     ChromaViewPlugin.obj
 0002:00002778       ??_R4AbstractInt32Id@U2@@6B@ 10012778     ChromaViewPlugin.obj
 0002:0000278c       ??_R3AbstractInt32Id@U2@@8 1001278c     ChromaViewPlugin.obj
 0002:0000279c       ??_R2AbstractInt32Id@U2@@8 1001279c     ChromaViewPlugin.obj
 0002:000027a8       ??_R1A@?0A@EA@AbstractInt32Id@U2@@8 100127a8     ChromaViewPlugin.obj
 0002:000027c4       ??_R1A@?0A@EA@?$AbstractId@H@U2@@8 100127c4     ChromaViewPlugin.obj
 0002:000027e0       ??_R3?$AbstractId@H@U2@@8  100127e0     ChromaViewPlugin.obj
 0002:000027f0       ??_R2?$AbstractId@H@U2@@8  100127f0     ChromaViewPlugin.obj
 0002:000027f8       ??_R4?$AbstractId@H@U2@@6B@ 100127f8     ChromaViewPlugin.obj
 0002:0000280c       ??_R4ServiceType@U2@@6B@   1001280c     ChromaViewPlugin.obj
 0002:00002820       ??_R3ServiceType@U2@@8     10012820     ChromaViewPlugin.obj
 0002:00002830       ??_R2ServiceType@U2@@8     10012830     ChromaViewPlugin.obj
 0002:00002840       ??_R1A@?0A@EA@ServiceType@U2@@8 10012840     ChromaViewPlugin.obj
 0002:0000285c       ??_R4ChromaViewPlugin@U2@@6B@ 1001285c     ChromaViewPlugin.obj
 0002:00002870       ??_R3ChromaViewPlugin@U2@@8 10012870     ChromaViewPlugin.obj
 0002:00002880       ??_R2ChromaViewPlugin@U2@@8 10012880     ChromaViewPlugin.obj
 0002:00002890       ??_R1A@?0A@EA@ChromaViewPlugin@U2@@8 10012890     ChromaViewPlugin.obj
 0002:000028ac       ??_R1A@?0A@EA@Plugin@U2@@8 100128ac     ChromaViewPlugin.obj
 0002:000028c8       ??_R3Plugin@U2@@8          100128c8     ChromaViewPlugin.obj
 0002:000028d8       ??_R2Plugin@U2@@8          100128d8     ChromaViewPlugin.obj
 0002:000028e4       ??_R1A@?0A@EA@QObject@@8   100128e4     ChromaViewPlugin.obj
 0002:00002900       ??_R3QObject@@8            10012900     ChromaViewPlugin.obj
 0002:00002910       ??_R2QObject@@8            10012910     ChromaViewPlugin.obj
 0002:00002918       ??_R4ChromaViewContext@U2@@6BQObject@@@ 10012918     ChromaViewPlugin.obj
 0002:0000292c       ??_R3ChromaViewContext@U2@@8 1001292c     ChromaViewPlugin.obj
 0002:0000293c       ??_R2ChromaViewContext@U2@@8 1001293c     ChromaViewPlugin.obj
 0002:00002950       ??_R1A@?0A@EA@ChromaViewContext@U2@@8 10012950     ChromaViewPlugin.obj
 0002:0000296c       ??_R1A@?0A@EA@GObjectViewWindowContext@U2@@8 1001296c     ChromaViewPlugin.obj
 0002:00002988       ??_R3GObjectViewWindowContext@U2@@8 10012988     ChromaViewPlugin.obj
 0002:00002998       ??_R2GObjectViewWindowContext@U2@@8 10012998     ChromaViewPlugin.obj
 0002:000029a8       ??_R17?0A@EA@GObjectViewObjectHandler@U2@@8 100129a8     ChromaViewPlugin.obj
 0002:000029c4       ??_R3GObjectViewObjectHandler@U2@@8 100129c4     ChromaViewPlugin.obj
 0002:000029d4       ??_R2GObjectViewObjectHandler@U2@@8 100129d4     ChromaViewPlugin.obj
 0002:000029dc       ??_R1A@?0A@EA@GObjectViewObjectHandler@U2@@8 100129dc     ChromaViewPlugin.obj
 0002:000029f8       ??_R4ChromaViewContext@U2@@6BGObjectViewObjectHandler@1@@ 100129f8     ChromaViewPlugin.obj
 0002:00002a0c       ??_R4ChromaViewAction@U2@@6B@ 10012a0c     ChromaViewPlugin.obj
 0002:00002a20       ??_R3ChromaViewAction@U2@@8 10012a20     ChromaViewPlugin.obj
 0002:00002a30       ??_R2ChromaViewAction@U2@@8 10012a30     ChromaViewPlugin.obj
 0002:00002a44       ??_R1A@?0A@EA@ChromaViewAction@U2@@8 10012a44     ChromaViewPlugin.obj
 0002:00002a60       ??_R1A@?0A@EA@ADVSequenceWidgetAction@U2@@8 10012a60     ChromaViewPlugin.obj
 0002:00002a7c       ??_R3ADVSequenceWidgetAction@U2@@8 10012a7c     ChromaViewPlugin.obj
 0002:00002a8c       ??_R2ADVSequenceWidgetAction@U2@@8 10012a8c     ChromaViewPlugin.obj
 0002:00002a9c       ??_R1A@?0A@EA@QAction@@8   10012a9c     ChromaViewPlugin.obj
 0002:00002ab8       ??_R3QAction@@8            10012ab8     ChromaViewPlugin.obj
 0002:00002ac8       ??_R2QAction@@8            10012ac8     ChromaViewPlugin.obj
 0002:00002ad4       ??_R4QAction@@6B@          10012ad4     ChromatogramView.obj
 0002:00002ae8       ??_R4LoadUnloadedDocumentTask@U2@@6B@ 10012ae8     ChromatogramView.obj
 0002:00002afc       ??_R3LoadUnloadedDocumentTask@U2@@8 10012afc     ChromatogramView.obj
 0002:00002b0c       ??_R2LoadUnloadedDocumentTask@U2@@8 10012b0c     ChromatogramView.obj
 0002:00002b20       ??_R1A@?0A@EA@LoadUnloadedDocumentTask@U2@@8 10012b20     ChromatogramView.obj
 0002:00002b3c       ??_R1A@?0A@EA@DocumentProviderTask@U2@@8 10012b3c     ChromatogramView.obj
 0002:00002b58       ??_R3DocumentProviderTask@U2@@8 10012b58     ChromatogramView.obj
 0002:00002b68       ??_R2DocumentProviderTask@U2@@8 10012b68     ChromatogramView.obj
 0002:00002b78       ??_R1A@?0A@EA@Task@U2@@8   10012b78     ChromatogramView.obj
 0002:00002b94       ??_R3Task@U2@@8            10012b94     ChromatogramView.obj
 0002:00002ba4       ??_R2Task@U2@@8            10012ba4     ChromatogramView.obj
 0002:00002bb0       ??_R4QMenu@@6BQObject@@@   10012bb0     ChromatogramView.obj
 0002:00002bc4       ??_R3QMenu@@8              10012bc4     ChromatogramView.obj
 0002:00002bd4       ??_R2QMenu@@8              10012bd4     ChromatogramView.obj
 0002:00002be8       ??_R1A@?0A@EA@QMenu@@8     10012be8     ChromatogramView.obj
 0002:00002c04       ??_R1A@?0A@EA@QWidget@@8   10012c04     ChromatogramView.obj
 0002:00002c20       ??_R3QWidget@@8            10012c20     ChromatogramView.obj
 0002:00002c30       ??_R2QWidget@@8            10012c30     ChromatogramView.obj
 0002:00002c40       ??_R17?0A@EA@QPaintDevice@@8 10012c40     ChromatogramView.obj
 0002:00002c5c       ??_R3QPaintDevice@@8       10012c5c     ChromatogramView.obj
 0002:00002c6c       ??_R2QPaintDevice@@8       10012c6c     ChromatogramView.obj
 0002:00002c74       ??_R1A@?0A@EA@QPaintDevice@@8 10012c74     ChromatogramView.obj
 0002:00002c90       ??_R4QMenu@@6BQPaintDevice@@@ 10012c90     ChromatogramView.obj
 0002:00002ca4       ??_R4TaskSignalMapper@U2@@6B@ 10012ca4     ChromatogramView.obj
 0002:00002cb8       ??_R3TaskSignalMapper@U2@@8 10012cb8     ChromatogramView.obj
 0002:00002cc8       ??_R2TaskSignalMapper@U2@@8 10012cc8     ChromatogramView.obj
 0002:00002cd4       ??_R1A@?0A@EA@TaskSignalMapper@U2@@8 10012cd4     ChromatogramView.obj
 0002:00002cf0       ??_R4QHBoxLayout@@6BQObject@@@ 10012cf0     ChromatogramView.obj
 0002:00002d04       ??_R3QHBoxLayout@@8        10012d04     ChromatogramView.obj
 0002:00002d14       ??_R2QHBoxLayout@@8        10012d14     ChromatogramView.obj
 0002:00002d2c       ??_R1A@?0A@EA@QHBoxLayout@@8 10012d2c     ChromatogramView.obj
 0002:00002d48       ??_R1A@?0A@EA@QBoxLayout@@8 10012d48     ChromatogramView.obj
 0002:00002d64       ??_R3QBoxLayout@@8         10012d64     ChromatogramView.obj
 0002:00002d74       ??_R2QBoxLayout@@8         10012d74     ChromatogramView.obj
 0002:00002d88       ??_R1A@?0A@EA@QLayout@@8   10012d88     ChromatogramView.obj
 0002:00002da4       ??_R3QLayout@@8            10012da4     ChromatogramView.obj
 0002:00002db4       ??_R2QLayout@@8            10012db4     ChromatogramView.obj
 0002:00002dc4       ??_R17?0A@EA@QLayoutItem@@8 10012dc4     ChromatogramView.obj
 0002:00002de0       ??_R3QLayoutItem@@8        10012de0     ChromatogramView.obj
 0002:00002df0       ??_R2QLayoutItem@@8        10012df0     ChromatogramView.obj
 0002:00002df8       ??_R1A@?0A@EA@QLayoutItem@@8 10012df8     ChromatogramView.obj
 0002:00002e14       ??_R4QHBoxLayout@@6BQLayoutItem@@@ 10012e14     ChromatogramView.obj
 0002:00002e28       ??_R4ScaleBar@U2@@6BQObject@@@ 10012e28     ChromatogramView.obj
 0002:00002e3c       ??_R3ScaleBar@U2@@8        10012e3c     ChromatogramView.obj
 0002:00002e4c       ??_R2ScaleBar@U2@@8        10012e4c     ChromatogramView.obj
 0002:00002e60       ??_R1A@?0A@EA@ScaleBar@U2@@8 10012e60     ChromatogramView.obj
 0002:00002e7c       ??_R4ScaleBar@U2@@6BQPaintDevice@@@ 10012e7c     ChromatogramView.obj
 0002:00002e90       ??_R4ChromatogramViewRenderArea@U2@@6BQObject@@@ 10012e90     ChromatogramView.obj
 0002:00002ea4       ??_R3ChromatogramViewRenderArea@U2@@8 10012ea4     ChromatogramView.obj
 0002:00002eb4       ??_R2ChromatogramViewRenderArea@U2@@8 10012eb4     ChromatogramView.obj
 0002:00002ecc       ??_R1A@?0A@EA@ChromatogramViewRenderArea@U2@@8 10012ecc     ChromatogramView.obj
 0002:00002ee8       ??_R1A@?0A@EA@GSequenceLineViewRenderArea@U2@@8 10012ee8     ChromatogramView.obj
 0002:00002f04       ??_R3GSequenceLineViewRenderArea@U2@@8 10012f04     ChromatogramView.obj
 0002:00002f14       ??_R2GSequenceLineViewRenderArea@U2@@8 10012f14     ChromatogramView.obj
 0002:00002f28       ??_R4ChromatogramViewRenderArea@U2@@6BQPaintDevice@@@ 10012f28     ChromatogramView.obj
 0002:00002f3c       ??_R4ChromatogramView@U2@@6BQObject@@@ 10012f3c     ChromatogramView.obj
 0002:00002f50       ??_R3ChromatogramView@U2@@8 10012f50     ChromatogramView.obj
 0002:00002f60       ??_R2ChromatogramView@U2@@8 10012f60     ChromatogramView.obj
 0002:00002f7c       ??_R1A@?0A@EA@ChromatogramView@U2@@8 10012f7c     ChromatogramView.obj
 0002:00002f98       ??_R1A@?0A@EA@GSequenceLineView@U2@@8 10012f98     ChromatogramView.obj
 0002:00002fb4       ??_R3GSequenceLineView@U2@@8 10012fb4     ChromatogramView.obj
 0002:00002fc4       ??_R2GSequenceLineView@U2@@8 10012fc4     ChromatogramView.obj
 0002:00002fdc       ??_R1A@?0A@EA@WidgetWithLocalToolbar@U2@@8 10012fdc     ChromatogramView.obj
 0002:00002ff8       ??_R3WidgetWithLocalToolbar@U2@@8 10012ff8     ChromatogramView.obj
 0002:00003008       ??_R2WidgetWithLocalToolbar@U2@@8 10013008     ChromatogramView.obj
 0002:0000301c       ??_R4ChromatogramView@U2@@6BQPaintDevice@@@ 1001301c     ChromatogramView.obj
 0002:00003030       ??_R4type_info@@6B@        10013030     MSVCRT:ti_inst.obj
 0002:00003044       ??_R3type_info@@8          10013044     MSVCRT:ti_inst.obj
 0002:00003054       ??_R2type_info@@8          10013054     MSVCRT:ti_inst.obj
 0002:0000305c       ??_R1A@?0A@EA@type_info@@8 1001305c     MSVCRT:ti_inst.obj
 0002:00003080       ___safe_se_handler_table   10013080     <linker-defined>
 0002:00003198       ___rtc_iaa                 10013198     MSVCRT:initsect.obj
 0002:0000319c       ___rtc_izz                 1001319c     MSVCRT:initsect.obj
 0002:000031a0       ___rtc_taa                 100131a0     MSVCRT:initsect.obj
 0002:000031a4       ___rtc_tzz                 100131a4     MSVCRT:initsect.obj
 0002:00004784       __IMPORT_DESCRIPTOR_U2Core 10014784     U2Core:U2Core.dll
 0002:00004798       __IMPORT_DESCRIPTOR_U2Gui  10014798     U2Gui:U2Gui.dll
 0002:000047ac       __IMPORT_DESCRIPTOR_U2View 100147ac     U2View:U2View.dll
 0002:000047c0       __IMPORT_DESCRIPTOR_Qt5Widgets 100147c0     Qt5Widgets:Qt5Widgets.dll
 0002:000047d4       __IMPORT_DESCRIPTOR_Qt5Gui 100147d4     Qt5Gui:Qt5Gui.dll
 0002:000047e8       __IMPORT_DESCRIPTOR_Qt5Core 100147e8     Qt5Core:Qt5Core.dll
 0002:000047fc       __IMPORT_DESCRIPTOR_MSVCP120 100147fc     msvcprt:MSVCP120.dll
 0002:00004810       __IMPORT_DESCRIPTOR_MSVCR120 10014810     MSVCRT:MSVCR120.dll
 0002:00004824       __IMPORT_DESCRIPTOR_KERNEL32 10014824     kernel32:KERNEL32.dll
 0002:00004838       __NULL_IMPORT_DESCRIPTOR   10014838     U2Core:U2Core.dll
 0003:00000000       ?_Generic_object@?$_Error_objects@H@std@@2V_Generic_error_category@2@A 1001b000     ChromaViewPlugin.obj
 0003:00000004       ?_Iostream_object@?$_Error_objects@H@std@@2V_Iostream_error_category@2@A 1001b004     ChromaViewPlugin.obj
 0003:00000008       ?_System_object@?$_Error_objects@H@std@@2V_System_error_category@2@A 1001b008     ChromaViewPlugin.obj
 0003:00000144       ?staticMetaObject@ChromaViewPlugin@U2@@2UQMetaObject@@B 1001b144     moc_ChromaViewPlugin.obj
 0003:0000015c       ?staticMetaObject@ChromaViewContext@U2@@2UQMetaObject@@B 1001b15c     moc_ChromaViewPlugin.obj
 0003:00000174       ?staticMetaObject@ChromaViewAction@U2@@2UQMetaObject@@B 1001b174     moc_ChromaViewPlugin.obj
 0003:0000018c       ?staticMetaObject@ChromatogramView@U2@@2UQMetaObject@@B 1001b18c     moc_ChromatogramView.obj
 0003:000001a4       ?staticMetaObject@ChromatogramViewRenderArea@U2@@2UQMetaObject@@B 1001b1a4     moc_ChromatogramView.obj
 0003:000001bc       ___security_cookie         1001b1bc     MSVCRT:gs_cookie.obj
 0003:000001c0       ___security_cookie_complement 1001b1c0     MSVCRT:gs_cookie.obj
 0003:000001d0       ___native_dllmain_reason   1001b1d0     MSVCRT:natstart.obj
 0003:000001d4       ??_R0?AVerror_category@std@@@8 1001b1d4     ChromaViewPlugin.obj
 0003:000001f8       ??_R0?AV_Generic_error_category@std@@@8 1001b1f8     ChromaViewPlugin.obj
 0003:00000224       ??_R0?AV_Iostream_error_category@std@@@8 1001b224     ChromaViewPlugin.obj
 0003:00000250       ??_R0?AV_System_error_category@std@@@8 1001b250     ChromaViewPlugin.obj
 0003:0000027c       ??_R0?AVAbstractInt32Id@U2@@@8 1001b27c     ChromaViewPlugin.obj
 0003:000002a0       ??_R0?AV?$AbstractId@H@U2@@@8 1001b2a0     ChromaViewPlugin.obj
 0003:000002c0       ??_R0?AVServiceType@U2@@@8 1001b2c0     ChromaViewPlugin.obj
 0003:000002e0       ??_R0?AVChromaViewPlugin@U2@@@8 1001b2e0     ChromaViewPlugin.obj
 0003:00000304       ??_R0?AVPlugin@U2@@@8      1001b304     ChromaViewPlugin.obj
 0003:0000031c       ??_R0?AVQObject@@@8        1001b31c     ChromaViewPlugin.obj
 0003:00000334       ??_R0?AVChromaViewContext@U2@@@8 1001b334     ChromaViewPlugin.obj
 0003:00000358       ??_R0?AVGObjectViewWindowContext@U2@@@8 1001b358     ChromaViewPlugin.obj
 0003:00000384       ??_R0?AVGObjectViewObjectHandler@U2@@@8 1001b384     ChromaViewPlugin.obj
 0003:000003b0       ??_R0?AVChromaViewAction@U2@@@8 1001b3b0     ChromaViewPlugin.obj
 0003:000003d4       ??_R0?AVADVSequenceWidgetAction@U2@@@8 1001b3d4     ChromaViewPlugin.obj
 0003:00000400       ??_R0?AVQAction@@@8        1001b400     ChromaViewPlugin.obj
 0003:00000418       ??_R0?AVLoadUnloadedDocumentTask@U2@@@8 1001b418     ChromatogramView.obj
 0003:00000444       ??_R0?AVDocumentProviderTask@U2@@@8 1001b444     ChromatogramView.obj
 0003:0000046c       ??_R0?AVTask@U2@@@8        1001b46c     ChromatogramView.obj
 0003:00000484       ??_R0?AVQMenu@@@8          1001b484     ChromatogramView.obj
 0003:00000498       ??_R0?AVQWidget@@@8        1001b498     ChromatogramView.obj
 0003:000004b0       ??_R0?AVQPaintDevice@@@8   1001b4b0     ChromatogramView.obj
 0003:000004cc       ??_R0?AVTaskSignalMapper@U2@@@8 1001b4cc     ChromatogramView.obj
 0003:000004f0       ??_R0?AVQHBoxLayout@@@8    1001b4f0     ChromatogramView.obj
 0003:0000050c       ??_R0?AVQBoxLayout@@@8     1001b50c     ChromatogramView.obj
 0003:00000528       ??_R0?AVQLayout@@@8        1001b528     ChromatogramView.obj
 0003:00000540       ??_R0?AVQLayoutItem@@@8    1001b540     ChromatogramView.obj
 0003:0000055c       ??_R0?AVScaleBar@U2@@@8    1001b55c     ChromatogramView.obj
 0003:00000578       ??_R0?AVChromatogramViewRenderArea@U2@@@8 1001b578     ChromatogramView.obj
 0003:000005a4       ??_R0?AVGSequenceLineViewRenderArea@U2@@@8 1001b5a4     ChromatogramView.obj
 0003:000005d4       ??_R0?AVChromatogramView@U2@@@8 1001b5d4     ChromatogramView.obj
 0003:000005f8       ??_R0?AVGSequenceLineView@U2@@@8 1001b5f8     ChromatogramView.obj
 0003:0000061c       ??_R0?AVWidgetWithLocalToolbar@U2@@@8 1001b61c     ChromatogramView.obj
 0003:00000644       ??_R0?AVtype_info@@@8      1001b644     MSVCRT:ti_inst.obj
 0003:000006ac       ?id@?$num_put@DV?$back_insert_iterator@V?$basic_string@DU?$char_traits@D@std@@V?$allocator@D@2@@std@@@std@@@std@@2V0locale@2@A 1001b6ac     ChromaViewPlugin.obj
 0003:000006b0       ?id@?$num_put@_WV?$back_insert_iterator@V?$basic_string@_WU?$char_traits@_W@std@@V?$allocator@_W@2@@std@@@std@@@std@@2V0locale@2@A 1001b6b0     ChromaViewPlugin.obj
 0003:000007e8       ?metatype_id@?1??qt_metatype_id@?$QMetaTypeIdQObject@PAVADVSequenceWidget@U2@@$00@@SAHXZ@4V?$QBasicAtomicInteger@H@@A 1001b7e8     moc_ChromaViewPlugin.obj
 0003:000007f0       ?metatype_id@?1??qt_metatype_id@?$QMetaTypeIdQObject@PAVQAction@@$00@@SAHXZ@4V?$QBasicAtomicInteger@H@@A 1001b7f0     moc_ChromatogramView.obj
 0003:000007f4       ?metatype_id@?1??qt_metatype_id@?$QMetaTypeIdQObject@PAVGObject@U2@@$00@@SAHXZ@4V?$QBasicAtomicInteger@H@@A 1001b7f4     moc_ChromatogramView.obj
 0003:000007f8       ?dummy@?A0xc45d533f@@3Uinitializer@1@A 1001b7f8     qrc_chroma_view.obj
 0003:00000b20       ?__type_info_root_node@@3U__type_info_node@@A 1001bb20     MSVCRT:tncleanup.obj
 0003:00000b28       ___native_startup_lock     1001bb28     <common>
 0003:00000b2c       ___native_startup_state    1001bb2c     <common>
 0003:00000b30       ___dyn_tls_init_callback   1001bb30     <common>
 0003:00000b34       ___onexitend               1001bb34     <common>
 0003:00000b38       ___onexitbegin             1001bb38     <common>

 entry point at        0001:0000ce9e

 Static symbols

 0000:fffe1000       .debug$S                   10000000     MSVCRT:MSVCR120.dll
 0000:fffe1000       .debug$S                   10000000     MSVCRT:MSVCR120.dll
 0000:fffe1000       .debug$S                   10000000     MSVCRT:MSVCR120.dll
 0000:fffe1000       .debug$S                   10000000     MSVCRT:MSVCR120.dll
 0000:fffe1000       .debug$S                   10000000     MSVCRT:MSVCR120.dll
 0000:fffe1000       .debug$S                   10000000     MSVCRT:MSVCR120.dll
 0000:fffe1000       .debug$S                   10000000     MSVCRT:MSVCR120.dll
 0000:fffe1000       .debug$S                   10000000     MSVCRT:MSVCR120.dll
 0000:fffe1000       .debug$S                   10000000     MSVCRT:MSVCR120.dll
 0000:fffe1000       .debug$S                   10000000     MSVCRT:MSVCR120.dll
 0002:ffff0000       ?_Iostream_object$initializer$@?$_Error_objects@H@std@@2P6AXXZA 10000000     ChromatogramView.obj
 0000:fffe1000       .debug$S                   10000000     MSVCRT:MSVCR120.dll
 0000:fffe1000       .debug$S                   10000000     MSVCRT:MSVCR120.dll
 0000:fffe1000       .debug$S                   10000000     MSVCRT:MSVCR120.dll
 0000:fffe1000       .debug$S                   10000000     MSVCRT:MSVCR120.dll
 0000:fffe1000       .debug$S                   10000000     MSVCRT:MSVCR120.dll
 0000:fffe1000       .debug$S                   10000000     MSVCRT:MSVCR120.dll
 0002:ffff0000       ?_System_object$initializer$@?$_Error_objects@H@std@@2P6AXXZA 10000000     ChromatogramView.obj
 0000:fffe1000       .debug$S                   10000000     U2Core:U2Core.dll
 0000:fffe1000       .debug$S                   10000000     U2Core:U2Core.dll
 0000:fffe1000       .debug$S                   10000000     MSVCRT:MSVCR120.dll
 0000:fffe1000       .debug$S                   10000000     U2Core:U2Core.dll
 0000:fffe1000       .debug$S                   10000000     MSVCRT:MSVCR120.dll
 0000:fffe1000       .debug$S                   10000000     U2Core:U2Core.dll
 0000:fffe1000       .debug$S                   10000000     MSVCRT:MSVCR120.dll
 0001:fffff000       __ehhandler$?_Copy@?$basic_string@DU?$char_traits@D@std@@V?$allocator@D@2@@std@@QAEXII@Z 10000000 f   moc_ChromatogramView.obj
 0000:fffe1000       .debug$S                   10000000     U2Core:U2Core.dll
 0000:fffe1000       .debug$S                   10000000     U2Core:U2Core.dll
 0000:fffe1000       .debug$S                   10000000     MSVCRT:MSVCR120.dll
 0000:fffe1000       .debug$S                   10000000     MSVCRT:MSVCR120.dll
 0000:fffe1000       .debug$S                   10000000     MSVCRT:MSVCR120.dll
 0000:fffe1000       .debug$S                   10000000     MSVCRT:MSVCR120.dll
 0000:fffe1000       .debug$S                   10000000     MSVCRT:MSVCR120.dll
 0000:fffe1000       .debug$S                   10000000     U2Core:U2Core.dll
 0000:fffe1000       .debug$S                   10000000     U2Core:U2Core.dll
 0000:fffe1000       .debug$S                   10000000     U2Core:U2Core.dll
 0000:fffe1000       .debug$S                   10000000     U2Core:U2Core.dll
 0002:ffff0000       __catchsym$?_Copy@?$basic_string@DU?$char_traits@D@std@@V?$allocator@D@2@@std@@QAEXII@Z$5 10000000     moc_ChromatogramView.obj
 0000:fffe1000       .debug$S                   10000000     MSVCRT:MSVCR120.dll
 0000:fffe1000       .debug$S                   10000000     MSVCRT:MSVCR120.dll
 0000:fffe1000       .debug$S                   10000000     MSVCRT:MSVCR120.dll
 0000:fffe1000       .debug$S                   10000000     MSVCRT:MSVCR120.dll
 0000:fffe1000       .debug$S                   10000000     msvcprt:MSVCP120.dll
 0000:fffe1000       .debug$S                   10000000     msvcprt:MSVCP120.dll
 0000:fffe1000       .debug$S                   10000000     msvcprt:MSVCP120.dll
 0000:fffe1000       .debug$S                   10000000     msvcprt:MSVCP120.dll
 0000:fffe1000       .debug$S                   10000000     msvcprt:MSVCP120.dll
 0000:fffe1000       .debug$S                   10000000     kernel32:KERNEL32.dll
 0002:ffff0000       ?_Generic_object$initializer$@?$_Error_objects@H@std@@2P6AXXZA 10000000     moc_ChromatogramView.obj
 0002:ffff0000       ?_Iostream_object$initializer$@?$_Error_objects@H@std@@2P6AXXZA 10000000     moc_ChromatogramView.obj
 0002:ffff0000       ?_System_object$initializer$@?$_Error_objects@H@std@@2P6AXXZA 10000000     moc_ChromatogramView.obj
 0000:fffe1000       .debug$S                   10000000     kernel32:KERNEL32.dll
 0000:fffe1000       .debug$S                   10000000     kernel32:KERNEL32.dll
 0000:fffe1000       .debug$S                   10000000     kernel32:KERNEL32.dll
 0000:fffe1000       .debug$S                   10000000     kernel32:KERNEL32.dll
 0000:fffe1000       .debug$S                   10000000     kernel32:KERNEL32.dll
 0000:fffe1000       .debug$S                   10000000     kernel32:KERNEL32.dll
 0000:fffe1000       .debug$S                   10000000     U2Core:U2Core.dll
 0000:fffe1000       .debug$S                   10000000     kernel32:KERNEL32.dll
 0000:fffe1000       .debug$S                   10000000     U2Core:U2Core.dll
 0000:fffe1000       .debug$S                   10000000     kernel32:KERNEL32.dll
 0000:fffe1000       .debug$S                   10000000     U2Core:U2Core.dll
 0000:fffe1000       .debug$S                   10000000     Qt5Core:Qt5Core.dll
 0000:fffe1000       .debug$S                   10000000     U2Core:U2Core.dll
 0000:fffe1000       .debug$S                   10000000     Qt5Core:Qt5Core.dll
 0000:fffe1000       .debug$S                   10000000     U2Core:U2Core.dll
 0000:fffe1000       .debug$S                   10000000     Qt5Core:Qt5Core.dll
 0000:fffe1000       .debug$S                   10000000     U2Core:U2Core.dll
 0000:fffe1000       .debug$S                   10000000     Qt5Core:Qt5Core.dll
 0000:fffe1000       .debug$S                   10000000     U2Core:U2Core.dll
 0000:fffe1000       .debug$S                   10000000     Qt5Core:Qt5Core.dll
 0000:fffe1000       .debug$S                   10000000     U2Core:U2Core.dll
 0000:fffe1000       .debug$S                   10000000     Qt5Core:Qt5Core.dll
 0000:fffe1000       .debug$S                   10000000     U2Core:U2Core.dll
 0000:fffe1000       .debug$S                   10000000     Qt5Core:Qt5Core.dll
 0000:fffe1000       .debug$S                   10000000     U2Core:U2Core.dll
 0000:fffe1000       .debug$S                   10000000     Qt5Core:Qt5Core.dll
 0000:fffe1000       .debug$S                   10000000     U2Core:U2Core.dll
 0000:fffe1000       .debug$S                   10000000     Qt5Core:Qt5Core.dll
 0000:fffe1000       .debug$S                   10000000     U2Core:U2Core.dll
 0000:fffe1000       .debug$S                   10000000     Qt5Core:Qt5Core.dll
 0000:fffe1000       .debug$S                   10000000     U2Core:U2Core.dll
 0000:fffe1000       .debug$S                   10000000     Qt5Core:Qt5Core.dll
 0000:fffe1000       .debug$S                   10000000     U2Core:U2Core.dll
 0000:fffe1000       .debug$S                   10000000     U2Core:U2Core.dll
 0000:fffe1000       .debug$S                   10000000     U2Core:U2Core.dll
 0000:fffe1000       .debug$S                   10000000     U2Core:U2Core.dll
 0000:fffe1000       .debug$S                   10000000     Qt5Core:Qt5Core.dll
 0000:fffe1000       .debug$S                   10000000     U2Core:U2Core.dll
 0000:fffe1000       .debug$S                   10000000     Qt5Core:Qt5Core.dll
 0000:fffe1000       .debug$S                   10000000     U2Core:U2Core.dll
 0000:fffe1000       .debug$S                   10000000     Qt5Core:Qt5Core.dll
 0001:fffff000       __ehhandler$?_Copy@?$basic_string@DU?$char_traits@D@std@@V?$allocator@D@2@@std@@QAEXII@Z 10000000 f   moc_ChromaViewPlugin.obj
 0000:fffe1000       .debug$S                   10000000     U2Core:U2Core.dll
 0000:fffe1000       .debug$S                   10000000     U2Core:U2Core.dll
 0000:fffe1000       .debug$S                   10000000     Qt5Core:Qt5Core.dll
 0000:fffe1000       .debug$S                   10000000     Qt5Core:Qt5Core.dll
 0000:fffe1000       .debug$S                   10000000     U2Core:U2Core.dll
 0000:fffe1000       .debug$S                   10000000     U2Core:U2Core.dll
 0000:fffe1000       .debug$S                   10000000     U2Core:U2Core.dll
 0000:fffe1000       .debug$S                   10000000     U2Core:U2Core.dll
 0002:ffff0000       __catchsym$?_Copy@?$basic_string@DU?$char_traits@D@std@@V?$allocator@D@2@@std@@QAEXII@Z$5 10000000     moc_ChromaViewPlugin.obj
 0000:fffe1000       .debug$S                   10000000     Qt5Core:Qt5Core.dll
 0000:fffe1000       .debug$S                   10000000     Qt5Core:Qt5Core.dll
 0000:fffe1000       .debug$S                   10000000     Qt5Core:Qt5Core.dll
 0000:fffe1000       .debug$S                   10000000     Qt5Core:Qt5Core.dll
 0000:fffe1000       .debug$S                   10000000     Qt5Core:Qt5Core.dll
 0000:fffe1000       .debug$S                   10000000     Qt5Core:Qt5Core.dll
 0000:fffe1000       .debug$S                   10000000     Qt5Core:Qt5Core.dll
 0000:fffe1000       .debug$S                   10000000     Qt5Core:Qt5Core.dll
 0000:fffe1000       .debug$S                   10000000     Qt5Core:Qt5Core.dll
 0000:fffe1000       .debug$S                   10000000     Qt5Core:Qt5Core.dll
 0000:fffe1000       .debug$S                   10000000     Qt5Core:Qt5Core.dll
 0000:fffe1000       .debug$S                   10000000     Qt5Core:Qt5Core.dll
 0000:fffe1000       .debug$S                   10000000     Qt5Core:Qt5Core.dll
 0000:fffe1000       .debug$S                   10000000     Qt5Core:Qt5Core.dll
 0000:fffe1000       .debug$S                   10000000     Qt5Core:Qt5Core.dll
 0000:fffe1000       .debug$S                   10000000     Qt5Core:Qt5Core.dll
 0000:fffe1000       .debug$S                   10000000     Qt5Core:Qt5Core.dll
 0000:fffe1000       .debug$S                   10000000     Qt5Core:Qt5Core.dll
 0000:fffe1000       .debug$S                   10000000     Qt5Core:Qt5Core.dll
 0000:fffe1000       .debug$S                   10000000     Qt5Core:Qt5Core.dll
 0000:fffe1000       .debug$S                   10000000     Qt5Core:Qt5Core.dll
 0000:fffe1000       .debug$S                   10000000     Qt5Core:Qt5Core.dll
 0000:fffe1000       .debug$S                   10000000     Qt5Core:Qt5Core.dll
 0000:fffe1000       .debug$S                   10000000     Qt5Core:Qt5Core.dll
 0000:fffe1000       .debug$S                   10000000     Qt5Core:Qt5Core.dll
 0000:fffe1000       .debug$S                   10000000     Qt5Core:Qt5Core.dll
 0000:fffe1000       .debug$S                   10000000     Qt5Core:Qt5Core.dll
 0000:fffe1000       .debug$S                   10000000     Qt5Core:Qt5Core.dll
 0000:fffe1000       .debug$S                   10000000     Qt5Core:Qt5Core.dll
 0000:fffe1000       .debug$S                   10000000     Qt5Core:Qt5Core.dll
 0000:fffe1000       .debug$S                   10000000     Qt5Core:Qt5Core.dll
 0000:fffe1000       .debug$S                   10000000     Qt5Core:Qt5Core.dll
 0000:fffe1000       .debug$S                   10000000     Qt5Core:Qt5Core.dll
 0000:fffe1000       .debug$S                   10000000     Qt5Core:Qt5Core.dll
 0000:fffe1000       .debug$S                   10000000     Qt5Core:Qt5Core.dll
 0002:ffff0000       ?_Generic_object$initializer$@?$_Error_objects@H@std@@2P6AXXZA 10000000     moc_ChromaViewPlugin.obj
 0002:ffff0000       ?_Iostream_object$initializer$@?$_Error_objects@H@std@@2P6AXXZA 10000000     moc_ChromaViewPlugin.obj
 0002:ffff0000       ?_System_object$initializer$@?$_Error_objects@H@std@@2P6AXXZA 10000000     moc_ChromaViewPlugin.obj
 0000:fffe1000       .debug$S                   10000000     U2Core:U2Core.dll
 0000:fffe1000       .debug$S                   10000000     Qt5Core:Qt5Core.dll
 0000:fffe1000       .debug$S                   10000000     U2Core:U2Core.dll
 0000:fffe1000       .debug$S                   10000000     Qt5Core:Qt5Core.dll
 0000:fffe1000       .debug$S                   10000000     U2Core:U2Core.dll
 0000:fffe1000       .debug$S                   10000000     Qt5Core:Qt5Core.dll
 0000:fffe1000       .debug$S                   10000000     U2Core:U2Core.dll
 0000:fffe1000       .debug$S                   10000000     Qt5Core:Qt5Core.dll
 0000:fffe1000       .debug$S                   10000000     U2Core:U2Core.dll
 0000:fffe1000       .debug$S                   10000000     Qt5Core:Qt5Core.dll
 0000:fffe1000       .debug$S                   10000000     U2Core:U2Core.dll
 0000:fffe1000       .debug$S                   10000000     Qt5Core:Qt5Core.dll
 0000:fffe1000       .debug$S                   10000000     U2Core:U2Core.dll
 0000:fffe1000       .debug$S                   10000000     Qt5Core:Qt5Core.dll
 0000:fffe1000       .debug$S                   10000000     U2Core:U2Core.dll
 0000:fffe1000       .debug$S                   10000000     Qt5Core:Qt5Core.dll
 0000:fffe1000       .debug$S                   10000000     U2Core:U2Core.dll
 0000:fffe1000       .debug$S                   10000000     Qt5Core:Qt5Core.dll
 0000:fffe1000       .debug$S                   10000000     U2Core:U2Core.dll
 0000:fffe1000       .debug$S                   10000000     Qt5Core:Qt5Core.dll
 0000:fffe1000       .debug$S                   10000000     U2Core:U2Core.dll
 0000:fffe1000       .debug$S                   10000000     Qt5Core:Qt5Core.dll
 0000:fffe1000       .debug$S                   10000000     U2Core:U2Core.dll
 0000:fffe1000       .debug$S                   10000000     Qt5Core:Qt5Core.dll
 0000:fffe1000       .debug$S                   10000000     U2Core:U2Core.dll
 0000:fffe1000       .debug$S                   10000000     Qt5Core:Qt5Core.dll
 0000:fffe1000       .debug$S                   10000000     U2Core:U2Core.dll
 0000:fffe1000       .debug$S                   10000000     Qt5Core:Qt5Core.dll
 0000:fffe1000       .debug$S                   10000000     U2Core:U2Core.dll
 0000:fffe1000       .debug$S                   10000000     Qt5Core:Qt5Core.dll
 0000:fffe1000       .debug$S                   10000000     U2Core:U2Core.dll
 0000:fffe1000       .debug$S                   10000000     Qt5Core:Qt5Core.dll
 0000:fffe1000       .debug$S                   10000000     U2Core:U2Core.dll
 0000:fffe1000       .debug$S                   10000000     Qt5Core:Qt5Core.dll
 0000:fffe1000       .debug$S                   10000000     U2Core:U2Core.dll
 0000:fffe1000       .debug$S                   10000000     Qt5Core:Qt5Core.dll
 0000:fffe1000       .debug$S                   10000000     U2Core:U2Core.dll
 0000:fffe1000       .debug$S                   10000000     Qt5Core:Qt5Core.dll
 0000:fffe1000       .debug$S                   10000000     U2Core:U2Core.dll
 0000:fffe1000       .debug$S                   10000000     Qt5Core:Qt5Core.dll
 0000:fffe1000       .debug$S                   10000000     U2Core:U2Core.dll
 0000:fffe1000       .debug$S                   10000000     Qt5Core:Qt5Core.dll
 0000:fffe1000       .debug$S                   10000000     U2Core:U2Core.dll
 0000:fffe1000       .debug$S                   10000000     Qt5Core:Qt5Core.dll
 0000:fffe1000       .debug$S                   10000000     Qt5Core:Qt5Core.dll
 0000:fffe1000       .debug$S                   10000000     U2Core:U2Core.dll
 0000:fffe1000       .debug$S                   10000000     Qt5Core:Qt5Core.dll
 0000:fffe1000       .debug$S                   10000000     U2Core:U2Core.dll
 0000:fffe1000       .debug$S                   10000000     Qt5Core:Qt5Core.dll
 0000:fffe1000       .debug$S                   10000000     U2Core:U2Core.dll
 0000:fffe1000       .debug$S                   10000000     Qt5Core:Qt5Core.dll
 0001:fffff000       __ehhandler$?_Copy@?$basic_string@DU?$char_traits@D@std@@V?$allocator@D@2@@std@@QAEXII@Z 10000000 f   ChromatogramView.obj
 0000:fffe1000       .debug$S                   10000000     U2Core:U2Core.dll
 0000:fffe1000       .debug$S                   10000000     U2Core:U2Core.dll
 0000:fffe1000       .debug$S                   10000000     Qt5Core:Qt5Core.dll
 0000:fffe1000       .debug$S                   10000000     Qt5Core:Qt5Core.dll
 0000:fffe1000       .debug$S                   10000000     Qt5Core:Qt5Core.dll
 0000:fffe1000       .debug$S                   10000000     Qt5Core:Qt5Core.dll
 0000:fffe1000       .debug$S                   10000000     Qt5Gui:Qt5Gui.dll
 0000:fffe1000       .debug$S                   10000000     Qt5Gui:Qt5Gui.dll
 0000:fffe1000       .debug$S                   10000000     Qt5Gui:Qt5Gui.dll
 0000:fffe1000       .debug$S                   10000000     Qt5Gui:Qt5Gui.dll
 0000:fffe1000       .debug$S                   10000000     Qt5Gui:Qt5Gui.dll
 0000:fffe1000       .debug$S                   10000000     Qt5Gui:Qt5Gui.dll
 0000:fffe1000       .debug$S                   10000000     Qt5Gui:Qt5Gui.dll
 0000:fffe1000       .debug$S                   10000000     Qt5Gui:Qt5Gui.dll
 0000:fffe1000       .debug$S                   10000000     Qt5Gui:Qt5Gui.dll
 0000:fffe1000       .debug$S                   10000000     Qt5Gui:Qt5Gui.dll
 0000:fffe1000       .debug$S                   10000000     Qt5Gui:Qt5Gui.dll
 0000:fffe1000       .debug$S                   10000000     Qt5Gui:Qt5Gui.dll
 0000:fffe1000       .debug$S                   10000000     Qt5Gui:Qt5Gui.dll
 0000:fffe1000       .debug$S                   10000000     Qt5Gui:Qt5Gui.dll
 0000:fffe1000       .debug$S                   10000000     Qt5Gui:Qt5Gui.dll
 0000:fffe1000       .debug$S                   10000000     Qt5Gui:Qt5Gui.dll
 0000:fffe1000       .debug$S                   10000000     Qt5Gui:Qt5Gui.dll
 0000:fffe1000       .debug$S                   10000000     Qt5Gui:Qt5Gui.dll
 0000:fffe1000       .debug$S                   10000000     Qt5Gui:Qt5Gui.dll
 0000:fffe1000       .debug$S                   10000000     Qt5Gui:Qt5Gui.dll
 0000:fffe1000       .debug$S                   10000000     Qt5Gui:Qt5Gui.dll
 0000:fffe1000       .debug$S                   10000000     Qt5Gui:Qt5Gui.dll
 0001:fffff000       __ehhandler$?detach_helper@?$QList@PAVGObject@U2@@@@AAEXH@Z 10000000 f   ChromatogramView.obj
 0000:fffe1000       .debug$S                   10000000     U2Core:U2Core.dll
 0000:fffe1000       .debug$S                   10000000     Qt5Gui:Qt5Gui.dll
 0000:fffe1000       .debug$S                   10000000     Qt5Gui:Qt5Gui.dll
 0000:fffe1000       .debug$S                   10000000     Qt5Gui:Qt5Gui.dll
 0000:fffe1000       .debug$S                   10000000     Qt5Gui:Qt5Gui.dll
 0000:fffe1000       .debug$S                   10000000     Qt5Gui:Qt5Gui.dll
 0000:fffe1000       .debug$S                   10000000     Qt5Gui:Qt5Gui.dll
 0000:fffe1000       .debug$S                   10000000     Qt5Gui:Qt5Gui.dll
 0000:fffe1000       .debug$S                   10000000     Qt5Gui:Qt5Gui.dll
 0000:fffe1000       .debug$S                   10000000     Qt5Gui:Qt5Gui.dll
 0000:fffe1000       .debug$S                   10000000     Qt5Gui:Qt5Gui.dll
 0000:fffe1000       .debug$S                   10000000     Qt5Gui:Qt5Gui.dll
 0000:fffe1000       .debug$S                   10000000     Qt5Gui:Qt5Gui.dll
 0000:fffe1000       .debug$S                   10000000     Qt5Gui:Qt5Gui.dll
 0000:fffe1000       .debug$S                   10000000     Qt5Gui:Qt5Gui.dll
 0000:fffe1000       .debug$S                   10000000     Qt5Gui:Qt5Gui.dll
 0000:fffe1000       .debug$S                   10000000     Qt5Gui:Qt5Gui.dll
 0000:fffe1000       .debug$S                   10000000     Qt5Gui:Qt5Gui.dll
 0000:fffe1000       .debug$S                   10000000     Qt5Gui:Qt5Gui.dll
 0000:fffe1000       .debug$S                   10000000     Qt5Gui:Qt5Gui.dll
 0000:fffe1000       .debug$S                   10000000     Qt5Gui:Qt5Gui.dll
 0000:fffe1000       .debug$S                   10000000     Qt5Gui:Qt5Gui.dll
 0000:fffe1000       .debug$S                   10000000     Qt5Gui:Qt5Gui.dll
 0000:fffe1000       .debug$S                   10000000     Qt5Gui:Qt5Gui.dll
 0000:fffe1000       .debug$S                   10000000     Qt5Gui:Qt5Gui.dll
 0000:fffe1000       .debug$S                   10000000     Qt5Gui:Qt5Gui.dll
 0000:fffe1000       .debug$S                   10000000     Qt5Widgets:Qt5Widgets.dll
 0000:fffe1000       .debug$S                   10000000     Qt5Widgets:Qt5Widgets.dll
 0000:fffe1000       .debug$S                   10000000     Qt5Widgets:Qt5Widgets.dll
 0000:fffe1000       .debug$S                   10000000     Qt5Widgets:Qt5Widgets.dll
 0000:fffe1000       .debug$S                   10000000     Qt5Widgets:Qt5Widgets.dll
 0000:fffe1000       .debug$S                   10000000     Qt5Widgets:Qt5Widgets.dll
 0000:fffe1000       .debug$S                   10000000     Qt5Widgets:Qt5Widgets.dll
 0000:fffe1000       .debug$S                   10000000     Qt5Widgets:Qt5Widgets.dll
 0000:fffe1000       .debug$S                   10000000     Qt5Widgets:Qt5Widgets.dll
 0000:fffe1000       .debug$S                   10000000     Qt5Widgets:Qt5Widgets.dll
 0000:fffe1000       .debug$S                   10000000     Qt5Widgets:Qt5Widgets.dll
 0000:fffe1000       .debug$S                   10000000     Qt5Widgets:Qt5Widgets.dll
 0000:fffe1000       .debug$S                   10000000     Qt5Widgets:Qt5Widgets.dll
 0000:fffe1000       .debug$S                   10000000     Qt5Widgets:Qt5Widgets.dll
 0000:fffe1000       .debug$S                   10000000     Qt5Widgets:Qt5Widgets.dll
 0000:fffe1000       .debug$S                   10000000     Qt5Widgets:Qt5Widgets.dll
 0000:fffe1000       .debug$S                   10000000     Qt5Widgets:Qt5Widgets.dll
 0000:fffe1000       .debug$S                   10000000     Qt5Widgets:Qt5Widgets.dll
 0000:fffe1000       .debug$S                   10000000     Qt5Widgets:Qt5Widgets.dll
 0000:fffe1000       .debug$S                   10000000     Qt5Widgets:Qt5Widgets.dll
 0000:fffe1000       .debug$S                   10000000     Qt5Widgets:Qt5Widgets.dll
 0000:fffe1000       .debug$S                   10000000     Qt5Widgets:Qt5Widgets.dll
 0000:fffe1000       .debug$S                   10000000     Qt5Widgets:Qt5Widgets.dll
 0000:fffe1000       .debug$S                   10000000     Qt5Widgets:Qt5Widgets.dll
 0000:fffe1000       .debug$S                   10000000     Qt5Widgets:Qt5Widgets.dll
 0000:fffe1000       .debug$S                   10000000     Qt5Widgets:Qt5Widgets.dll
 0000:fffe1000       .debug$S                   10000000     Qt5Widgets:Qt5Widgets.dll
 0000:fffe1000       .debug$S                   10000000     Qt5Widgets:Qt5Widgets.dll
 0000:fffe1000       .debug$S                   10000000     Qt5Widgets:Qt5Widgets.dll
 0000:fffe1000       .debug$S                   10000000     Qt5Widgets:Qt5Widgets.dll
 0000:fffe1000       .debug$S                   10000000     Qt5Widgets:Qt5Widgets.dll
 0000:fffe1000       .debug$S                   10000000     Qt5Widgets:Qt5Widgets.dll
 0000:fffe1000       .debug$S                   10000000     Qt5Widgets:Qt5Widgets.dll
 0000:fffe1000       .debug$S                   10000000     Qt5Widgets:Qt5Widgets.dll
 0000:fffe1000       .debug$S                   10000000     Qt5Widgets:Qt5Widgets.dll
 0000:fffe1000       .debug$S                   10000000     Qt5Widgets:Qt5Widgets.dll
 0000:fffe1000       .debug$S                   10000000     Qt5Widgets:Qt5Widgets.dll
 0000:fffe1000       .debug$S                   10000000     Qt5Widgets:Qt5Widgets.dll
 0000:fffe1000       .debug$S                   10000000     Qt5Widgets:Qt5Widgets.dll
 0000:fffe1000       .debug$S                   10000000     Qt5Widgets:Qt5Widgets.dll
 0000:fffe1000       .debug$S                   10000000     Qt5Widgets:Qt5Widgets.dll
 0000:fffe1000       .debug$S                   10000000     Qt5Widgets:Qt5Widgets.dll
 0000:fffe1000       .debug$S                   10000000     Qt5Widgets:Qt5Widgets.dll
 0000:fffe1000       .debug$S                   10000000     Qt5Widgets:Qt5Widgets.dll
 0000:fffe1000       .debug$S                   10000000     Qt5Widgets:Qt5Widgets.dll
 0000:fffe1000       .debug$S                   10000000     Qt5Widgets:Qt5Widgets.dll
 0000:fffe1000       .debug$S                   10000000     Qt5Widgets:Qt5Widgets.dll
 0000:fffe1000       .debug$S                   10000000     Qt5Widgets:Qt5Widgets.dll
 0000:fffe1000       .debug$S                   10000000     Qt5Widgets:Qt5Widgets.dll
 0000:fffe1000       .debug$S                   10000000     Qt5Widgets:Qt5Widgets.dll
 0000:fffe1000       .debug$S                   10000000     Qt5Widgets:Qt5Widgets.dll
 0000:fffe1000       .debug$S                   10000000     Qt5Widgets:Qt5Widgets.dll
 0000:fffe1000       .debug$S                   10000000     Qt5Widgets:Qt5Widgets.dll
 0000:fffe1000       .debug$S                   10000000     Qt5Widgets:Qt5Widgets.dll
 0000:fffe1000       .debug$S                   10000000     Qt5Widgets:Qt5Widgets.dll
 0000:fffe1000       .debug$S                   10000000     Qt5Widgets:Qt5Widgets.dll
 0000:fffe1000       .debug$S                   10000000     Qt5Widgets:Qt5Widgets.dll
 0000:fffe1000       .debug$S                   10000000     Qt5Widgets:Qt5Widgets.dll
 0000:fffe1000       .debug$S                   10000000     Qt5Widgets:Qt5Widgets.dll
 0000:fffe1000       .debug$S                   10000000     Qt5Widgets:Qt5Widgets.dll
 0000:fffe1000       .debug$S                   10000000     Qt5Widgets:Qt5Widgets.dll
 0000:fffe1000       .debug$S                   10000000     Qt5Widgets:Qt5Widgets.dll
 0000:fffe1000       .debug$S                   10000000     Qt5Widgets:Qt5Widgets.dll
 0000:fffe1000       .debug$S                   10000000     Qt5Widgets:Qt5Widgets.dll
 0000:fffe1000       .debug$S                   10000000     Qt5Widgets:Qt5Widgets.dll
 0000:fffe1000       .debug$S                   10000000     Qt5Widgets:Qt5Widgets.dll
 0000:fffe1000       .debug$S                   10000000     Qt5Widgets:Qt5Widgets.dll
 0000:fffe1000       .debug$S                   10000000     Qt5Widgets:Qt5Widgets.dll
 0000:fffe1000       .debug$S                   10000000     Qt5Widgets:Qt5Widgets.dll
 0000:fffe1000       .debug$S                   10000000     Qt5Widgets:Qt5Widgets.dll
 0000:fffe1000       .debug$S                   10000000     Qt5Widgets:Qt5Widgets.dll
 0000:fffe1000       .debug$S                   10000000     Qt5Widgets:Qt5Widgets.dll
 0000:fffe1000       .debug$S                   10000000     Qt5Widgets:Qt5Widgets.dll
 0000:fffe1000       .debug$S                   10000000     Qt5Widgets:Qt5Widgets.dll
 0000:fffe1000       .debug$S                   10000000     Qt5Widgets:Qt5Widgets.dll
 0000:fffe1000       .debug$S                   10000000     Qt5Widgets:Qt5Widgets.dll
 0000:fffe1000       .debug$S                   10000000     Qt5Widgets:Qt5Widgets.dll
 0000:fffe1000       .debug$S                   10000000     Qt5Widgets:Qt5Widgets.dll
 0000:fffe1000       .debug$S                   10000000     Qt5Widgets:Qt5Widgets.dll
 0000:fffe1000       .debug$S                   10000000     Qt5Widgets:Qt5Widgets.dll
 0000:fffe1000       .debug$S                   10000000     Qt5Widgets:Qt5Widgets.dll
 0000:fffe1000       .debug$S                   10000000     Qt5Widgets:Qt5Widgets.dll
 0000:fffe1000       .debug$S                   10000000     Qt5Widgets:Qt5Widgets.dll
 0000:fffe1000       .debug$S                   10000000     Qt5Widgets:Qt5Widgets.dll
 0000:fffe1000       .debug$S                   10000000     Qt5Widgets:Qt5Widgets.dll
 0000:fffe1000       .debug$S                   10000000     Qt5Widgets:Qt5Widgets.dll
 0000:fffe1000       .debug$S                   10000000     Qt5Widgets:Qt5Widgets.dll
 0000:fffe1000       .debug$S                   10000000     Qt5Widgets:Qt5Widgets.dll
 0000:fffe1000       .debug$S                   10000000     Qt5Widgets:Qt5Widgets.dll
 0000:fffe1000       .debug$S                   10000000     Qt5Widgets:Qt5Widgets.dll
 0000:fffe1000       .debug$S                   10000000     Qt5Widgets:Qt5Widgets.dll
 0000:fffe1000       .debug$S                   10000000     Qt5Widgets:Qt5Widgets.dll
 0000:fffe1000       .debug$S                   10000000     Qt5Widgets:Qt5Widgets.dll
 0000:fffe1000       .debug$S                   10000000     Qt5Widgets:Qt5Widgets.dll
 0000:fffe1000       .debug$S                   10000000     Qt5Widgets:Qt5Widgets.dll
 0000:fffe1000       .debug$S                   10000000     Qt5Widgets:Qt5Widgets.dll
 0000:fffe1000       .debug$S                   10000000     Qt5Widgets:Qt5Widgets.dll
 0000:fffe1000       .debug$S                   10000000     Qt5Widgets:Qt5Widgets.dll
 0000:fffe1000       .debug$S                   10000000     Qt5Widgets:Qt5Widgets.dll
 0000:fffe1000       .debug$S                   10000000     Qt5Widgets:Qt5Widgets.dll
 0000:fffe1000       .debug$S                   10000000     Qt5Widgets:Qt5Widgets.dll
 0000:fffe1000       .debug$S                   10000000     Qt5Widgets:Qt5Widgets.dll
 0000:fffe1000       .debug$S                   10000000     Qt5Widgets:Qt5Widgets.dll
 0000:fffe1000       .debug$S                   10000000     Qt5Widgets:Qt5Widgets.dll
 0000:fffe1000       .debug$S                   10000000     Qt5Widgets:Qt5Widgets.dll
 0000:fffe1000       .debug$S                   10000000     Qt5Widgets:Qt5Widgets.dll
 0000:fffe1000       .debug$S                   10000000     Qt5Widgets:Qt5Widgets.dll
 0000:fffe1000       .debug$S                   10000000     Qt5Widgets:Qt5Widgets.dll
 0000:fffe1000       .debug$S                   10000000     Qt5Widgets:Qt5Widgets.dll
 0000:fffe1000       .debug$S                   10000000     Qt5Widgets:Qt5Widgets.dll
 0000:fffe1000       .debug$S                   10000000     Qt5Widgets:Qt5Widgets.dll
 0000:fffe1000       .debug$S                   10000000     Qt5Widgets:Qt5Widgets.dll
 0000:fffe1000       .debug$S                   10000000     Qt5Widgets:Qt5Widgets.dll
 0000:fffe1000       .debug$S                   10000000     Qt5Widgets:Qt5Widgets.dll
 0000:fffe1000       .debug$S                   10000000     Qt5Widgets:Qt5Widgets.dll
 0000:fffe1000       .debug$S                   10000000     Qt5Widgets:Qt5Widgets.dll
 0000:fffe1000       .debug$S                   10000000     Qt5Widgets:Qt5Widgets.dll
 0000:fffe1000       .debug$S                   10000000     Qt5Widgets:Qt5Widgets.dll
 0000:fffe1000       .debug$S                   10000000     Qt5Widgets:Qt5Widgets.dll
 0000:fffe1000       .debug$S                   10000000     Qt5Widgets:Qt5Widgets.dll
 0000:fffe1000       .debug$S                   10000000     Qt5Widgets:Qt5Widgets.dll
 0000:fffe1000       .debug$S                   10000000     Qt5Widgets:Qt5Widgets.dll
 0000:fffe1000       .debug$S                   10000000     Qt5Widgets:Qt5Widgets.dll
 0000:fffe1000       .debug$S                   10000000     Qt5Widgets:Qt5Widgets.dll
 0000:fffe1000       .debug$S                   10000000     Qt5Widgets:Qt5Widgets.dll
 0000:fffe1000       .debug$S                   10000000     Qt5Widgets:Qt5Widgets.dll
 0000:fffe1000       .debug$S                   10000000     Qt5Widgets:Qt5Widgets.dll
 0000:fffe1000       .debug$S                   10000000     Qt5Widgets:Qt5Widgets.dll
 0000:fffe1000       .debug$S                   10000000     U2View:U2View.dll
 0000:fffe1000       .debug$S                   10000000     U2View:U2View.dll
 0000:fffe1000       .debug$S                   10000000     U2View:U2View.dll
 0000:fffe1000       .debug$S                   10000000     U2View:U2View.dll
 0000:fffe1000       .debug$S                   10000000     U2View:U2View.dll
 0000:fffe1000       .debug$S                   10000000     U2View:U2View.dll
 0000:fffe1000       .debug$S                   10000000     U2View:U2View.dll
 0000:fffe1000       .debug$S                   10000000     U2View:U2View.dll
 0000:fffe1000       .debug$S                   10000000     U2View:U2View.dll
 0000:fffe1000       .debug$S                   10000000     U2View:U2View.dll
 0000:fffe1000       .debug$S                   10000000     U2View:U2View.dll
 0000:fffe1000       .debug$S                   10000000     U2View:U2View.dll
 0000:fffe1000       .debug$S                   10000000     U2View:U2View.dll
 0000:fffe1000       .debug$S                   10000000     U2View:U2View.dll
 0000:fffe1000       .debug$S                   10000000     U2View:U2View.dll
 0000:fffe1000       .debug$S                   10000000     U2View:U2View.dll
 0000:fffe1000       .debug$S                   10000000     U2View:U2View.dll
 0000:fffe1000       .debug$S                   10000000     U2View:U2View.dll
 0000:fffe1000       .debug$S                   10000000     U2View:U2View.dll
 0000:fffe1000       .debug$S                   10000000     U2View:U2View.dll
 0000:fffe1000       .debug$S                   10000000     U2View:U2View.dll
 0000:fffe1000       .debug$S                   10000000     U2View:U2View.dll
 0000:fffe1000       .debug$S                   10000000     U2View:U2View.dll
 0000:fffe1000       .debug$S                   10000000     U2View:U2View.dll
 0000:fffe1000       .debug$S                   10000000     U2View:U2View.dll
 0000:fffe1000       .debug$S                   10000000     U2View:U2View.dll
 0000:fffe1000       .debug$S                   10000000     U2View:U2View.dll
 0000:fffe1000       .debug$S                   10000000     U2View:U2View.dll
 0000:fffe1000       .debug$S                   10000000     U2View:U2View.dll
 0000:fffe1000       .debug$S                   10000000     U2View:U2View.dll
 0000:fffe1000       .debug$S                   10000000     U2View:U2View.dll
 0000:fffe1000       .debug$S                   10000000     U2View:U2View.dll
 0000:fffe1000       .debug$S                   10000000     U2View:U2View.dll
 0000:fffe1000       .debug$S                   10000000     U2View:U2View.dll
 0000:fffe1000       .debug$S                   10000000     U2View:U2View.dll
 0000:fffe1000       .debug$S                   10000000     U2View:U2View.dll
 0000:fffe1000       .debug$S                   10000000     U2View:U2View.dll
 0000:fffe1000       .debug$S                   10000000     U2View:U2View.dll
 0000:fffe1000       .debug$S                   10000000     U2View:U2View.dll
 0000:fffe1000       .debug$S                   10000000     U2View:U2View.dll
 0000:fffe1000       .debug$S                   10000000     U2View:U2View.dll
 0000:fffe1000       .debug$S                   10000000     U2View:U2View.dll
 0000:fffe1000       .debug$S                   10000000     U2View:U2View.dll
 0000:fffe1000       .debug$S                   10000000     U2View:U2View.dll
 0000:fffe1000       .debug$S                   10000000     U2View:U2View.dll
 0000:fffe1000       .debug$S                   10000000     U2View:U2View.dll
 0000:fffe1000       .debug$S                   10000000     U2View:U2View.dll
 0000:fffe1000       .debug$S                   10000000     U2View:U2View.dll
 0000:fffe1000       .debug$S                   10000000     U2View:U2View.dll
 0000:fffe1000       .debug$S                   10000000     U2View:U2View.dll
 0000:fffe1000       .debug$S                   10000000     U2View:U2View.dll
 0000:fffe1000       .debug$S                   10000000     U2View:U2View.dll
 0000:fffe1000       .debug$S                   10000000     U2View:U2View.dll
 0000:fffe1000       .debug$S                   10000000     U2View:U2View.dll
 0000:fffe1000       .debug$S                   10000000     U2View:U2View.dll
 0000:fffe1000       .debug$S                   10000000     U2View:U2View.dll
 0000:fffe1000       .debug$S                   10000000     U2View:U2View.dll
 0000:fffe1000       .debug$S                   10000000     U2View:U2View.dll
 0000:fffe1000       .debug$S                   10000000     U2View:U2View.dll
 0000:fffe1000       .debug$S                   10000000     U2Core:U2Core.dll
 0000:fffe1000       .debug$S                   10000000     U2Core:U2Core.dll
 0000:fffe1000       .debug$S                   10000000     U2Core:U2Core.dll
 0000:fffe1000       .debug$S                   10000000     U2Core:U2Core.dll
 0002:ffff0000       __catchsym$?_Copy@?$basic_string@DU?$char_traits@D@std@@V?$allocator@D@2@@std@@QAEXII@Z$5 10000000     ChromatogramView.obj
 0000:fffe1000       .debug$S                   10000000     U2View:U2View.dll
 0000:fffe1000       .debug$S                   10000000     U2View:U2View.dll
 0000:fffe1000       .debug$S                   10000000     U2View:U2View.dll
 0000:fffe1000       .debug$S                   10000000     U2View:U2View.dll
 0000:fffe1000       .debug$S                   10000000     U2View:U2View.dll
 0000:fffe1000       .debug$S                   10000000     U2Gui:U2Gui.dll
 0000:fffe1000       .debug$S                   10000000     U2Gui:U2Gui.dll
 0000:fffe1000       .debug$S                   10000000     U2Gui:U2Gui.dll
 0000:fffe1000       .debug$S                   10000000     U2Gui:U2Gui.dll
 0000:fffe1000       .debug$S                   10000000     U2Gui:U2Gui.dll
 0000:fffe1000       .debug$S                   10000000     U2Gui:U2Gui.dll
 0000:fffe1000       .debug$S                   10000000     U2Gui:U2Gui.dll
 0000:fffe1000       .debug$S                   10000000     U2Gui:U2Gui.dll
 0000:fffe1000       .debug$S                   10000000     U2Gui:U2Gui.dll
 0000:fffe1000       .debug$S                   10000000     U2Gui:U2Gui.dll
 0000:fffe1000       .debug$S                   10000000     U2Gui:U2Gui.dll
 0000:fffe1000       .debug$S                   10000000     U2Gui:U2Gui.dll
 0000:fffe1000       .debug$S                   10000000     U2Gui:U2Gui.dll
 0000:fffe1000       .debug$S                   10000000     U2Gui:U2Gui.dll
 0000:fffe1000       .debug$S                   10000000     U2Gui:U2Gui.dll
 0000:fffe1000       .debug$S                   10000000     U2Gui:U2Gui.dll
 0000:fffe1000       .debug$S                   10000000     U2Gui:U2Gui.dll
 0000:fffe1000       .debug$S                   10000000     U2Gui:U2Gui.dll
 0000:fffe1000       .debug$S                   10000000     U2Gui:U2Gui.dll
 0000:fffe1000       .debug$S                   10000000     U2Gui:U2Gui.dll
 0000:fffe1000       .debug$S                   10000000     U2Gui:U2Gui.dll
 0000:fffe1000       .debug$S                   10000000     U2Gui:U2Gui.dll
 0000:fffe1000       .debug$S                   10000000     U2Gui:U2Gui.dll
 0000:fffe1000       .debug$S                   10000000     U2Gui:U2Gui.dll
 0000:fffe1000       .debug$S                   10000000     U2Gui:U2Gui.dll
 0000:fffe1000       .debug$S                   10000000     U2Core:U2Core.dll
 0000:fffe1000       .debug$S                   10000000     U2Core:U2Core.dll
 0000:fffe1000       .debug$S                   10000000     U2Core:U2Core.dll
 0002:ffff0000       __catchsym$?detach_helper@?$QList@PAVGObject@U2@@@@AAEXH@Z$2 10000000     ChromatogramView.obj
 0000:fffe1000       .debug$S                   10000000     U2Gui:U2Gui.dll
 0000:fffe1000       .debug$S                   10000000     U2Gui:U2Gui.dll
 0000:fffe1000       .debug$S                   10000000     U2Gui:U2Gui.dll
 0000:fffe1000       .debug$S                   10000000     U2Core:U2Core.dll
 0000:fffe1000       .debug$S                   10000000     U2Core:U2Core.dll
 0000:fffe1000       .debug$S                   10000000     U2Core:U2Core.dll
 0000:fffe1000       .debug$S                   10000000     U2Core:U2Core.dll
 0000:fffe1000       .debug$S                   10000000     U2Core:U2Core.dll
 0000:fffe1000       .debug$S                   10000000     U2Core:U2Core.dll
 0000:fffe1000       .debug$S                   10000000     U2Core:U2Core.dll
 0000:fffe1000       .debug$S                   10000000     U2Core:U2Core.dll
 0000:fffe1000       .debug$S                   10000000     U2Core:U2Core.dll
 0000:fffe1000       .debug$S                   10000000     U2Core:U2Core.dll
 0000:fffe1000       .debug$S                   10000000     U2Core:U2Core.dll
 0000:fffe1000       .debug$S                   10000000     U2Core:U2Core.dll
 0000:fffe1000       .debug$S                   10000000     U2Core:U2Core.dll
 0000:fffe1000       .debug$S                   10000000     U2Core:U2Core.dll
 0000:fffe1000       .debug$S                   10000000     U2Core:U2Core.dll
 0000:fffe1000       .debug$S                   10000000     U2Core:U2Core.dll
 0000:fffe1000       .debug$S                   10000000     U2Core:U2Core.dll
 0000:fffe1000       .debug$S                   10000000     U2Core:U2Core.dll
 0000:fffe1000       .debug$S                   10000000     U2Core:U2Core.dll
 0000:fffe1000       .debug$S                   10000000     U2Core:U2Core.dll
 0000:fffe1000       .debug$S                   10000000     U2Core:U2Core.dll
 0000:fffe1000       .debug$S                   10000000     U2Core:U2Core.dll
 0000:fffe1000       .debug$S                   10000000     U2Core:U2Core.dll
 0000:fffe1000       .debug$S                   10000000     U2Core:U2Core.dll
 0000:fffe1000       .debug$S                   10000000     U2Core:U2Core.dll
 0002:ffff0000       ?_Generic_object$initializer$@?$_Error_objects@H@std@@2P6AXXZA 10000000     ChromatogramView.obj
 0002:ffff0010       __unwindtable$?detach_helper@?$QList@PAVGObject@U2@@@@AAEXH@Z 10000010     ChromatogramView.obj
 0002:ffff0010       __catchsym$?_Copy@?$basic_string@DU?$char_traits@D@std@@V?$allocator@D@2@@std@@QAEXII@Z$4 10000010     moc_ChromatogramView.obj
 0002:ffff0010       __catchsym$?_Copy@?$basic_string@DU?$char_traits@D@std@@V?$allocator@D@2@@std@@QAEXII@Z$4 10000010     ChromatogramView.obj
 0002:ffff0010       __catchsym$?_Copy@?$basic_string@DU?$char_traits@D@std@@V?$allocator@D@2@@std@@QAEXII@Z$4 10000010     moc_ChromaViewPlugin.obj
 0002:ffff0020       __tryblocktable$?detach_helper@?$QList@PAVGObject@U2@@@@AAEXH@Z 10000020     ChromatogramView.obj
 0002:ffff0020       __unwindtable$?_Copy@?$basic_string@DU?$char_traits@D@std@@V?$allocator@D@2@@std@@QAEXII@Z 10000020     moc_ChromaViewPlugin.obj
 0002:ffff0020       __unwindtable$?_Copy@?$basic_string@DU?$char_traits@D@std@@V?$allocator@D@2@@std@@QAEXII@Z 10000020     ChromatogramView.obj
 0002:ffff0020       __unwindtable$?_Copy@?$basic_string@DU?$char_traits@D@std@@V?$allocator@D@2@@std@@QAEXII@Z 10000020     moc_ChromatogramView.obj
 0002:ffff0034       __ehfuncinfo$?detach_helper@?$QList@PAVGObject@U2@@@@AAEXH@Z 10000034     ChromatogramView.obj
 0002:ffff0040       __ehfuncinfo$?_Copy@?$basic_string@DU?$char_traits@D@std@@V?$allocator@D@2@@std@@QAEXII@Z 10000040     moc_ChromatogramView.obj
 0002:ffff0040       __ehfuncinfo$?_Copy@?$basic_string@DU?$char_traits@D@std@@V?$allocator@D@2@@std@@QAEXII@Z 10000040     moc_ChromaViewPlugin.obj
 0002:ffff0040       __ehfuncinfo$?_Copy@?$basic_string@DU?$char_traits@D@std@@V?$allocator@D@2@@std@@QAEXII@Z 10000040     ChromatogramView.obj
 0002:ffff0064       __tryblocktable$?_Copy@?$basic_string@DU?$char_traits@D@std@@V?$allocator@D@2@@std@@QAEXII@Z 10000064     moc_ChromatogramView.obj
 0002:ffff0064       __tryblocktable$?_Copy@?$basic_string@DU?$char_traits@D@std@@V?$allocator@D@2@@std@@QAEXII@Z 10000064     ChromatogramView.obj
 0002:ffff0064       __tryblocktable$?_Copy@?$basic_string@DU?$char_traits@D@std@@V?$allocator@D@2@@std@@QAEXII@Z 10000064     moc_ChromaViewPlugin.obj
 0001:fffff096       __catch$?_Copy@?$basic_string@DU?$char_traits@D@std@@V?$allocator@D@2@@std@@QAEXII@Z$0 10000096 f   moc_ChromatogramView.obj
 0001:fffff096       __catch$?_Copy@?$basic_string@DU?$char_traits@D@std@@V?$allocator@D@2@@std@@QAEXII@Z$0 10000096 f   moc_ChromaViewPlugin.obj
 0001:fffff096       __catch$?_Copy@?$basic_string@DU?$char_traits@D@std@@V?$allocator@D@2@@std@@QAEXII@Z$0 10000096 f   ChromatogramView.obj
 0001:fffff0ac       __catch$?detach_helper@?$QList@PAVGObject@U2@@@@AAEXH@Z$0 100000ac f   ChromatogramView.obj
 0001:fffff0d3       __catch$?_Copy@?$basic_string@DU?$char_traits@D@std@@V?$allocator@D@2@@std@@QAEXII@Z$1 100000d3 f   moc_ChromatogramView.obj
 0001:fffff0d3       __catch$?_Copy@?$basic_string@DU?$char_traits@D@std@@V?$allocator@D@2@@std@@QAEXII@Z$1 100000d3 f   ChromatogramView.obj
 0001:fffff0d3       __catch$?_Copy@?$basic_string@DU?$char_traits@D@std@@V?$allocator@D@2@@std@@QAEXII@Z$1 100000d3 f   moc_ChromaViewPlugin.obj
 0001:00000000       ??__E?_Generic_object@?$_Error_objects@H@std@@2V_Generic_error_category@2@A@@YAXXZ 10001000 f   ChromaViewPlugin.obj
 0001:00000010       ??__E?_Iostream_object@?$_Error_objects@H@std@@2V_Iostream_error_category@2@A@@YAXXZ 10001010 f   ChromaViewPlugin.obj
 0001:00000020       ??__E?_System_object@?$_Error_objects@H@std@@2V_System_error_category@2@A@@YAXXZ 10001020 f   ChromaViewPlugin.obj
 0001:00000030       ??__EService_DNAExport@U2@@YAXXZ 10001030 f   ChromaViewPlugin.obj
 0001:00000040       ??__EService_DNAGraphPack@U2@@YAXXZ 10001040 f   ChromaViewPlugin.obj
 0001:00000050       ??__EService_ExternalToolSupport@U2@@YAXXZ 10001050 f   ChromaViewPlugin.obj
 0001:00000060       ??__EService_GUITesting@U2@@YAXXZ 10001060 f   ChromaViewPlugin.obj
 0001:00000070       ??__EService_MaxCoreServiceId@U2@@YAXXZ 10001070 f   ChromaViewPlugin.obj
 0001:00000080       ??__EService_MinCoreServiceId@U2@@YAXXZ 10001080 f   ChromaViewPlugin.obj
 0001:00000090       ??__EService_PluginViewer@U2@@YAXXZ 10001090 f   ChromaViewPlugin.obj
 0001:000000a0       ??__EService_Project@U2@@YAXXZ 100010a0 f   ChromaViewPlugin.obj
 0001:000000b0       ??__EService_ProjectView@U2@@YAXXZ 100010b0 f   ChromaViewPlugin.obj
 0001:000000c0       ??__EService_QueryDesigner@U2@@YAXXZ 100010c0 f   ChromaViewPlugin.obj
 0001:000000d0       ??__EService_ScriptRegistry@U2@@YAXXZ 100010d0 f   ChromaViewPlugin.obj
 0001:000000e0       ??__EService_TestRunner@U2@@YAXXZ 100010e0 f   ChromaViewPlugin.obj
 0001:000000f0       ??__EService_WorkflowDesigner@U2@@YAXXZ 100010f0 f   ChromaViewPlugin.obj
 0001:00000100       ??__EalgoLog@U2@@YAXXZ     10001100 f   ChromaViewPlugin.obj
 0001:00000180       ??__EcmdLog@U2@@YAXXZ      10001180 f   ChromaViewPlugin.obj
 0001:00000200       ??__EcoreLog@U2@@YAXXZ     10001200 f   ChromaViewPlugin.obj
 0001:00000280       ??__EioLog@U2@@YAXXZ       10001280 f   ChromaViewPlugin.obj
 0001:00000300       ??__EperfLog@U2@@YAXXZ     10001300 f   ChromaViewPlugin.obj
 0001:00000380       ??__EscriptLog@U2@@YAXXZ   10001380 f   ChromaViewPlugin.obj
 0001:00000400       ??__EtaskLog@U2@@YAXXZ     10001400 f   ChromaViewPlugin.obj
 0001:00000480       ??__EuiLog@U2@@YAXXZ       10001480 f   ChromaViewPlugin.obj
 0001:00000500       ??__EuserActLog@U2@@YAXXZ  10001500 f   ChromaViewPlugin.obj
 0001:00000580       ??__E?_Generic_object@?$_Error_objects@H@std@@2V_Generic_error_category@2@A@@YAXXZ 10001580 f   ChromatogramView.obj
 0001:00000590       ??__E?_Iostream_object@?$_Error_objects@H@std@@2V_Iostream_error_category@2@A@@YAXXZ 10001590 f   ChromatogramView.obj
 0001:000005a0       ??__E?_System_object@?$_Error_objects@H@std@@2V_System_error_category@2@A@@YAXXZ 100015a0 f   ChromatogramView.obj
 0001:000005b0       ??__EService_DNAExport@U2@@YAXXZ 100015b0 f   ChromatogramView.obj
 0001:000005c0       ??__EService_DNAGraphPack@U2@@YAXXZ 100015c0 f   ChromatogramView.obj
 0001:000005d0       ??__EService_ExternalToolSupport@U2@@YAXXZ 100015d0 f   ChromatogramView.obj
 0001:000005e0       ??__EService_GUITesting@U2@@YAXXZ 100015e0 f   ChromatogramView.obj
 0001:000005f0       ??__EService_MaxCoreServiceId@U2@@YAXXZ 100015f0 f   ChromatogramView.obj
 0001:00000600       ??__EService_MinCoreServiceId@U2@@YAXXZ 10001600 f   ChromatogramView.obj
 0001:00000610       ??__EService_PluginViewer@U2@@YAXXZ 10001610 f   ChromatogramView.obj
 0001:00000620       ??__EService_Project@U2@@YAXXZ 10001620 f   ChromatogramView.obj
 0001:00000630       ??__EService_ProjectView@U2@@YAXXZ 10001630 f   ChromatogramView.obj
 0001:00000640       ??__EService_QueryDesigner@U2@@YAXXZ 10001640 f   ChromatogramView.obj
 0001:00000650       ??__EService_ScriptRegistry@U2@@YAXXZ 10001650 f   ChromatogramView.obj
 0001:00000660       ??__EService_TestRunner@U2@@YAXXZ 10001660 f   ChromatogramView.obj
 0001:00000670       ??__EService_WorkflowDesigner@U2@@YAXXZ 10001670 f   ChromatogramView.obj
 0001:00000680       ??__EalgoLog@U2@@YAXXZ     10001680 f   ChromatogramView.obj
 0001:00000700       ??__EcmdLog@U2@@YAXXZ      10001700 f   ChromatogramView.obj
 0001:00000780       ??__EcoreLog@U2@@YAXXZ     10001780 f   ChromatogramView.obj
 0001:00000800       ??__EioLog@U2@@YAXXZ       10001800 f   ChromatogramView.obj
 0001:00000880       ??__EperfLog@U2@@YAXXZ     10001880 f   ChromatogramView.obj
 0001:00000900       ??__EscriptLog@U2@@YAXXZ   10001900 f   ChromatogramView.obj
 0001:00000980       ??__EtaskLog@U2@@YAXXZ     10001980 f   ChromatogramView.obj
 0001:00000a00       ??__EuiLog@U2@@YAXXZ       10001a00 f   ChromatogramView.obj
 0001:00000a80       ??__EuserActLog@U2@@YAXXZ  10001a80 f   ChromatogramView.obj
 0001:00000b00       ??__E?_Generic_object@?$_Error_objects@H@std@@2V_Generic_error_category@2@A@@YAXXZ 10001b00 f   moc_ChromaViewPlugin.obj
 0001:00000b10       ??__E?_Iostream_object@?$_Error_objects@H@std@@2V_Iostream_error_category@2@A@@YAXXZ 10001b10 f   moc_ChromaViewPlugin.obj
 0001:00000b20       ??__E?_System_object@?$_Error_objects@H@std@@2V_System_error_category@2@A@@YAXXZ 10001b20 f   moc_ChromaViewPlugin.obj
 0001:00000b30       ??__E?staticMetaObject@ChromaViewAction@U2@@2UQMetaObject@@B@@YAXXZ 10001b30 f   moc_ChromaViewPlugin.obj
 0001:00000b40       ??__E?staticMetaObject@ChromaViewContext@U2@@2UQMetaObject@@B@@YAXXZ 10001b40 f   moc_ChromaViewPlugin.obj
 0001:00000b50       ??__E?staticMetaObject@ChromaViewPlugin@U2@@2UQMetaObject@@B@@YAXXZ 10001b50 f   moc_ChromaViewPlugin.obj
 0001:00000b60       ??__EService_DNAExport@U2@@YAXXZ 10001b60 f   moc_ChromaViewPlugin.obj
 0001:00000b70       ??__EService_DNAGraphPack@U2@@YAXXZ 10001b70 f   moc_ChromaViewPlugin.obj
 0001:00000b80       ??__EService_ExternalToolSupport@U2@@YAXXZ 10001b80 f   moc_ChromaViewPlugin.obj
 0001:00000b90       ??__EService_GUITesting@U2@@YAXXZ 10001b90 f   moc_ChromaViewPlugin.obj
 0001:00000ba0       ??__EService_MaxCoreServiceId@U2@@YAXXZ 10001ba0 f   moc_ChromaViewPlugin.obj
 0001:00000bb0       ??__EService_MinCoreServiceId@U2@@YAXXZ 10001bb0 f   moc_ChromaViewPlugin.obj
 0001:00000bc0       ??__EService_PluginViewer@U2@@YAXXZ 10001bc0 f   moc_ChromaViewPlugin.obj
 0001:00000bd0       ??__EService_Project@U2@@YAXXZ 10001bd0 f   moc_ChromaViewPlugin.obj
 0001:00000be0       ??__EService_ProjectView@U2@@YAXXZ 10001be0 f   moc_ChromaViewPlugin.obj
 0001:00000bf0       ??__EService_QueryDesigner@U2@@YAXXZ 10001bf0 f   moc_ChromaViewPlugin.obj
 0001:00000c00       ??__EService_ScriptRegistry@U2@@YAXXZ 10001c00 f   moc_ChromaViewPlugin.obj
 0001:00000c10       ??__EService_TestRunner@U2@@YAXXZ 10001c10 f   moc_ChromaViewPlugin.obj
 0001:00000c20       ??__EService_WorkflowDesigner@U2@@YAXXZ 10001c20 f   moc_ChromaViewPlugin.obj
 0001:00000c30       ??__E?_Generic_object@?$_Error_objects@H@std@@2V_Generic_error_category@2@A@@YAXXZ 10001c30 f   moc_ChromatogramView.obj
 0001:00000c40       ??__E?_Iostream_object@?$_Error_objects@H@std@@2V_Iostream_error_category@2@A@@YAXXZ 10001c40 f   moc_ChromatogramView.obj
 0001:00000c50       ??__E?_System_object@?$_Error_objects@H@std@@2V_System_error_category@2@A@@YAXXZ 10001c50 f   moc_ChromatogramView.obj
 0001:00000c60       ??__E?staticMetaObject@ChromatogramView@U2@@2UQMetaObject@@B@@YAXXZ 10001c60 f   moc_ChromatogramView.obj
 0001:00000c70       ??__E?staticMetaObject@ChromatogramViewRenderArea@U2@@2UQMetaObject@@B@@YAXXZ 10001c70 f   moc_ChromatogramView.obj
 0001:00000c80       ??__Edummy@?A0xc45d533f@@YAXXZ 10001c80 f   qrc_chroma_view.obj
 0001:00000f6e       __catch$??0?$QList@PAVADVSequenceWidget@U2@@@@QAE@ABV0@@Z$0 10001f6e f i ChromaViewPlugin.obj
 0001:00001836       __catch$?_Copy@?$basic_string@DU?$char_traits@D@std@@V?$allocator@D@2@@std@@QAEXII@Z$0 10002836 f i ChromaViewPlugin.obj
 0001:00001873       __catch$?_Copy@?$basic_string@DU?$char_traits@D@std@@V?$allocator@D@2@@std@@QAEXII@Z$1 10002873 f i ChromaViewPlugin.obj
 0001:0000201c       __catch$?detach_helper@?$QList@PAVGObject@U2@@@@AAEXH@Z$0 1000301c f i ChromaViewPlugin.obj
 0001:000021b0       ?findChromaObj@U2@@YAPAVDNAChromatogramObject@1@PAVADVSingleSequenceWidget@1@@Z 100031b0 f   ChromaViewPlugin.obj
 0001:00002f6e       __catch$??0?$QList@H@@QAE@ABV0@@Z$0 10003f6e f i ChromatogramView.obj
 0001:0000303e       __catch$??0?$QList@PAVGObject@U2@@@@QAE@ABV0@@Z$0 1000403e f i ChromatogramView.obj
 0001:000030fe       __catch$??0?$QList@PAVQAction@@@@QAE@ABV0@@Z$0 100040fe f i ChromatogramView.obj
 0001:00004f15       __catch$?append@?$QList@H@@QAEXABH@Z$4 10005f15 f i ChromatogramView.obj
 0001:00004f9c       __catch$?append@?$QList@V?$QPointer@VGObject@U2@@@@@@QAEXABV?$QPointer@VGObject@U2@@@@@Z$2 10005f9c f i ChromatogramView.obj
 0001:00004f9c       __catch$?append@?$QList@V?$QPointer@VGObject@U2@@@@@@QAEXABV?$QPointer@VGObject@U2@@@@@Z$0 10005f9c f i ChromatogramView.obj
 0001:00005d7c       __catch$?detach_helper@?$QList@H@@AAEXH@Z$0 10006d7c f i ChromatogramView.obj
 0001:00005ea1       __catch$?detach_helper_grow@?$QList@H@@AAEPAUNode@1@HH@Z$0 10006ea1 f i ChromatogramView.obj
 0001:00005ea1       __catch$?detach_helper_grow@?$QList@H@@AAEPAUNode@1@HH@Z$2 10006ea1 f i ChromatogramView.obj
 0001:00005fcc       __catch$?detach_helper_grow@?$QList@V?$QPointer@VGObject@U2@@@@@@AAEPAUNode@1@HH@Z$2 10006fcc f i ChromatogramView.obj
 0001:00006007       __catch$?detach_helper_grow@?$QList@V?$QPointer@VGObject@U2@@@@@@AAEPAUNode@1@HH@Z$0 10007007 f i ChromatogramView.obj
 0001:00006f68       $LN86                      10007f68     ChromatogramView.obj
 0001:00006f80       $LN82                      10007f80     ChromatogramView.obj
 0001:00008158       $LN316                     10009158     ChromatogramView.obj
 0001:0000816c       $LN309                     1000916c     ChromatogramView.obj
 0001:0000857c       $LN13                      1000957c     ChromatogramView.obj
 0001:00008590       $LN10                      10009590     ChromatogramView.obj
 0001:00008e85       __catch$?node_copy@?$QList@V?$QPointer@VGObject@U2@@@@@@AAEXPAUNode@1@00@Z$0 10009e85 f i ChromatogramView.obj
 0001:00009373       __catch$?reallocData@?$QVector@D@@AAEXHHV?$QFlags@W4AllocationOption@QArrayData@@@@@Z$0 1000a373 f i ChromatogramView.obj
 0001:00009385       __catch$?reallocData@?$QVector@D@@AAEXHHV?$QFlags@W4AllocationOption@QArrayData@@@@@Z$2 1000a385 f i ChromatogramView.obj
 0001:000095b3       __catch$?reallocData@?$QVector@G@@AAEXHHV?$QFlags@W4AllocationOption@QArrayData@@@@@Z$0 1000a5b3 f i ChromatogramView.obj
 0001:000095c5       __catch$?reallocData@?$QVector@G@@AAEXHHV?$QFlags@W4AllocationOption@QArrayData@@@@@Z$2 1000a5c5 f i ChromatogramView.obj
 0001:0000ba8c       $LN50                      1000ca8c     moc_ChromatogramView.obj
 0001:0000c7ff       ?ArrayUnwindFilter@@YAHPAU_EXCEPTION_POINTERS@@@Z 1000d7ff f   MSVCRT:ehvecdtr.obj
 0001:0000c880       $$000000                   1000d880     MSVCRT:ftol3.obj
 0001:0000cc54       _pre_c_init                1000dc54 f   MSVCRT:crtdll.obj
 0001:0000cec1       ___DllMainCRTStartup       1000dec1 f   MSVCRT:crtdll.obj
 0001:0000d010       $$000000                   1000e010     MSVCRT:sehprolg4.obj
 0001:0000d6a0       __ehhandler$??0?$QList@PAVADVSequenceWidget@U2@@@@QAE@ABV0@@Z 1000e6a0 f   ChromaViewPlugin.obj
 0001:0000d6c0       __unwindfunclet$??0ChromaViewAction@U2@@QAE@XZ$0 1000e6c0 f   ChromaViewPlugin.obj
 0001:0000d6c9       __unwindfunclet$??0ChromaViewAction@U2@@QAE@XZ$1 1000e6c9 f   ChromaViewPlugin.obj
 0001:0000d6d2       __unwindfunclet$??0ChromaViewAction@U2@@QAE@XZ$2 1000e6d2 f   ChromaViewPlugin.obj
 0001:0000d6db       __ehhandler$??0ChromaViewAction@U2@@QAE@XZ 1000e6db f   ChromaViewPlugin.obj
 0001:0000d700       __unwindfunclet$??0ChromaViewContext@U2@@QAE@PAVQObject@@@Z$0 1000e700 f   ChromaViewPlugin.obj
 0001:0000d708       __unwindfunclet$??0ChromaViewContext@U2@@QAE@PAVQObject@@@Z$1 1000e708 f   ChromaViewPlugin.obj
 0001:0000d711       __ehhandler$??0ChromaViewContext@U2@@QAE@PAVQObject@@@Z 1000e711 f   ChromaViewPlugin.obj
 0001:0000d730       __unwindfunclet$??0ChromaViewPlugin@U2@@QAE@XZ$0 1000e730 f   ChromaViewPlugin.obj
 0001:0000d739       __unwindfunclet$??0ChromaViewPlugin@U2@@QAE@XZ$1 1000e739 f   ChromaViewPlugin.obj
 0001:0000d742       __unwindfunclet$??0ChromaViewPlugin@U2@@QAE@XZ$2 1000e742 f   ChromaViewPlugin.obj
 0001:0000d74b       __unwindfunclet$??0ChromaViewPlugin@U2@@QAE@XZ$3 1000e74b f   ChromaViewPlugin.obj
 0001:0000d756       __unwindfunclet$??0ChromaViewPlugin@U2@@QAE@XZ$4 1000e756 f   ChromaViewPlugin.obj
 0001:0000d75e       __unwindfunclet$??0ChromaViewPlugin@U2@@QAE@XZ$5 1000e75e f   ChromaViewPlugin.obj
 0001:0000d767       __ehhandler$??0ChromaViewPlugin@U2@@QAE@XZ 1000e767 f   ChromaViewPlugin.obj
 0001:0000d790       __unwindfunclet$??__EalgoLog@U2@@YAXXZ$0 1000e790 f   ChromaViewPlugin.obj
 0001:0000d799       __ehhandler$??__EalgoLog@U2@@YAXXZ 1000e799 f   ChromaViewPlugin.obj
 0001:0000d7c0       __unwindfunclet$??__EcmdLog@U2@@YAXXZ$0 1000e7c0 f   ChromaViewPlugin.obj
 0001:0000d7c9       __ehhandler$??__EcmdLog@U2@@YAXXZ 1000e7c9 f   ChromaViewPlugin.obj
 0001:0000d7f0       __unwindfunclet$??__EcoreLog@U2@@YAXXZ$0 1000e7f0 f   ChromaViewPlugin.obj
 0001:0000d7f9       __ehhandler$??__EcoreLog@U2@@YAXXZ 1000e7f9 f   ChromaViewPlugin.obj
 0001:0000d820       __unwindfunclet$??__EioLog@U2@@YAXXZ$0 1000e820 f   ChromaViewPlugin.obj
 0001:0000d829       __ehhandler$??__EioLog@U2@@YAXXZ 1000e829 f   ChromaViewPlugin.obj
 0001:0000d850       __unwindfunclet$??__EperfLog@U2@@YAXXZ$0 1000e850 f   ChromaViewPlugin.obj
 0001:0000d859       __ehhandler$??__EperfLog@U2@@YAXXZ 1000e859 f   ChromaViewPlugin.obj
 0001:0000d880       __unwindfunclet$??__EscriptLog@U2@@YAXXZ$0 1000e880 f   ChromaViewPlugin.obj
 0001:0000d889       __ehhandler$??__EscriptLog@U2@@YAXXZ 1000e889 f   ChromaViewPlugin.obj
 0001:0000d8b0       __unwindfunclet$??__EtaskLog@U2@@YAXXZ$0 1000e8b0 f   ChromaViewPlugin.obj
 0001:0000d8b9       __ehhandler$??__EtaskLog@U2@@YAXXZ 1000e8b9 f   ChromaViewPlugin.obj
 0001:0000d8e0       __unwindfunclet$??__EuiLog@U2@@YAXXZ$0 1000e8e0 f   ChromaViewPlugin.obj
 0001:0000d8e9       __ehhandler$??__EuiLog@U2@@YAXXZ 1000e8e9 f   ChromaViewPlugin.obj
 0001:0000d910       __unwindfunclet$??__EuserActLog@U2@@YAXXZ$0 1000e910 f   ChromaViewPlugin.obj
 0001:0000d919       __ehhandler$??__EuserActLog@U2@@YAXXZ 1000e919 f   ChromaViewPlugin.obj
 0001:0000d940       __ehhandler$?_Copy@?$basic_string@DU?$char_traits@D@std@@V?$allocator@D@2@@std@@QAEXII@Z 1000e940 f   ChromaViewPlugin.obj
 0001:0000d960       __ehhandler$?detach_helper@?$QList@PAVGObject@U2@@@@AAEXH@Z 1000e960 f   ChromaViewPlugin.obj
 0001:0000d980       __unwindfunclet$?findChromaObj@U2@@YAPAVDNAChromatogramObject@1@PAVADVSingleSequenceWidget@1@@Z$1 1000e980 f   ChromaViewPlugin.obj
 0001:0000d988       __unwindfunclet$?findChromaObj@U2@@YAPAVDNAChromatogramObject@1@PAVADVSingleSequenceWidget@1@@Z$3 1000e988 f   ChromaViewPlugin.obj
 0001:0000d990       __ehhandler$?findChromaObj@U2@@YAPAVDNAChromatogramObject@1@PAVADVSingleSequenceWidget@1@@Z 1000e990 f   ChromaViewPlugin.obj
 0001:0000d9b0       __unwindfunclet$?initViewContext@ChromaViewContext@U2@@MAEXPAVGObjectView@2@@Z$0 1000e9b0 f   ChromaViewPlugin.obj
 0001:0000d9b8       __unwindfunclet$?initViewContext@ChromaViewContext@U2@@MAEXPAVGObjectView@2@@Z$1 1000e9b8 f   ChromaViewPlugin.obj
 0001:0000d9c0       __ehhandler$?initViewContext@ChromaViewContext@U2@@MAEXPAVGObjectView@2@@Z 1000e9c0 f   ChromaViewPlugin.obj
 0001:0000d9e0       __unwindfunclet$?sl_sequenceWidgetAdded@ChromaViewContext@U2@@IAEXPAVADVSequenceWidget@2@@Z$0 1000e9e0 f   ChromaViewPlugin.obj
 0001:0000d9eb       __unwindfunclet$?sl_sequenceWidgetAdded@ChromaViewContext@U2@@IAEXPAVADVSequenceWidget@2@@Z$1 1000e9eb f   ChromaViewPlugin.obj
 0001:0000d9f4       __unwindfunclet$?sl_sequenceWidgetAdded@ChromaViewContext@U2@@IAEXPAVADVSequenceWidget@2@@Z$2 1000e9f4 f   ChromaViewPlugin.obj
 0001:0000d9fd       __ehhandler$?sl_sequenceWidgetAdded@ChromaViewContext@U2@@IAEXPAVADVSequenceWidget@2@@Z 1000e9fd f   ChromaViewPlugin.obj
 0001:0000da20       __unwindfunclet$?sl_showChromatogram@ChromaViewContext@U2@@IAEXXZ$1 1000ea20 f   ChromaViewPlugin.obj
 0001:0000da2b       __ehhandler$?sl_showChromatogram@ChromaViewContext@U2@@IAEXXZ 1000ea2b f   ChromaViewPlugin.obj
 0001:0000da50       __ehhandler$??0?$QList@H@@QAE@ABV0@@Z 1000ea50 f   ChromatogramView.obj
 0001:0000da70       __ehhandler$??0?$QList@PAVGObject@U2@@@@QAE@ABV0@@Z 1000ea70 f   ChromatogramView.obj
 0001:0000da90       __ehhandler$??0?$QList@PAVQAction@@@@QAE@ABV0@@Z 1000ea90 f   ChromatogramView.obj
 0001:0000dab0       __unwindfunclet$??0ChromatogramView@U2@@QAE@PAVQWidget@@PAVADVSequenceObjectContext@1@PAVGSequenceLineView@1@ABVDNAChromatogram@1@@Z$0 1000eab0 f   ChromatogramView.obj
 0001:0000dab9       __unwindfunclet$??0ChromatogramView@U2@@QAE@PAVQWidget@@PAVADVSequenceObjectContext@1@PAVGSequenceLineView@1@ABVDNAChromatogram@1@@Z$1 1000eab9 f   ChromatogramView.obj
 0001:0000dac8       __unwindfunclet$??0ChromatogramView@U2@@QAE@PAVQWidget@@PAVADVSequenceObjectContext@1@PAVGSequenceLineView@1@ABVDNAChromatogram@1@@Z$2 1000eac8 f   ChromatogramView.obj
 0001:0000dad6       __unwindfunclet$??0ChromatogramView@U2@@QAE@PAVQWidget@@PAVADVSequenceObjectContext@1@PAVGSequenceLineView@1@ABVDNAChromatogram@1@@Z$3 1000ead6 f   ChromatogramView.obj
 0001:0000dae4       __unwindfunclet$??0ChromatogramView@U2@@QAE@PAVQWidget@@PAVADVSequenceObjectContext@1@PAVGSequenceLineView@1@ABVDNAChromatogram@1@@Z$4 1000eae4 f   ChromatogramView.obj
 0001:0000daed       __unwindfunclet$??0ChromatogramView@U2@@QAE@PAVQWidget@@PAVADVSequenceObjectContext@1@PAVGSequenceLineView@1@ABVDNAChromatogram@1@@Z$5 1000eaed f   ChromatogramView.obj
 0001:0000daf8       __unwindfunclet$??0ChromatogramView@U2@@QAE@PAVQWidget@@PAVADVSequenceObjectContext@1@PAVGSequenceLineView@1@ABVDNAChromatogram@1@@Z$6 1000eaf8 f   ChromatogramView.obj
 0001:0000db12       __unwindfunclet$??0ChromatogramView@U2@@QAE@PAVQWidget@@PAVADVSequenceObjectContext@1@PAVGSequenceLineView@1@ABVDNAChromatogram@1@@Z$7 1000eb12 f   ChromatogramView.obj
 0001:0000db1b       __unwindfunclet$??0ChromatogramView@U2@@QAE@PAVQWidget@@PAVADVSequenceObjectContext@1@PAVGSequenceLineView@1@ABVDNAChromatogram@1@@Z$8 1000eb1b f   ChromatogramView.obj
 0001:0000db24       __unwindfunclet$??0ChromatogramView@U2@@QAE@PAVQWidget@@PAVADVSequenceObjectContext@1@PAVGSequenceLineView@1@ABVDNAChromatogram@1@@Z$10 1000eb24 f   ChromatogramView.obj
 0001:0000db2f       __unwindfunclet$??0ChromatogramView@U2@@QAE@PAVQWidget@@PAVADVSequenceObjectContext@1@PAVGSequenceLineView@1@ABVDNAChromatogram@1@@Z$11 1000eb2f f   ChromatogramView.obj
 0001:0000db49       __unwindfunclet$??0ChromatogramView@U2@@QAE@PAVQWidget@@PAVADVSequenceObjectContext@1@PAVGSequenceLineView@1@ABVDNAChromatogram@1@@Z$13 1000eb49 f   ChromatogramView.obj
 0001:0000db54       __unwindfunclet$??0ChromatogramView@U2@@QAE@PAVQWidget@@PAVADVSequenceObjectContext@1@PAVGSequenceLineView@1@ABVDNAChromatogram@1@@Z$14 1000eb54 f   ChromatogramView.obj
 0001:0000db6e       __unwindfunclet$??0ChromatogramView@U2@@QAE@PAVQWidget@@PAVADVSequenceObjectContext@1@PAVGSequenceLineView@1@ABVDNAChromatogram@1@@Z$15 1000eb6e f   ChromatogramView.obj
 0001:0000db77       __unwindfunclet$??0ChromatogramView@U2@@QAE@PAVQWidget@@PAVADVSequenceObjectContext@1@PAVGSequenceLineView@1@ABVDNAChromatogram@1@@Z$16 1000eb77 f   ChromatogramView.obj
 0001:0000db80       __unwindfunclet$??0ChromatogramView@U2@@QAE@PAVQWidget@@PAVADVSequenceObjectContext@1@PAVGSequenceLineView@1@ABVDNAChromatogram@1@@Z$17 1000eb80 f   ChromatogramView.obj
 0001:0000db89       __unwindfunclet$??0ChromatogramView@U2@@QAE@PAVQWidget@@PAVADVSequenceObjectContext@1@PAVGSequenceLineView@1@ABVDNAChromatogram@1@@Z$18 1000eb89 f   ChromatogramView.obj
 0001:0000db92       __unwindfunclet$??0ChromatogramView@U2@@QAE@PAVQWidget@@PAVADVSequenceObjectContext@1@PAVGSequenceLineView@1@ABVDNAChromatogram@1@@Z$19 1000eb92 f   ChromatogramView.obj
 0001:0000db9d       __unwindfunclet$??0ChromatogramView@U2@@QAE@PAVQWidget@@PAVADVSequenceObjectContext@1@PAVGSequenceLineView@1@ABVDNAChromatogram@1@@Z$20 1000eb9d f   ChromatogramView.obj
 0001:0000dba8       __unwindfunclet$??0ChromatogramView@U2@@QAE@PAVQWidget@@PAVADVSequenceObjectContext@1@PAVGSequenceLineView@1@ABVDNAChromatogram@1@@Z$22 1000eba8 f   ChromatogramView.obj
 0001:0000dbb3       __unwindfunclet$??0ChromatogramView@U2@@QAE@PAVQWidget@@PAVADVSequenceObjectContext@1@PAVGSequenceLineView@1@ABVDNAChromatogram@1@@Z$23 1000ebb3 f   ChromatogramView.obj
 0001:0000dbbc       __unwindfunclet$??0ChromatogramView@U2@@QAE@PAVQWidget@@PAVADVSequenceObjectContext@1@PAVGSequenceLineView@1@ABVDNAChromatogram@1@@Z$24 1000ebbc f   ChromatogramView.obj
 0001:0000dbc5       __unwindfunclet$??0ChromatogramView@U2@@QAE@PAVQWidget@@PAVADVSequenceObjectContext@1@PAVGSequenceLineView@1@ABVDNAChromatogram@1@@Z$25 1000ebc5 f   ChromatogramView.obj
 0001:0000dbce       __unwindfunclet$??0ChromatogramView@U2@@QAE@PAVQWidget@@PAVADVSequenceObjectContext@1@PAVGSequenceLineView@1@ABVDNAChromatogram@1@@Z$26 1000ebce f   ChromatogramView.obj
 0001:0000dbd7       __unwindfunclet$??0ChromatogramView@U2@@QAE@PAVQWidget@@PAVADVSequenceObjectContext@1@PAVGSequenceLineView@1@ABVDNAChromatogram@1@@Z$27 1000ebd7 f   ChromatogramView.obj
 0001:0000dbe0       __unwindfunclet$??0ChromatogramView@U2@@QAE@PAVQWidget@@PAVADVSequenceObjectContext@1@PAVGSequenceLineView@1@ABVDNAChromatogram@1@@Z$28 1000ebe0 f   ChromatogramView.obj
 0001:0000dbe9       __unwindfunclet$??0ChromatogramView@U2@@QAE@PAVQWidget@@PAVADVSequenceObjectContext@1@PAVGSequenceLineView@1@ABVDNAChromatogram@1@@Z$30 1000ebe9 f   ChromatogramView.obj
 0001:0000dbf4       __unwindfunclet$??0ChromatogramView@U2@@QAE@PAVQWidget@@PAVADVSequenceObjectContext@1@PAVGSequenceLineView@1@ABVDNAChromatogram@1@@Z$31 1000ebf4 f   ChromatogramView.obj
 0001:0000dc0e       __unwindfunclet$??0ChromatogramView@U2@@QAE@PAVQWidget@@PAVADVSequenceObjectContext@1@PAVGSequenceLineView@1@ABVDNAChromatogram@1@@Z$33 1000ec0e f   ChromatogramView.obj
 0001:0000dc19       __unwindfunclet$??0ChromatogramView@U2@@QAE@PAVQWidget@@PAVADVSequenceObjectContext@1@PAVGSequenceLineView@1@ABVDNAChromatogram@1@@Z$34 1000ec19 f   ChromatogramView.obj
 0001:0000dc33       __unwindfunclet$??0ChromatogramView@U2@@QAE@PAVQWidget@@PAVADVSequenceObjectContext@1@PAVGSequenceLineView@1@ABVDNAChromatogram@1@@Z$36 1000ec33 f   ChromatogramView.obj
 0001:0000dc3e       __unwindfunclet$??0ChromatogramView@U2@@QAE@PAVQWidget@@PAVADVSequenceObjectContext@1@PAVGSequenceLineView@1@ABVDNAChromatogram@1@@Z$37 1000ec3e f   ChromatogramView.obj
 0001:0000dc58       __unwindfunclet$??0ChromatogramView@U2@@QAE@PAVQWidget@@PAVADVSequenceObjectContext@1@PAVGSequenceLineView@1@ABVDNAChromatogram@1@@Z$39 1000ec58 f   ChromatogramView.obj
 0001:0000dc63       __unwindfunclet$??0ChromatogramView@U2@@QAE@PAVQWidget@@PAVADVSequenceObjectContext@1@PAVGSequenceLineView@1@ABVDNAChromatogram@1@@Z$40 1000ec63 f   ChromatogramView.obj
 0001:0000dc7d       __unwindfunclet$??0ChromatogramView@U2@@QAE@PAVQWidget@@PAVADVSequenceObjectContext@1@PAVGSequenceLineView@1@ABVDNAChromatogram@1@@Z$43 1000ec7d f   ChromatogramView.obj
 0001:0000dc86       __unwindfunclet$??0ChromatogramView@U2@@QAE@PAVQWidget@@PAVADVSequenceObjectContext@1@PAVGSequenceLineView@1@ABVDNAChromatogram@1@@Z$44 1000ec86 f   ChromatogramView.obj
 0001:0000dc8f       __ehhandler$??0ChromatogramView@U2@@QAE@PAVQWidget@@PAVADVSequenceObjectContext@1@PAVGSequenceLineView@1@ABVDNAChromatogram@1@@Z 1000ec8f f   ChromatogramView.obj
 0001:0000dcb0       __unwindfunclet$??0ChromatogramViewRenderArea@U2@@QAE@PAVChromatogramView@1@ABVDNAChromatogram@1@@Z$0 1000ecb0 f   ChromatogramView.obj
 0001:0000dcb9       __unwindfunclet$??0ChromatogramViewRenderArea@U2@@QAE@PAVChromatogramView@1@ABVDNAChromatogram@1@@Z$1 1000ecb9 f   ChromatogramView.obj
 0001:0000dcc8       __unwindfunclet$??0ChromatogramViewRenderArea@U2@@QAE@PAVChromatogramView@1@ABVDNAChromatogram@1@@Z$2 1000ecc8 f   ChromatogramView.obj
 0001:0000dcd1       __unwindfunclet$??0ChromatogramViewRenderArea@U2@@QAE@PAVChromatogramView@1@ABVDNAChromatogram@1@@Z$3 1000ecd1 f   ChromatogramView.obj
 0001:0000dce0       __unwindfunclet$??0ChromatogramViewRenderArea@U2@@QAE@PAVChromatogramView@1@ABVDNAChromatogram@1@@Z$4 1000ece0 f   ChromatogramView.obj
 0001:0000dcef       __unwindfunclet$??0ChromatogramViewRenderArea@U2@@QAE@PAVChromatogramView@1@ABVDNAChromatogram@1@@Z$5 1000ecef f   ChromatogramView.obj
 0001:0000dcfe       __unwindfunclet$??0ChromatogramViewRenderArea@U2@@QAE@PAVChromatogramView@1@ABVDNAChromatogram@1@@Z$6 1000ecfe f   ChromatogramView.obj
 0001:0000dd07       __unwindfunclet$??0ChromatogramViewRenderArea@U2@@QAE@PAVChromatogramView@1@ABVDNAChromatogram@1@@Z$7 1000ed07 f   ChromatogramView.obj
 0001:0000dd10       __ehhandler$??0ChromatogramViewRenderArea@U2@@QAE@PAVChromatogramView@1@ABVDNAChromatogram@1@@Z 1000ed10 f   ChromatogramView.obj
 0001:0000dd30       __unwindfunclet$??0DocumentFormatConstraints@U2@@QAE@XZ$0 1000ed30 f   ChromatogramView.obj
 0001:0000dd3b       __ehhandler$??0DocumentFormatConstraints@U2@@QAE@XZ 1000ed3b f   ChromatogramView.obj
 0001:0000dd60       __unwindfunclet$??1ChromatogramView@U2@@UAE@XZ$0 1000ed60 f   ChromatogramView.obj
 0001:0000dd69       __unwindfunclet$??1ChromatogramView@U2@@UAE@XZ$1 1000ed69 f   ChromatogramView.obj
 0001:0000dd78       __unwindfunclet$??1ChromatogramView@U2@@UAE@XZ$2 1000ed78 f   ChromatogramView.obj
 0001:0000dd86       __ehhandler$??1ChromatogramView@U2@@UAE@XZ 1000ed86 f   ChromatogramView.obj
 0001:0000ddb0       __unwindfunclet$??1ChromatogramViewRenderArea@U2@@UAE@XZ$0 1000edb0 f   ChromatogramView.obj
 0001:0000ddb9       __unwindfunclet$??1ChromatogramViewRenderArea@U2@@UAE@XZ$1 1000edb9 f   ChromatogramView.obj
 0001:0000ddc8       __unwindfunclet$??1ChromatogramViewRenderArea@U2@@UAE@XZ$2 1000edc8 f   ChromatogramView.obj
 0001:0000ddd7       __unwindfunclet$??1ChromatogramViewRenderArea@U2@@UAE@XZ$3 1000edd7 f   ChromatogramView.obj
 0001:0000dde6       __ehhandler$??1ChromatogramViewRenderArea@U2@@UAE@XZ 1000ede6 f   ChromatogramView.obj
 0001:0000de10       __unwindfunclet$??1DocumentFormatConstraints@U2@@QAE@XZ$0 1000ee10 f   ChromatogramView.obj
 0001:0000de1b       __unwindfunclet$??1DocumentFormatConstraints@U2@@QAE@XZ$1 1000ee1b f   ChromatogramView.obj
 0001:0000de27       __ehhandler$??1DocumentFormatConstraints@U2@@QAE@XZ 1000ee27 f   ChromatogramView.obj
 0001:0000de50       __unwindfunclet$??H@YA?BVQString@@ABV0@0@Z$0 1000ee50 f   ChromatogramView.obj
 0001:0000de6a       __ehhandler$??H@YA?BVQString@@ABV0@0@Z 1000ee6a f   ChromatogramView.obj
 0001:0000de90       __unwindfunclet$??H@YA?BVQString@@ABV0@PBD@Z$0 1000ee90 f   ChromatogramView.obj
 0001:0000deaa       __unwindfunclet$??H@YA?BVQString@@ABV0@PBD@Z$1 1000eeaa f   ChromatogramView.obj
 0001:0000deb3       __ehhandler$??H@YA?BVQString@@ABV0@PBD@Z 1000eeb3 f   ChromatogramView.obj
 0001:0000ded0       __unwindfunclet$??H@YA?BVQString@@PBDABV0@@Z$0 1000eed0 f   ChromatogramView.obj
 0001:0000deea       __ehhandler$??H@YA?BVQString@@PBDABV0@@Z 1000eeea f   ChromatogramView.obj
 0001:0000df10       __unwindfunclet$??__EalgoLog@U2@@YAXXZ$0 1000ef10 f   ChromatogramView.obj
 0001:0000df19       __ehhandler$??__EalgoLog@U2@@YAXXZ 1000ef19 f   ChromatogramView.obj
 0001:0000df40       __unwindfunclet$??__EcmdLog@U2@@YAXXZ$0 1000ef40 f   ChromatogramView.obj
 0001:0000df49       __ehhandler$??__EcmdLog@U2@@YAXXZ 1000ef49 f   ChromatogramView.obj
 0001:0000df70       __unwindfunclet$??__EcoreLog@U2@@YAXXZ$0 1000ef70 f   ChromatogramView.obj
 0001:0000df79       __ehhandler$??__EcoreLog@U2@@YAXXZ 1000ef79 f   ChromatogramView.obj
 0001:0000dfa0       __unwindfunclet$??__EioLog@U2@@YAXXZ$0 1000efa0 f   ChromatogramView.obj
 0001:0000dfa9       __ehhandler$??__EioLog@U2@@YAXXZ 1000efa9 f   ChromatogramView.obj
 0001:0000dfd0       __unwindfunclet$??__EperfLog@U2@@YAXXZ$0 1000efd0 f   ChromatogramView.obj
 0001:0000dfd9       __ehhandler$??__EperfLog@U2@@YAXXZ 1000efd9 f   ChromatogramView.obj
 0001:0000e000       __unwindfunclet$??__EscriptLog@U2@@YAXXZ$0 1000f000 f   ChromatogramView.obj
 0001:0000e009       __ehhandler$??__EscriptLog@U2@@YAXXZ 1000f009 f   ChromatogramView.obj
 0001:0000e030       __unwindfunclet$??__EtaskLog@U2@@YAXXZ$0 1000f030 f   ChromatogramView.obj
 0001:0000e039       __ehhandler$??__EtaskLog@U2@@YAXXZ 1000f039 f   ChromatogramView.obj
 0001:0000e060       __unwindfunclet$??__EuiLog@U2@@YAXXZ$0 1000f060 f   ChromatogramView.obj
 0001:0000e069       __ehhandler$??__EuiLog@U2@@YAXXZ 1000f069 f   ChromatogramView.obj
 0001:0000e090       __unwindfunclet$??__EuserActLog@U2@@YAXXZ$0 1000f090 f   ChromatogramView.obj
 0001:0000e099       __ehhandler$??__EuserActLog@U2@@YAXXZ 1000f099 f   ChromatogramView.obj
 0001:0000e0c0       __ehhandler$?append@?$QList@H@@QAEXABH@Z 1000f0c0 f   ChromatogramView.obj
 0001:0000e0e0       __ehhandler$?append@?$QList@V?$QPointer@VGObject@U2@@@@@@QAEXABV?$QPointer@VGObject@U2@@@@@Z 1000f0e0 f   ChromatogramView.obj
 0001:0000e100       __unwindfunclet$?buildPopupMenu@ChromatogramView@U2@@UAEXAAVQMenu@@@Z$0 1000f100 f   ChromatogramView.obj
 0001:0000e109       __unwindfunclet$?buildPopupMenu@ChromatogramView@U2@@UAEXAAVQMenu@@@Z$1 1000f109 f   ChromatogramView.obj
 0001:0000e111       __ehhandler$?buildPopupMenu@ChromatogramView@U2@@UAEXAAVQMenu@@@Z 1000f111 f   ChromatogramView.obj
 0001:0000e130       __unwindfunclet$?createNode@?$QHash@VQString@@UQHashDummyValue@@@@AAEPAU?$QHashNode@VQString@@UQHashDummyValue@@@@IABVQString@@ABUQHashDummyValue@@PAPAU2@@Z$0 1000f130 f   ChromatogramView.obj
 0001:0000e141       __ehhandler$?createNode@?$QHash@VQString@@UQHashDummyValue@@@@AAEPAU?$QHashNode@VQString@@UQHashDummyValue@@@@IABVQString@@ABUQHashDummyValue@@PAPAU2@@Z 1000f141 f   ChromatogramView.obj
 0001:0000e160       __unwindfunclet$?createToggleTraceAction@ChromatogramView@U2@@AAEPAVQAction@@ABVQString@@@Z$0 1000f160 f   ChromatogramView.obj
 0001:0000e16b       __ehhandler$?createToggleTraceAction@ChromatogramView@U2@@AAEPAVQAction@@ABVQString@@@Z 1000f16b f   ChromatogramView.obj
 0001:0000e190       __ehhandler$?detach_helper@?$QList@H@@AAEXH@Z 1000f190 f   ChromatogramView.obj
 0001:0000e1b0       __ehhandler$?detach_helper_grow@?$QList@H@@AAEPAUNode@1@HH@Z 1000f1b0 f   ChromatogramView.obj
 0001:0000e1d0       __ehhandler$?detach_helper_grow@?$QList@V?$QPointer@VGObject@U2@@@@@@AAEPAUNode@1@HH@Z 1000f1d0 f   ChromatogramView.obj
 0001:0000e1f0       __unwindfunclet$?drawAll@ChromatogramViewRenderArea@U2@@MAEXPAVQPaintDevice@@@Z$0 1000f1f0 f   ChromatogramView.obj
 0001:0000e1fe       __unwindfunclet$?drawAll@ChromatogramViewRenderArea@U2@@MAEXPAVQPaintDevice@@@Z$1 1000f1fe f   ChromatogramView.obj
 0001:0000e20c       __unwindfunclet$?drawAll@ChromatogramViewRenderArea@U2@@MAEXPAVQPaintDevice@@@Z$2 1000f20c f   ChromatogramView.obj
 0001:0000e217       __unwindfunclet$?drawAll@ChromatogramViewRenderArea@U2@@MAEXPAVQPaintDevice@@@Z$3 1000f217 f   ChromatogramView.obj
 0001:0000e222       __unwindfunclet$?drawAll@ChromatogramViewRenderArea@U2@@MAEXPAVQPaintDevice@@@Z$4 1000f222 f   ChromatogramView.obj
 0001:0000e22d       __unwindfunclet$?drawAll@ChromatogramViewRenderArea@U2@@MAEXPAVQPaintDevice@@@Z$6 1000f22d f   ChromatogramView.obj
 0001:0000e239       __unwindfunclet$?drawAll@ChromatogramViewRenderArea@U2@@MAEXPAVQPaintDevice@@@Z$7 1000f239 f   ChromatogramView.obj
 0001:0000e242       __unwindfunclet$?drawAll@ChromatogramViewRenderArea@U2@@MAEXPAVQPaintDevice@@@Z$8 1000f242 f   ChromatogramView.obj
 0001:0000e24b       __unwindfunclet$?drawAll@ChromatogramViewRenderArea@U2@@MAEXPAVQPaintDevice@@@Z$9 1000f24b f   ChromatogramView.obj
 0001:0000e254       __unwindfunclet$?drawAll@ChromatogramViewRenderArea@U2@@MAEXPAVQPaintDevice@@@Z$10 1000f254 f   ChromatogramView.obj
 0001:0000e25d       __unwindfunclet$?drawAll@ChromatogramViewRenderArea@U2@@MAEXPAVQPaintDevice@@@Z$11 1000f25d f   ChromatogramView.obj
 0001:0000e266       __unwindfunclet$?drawAll@ChromatogramViewRenderArea@U2@@MAEXPAVQPaintDevice@@@Z$12 1000f266 f   ChromatogramView.obj
 0001:0000e26f       __unwindfunclet$?drawAll@ChromatogramViewRenderArea@U2@@MAEXPAVQPaintDevice@@@Z$13 1000f26f f   ChromatogramView.obj
 0001:0000e278       __unwindfunclet$?drawAll@ChromatogramViewRenderArea@U2@@MAEXPAVQPaintDevice@@@Z$14 1000f278 f   ChromatogramView.obj
 0001:0000e281       __unwindfunclet$?drawAll@ChromatogramViewRenderArea@U2@@MAEXPAVQPaintDevice@@@Z$15 1000f281 f   ChromatogramView.obj
 0001:0000e28a       __unwindfunclet$?drawAll@ChromatogramViewRenderArea@U2@@MAEXPAVQPaintDevice@@@Z$16 1000f28a f   ChromatogramView.obj
 0001:0000e293       __unwindfunclet$?drawAll@ChromatogramViewRenderArea@U2@@MAEXPAVQPaintDevice@@@Z$17 1000f293 f   ChromatogramView.obj
 0001:0000e29c       __unwindfunclet$?drawAll@ChromatogramViewRenderArea@U2@@MAEXPAVQPaintDevice@@@Z$18 1000f29c f   ChromatogramView.obj
 0001:0000e2a5       __ehhandler$?drawAll@ChromatogramViewRenderArea@U2@@MAEXPAVQPaintDevice@@@Z 1000f2a5 f   ChromatogramView.obj
 0001:0000e2d0       __unwindfunclet$?drawChromatogramBaseCallsLines@ChromatogramViewRenderArea@U2@@AAEXNNNNAAVQPainter@@ABVU2Region@2@ABVQByteArray@@ABUChromatogramViewSettings@2@@Z$0 1000f2d0 f   ChromatogramView.obj
 0001:0000e2de       __ehhandler$?drawChromatogramBaseCallsLines@ChromatogramViewRenderArea@U2@@AAEXNNNNAAVQPainter@@ABVU2Region@2@ABVQByteArray@@ABUChromatogramViewSettings@2@@Z 1000f2de f   ChromatogramView.obj
 0001:0000e300       __unwindfunclet$?drawChromatogramTrace@ChromatogramViewRenderArea@U2@@AAEXNNNNAAVQPainter@@ABVU2Region@2@ABUChromatogramViewSettings@2@@Z$0 1000f300 f   ChromatogramView.obj
 0001:0000e30e       __unwindfunclet$?drawChromatogramTrace@ChromatogramViewRenderArea@U2@@AAEXNNNNAAVQPainter@@ABVU2Region@2@ABUChromatogramViewSettings@2@@Z$1 1000f30e f   ChromatogramView.obj
 0001:0000e317       __unwindfunclet$?drawChromatogramTrace@ChromatogramViewRenderArea@U2@@AAEXNNNNAAVQPainter@@ABVU2Region@2@ABUChromatogramViewSettings@2@@Z$2 1000f317 f   ChromatogramView.obj
 0001:0000e320       __unwindfunclet$?drawChromatogramTrace@ChromatogramViewRenderArea@U2@@AAEXNNNNAAVQPainter@@ABVU2Region@2@ABUChromatogramViewSettings@2@@Z$3 1000f320 f   ChromatogramView.obj
 0001:0000e329       __unwindfunclet$?drawChromatogramTrace@ChromatogramViewRenderArea@U2@@AAEXNNNNAAVQPainter@@ABVU2Region@2@ABUChromatogramViewSettings@2@@Z$4 1000f329 f   ChromatogramView.obj
 0001:0000e332       __ehhandler$?drawChromatogramTrace@ChromatogramViewRenderArea@U2@@AAEXNNNNAAVQPainter@@ABVU2Region@2@ABUChromatogramViewSettings@2@@Z 1000f332 f   ChromatogramView.obj
 0001:0000e350       __unwindfunclet$?drawOriginalBaseCalls@ChromatogramViewRenderArea@U2@@AAEXNNNNAAVQPainter@@ABVU2Region@2@ABVQByteArray@@_N@Z$0 1000f350 f   ChromatogramView.obj
 0001:0000e359       __unwindfunclet$?drawOriginalBaseCalls@ChromatogramViewRenderArea@U2@@AAEXNNNNAAVQPainter@@ABVU2Region@2@ABVQByteArray@@_N@Z$1 1000f359 f   ChromatogramView.obj
 0001:0000e362       __unwindfunclet$?drawOriginalBaseCalls@ChromatogramViewRenderArea@U2@@AAEXNNNNAAVQPainter@@ABVU2Region@2@ABVQByteArray@@_N@Z$2 1000f362 f   ChromatogramView.obj
 0001:0000e36b       __unwindfunclet$?drawOriginalBaseCalls@ChromatogramViewRenderArea@U2@@AAEXNNNNAAVQPainter@@ABVU2Region@2@ABVQByteArray@@_N@Z$3 1000f36b f   ChromatogramView.obj
 0001:0000e374       __ehhandler$?drawOriginalBaseCalls@ChromatogramViewRenderArea@U2@@AAEXNNNNAAVQPainter@@ABVU2Region@2@ABVQByteArray@@_N@Z 1000f374 f   ChromatogramView.obj
 0001:0000e3a0       __unwindfunclet$?drawQualityValues@ChromatogramViewRenderArea@U2@@AAEXNNNNAAVQPainter@@ABVU2Region@2@ABVQByteArray@@@Z$0 1000f3a0 f   ChromatogramView.obj
 0001:0000e3a9       __unwindfunclet$?drawQualityValues@ChromatogramViewRenderArea@U2@@AAEXNNNNAAVQPainter@@ABVU2Region@2@ABVQByteArray@@@Z$1 1000f3a9 f   ChromatogramView.obj
 0001:0000e3b5       __ehhandler$?drawQualityValues@ChromatogramViewRenderArea@U2@@AAEXNNNNAAVQPainter@@ABVU2Region@2@ABVQByteArray@@@Z 1000f3b5 f   ChromatogramView.obj
 0001:0000e3e0       __unwindfunclet$?duplicateNode@?$QHash@VQString@@UQHashDummyValue@@@@CAXPAUNode@QHashData@@PAX@Z$0 1000f3e0 f   ChromatogramView.obj
 0001:0000e3f1       __ehhandler$?duplicateNode@?$QHash@VQString@@UQHashDummyValue@@@@CAXPAUNode@QHashData@@PAX@Z 1000f3f1 f   ChromatogramView.obj
 0001:0000e410       __unwindfunclet$?insert@?$QHash@VQString@@UQHashDummyValue@@@@QAE?AViterator@1@ABVQString@@ABUQHashDummyValue@@@Z$0 1000f410 f   ChromatogramView.obj
 0001:0000e421       __ehhandler$?insert@?$QHash@VQString@@UQHashDummyValue@@@@QAE?AViterator@1@ABVQString@@ABUQHashDummyValue@@@Z 1000f421 f   ChromatogramView.obj
 0001:0000e440       __ehhandler$?node_copy@?$QList@V?$QPointer@VGObject@U2@@@@@@AAEXPAUNode@1@00@Z 1000f440 f   ChromatogramView.obj
 0001:0000e460       __unwindfunclet$?pack@ChromatogramView@U2@@MAEXXZ$0 1000f460 f   ChromatogramView.obj
 0001:0000e46b       __ehhandler$?pack@ChromatogramView@U2@@MAEXXZ 1000f46b f   ChromatogramView.obj
 0001:0000e490       __ehhandler$?reallocData@?$QVector@D@@AAEXHHV?$QFlags@W4AllocationOption@QArrayData@@@@@Z 1000f490 f   ChromatogramView.obj
 0001:0000e4b0       __ehhandler$?reallocData@?$QVector@G@@AAEXHHV?$QFlags@W4AllocationOption@QArrayData@@@@@Z 1000f4b0 f   ChromatogramView.obj
 0001:0000e4d0       __unwindfunclet$?sl_addNewSequenceObject@ChromatogramView@U2@@AAEXXZ$0 1000f4d0 f   ChromatogramView.obj
 0001:0000e4d9       __unwindfunclet$?sl_addNewSequenceObject@ChromatogramView@U2@@AAEXXZ$2 1000f4d9 f   ChromatogramView.obj
 0001:0000e4e2       __unwindfunclet$?sl_addNewSequenceObject@ChromatogramView@U2@@AAEXXZ$27 1000f4e2 f   ChromatogramView.obj
 0001:0000e4ea       __unwindfunclet$?sl_addNewSequenceObject@ChromatogramView@U2@@AAEXXZ$3 1000f4ea f   ChromatogramView.obj
 0001:0000e4f2       __unwindfunclet$?sl_addNewSequenceObject@ChromatogramView@U2@@AAEXXZ$4 1000f4f2 f   ChromatogramView.obj
 0001:0000e4fb       __unwindfunclet$?sl_addNewSequenceObject@ChromatogramView@U2@@AAEXXZ$5 1000f4fb f   ChromatogramView.obj
 0001:0000e503       __unwindfunclet$?sl_addNewSequenceObject@ChromatogramView@U2@@AAEXXZ$6 1000f503 f   ChromatogramView.obj
 0001:0000e50c       __unwindfunclet$?sl_addNewSequenceObject@ChromatogramView@U2@@AAEXXZ$7 1000f50c f   ChromatogramView.obj
 0001:0000e515       __unwindfunclet$?sl_addNewSequenceObject@ChromatogramView@U2@@AAEXXZ$8 1000f515 f   ChromatogramView.obj
 0001:0000e51e       __unwindfunclet$?sl_addNewSequenceObject@ChromatogramView@U2@@AAEXXZ$9 1000f51e f   ChromatogramView.obj
 0001:0000e527       __unwindfunclet$?sl_addNewSequenceObject@ChromatogramView@U2@@AAEXXZ$10 1000f527 f   ChromatogramView.obj
 0001:0000e530       __unwindfunclet$?sl_addNewSequenceObject@ChromatogramView@U2@@AAEXXZ$11 1000f530 f   ChromatogramView.obj
 0001:0000e539       __unwindfunclet$?sl_addNewSequenceObject@ChromatogramView@U2@@AAEXXZ$13 1000f539 f   ChromatogramView.obj
 0001:0000e542       __unwindfunclet$?sl_addNewSequenceObject@ChromatogramView@U2@@AAEXXZ$14 1000f542 f   ChromatogramView.obj
 0001:0000e54b       __unwindfunclet$?sl_addNewSequenceObject@ChromatogramView@U2@@AAEXXZ$15 1000f54b f   ChromatogramView.obj
 0001:0000e554       __unwindfunclet$?sl_addNewSequenceObject@ChromatogramView@U2@@AAEXXZ$16 1000f554 f   ChromatogramView.obj
 0001:0000e55d       __unwindfunclet$?sl_addNewSequenceObject@ChromatogramView@U2@@AAEXXZ$17 1000f55d f   ChromatogramView.obj
 0001:0000e566       __unwindfunclet$?sl_addNewSequenceObject@ChromatogramView@U2@@AAEXXZ$18 1000f566 f   ChromatogramView.obj
 0001:0000e56f       __unwindfunclet$?sl_addNewSequenceObject@ChromatogramView@U2@@AAEXXZ$19 1000f56f f   ChromatogramView.obj
 0001:0000e578       __unwindfunclet$?sl_addNewSequenceObject@ChromatogramView@U2@@AAEXXZ$21 1000f578 f   ChromatogramView.obj
 0001:0000e584       __unwindfunclet$?sl_addNewSequenceObject@ChromatogramView@U2@@AAEXXZ$22 1000f584 f   ChromatogramView.obj
 0001:0000e58d       __unwindfunclet$?sl_addNewSequenceObject@ChromatogramView@U2@@AAEXXZ$23 1000f58d f   ChromatogramView.obj
 0001:0000e595       __unwindfunclet$?sl_addNewSequenceObject@ChromatogramView@U2@@AAEXXZ$24 1000f595 f   ChromatogramView.obj
 0001:0000e59d       __unwindfunclet$?sl_addNewSequenceObject@ChromatogramView@U2@@AAEXXZ$25 1000f59d f   ChromatogramView.obj
 0001:0000e5a6       __ehhandler$?sl_addNewSequenceObject@ChromatogramView@U2@@AAEXXZ 1000f5a6 f   ChromatogramView.obj
 0001:0000e5d0       __unwindfunclet$?sl_onAddExistingSequenceObject@ChromatogramView@U2@@AAEXXZ$0 1000f5d0 f   ChromatogramView.obj
 0001:0000e5dc       __unwindfunclet$?sl_onAddExistingSequenceObject@ChromatogramView@U2@@AAEXXZ$1 1000f5dc f   ChromatogramView.obj
 0001:0000e5e5       __unwindfunclet$?sl_onAddExistingSequenceObject@ChromatogramView@U2@@AAEXXZ$2 1000f5e5 f   ChromatogramView.obj
 0001:0000e5ed       __unwindfunclet$?sl_onAddExistingSequenceObject@ChromatogramView@U2@@AAEXXZ$3 1000f5ed f   ChromatogramView.obj
 0001:0000e5f5       __unwindfunclet$?sl_onAddExistingSequenceObject@ChromatogramView@U2@@AAEXXZ$4 1000f5f5 f   ChromatogramView.obj
 0001:0000e5fd       __unwindfunclet$?sl_onAddExistingSequenceObject@ChromatogramView@U2@@AAEXXZ$5 1000f5fd f   ChromatogramView.obj
 0001:0000e606       __unwindfunclet$?sl_onAddExistingSequenceObject@ChromatogramView@U2@@AAEXXZ$6 1000f606 f   ChromatogramView.obj
 0001:0000e60f       __unwindfunclet$?sl_onAddExistingSequenceObject@ChromatogramView@U2@@AAEXXZ$7 1000f60f f   ChromatogramView.obj
 0001:0000e618       __unwindfunclet$?sl_onAddExistingSequenceObject@ChromatogramView@U2@@AAEXXZ$8 1000f618 f   ChromatogramView.obj
 0001:0000e623       __unwindfunclet$?sl_onAddExistingSequenceObject@ChromatogramView@U2@@AAEXXZ$9 1000f623 f   ChromatogramView.obj
 0001:0000e640       __unwindfunclet$?sl_onAddExistingSequenceObject@ChromatogramView@U2@@AAEXXZ$10 1000f640 f   ChromatogramView.obj
 0001:0000e65d       __unwindfunclet$?sl_onAddExistingSequenceObject@ChromatogramView@U2@@AAEXXZ$11 1000f65d f   ChromatogramView.obj
 0001:0000e668       __ehhandler$?sl_onAddExistingSequenceObject@ChromatogramView@U2@@AAEXXZ 1000f668 f   ChromatogramView.obj
 0001:0000e690       __unwindfunclet$?sl_onPopupMenuCkicked@ChromatogramView@U2@@AAEXPAVQAction@@@Z$0 1000f690 f   ChromatogramView.obj
 0001:0000e699       __unwindfunclet$?sl_onPopupMenuCkicked@ChromatogramView@U2@@AAEXPAVQAction@@@Z$1 1000f699 f   ChromatogramView.obj
 0001:0000e6a2       __unwindfunclet$?sl_onPopupMenuCkicked@ChromatogramView@U2@@AAEXPAVQAction@@@Z$2 1000f6a2 f   ChromatogramView.obj
 0001:0000e6ab       __unwindfunclet$?sl_onPopupMenuCkicked@ChromatogramView@U2@@AAEXPAVQAction@@@Z$3 1000f6ab f   ChromatogramView.obj
 0001:0000e6b4       __unwindfunclet$?sl_onPopupMenuCkicked@ChromatogramView@U2@@AAEXPAVQAction@@@Z$4 1000f6b4 f   ChromatogramView.obj
 0001:0000e6bd       __unwindfunclet$?sl_onPopupMenuCkicked@ChromatogramView@U2@@AAEXPAVQAction@@@Z$5 1000f6bd f   ChromatogramView.obj
 0001:0000e6c6       __unwindfunclet$?sl_onPopupMenuCkicked@ChromatogramView@U2@@AAEXPAVQAction@@@Z$6 1000f6c6 f   ChromatogramView.obj
 0001:0000e6cf       __unwindfunclet$?sl_onPopupMenuCkicked@ChromatogramView@U2@@AAEXPAVQAction@@@Z$7 1000f6cf f   ChromatogramView.obj
 0001:0000e6d8       __unwindfunclet$?sl_onPopupMenuCkicked@ChromatogramView@U2@@AAEXPAVQAction@@@Z$8 1000f6d8 f   ChromatogramView.obj
 0001:0000e6e1       __unwindfunclet$?sl_onPopupMenuCkicked@ChromatogramView@U2@@AAEXPAVQAction@@@Z$9 1000f6e1 f   ChromatogramView.obj
 0001:0000e6ea       __unwindfunclet$?sl_onPopupMenuCkicked@ChromatogramView@U2@@AAEXPAVQAction@@@Z$10 1000f6ea f   ChromatogramView.obj
 0001:0000e6f3       __unwindfunclet$?sl_onPopupMenuCkicked@ChromatogramView@U2@@AAEXPAVQAction@@@Z$11 1000f6f3 f   ChromatogramView.obj
 0001:0000e6fc       __unwindfunclet$?sl_onPopupMenuCkicked@ChromatogramView@U2@@AAEXPAVQAction@@@Z$12 1000f6fc f   ChromatogramView.obj
 0001:0000e705       __unwindfunclet$?sl_onPopupMenuCkicked@ChromatogramView@U2@@AAEXPAVQAction@@@Z$13 1000f705 f   ChromatogramView.obj
 0001:0000e70e       __unwindfunclet$?sl_onPopupMenuCkicked@ChromatogramView@U2@@AAEXPAVQAction@@@Z$14 1000f70e f   ChromatogramView.obj
 0001:0000e717       __unwindfunclet$?sl_onPopupMenuCkicked@ChromatogramView@U2@@AAEXPAVQAction@@@Z$15 1000f717 f   ChromatogramView.obj
 0001:0000e720       __unwindfunclet$?sl_onPopupMenuCkicked@ChromatogramView@U2@@AAEXPAVQAction@@@Z$16 1000f720 f   ChromatogramView.obj
 0001:0000e729       __ehhandler$?sl_onPopupMenuCkicked@ChromatogramView@U2@@AAEXPAVQAction@@@Z 1000f729 f   ChromatogramView.obj
 0001:0000e750       __unwindfunclet$?sl_onSequenceObjectLoaded@ChromatogramView@U2@@AAEXPAVTask@2@@Z$0 1000f750 f   ChromatogramView.obj
 0001:0000e759       __ehhandler$?sl_onSequenceObjectLoaded@ChromatogramView@U2@@AAEXPAVTask@2@@Z 1000f759 f   ChromatogramView.obj
 0001:0000e780       __unwindfunclet$?sl_removeChanges@ChromatogramView@U2@@AAEXXZ$0 1000f780 f   ChromatogramView.obj
 0001:0000e789       __unwindfunclet$?sl_removeChanges@ChromatogramView@U2@@AAEXXZ$1 1000f789 f   ChromatogramView.obj
 0001:0000e792       __unwindfunclet$?sl_removeChanges@ChromatogramView@U2@@AAEXXZ$2 1000f792 f   ChromatogramView.obj
 0001:0000e79b       __unwindfunclet$?sl_removeChanges@ChromatogramView@U2@@AAEXXZ$3 1000f79b f   ChromatogramView.obj
 0001:0000e7a4       __unwindfunclet$?sl_removeChanges@ChromatogramView@U2@@AAEXXZ$4 1000f7a4 f   ChromatogramView.obj
 0001:0000e7ad       __ehhandler$?sl_removeChanges@ChromatogramView@U2@@AAEXXZ 1000f7ad f   ChromatogramView.obj
 0001:0000e7d0       __unwindfunclet$?sl_showAllTraces@ChromatogramView@U2@@AAEXXZ$0 1000f7d0 f   ChromatogramView.obj
 0001:0000e7d8       __unwindfunclet$?sl_showAllTraces@ChromatogramView@U2@@AAEXXZ$1 1000f7d8 f   ChromatogramView.obj
 0001:0000e7e0       __ehhandler$?sl_showAllTraces@ChromatogramView@U2@@AAEXXZ 1000f7e0 f   ChromatogramView.obj
 0001:0000e800       __unwindfunclet$?sl_showHideTrace@ChromatogramView@U2@@AAEXXZ$0 1000f800 f   ChromatogramView.obj
 0001:0000e809       __unwindfunclet$?sl_showHideTrace@ChromatogramView@U2@@AAEXXZ$1 1000f809 f   ChromatogramView.obj
 0001:0000e812       __unwindfunclet$?sl_showHideTrace@ChromatogramView@U2@@AAEXXZ$2 1000f812 f   ChromatogramView.obj
 0001:0000e81b       __unwindfunclet$?sl_showHideTrace@ChromatogramView@U2@@AAEXXZ$3 1000f81b f   ChromatogramView.obj
 0001:0000e824       __ehhandler$?sl_showHideTrace@ChromatogramView@U2@@AAEXXZ 1000f824 f   ChromatogramView.obj
 0001:0000e840       __unwindfunclet$?qt_metatype_id@?$QMetaTypeIdQObject@PAVADVSequenceWidget@U2@@$00@@SAHXZ$0 1000f840 f   moc_ChromaViewPlugin.obj
 0001:0000e849       __ehhandler$?qt_metatype_id@?$QMetaTypeIdQObject@PAVADVSequenceWidget@U2@@$00@@SAHXZ 1000f849 f   moc_ChromaViewPlugin.obj
 0001:0000e870       __unwindfunclet$?qt_metatype_id@?$QMetaTypeIdQObject@PAVGObject@U2@@$00@@SAHXZ$0 1000f870 f   moc_ChromatogramView.obj
 0001:0000e879       __ehhandler$?qt_metatype_id@?$QMetaTypeIdQObject@PAVGObject@U2@@$00@@SAHXZ 1000f879 f   moc_ChromatogramView.obj
 0001:0000e8a0       __unwindfunclet$?qt_metatype_id@?$QMetaTypeIdQObject@PAVQAction@@$00@@SAHXZ$0 1000f8a0 f   moc_ChromatogramView.obj
 0001:0000e8a9       __ehhandler$?qt_metatype_id@?$QMetaTypeIdQObject@PAVQAction@@$00@@SAHXZ 1000f8a9 f   moc_ChromatogramView.obj
 0001:0000e8d0       ??__F?_Generic_object@?$_Error_objects@H@std@@2V_Generic_error_category@2@A@@YAXXZ 1000f8d0 f   ChromaViewPlugin.obj
 0001:0000e8e0       ??__F?_Iostream_object@?$_Error_objects@H@std@@2V_Iostream_error_category@2@A@@YAXXZ 1000f8e0 f   ChromaViewPlugin.obj
 0001:0000e8f0       ??__F?_System_object@?$_Error_objects@H@std@@2V_System_error_category@2@A@@YAXXZ 1000f8f0 f   ChromaViewPlugin.obj
 0001:0000e900       ??__FService_DNAExport@U2@@YAXXZ 1000f900 f   ChromaViewPlugin.obj
 0001:0000e910       ??__FService_DNAGraphPack@U2@@YAXXZ 1000f910 f   ChromaViewPlugin.obj
 0001:0000e920       ??__FService_ExternalToolSupport@U2@@YAXXZ 1000f920 f   ChromaViewPlugin.obj
 0001:0000e930       ??__FService_GUITesting@U2@@YAXXZ 1000f930 f   ChromaViewPlugin.obj
 0001:0000e940       ??__FService_MaxCoreServiceId@U2@@YAXXZ 1000f940 f   ChromaViewPlugin.obj
 0001:0000e950       ??__FService_MinCoreServiceId@U2@@YAXXZ 1000f950 f   ChromaViewPlugin.obj
 0001:0000e960       ??__FService_PluginViewer@U2@@YAXXZ 1000f960 f   ChromaViewPlugin.obj
 0001:0000e970       ??__FService_Project@U2@@YAXXZ 1000f970 f   ChromaViewPlugin.obj
 0001:0000e980       ??__FService_ProjectView@U2@@YAXXZ 1000f980 f   ChromaViewPlugin.obj
 0001:0000e990       ??__FService_QueryDesigner@U2@@YAXXZ 1000f990 f   ChromaViewPlugin.obj
 0001:0000e9a0       ??__FService_ScriptRegistry@U2@@YAXXZ 1000f9a0 f   ChromaViewPlugin.obj
 0001:0000e9b0       ??__FService_TestRunner@U2@@YAXXZ 1000f9b0 f   ChromaViewPlugin.obj
 0001:0000e9c0       ??__FService_WorkflowDesigner@U2@@YAXXZ 1000f9c0 f   ChromaViewPlugin.obj
 0001:0000e9d0       ??__FalgoLog@U2@@YAXXZ     1000f9d0 f   ChromaViewPlugin.obj
 0001:0000e9e0       ??__FcmdLog@U2@@YAXXZ      1000f9e0 f   ChromaViewPlugin.obj
 0001:0000e9f0       ??__FcoreLog@U2@@YAXXZ     1000f9f0 f   ChromaViewPlugin.obj
 0001:0000ea00       ??__FioLog@U2@@YAXXZ       1000fa00 f   ChromaViewPlugin.obj
 0001:0000ea10       ??__FperfLog@U2@@YAXXZ     1000fa10 f   ChromaViewPlugin.obj
 0001:0000ea20       ??__FscriptLog@U2@@YAXXZ   1000fa20 f   ChromaViewPlugin.obj
 0001:0000ea30       ??__FtaskLog@U2@@YAXXZ     1000fa30 f   ChromaViewPlugin.obj
 0001:0000ea40       ??__FuiLog@U2@@YAXXZ       1000fa40 f   ChromaViewPlugin.obj
 0001:0000ea50       ??__FuserActLog@U2@@YAXXZ  1000fa50 f   ChromaViewPlugin.obj
 0001:0000ea60       ??__F?_Generic_object@?$_Error_objects@H@std@@2V_Generic_error_category@2@A@@YAXXZ 1000fa60 f   ChromatogramView.obj
 0001:0000ea70       ??__F?_Iostream_object@?$_Error_objects@H@std@@2V_Iostream_error_category@2@A@@YAXXZ 1000fa70 f   ChromatogramView.obj
 0001:0000ea80       ??__F?_System_object@?$_Error_objects@H@std@@2V_System_error_category@2@A@@YAXXZ 1000fa80 f   ChromatogramView.obj
 0001:0000ea90       ??__FService_DNAExport@U2@@YAXXZ 1000fa90 f   ChromatogramView.obj
 0001:0000eaa0       ??__FService_DNAGraphPack@U2@@YAXXZ 1000faa0 f   ChromatogramView.obj
 0001:0000eab0       ??__FService_ExternalToolSupport@U2@@YAXXZ 1000fab0 f   ChromatogramView.obj
 0001:0000eac0       ??__FService_GUITesting@U2@@YAXXZ 1000fac0 f   ChromatogramView.obj
 0001:0000ead0       ??__FService_MaxCoreServiceId@U2@@YAXXZ 1000fad0 f   ChromatogramView.obj
 0001:0000eae0       ??__FService_MinCoreServiceId@U2@@YAXXZ 1000fae0 f   ChromatogramView.obj
 0001:0000eaf0       ??__FService_PluginViewer@U2@@YAXXZ 1000faf0 f   ChromatogramView.obj
 0001:0000eb00       ??__FService_Project@U2@@YAXXZ 1000fb00 f   ChromatogramView.obj
 0001:0000eb10       ??__FService_ProjectView@U2@@YAXXZ 1000fb10 f   ChromatogramView.obj
 0001:0000eb20       ??__FService_QueryDesigner@U2@@YAXXZ 1000fb20 f   ChromatogramView.obj
 0001:0000eb30       ??__FService_ScriptRegistry@U2@@YAXXZ 1000fb30 f   ChromatogramView.obj
 0001:0000eb40       ??__FService_TestRunner@U2@@YAXXZ 1000fb40 f   ChromatogramView.obj
 0001:0000eb50       ??__FService_WorkflowDesigner@U2@@YAXXZ 1000fb50 f   ChromatogramView.obj
 0001:0000eb60       ??__FalgoLog@U2@@YAXXZ     1000fb60 f   ChromatogramView.obj
 0001:0000eb70       ??__FbaseForIds@?1??drawAll@ChromatogramViewRenderArea@U2@@MAEXPAVQPaintDevice@@@Z@YAXXZ 1000fb70 f   ChromatogramView.obj
 0001:0000eb90       ??__FcmdLog@U2@@YAXXZ      1000fb90 f   ChromatogramView.obj
 0001:0000eba0       ??__FcoreLog@U2@@YAXXZ     1000fba0 f   ChromatogramView.obj
 0001:0000ebb0       ??__FioLog@U2@@YAXXZ       1000fbb0 f   ChromatogramView.obj
 0001:0000ebc0       ??__FperfLog@U2@@YAXXZ     1000fbc0 f   ChromatogramView.obj
 0001:0000ebd0       ??__FscriptLog@U2@@YAXXZ   1000fbd0 f   ChromatogramView.obj
 0001:0000ebe0       ??__FtaskLog@U2@@YAXXZ     1000fbe0 f   ChromatogramView.obj
 0001:0000ebf0       ??__FuiLog@U2@@YAXXZ       1000fbf0 f   ChromatogramView.obj
 0001:0000ec00       ??__FuserActLog@U2@@YAXXZ  1000fc00 f   ChromatogramView.obj
 0001:0000ec10       ??__F?_Generic_object@?$_Error_objects@H@std@@2V_Generic_error_category@2@A@@YAXXZ 1000fc10 f   moc_ChromaViewPlugin.obj
 0001:0000ec20       ??__F?_Iostream_object@?$_Error_objects@H@std@@2V_Iostream_error_category@2@A@@YAXXZ 1000fc20 f   moc_ChromaViewPlugin.obj
 0001:0000ec30       ??__F?_System_object@?$_Error_objects@H@std@@2V_System_error_category@2@A@@YAXXZ 1000fc30 f   moc_ChromaViewPlugin.obj
 0001:0000ec40       ??__FService_DNAExport@U2@@YAXXZ 1000fc40 f   moc_ChromaViewPlugin.obj
 0001:0000ec50       ??__FService_DNAGraphPack@U2@@YAXXZ 1000fc50 f   moc_ChromaViewPlugin.obj
 0001:0000ec60       ??__FService_ExternalToolSupport@U2@@YAXXZ 1000fc60 f   moc_ChromaViewPlugin.obj
 0001:0000ec70       ??__FService_GUITesting@U2@@YAXXZ 1000fc70 f   moc_ChromaViewPlugin.obj
 0001:0000ec80       ??__FService_MaxCoreServiceId@U2@@YAXXZ 1000fc80 f   moc_ChromaViewPlugin.obj
 0001:0000ec90       ??__FService_MinCoreServiceId@U2@@YAXXZ 1000fc90 f   moc_ChromaViewPlugin.obj
 0001:0000eca0       ??__FService_PluginViewer@U2@@YAXXZ 1000fca0 f   moc_ChromaViewPlugin.obj
 0001:0000ecb0       ??__FService_Project@U2@@YAXXZ 1000fcb0 f   moc_ChromaViewPlugin.obj
 0001:0000ecc0       ??__FService_ProjectView@U2@@YAXXZ 1000fcc0 f   moc_ChromaViewPlugin.obj
 0001:0000ecd0       ??__FService_QueryDesigner@U2@@YAXXZ 1000fcd0 f   moc_ChromaViewPlugin.obj
 0001:0000ece0       ??__FService_ScriptRegistry@U2@@YAXXZ 1000fce0 f   moc_ChromaViewPlugin.obj
 0001:0000ecf0       ??__FService_TestRunner@U2@@YAXXZ 1000fcf0 f   moc_ChromaViewPlugin.obj
 0001:0000ed00       ??__FService_WorkflowDesigner@U2@@YAXXZ 1000fd00 f   moc_ChromaViewPlugin.obj
 0001:0000ed10       ??__F?_Generic_object@?$_Error_objects@H@std@@2V_Generic_error_category@2@A@@YAXXZ 1000fd10 f   moc_ChromatogramView.obj
 0001:0000ed20       ??__F?_Iostream_object@?$_Error_objects@H@std@@2V_Iostream_error_category@2@A@@YAXXZ 1000fd20 f   moc_ChromatogramView.obj
 0001:0000ed30       ??__F?_System_object@?$_Error_objects@H@std@@2V_System_error_category@2@A@@YAXXZ 1000fd30 f   moc_ChromatogramView.obj
 0001:0000ed40       ??__Fdummy@?A0xc45d533f@@YAXXZ 1000fd40 f   qrc_chroma_view.obj
 0002:000007bc       _Service_PluginViewer$initializer$ 100107bc     ChromaViewPlugin.obj
 0002:000007c0       _Service_Project$initializer$ 100107c0     ChromaViewPlugin.obj
 0002:000007c4       _Service_ProjectView$initializer$ 100107c4     ChromaViewPlugin.obj
 0002:000007c8       _Service_DNAGraphPack$initializer$ 100107c8     ChromaViewPlugin.obj
 0002:000007cc       _Service_DNAExport$initializer$ 100107cc     ChromaViewPlugin.obj
 0002:000007d0       _Service_TestRunner$initializer$ 100107d0     ChromaViewPlugin.obj
 0002:000007d4       _Service_ScriptRegistry$initializer$ 100107d4     ChromaViewPlugin.obj
 0002:000007d8       _Service_ExternalToolSupport$initializer$ 100107d8     ChromaViewPlugin.obj
 0002:000007dc       _Service_GUITesting$initializer$ 100107dc     ChromaViewPlugin.obj
 0002:000007e0       _Service_WorkflowDesigner$initializer$ 100107e0     ChromaViewPlugin.obj
 0002:000007e4       _Service_QueryDesigner$initializer$ 100107e4     ChromaViewPlugin.obj
 0002:000007e8       _Service_MinCoreServiceId$initializer$ 100107e8     ChromaViewPlugin.obj
 0002:000007ec       _Service_MaxCoreServiceId$initializer$ 100107ec     ChromaViewPlugin.obj
 0002:000007f0       _algoLog$initializer$      100107f0     ChromaViewPlugin.obj
 0002:000007f4       _cmdLog$initializer$       100107f4     ChromaViewPlugin.obj
 0002:000007f8       _coreLog$initializer$      100107f8     ChromaViewPlugin.obj
 0002:000007fc       _ioLog$initializer$        100107fc     ChromaViewPlugin.obj
 0002:00000800       _perfLog$initializer$      10010800     ChromaViewPlugin.obj
 0002:00000804       _scriptLog$initializer$    10010804     ChromaViewPlugin.obj
 0002:00000808       _taskLog$initializer$      10010808     ChromaViewPlugin.obj
 0002:0000080c       _uiLog$initializer$        1001080c     ChromaViewPlugin.obj
 0002:00000810       _userActLog$initializer$   10010810     ChromaViewPlugin.obj
 0002:00000814       ?_Generic_object$initializer$@?$_Error_objects@H@std@@2P6AXXZA 10010814     ChromaViewPlugin.obj
 0002:00000818       ?_Iostream_object$initializer$@?$_Error_objects@H@std@@2P6AXXZA 10010818     ChromaViewPlugin.obj
 0002:0000081c       ?_System_object$initializer$@?$_Error_objects@H@std@@2P6AXXZA 1001081c     ChromaViewPlugin.obj
 0002:00000820       _algoLog$initializer$      10010820     ChromatogramView.obj
 0002:00000824       _cmdLog$initializer$       10010824     ChromatogramView.obj
 0002:00000828       _coreLog$initializer$      10010828     ChromatogramView.obj
 0002:0000082c       _ioLog$initializer$        1001082c     ChromatogramView.obj
 0002:00000830       _perfLog$initializer$      10010830     ChromatogramView.obj
 0002:00000834       _scriptLog$initializer$    10010834     ChromatogramView.obj
 0002:00000838       _taskLog$initializer$      10010838     ChromatogramView.obj
 0002:0000083c       _uiLog$initializer$        1001083c     ChromatogramView.obj
 0002:00000840       _userActLog$initializer$   10010840     ChromatogramView.obj
 0002:00000844       _Service_PluginViewer$initializer$ 10010844     ChromatogramView.obj
 0002:00000848       _Service_Project$initializer$ 10010848     ChromatogramView.obj
 0002:0000084c       _Service_ProjectView$initializer$ 1001084c     ChromatogramView.obj
 0002:00000850       _Service_DNAGraphPack$initializer$ 10010850     ChromatogramView.obj
 0002:00000854       _Service_DNAExport$initializer$ 10010854     ChromatogramView.obj
 0002:00000858       _Service_TestRunner$initializer$ 10010858     ChromatogramView.obj
 0002:0000085c       _Service_ScriptRegistry$initializer$ 1001085c     ChromatogramView.obj
 0002:00000860       _Service_ExternalToolSupport$initializer$ 10010860     ChromatogramView.obj
 0002:00000864       _Service_GUITesting$initializer$ 10010864     ChromatogramView.obj
 0002:00000868       _Service_WorkflowDesigner$initializer$ 10010868     ChromatogramView.obj
 0002:0000086c       _Service_QueryDesigner$initializer$ 1001086c     ChromatogramView.obj
 0002:00000870       _Service_MinCoreServiceId$initializer$ 10010870     ChromatogramView.obj
 0002:00000874       _Service_MaxCoreServiceId$initializer$ 10010874     ChromatogramView.obj
 0002:00000878       _Service_PluginViewer$initializer$ 10010878     moc_ChromaViewPlugin.obj
 0002:0000087c       _Service_Project$initializer$ 1001087c     moc_ChromaViewPlugin.obj
 0002:00000880       _Service_ProjectView$initializer$ 10010880     moc_ChromaViewPlugin.obj
 0002:00000884       _Service_DNAGraphPack$initializer$ 10010884     moc_ChromaViewPlugin.obj
 0002:00000888       _Service_DNAExport$initializer$ 10010888     moc_ChromaViewPlugin.obj
 0002:0000088c       _Service_TestRunner$initializer$ 1001088c     moc_ChromaViewPlugin.obj
 0002:00000890       _Service_ScriptRegistry$initializer$ 10010890     moc_ChromaViewPlugin.obj
 0002:00000894       _Service_ExternalToolSupport$initializer$ 10010894     moc_ChromaViewPlugin.obj
 0002:00000898       _Service_GUITesting$initializer$ 10010898     moc_ChromaViewPlugin.obj
 0002:0000089c       _Service_WorkflowDesigner$initializer$ 1001089c     moc_ChromaViewPlugin.obj
 0002:000008a0       _Service_QueryDesigner$initializer$ 100108a0     moc_ChromaViewPlugin.obj
 0002:000008a4       _Service_MinCoreServiceId$initializer$ 100108a4     moc_ChromaViewPlugin.obj
 0002:000008a8       _Service_MaxCoreServiceId$initializer$ 100108a8     moc_ChromaViewPlugin.obj
 0002:000008ac       ?staticMetaObject$initializer$@ChromaViewPlugin@U2@@2P6AXXZA 100108ac     moc_ChromaViewPlugin.obj
 0002:000008b0       ?staticMetaObject$initializer$@ChromaViewContext@U2@@2P6AXXZA 100108b0     moc_ChromaViewPlugin.obj
 0002:000008b4       ?staticMetaObject$initializer$@ChromaViewAction@U2@@2P6AXXZA 100108b4     moc_ChromaViewPlugin.obj
 0002:000008b8       ?staticMetaObject$initializer$@ChromatogramView@U2@@2P6AXXZA 100108b8     moc_ChromatogramView.obj
 0002:000008bc       ?staticMetaObject$initializer$@ChromatogramViewRenderArea@U2@@2P6AXXZA 100108bc     moc_ChromatogramView.obj
 0002:000008c0       _dummy$initializer$        100108c0     qrc_chroma_view.obj
 0002:000008cc       _pcinit                    100108cc     MSVCRT:crtdll.obj
 0002:000008d0       _pinit                     100108d0     MSVCRT:atonexit.obj
 0002:00001630       _qt_meta_stringdata_U2__ChromaViewPlugin 10011630     moc_ChromaViewPlugin.obj
 0002:00001658       _qt_meta_data_U2__ChromaViewPlugin 10011658     moc_ChromaViewPlugin.obj
 0002:00001694       _qt_meta_data_U2__ChromaViewAction 10011694     moc_ChromaViewPlugin.obj
 0002:000016d0       _qt_meta_stringdata_U2__ChromaViewContext 100116d0     moc_ChromaViewPlugin.obj
 0002:00001778       _qt_meta_data_U2__ChromaViewContext 10011778     moc_ChromaViewPlugin.obj
 0002:000017ec       _qt_meta_stringdata_U2__ChromaViewAction 100117ec     moc_ChromaViewPlugin.obj
 0002:00001818       _qt_meta_data_U2__ChromatogramView 10011818     moc_ChromatogramView.obj
 0002:0000196c       _qt_meta_stringdata_U2__ChromatogramViewRenderArea 1001196c     moc_ChromatogramView.obj
 0002:0000199c       _qt_meta_data_U2__ChromatogramViewRenderArea 1001199c     moc_ChromatogramView.obj
 0002:000019d8       _qt_meta_stringdata_U2__ChromatogramView 100119d8     moc_ChromatogramView.obj
 0002:00001c18       _qt_resource_data          10011c18     qrc_chroma_view.obj
 0002:00002408       _qt_resource_name          10012408     qrc_chroma_view.obj
 0002:00002478       _qt_resource_struct        10012478     qrc_chroma_view.obj
 0002:000024e0       _Int32ToUInt32             100124e0     MSVCRT:ftol3.obj
 0002:000024f0       _MantissaMask              100124f0     MSVCRT:ftol3.obj
 0002:000024f8       _IntegerBit                100124f8     MSVCRT:ftol3.obj
 0002:00002500       _SignBit64                 10012500     MSVCRT:ftol3.obj
 0002:00002508       _MinFP64                   10012508     MSVCRT:ftol3.obj
 0002:00002510       _MinInt64                  10012510     MSVCRT:ftol3.obj
 0002:00002518       _MaxInt64                  10012518     MSVCRT:ftol3.obj
 0002:00002520       _MaxUInt64                 10012520     MSVCRT:ftol3.obj
 0002:00002528       _MaxFP32                   10012528     MSVCRT:ftol3.obj
 0002:00002530       _MinFP32                   10012530     MSVCRT:ftol3.obj
 0002:00002538       _MinSubInexact             10012538     MSVCRT:ftol3.obj
 0002:00002540       _FpExcptTable              10012540     MSVCRT:ftol3.obj
 0002:00002550       _i1075                     10012550     MSVCRT:ftol3.obj
 0002:00002554       _i1087                     10012554     MSVCRT:ftol3.obj
 0002:00002558       _x0800                     10012558     MSVCRT:ftol3.obj
 0002:0000255c       _x17FF                     1001255c     MSVCRT:ftol3.obj
 0002:00002560       _CWMask                    10012560     MSVCRT:ftol3.obj
 0002:00002568       _GS_ExceptionPointers      10012568     MSVCRT:gs_report.obj
 0002:000031a8       __catchsym$?_Copy@?$basic_string@DU?$char_traits@D@std@@V?$allocator@D@2@@std@@QAEXII@Z$5 100131a8     ChromaViewPlugin.obj
 0002:000031b8       __catchsym$?_Copy@?$basic_string@DU?$char_traits@D@std@@V?$allocator@D@2@@std@@QAEXII@Z$4 100131b8     ChromaViewPlugin.obj
 0002:000031c8       __unwindtable$?_Copy@?$basic_string@DU?$char_traits@D@std@@V?$allocator@D@2@@std@@QAEXII@Z 100131c8     ChromaViewPlugin.obj
 0002:000031e8       __ehfuncinfo$?_Copy@?$basic_string@DU?$char_traits@D@std@@V?$allocator@D@2@@std@@QAEXII@Z 100131e8     ChromaViewPlugin.obj
 0002:0000320c       __tryblocktable$?_Copy@?$basic_string@DU?$char_traits@D@std@@V?$allocator@D@2@@std@@QAEXII@Z 1001320c     ChromaViewPlugin.obj
 0002:00003234       __catchsym$?detach_helper@?$QList@PAVGObject@U2@@@@AAEXH@Z$2 10013234     ChromaViewPlugin.obj
 0002:00003244       __unwindtable$?detach_helper@?$QList@PAVGObject@U2@@@@AAEXH@Z 10013244     ChromaViewPlugin.obj
 0002:00003254       __tryblocktable$?detach_helper@?$QList@PAVGObject@U2@@@@AAEXH@Z 10013254     ChromaViewPlugin.obj
 0002:00003268       __ehfuncinfo$?detach_helper@?$QList@PAVGObject@U2@@@@AAEXH@Z 10013268     ChromaViewPlugin.obj
 0002:0000328c       __ehfuncinfo$??0ChromaViewPlugin@U2@@QAE@XZ 1001328c     ChromaViewPlugin.obj
 0002:000032b0       __unwindtable$??0ChromaViewPlugin@U2@@QAE@XZ 100132b0     ChromaViewPlugin.obj
 0002:000032f8       __unwindtable$??0ChromaViewContext@U2@@QAE@PAVQObject@@@Z 100132f8     ChromaViewPlugin.obj
 0002:00003310       __ehfuncinfo$??0ChromaViewContext@U2@@QAE@PAVQObject@@@Z 10013310     ChromaViewPlugin.obj
 0002:00003334       __unwindtable$?sl_showChromatogram@ChromaViewContext@U2@@IAEXXZ 10013334     ChromaViewPlugin.obj
 0002:0000333c       __ehfuncinfo$?sl_showChromatogram@ChromaViewContext@U2@@IAEXXZ 1001333c     ChromaViewPlugin.obj
 0002:00003360       __unwindtable$?sl_sequenceWidgetAdded@ChromaViewContext@U2@@IAEXPAVADVSequenceWidget@2@@Z 10013360     ChromaViewPlugin.obj
 0002:00003378       __ehfuncinfo$?sl_sequenceWidgetAdded@ChromaViewContext@U2@@IAEXPAVADVSequenceWidget@2@@Z 10013378     ChromaViewPlugin.obj
 0002:0000339c       __unwindtable$?initViewContext@ChromaViewContext@U2@@MAEXPAVGObjectView@2@@Z 1001339c     ChromaViewPlugin.obj
 0002:000033b4       __ehfuncinfo$?initViewContext@ChromaViewContext@U2@@MAEXPAVGObjectView@2@@Z 100133b4     ChromaViewPlugin.obj
 0002:000033d8       __ehfuncinfo$??0ChromaViewAction@U2@@QAE@XZ 100133d8     ChromaViewPlugin.obj
 0002:000033fc       __unwindtable$??0ChromaViewAction@U2@@QAE@XZ 100133fc     ChromaViewPlugin.obj
 0002:00003424       __unwindtable$??__EalgoLog@U2@@YAXXZ 10013424     ChromaViewPlugin.obj
 0002:0000342c       __ehfuncinfo$??__EalgoLog@U2@@YAXXZ 1001342c     ChromaViewPlugin.obj
 0002:00003450       __unwindtable$??__EcmdLog@U2@@YAXXZ 10013450     ChromaViewPlugin.obj
 0002:00003458       __ehfuncinfo$??__EcmdLog@U2@@YAXXZ 10013458     ChromaViewPlugin.obj
 0002:0000347c       __unwindtable$??__EcoreLog@U2@@YAXXZ 1001347c     ChromaViewPlugin.obj
 0002:00003484       __ehfuncinfo$??__EcoreLog@U2@@YAXXZ 10013484     ChromaViewPlugin.obj
 0002:000034a8       __unwindtable$??__EioLog@U2@@YAXXZ 100134a8     ChromaViewPlugin.obj
 0002:000034b0       __ehfuncinfo$??__EioLog@U2@@YAXXZ 100134b0     ChromaViewPlugin.obj
 0002:000034d4       __unwindtable$??__EperfLog@U2@@YAXXZ 100134d4     ChromaViewPlugin.obj
 0002:000034dc       __ehfuncinfo$??__EperfLog@U2@@YAXXZ 100134dc     ChromaViewPlugin.obj
 0002:00003500       __unwindtable$??__EscriptLog@U2@@YAXXZ 10013500     ChromaViewPlugin.obj
 0002:00003508       __ehfuncinfo$??__EscriptLog@U2@@YAXXZ 10013508     ChromaViewPlugin.obj
 0002:0000352c       __unwindtable$??__EtaskLog@U2@@YAXXZ 1001352c     ChromaViewPlugin.obj
 0002:00003534       __ehfuncinfo$??__EtaskLog@U2@@YAXXZ 10013534     ChromaViewPlugin.obj
 0002:00003558       __unwindtable$??__EuiLog@U2@@YAXXZ 10013558     ChromaViewPlugin.obj
 0002:00003560       __ehfuncinfo$??__EuiLog@U2@@YAXXZ 10013560     ChromaViewPlugin.obj
 0002:00003584       __unwindtable$??__EuserActLog@U2@@YAXXZ 10013584     ChromaViewPlugin.obj
 0002:0000358c       __ehfuncinfo$??__EuserActLog@U2@@YAXXZ 1001358c     ChromaViewPlugin.obj
 0002:000035b0       __catchsym$??0?$QList@PAVADVSequenceWidget@U2@@@@QAE@ABV0@@Z$2 100135b0     ChromaViewPlugin.obj
 0002:000035c0       __unwindtable$??0?$QList@PAVADVSequenceWidget@U2@@@@QAE@ABV0@@Z 100135c0     ChromaViewPlugin.obj
 0002:000035d0       __tryblocktable$??0?$QList@PAVADVSequenceWidget@U2@@@@QAE@ABV0@@Z 100135d0     ChromaViewPlugin.obj
 0002:000035e4       __ehfuncinfo$??0?$QList@PAVADVSequenceWidget@U2@@@@QAE@ABV0@@Z 100135e4     ChromaViewPlugin.obj
 0002:00003608       __unwindtable$?findChromaObj@U2@@YAPAVDNAChromatogramObject@1@PAVADVSingleSequenceWidget@1@@Z 10013608     ChromaViewPlugin.obj
 0002:00003618       __ehfuncinfo$?findChromaObj@U2@@YAPAVDNAChromatogramObject@1@PAVADVSingleSequenceWidget@1@@Z 10013618     ChromaViewPlugin.obj
 0002:0000363c       __unwindtable$??H@YA?BVQString@@ABV0@0@Z 1001363c     ChromatogramView.obj
 0002:00003644       __ehfuncinfo$??H@YA?BVQString@@ABV0@0@Z 10013644     ChromatogramView.obj
 0002:00003668       __unwindtable$??H@YA?BVQString@@ABV0@PBD@Z 10013668     ChromatogramView.obj
 0002:00003678       __ehfuncinfo$??H@YA?BVQString@@ABV0@PBD@Z 10013678     ChromatogramView.obj
 0002:0000369c       __unwindtable$??H@YA?BVQString@@PBDABV0@@Z 1001369c     ChromatogramView.obj
 0002:000036a4       __ehfuncinfo$??H@YA?BVQString@@PBDABV0@@Z 100136a4     ChromatogramView.obj
 0002:000036c8       __catchsym$?reallocData@?$QVector@G@@AAEXHHV?$QFlags@W4AllocationOption@QArrayData@@@@@Z$5 100136c8     ChromatogramView.obj
 0002:000036d8       __catchsym$?reallocData@?$QVector@G@@AAEXHHV?$QFlags@W4AllocationOption@QArrayData@@@@@Z$4 100136d8     ChromatogramView.obj
 0002:000036e8       __unwindtable$?reallocData@?$QVector@G@@AAEXHHV?$QFlags@W4AllocationOption@QArrayData@@@@@Z 100136e8     ChromatogramView.obj
 0002:00003708       __ehfuncinfo$?reallocData@?$QVector@G@@AAEXHHV?$QFlags@W4AllocationOption@QArrayData@@@@@Z 10013708     ChromatogramView.obj
 0002:0000372c       __tryblocktable$?reallocData@?$QVector@G@@AAEXHHV?$QFlags@W4AllocationOption@QArrayData@@@@@Z 1001372c     ChromatogramView.obj
 0002:00003754       __catchsym$?reallocData@?$QVector@D@@AAEXHHV?$QFlags@W4AllocationOption@QArrayData@@@@@Z$5 10013754     ChromatogramView.obj
 0002:00003764       __catchsym$?reallocData@?$QVector@D@@AAEXHHV?$QFlags@W4AllocationOption@QArrayData@@@@@Z$4 10013764     ChromatogramView.obj
 0002:00003774       __unwindtable$?reallocData@?$QVector@D@@AAEXHHV?$QFlags@W4AllocationOption@QArrayData@@@@@Z 10013774     ChromatogramView.obj
 0002:00003794       __ehfuncinfo$?reallocData@?$QVector@D@@AAEXHHV?$QFlags@W4AllocationOption@QArrayData@@@@@Z 10013794     ChromatogramView.obj
 0002:000037b8       __tryblocktable$?reallocData@?$QVector@D@@AAEXHHV?$QFlags@W4AllocationOption@QArrayData@@@@@Z 100137b8     ChromatogramView.obj
 0002:000037e0       __unwindtable$?insert@?$QHash@VQString@@UQHashDummyValue@@@@QAE?AViterator@1@ABVQString@@ABUQHashDummyValue@@@Z 100137e0     ChromatogramView.obj
 0002:000037e8       __ehfuncinfo$?insert@?$QHash@VQString@@UQHashDummyValue@@@@QAE?AViterator@1@ABVQString@@ABUQHashDummyValue@@@Z 100137e8     ChromatogramView.obj
 0002:0000380c       __unwindtable$?createNode@?$QHash@VQString@@UQHashDummyValue@@@@AAEPAU?$QHashNode@VQString@@UQHashDummyValue@@@@IABVQString@@ABUQHashDummyValue@@PAPAU2@@Z 1001380c     ChromatogramView.obj
 0002:00003814       __ehfuncinfo$?createNode@?$QHash@VQString@@UQHashDummyValue@@@@AAEPAU?$QHashNode@VQString@@UQHashDummyValue@@@@IABVQString@@ABUQHashDummyValue@@PAPAU2@@Z 10013814     ChromatogramView.obj
 0002:00003838       __unwindtable$?duplicateNode@?$QHash@VQString@@UQHashDummyValue@@@@CAXPAUNode@QHashData@@PAX@Z 10013838     ChromatogramView.obj
 0002:00003840       __ehfuncinfo$?duplicateNode@?$QHash@VQString@@UQHashDummyValue@@@@CAXPAUNode@QHashData@@PAX@Z 10013840     ChromatogramView.obj
 0002:00003864       __unwindtable$??0DocumentFormatConstraints@U2@@QAE@XZ 10013864     ChromatogramView.obj
 0002:0000386c       __ehfuncinfo$??0DocumentFormatConstraints@U2@@QAE@XZ 1001386c     ChromatogramView.obj
 0002:00003890       __unwindtable$??1DocumentFormatConstraints@U2@@QAE@XZ 10013890     ChromatogramView.obj
 0002:000038a0       __ehfuncinfo$??1DocumentFormatConstraints@U2@@QAE@XZ 100138a0     ChromatogramView.obj
 0002:000038c4       __catchsym$??0?$QList@PAVGObject@U2@@@@QAE@ABV0@@Z$2 100138c4     ChromatogramView.obj
 0002:000038d4       __unwindtable$??0?$QList@PAVGObject@U2@@@@QAE@ABV0@@Z 100138d4     ChromatogramView.obj
 0002:000038e4       __tryblocktable$??0?$QList@PAVGObject@U2@@@@QAE@ABV0@@Z 100138e4     ChromatogramView.obj
 0002:000038f8       __ehfuncinfo$??0?$QList@PAVGObject@U2@@@@QAE@ABV0@@Z 100138f8     ChromatogramView.obj
 0002:0000391c       __unwindtable$??__EalgoLog@U2@@YAXXZ 1001391c     ChromatogramView.obj
 0002:00003924       __ehfuncinfo$??__EalgoLog@U2@@YAXXZ 10013924     ChromatogramView.obj
 0002:00003948       __unwindtable$??__EcmdLog@U2@@YAXXZ 10013948     ChromatogramView.obj
 0002:00003950       __ehfuncinfo$??__EcmdLog@U2@@YAXXZ 10013950     ChromatogramView.obj
 0002:00003974       __unwindtable$??__EcoreLog@U2@@YAXXZ 10013974     ChromatogramView.obj
 0002:0000397c       __ehfuncinfo$??__EcoreLog@U2@@YAXXZ 1001397c     ChromatogramView.obj
 0002:000039a0       __unwindtable$??__EioLog@U2@@YAXXZ 100139a0     ChromatogramView.obj
 0002:000039a8       __ehfuncinfo$??__EioLog@U2@@YAXXZ 100139a8     ChromatogramView.obj
 0002:000039cc       __unwindtable$??__EperfLog@U2@@YAXXZ 100139cc     ChromatogramView.obj
 0002:000039d4       __ehfuncinfo$??__EperfLog@U2@@YAXXZ 100139d4     ChromatogramView.obj
 0002:000039f8       __unwindtable$??__EscriptLog@U2@@YAXXZ 100139f8     ChromatogramView.obj
 0002:00003a00       __ehfuncinfo$??__EscriptLog@U2@@YAXXZ 10013a00     ChromatogramView.obj
 0002:00003a24       __unwindtable$??__EtaskLog@U2@@YAXXZ 10013a24     ChromatogramView.obj
 0002:00003a2c       __ehfuncinfo$??__EtaskLog@U2@@YAXXZ 10013a2c     ChromatogramView.obj
 0002:00003a50       __unwindtable$??__EuiLog@U2@@YAXXZ 10013a50     ChromatogramView.obj
 0002:00003a58       __ehfuncinfo$??__EuiLog@U2@@YAXXZ 10013a58     ChromatogramView.obj
 0002:00003a7c       __unwindtable$??__EuserActLog@U2@@YAXXZ 10013a7c     ChromatogramView.obj
 0002:00003a84       __ehfuncinfo$??__EuserActLog@U2@@YAXXZ 10013a84     ChromatogramView.obj
 0002:00003aa8       __catchsym$?append@?$QList@V?$QPointer@VGObject@U2@@@@@@QAEXABV?$QPointer@VGObject@U2@@@@@Z$13 10013aa8     ChromatogramView.obj
 0002:00003ab8       __catchsym$?append@?$QList@V?$QPointer@VGObject@U2@@@@@@QAEXABV?$QPointer@VGObject@U2@@@@@Z$12 10013ab8     ChromatogramView.obj
 0002:00003ac8       __ehfuncinfo$?append@?$QList@V?$QPointer@VGObject@U2@@@@@@QAEXABV?$QPointer@VGObject@U2@@@@@Z 10013ac8     ChromatogramView.obj
 0002:00003aec       __tryblocktable$?append@?$QList@V?$QPointer@VGObject@U2@@@@@@QAEXABV?$QPointer@VGObject@U2@@@@@Z 10013aec     ChromatogramView.obj
 0002:00003b14       __unwindtable$?append@?$QList@V?$QPointer@VGObject@U2@@@@@@QAEXABV?$QPointer@VGObject@U2@@@@@Z 10013b14     ChromatogramView.obj
 0002:00003b44       __catchsym$?detach_helper_grow@?$QList@V?$QPointer@VGObject@U2@@@@@@AAEPAUNode@1@HH@Z$5 10013b44     ChromatogramView.obj
 0002:00003b54       __catchsym$?detach_helper_grow@?$QList@V?$QPointer@VGObject@U2@@@@@@AAEPAUNode@1@HH@Z$4 10013b54     ChromatogramView.obj
 0002:00003b64       __unwindtable$?detach_helper_grow@?$QList@V?$QPointer@VGObject@U2@@@@@@AAEPAUNode@1@HH@Z 10013b64     ChromatogramView.obj
 0002:00003b84       __ehfuncinfo$?detach_helper_grow@?$QList@V?$QPointer@VGObject@U2@@@@@@AAEPAUNode@1@HH@Z 10013b84     ChromatogramView.obj
 0002:00003ba8       __tryblocktable$?detach_helper_grow@?$QList@V?$QPointer@VGObject@U2@@@@@@AAEPAUNode@1@HH@Z 10013ba8     ChromatogramView.obj
 0002:00003bd0       __catchsym$?node_copy@?$QList@V?$QPointer@VGObject@U2@@@@@@AAEXPAUNode@1@00@Z$6 10013bd0     ChromatogramView.obj
 0002:00003be0       __tryblocktable$?node_copy@?$QList@V?$QPointer@VGObject@U2@@@@@@AAEXPAUNode@1@00@Z 10013be0     ChromatogramView.obj
 0002:00003bf4       __unwindtable$?node_copy@?$QList@V?$QPointer@VGObject@U2@@@@@@AAEXPAUNode@1@00@Z 10013bf4     ChromatogramView.obj
 0002:00003c14       __ehfuncinfo$?node_copy@?$QList@V?$QPointer@VGObject@U2@@@@@@AAEXPAUNode@1@00@Z 10013c14     ChromatogramView.obj
 0002:00003c38       __catchsym$??0?$QList@H@@QAE@ABV0@@Z$2 10013c38     ChromatogramView.obj
 0002:00003c48       __unwindtable$??0?$QList@H@@QAE@ABV0@@Z 10013c48     ChromatogramView.obj
 0002:00003c58       __tryblocktable$??0?$QList@H@@QAE@ABV0@@Z 10013c58     ChromatogramView.obj
 0002:00003c6c       __ehfuncinfo$??0?$QList@H@@QAE@ABV0@@Z 10013c6c     ChromatogramView.obj
 0002:00003c90       __catchsym$?append@?$QList@H@@QAEXABH@Z$6 10013c90     ChromatogramView.obj
 0002:00003ca0       __tryblocktable$?append@?$QList@H@@QAEXABH@Z 10013ca0     ChromatogramView.obj
 0002:00003cb4       __ehfuncinfo$?append@?$QList@H@@QAEXABH@Z 10013cb4     ChromatogramView.obj
 0002:00003cd8       __unwindtable$?append@?$QList@H@@QAEXABH@Z 10013cd8     ChromatogramView.obj
 0002:00003d08       __catchsym$?detach_helper_grow@?$QList@H@@AAEPAUNode@1@HH@Z$5 10013d08     ChromatogramView.obj
 0002:00003d18       __catchsym$?detach_helper_grow@?$QList@H@@AAEPAUNode@1@HH@Z$4 10013d18     ChromatogramView.obj
 0002:00003d28       __unwindtable$?detach_helper_grow@?$QList@H@@AAEPAUNode@1@HH@Z 10013d28     ChromatogramView.obj
 0002:00003d48       __ehfuncinfo$?detach_helper_grow@?$QList@H@@AAEPAUNode@1@HH@Z 10013d48     ChromatogramView.obj
 0002:00003d6c       __tryblocktable$?detach_helper_grow@?$QList@H@@AAEPAUNode@1@HH@Z 10013d6c     ChromatogramView.obj
 0002:00003d94       __catchsym$?detach_helper@?$QList@H@@AAEXH@Z$2 10013d94     ChromatogramView.obj
 0002:00003da4       __unwindtable$?detach_helper@?$QList@H@@AAEXH@Z 10013da4     ChromatogramView.obj
 0002:00003db4       __tryblocktable$?detach_helper@?$QList@H@@AAEXH@Z 10013db4     ChromatogramView.obj
 0002:00003dc8       __ehfuncinfo$?detach_helper@?$QList@H@@AAEXH@Z 10013dc8     ChromatogramView.obj
 0002:00003dec       __ehfuncinfo$??0ChromatogramView@U2@@QAE@PAVQWidget@@PAVADVSequenceObjectContext@1@PAVGSequenceLineView@1@ABVDNAChromatogram@1@@Z 10013dec     ChromatogramView.obj
 0002:00003e10       __unwindtable$??0ChromatogramView@U2@@QAE@PAVQWidget@@PAVADVSequenceObjectContext@1@PAVGSequenceLineView@1@ABVDNAChromatogram@1@@Z 10013e10     ChromatogramView.obj
 0002:00003f68       __unwindtable$?buildPopupMenu@ChromatogramView@U2@@UAEXAAVQMenu@@@Z 10013f68     ChromatogramView.obj
 0002:00003f78       __ehfuncinfo$?buildPopupMenu@ChromatogramView@U2@@UAEXAAVQMenu@@@Z 10013f78     ChromatogramView.obj
 0002:00003f9c       __unwindtable$?pack@ChromatogramView@U2@@MAEXXZ 10013f9c     ChromatogramView.obj
 0002:00003fa4       __ehfuncinfo$?pack@ChromatogramView@U2@@MAEXXZ 10013fa4     ChromatogramView.obj
 0002:00003fc8       __ehfuncinfo$?sl_onPopupMenuCkicked@ChromatogramView@U2@@AAEXPAVQAction@@@Z 10013fc8     ChromatogramView.obj
 0002:00003fec       __unwindtable$?sl_onPopupMenuCkicked@ChromatogramView@U2@@AAEXPAVQAction@@@Z 10013fec     ChromatogramView.obj
 0002:00004074       __ehfuncinfo$?sl_addNewSequenceObject@ChromatogramView@U2@@AAEXXZ 10014074     ChromatogramView.obj
 0002:00004098       __unwindtable$?sl_addNewSequenceObject@ChromatogramView@U2@@AAEXXZ 10014098     ChromatogramView.obj
 0002:00004160       __ehfuncinfo$?sl_onAddExistingSequenceObject@ChromatogramView@U2@@AAEXXZ 10014160     ChromatogramView.obj
 0002:00004184       __unwindtable$?sl_onAddExistingSequenceObject@ChromatogramView@U2@@AAEXXZ 10014184     ChromatogramView.obj
 0002:000041f4       __unwindtable$?sl_onSequenceObjectLoaded@ChromatogramView@U2@@AAEXPAVTask@2@@Z 100141f4     ChromatogramView.obj
 0002:000041fc       __ehfuncinfo$?sl_onSequenceObjectLoaded@ChromatogramView@U2@@AAEXPAVTask@2@@Z 100141fc     ChromatogramView.obj
 0002:00004220       __ehfuncinfo$?sl_removeChanges@ChromatogramView@U2@@AAEXXZ 10014220     ChromatogramView.obj
 0002:00004244       __unwindtable$?sl_removeChanges@ChromatogramView@U2@@AAEXXZ 10014244     ChromatogramView.obj
 0002:0000426c       __unwindtable$?sl_showHideTrace@ChromatogramView@U2@@AAEXXZ 1001426c     ChromatogramView.obj
 0002:0000428c       __ehfuncinfo$?sl_showHideTrace@ChromatogramView@U2@@AAEXXZ 1001428c     ChromatogramView.obj
 0002:000042b0       __unwindtable$?sl_showAllTraces@ChromatogramView@U2@@AAEXXZ 100142b0     ChromatogramView.obj
 0002:000042c0       __ehfuncinfo$?sl_showAllTraces@ChromatogramView@U2@@AAEXXZ 100142c0     ChromatogramView.obj
 0002:000042e4       __unwindtable$?createToggleTraceAction@ChromatogramView@U2@@AAEPAVQAction@@ABVQString@@@Z 100142e4     ChromatogramView.obj
 0002:000042ec       __ehfuncinfo$?createToggleTraceAction@ChromatogramView@U2@@AAEPAVQAction@@ABVQString@@@Z 100142ec     ChromatogramView.obj
 0002:00004310       __unwindtable$??1ChromatogramView@U2@@UAE@XZ 10014310     ChromatogramView.obj
 0002:00004328       __ehfuncinfo$??1ChromatogramView@U2@@UAE@XZ 10014328     ChromatogramView.obj
 0002:0000434c       __ehfuncinfo$??0ChromatogramViewRenderArea@U2@@QAE@PAVChromatogramView@1@ABVDNAChromatogram@1@@Z 1001434c     ChromatogramView.obj
 0002:00004370       __unwindtable$??0ChromatogramViewRenderArea@U2@@QAE@PAVChromatogramView@1@ABVDNAChromatogram@1@@Z 10014370     ChromatogramView.obj
 0002:000043b8       __unwindtable$??1ChromatogramViewRenderArea@U2@@UAE@XZ 100143b8     ChromatogramView.obj
 0002:000043d8       __ehfuncinfo$??1ChromatogramViewRenderArea@U2@@UAE@XZ 100143d8     ChromatogramView.obj
 0002:000043fc       __ehfuncinfo$?drawAll@ChromatogramViewRenderArea@U2@@MAEXPAVQPaintDevice@@@Z 100143fc     ChromatogramView.obj
 0002:00004420       __unwindtable$?drawAll@ChromatogramViewRenderArea@U2@@MAEXPAVQPaintDevice@@@Z 10014420     ChromatogramView.obj
 0002:000044b8       __ehfuncinfo$?drawChromatogramTrace@ChromatogramViewRenderArea@U2@@AAEXNNNNAAVQPainter@@ABVU2Region@2@ABUChromatogramViewSettings@2@@Z 100144b8     ChromatogramView.obj
 0002:000044dc       __unwindtable$?drawChromatogramTrace@ChromatogramViewRenderArea@U2@@AAEXNNNNAAVQPainter@@ABVU2Region@2@ABUChromatogramViewSettings@2@@Z 100144dc     ChromatogramView.obj
 0002:00004504       __unwindtable$?drawOriginalBaseCalls@ChromatogramViewRenderArea@U2@@AAEXNNNNAAVQPainter@@ABVU2Region@2@ABVQByteArray@@_N@Z 10014504     ChromatogramView.obj
 0002:00004524       __ehfuncinfo$?drawOriginalBaseCalls@ChromatogramViewRenderArea@U2@@AAEXNNNNAAVQPainter@@ABVU2Region@2@ABVQByteArray@@_N@Z 10014524     ChromatogramView.obj
 0002:00004548       __unwindtable$?drawQualityValues@ChromatogramViewRenderArea@U2@@AAEXNNNNAAVQPainter@@ABVU2Region@2@ABVQByteArray@@@Z 10014548     ChromatogramView.obj
 0002:00004558       __ehfuncinfo$?drawQualityValues@ChromatogramViewRenderArea@U2@@AAEXNNNNAAVQPainter@@ABVU2Region@2@ABVQByteArray@@@Z 10014558     ChromatogramView.obj
 0002:0000457c       __unwindtable$?drawChromatogramBaseCallsLines@ChromatogramViewRenderArea@U2@@AAEXNNNNAAVQPainter@@ABVU2Region@2@ABVQByteArray@@ABUChromatogramViewSettings@2@@Z 1001457c     ChromatogramView.obj
 0002:00004584       __ehfuncinfo$?drawChromatogramBaseCallsLines@ChromatogramViewRenderArea@U2@@AAEXNNNNAAVQPainter@@ABVU2Region@2@ABVQByteArray@@ABUChromatogramViewSettings@2@@Z 10014584     ChromatogramView.obj
 0002:000045a8       __catchsym$??0?$QList@PAVQAction@@@@QAE@ABV0@@Z$2 100145a8     ChromatogramView.obj
 0002:000045b8       __unwindtable$??0?$QList@PAVQAction@@@@QAE@ABV0@@Z 100145b8     ChromatogramView.obj
 0002:000045c8       __tryblocktable$??0?$QList@PAVQAction@@@@QAE@ABV0@@Z 100145c8     ChromatogramView.obj
 0002:000045dc       __ehfuncinfo$??0?$QList@PAVQAction@@@@QAE@ABV0@@Z 100145dc     ChromatogramView.obj
 0002:00004600       __unwindtable$?qt_metatype_id@?$QMetaTypeIdQObject@PAVADVSequenceWidget@U2@@$00@@SAHXZ 10014600     moc_ChromaViewPlugin.obj
 0002:00004608       __ehfuncinfo$?qt_metatype_id@?$QMetaTypeIdQObject@PAVADVSequenceWidget@U2@@$00@@SAHXZ 10014608     moc_ChromaViewPlugin.obj
 0002:0000462c       __unwindtable$?qt_metatype_id@?$QMetaTypeIdQObject@PAVQAction@@$00@@SAHXZ 1001462c     moc_ChromatogramView.obj
 0002:00004634       __ehfuncinfo$?qt_metatype_id@?$QMetaTypeIdQObject@PAVQAction@@$00@@SAHXZ 10014634     moc_ChromatogramView.obj
 0002:00004658       __unwindtable$?qt_metatype_id@?$QMetaTypeIdQObject@PAVGObject@U2@@$00@@SAHXZ 10014658     moc_ChromatogramView.obj
 0002:00004660       __ehfuncinfo$?qt_metatype_id@?$QMetaTypeIdQObject@PAVGObject@U2@@$00@@SAHXZ 10014660     moc_ChromatogramView.obj
 0002:00004688       __sehtable$__onexit        10014688     MSVCRT:atonexit.obj
 0002:000046a8       __sehtable$??_M@YGXPAXIHP6EX0@Z@Z 100146a8     MSVCRT:ehvecdtr.obj
 0002:000046c8       __sehtable$?__ArrayUnwind@@YGXPAXIHP6EX0@Z@Z 100146c8     MSVCRT:ehvecdtr.obj
 0002:000046e8       __sehtable$___DllMainCRTStartup 100146e8     MSVCRT:crtdll.obj
 0002:00004710       __sehtable$__IsNonwritableInCurrentImage 10014710     MSVCRT:pesect.obj
 0002:00004730       .edata                     10014730     chroma_view.exp
 0002:00004758       rgpv                       10014758     chroma_view.exp
 0002:0000475c       rgszName                   1001475c     chroma_view.exp
 0002:00004760       rgwOrd                     10014760     chroma_view.exp
 0002:00004762       szName                     10014762     chroma_view.exp
 0002:00004772       $N00001                    10014772     chroma_view.exp
 0002:00006354       .idata$6                   10016354     U2Core:U2Core.dll
 0002:00006adc       .idata$6                   10016adc     U2Gui:U2Gui.dll
 0002:00007a9e       .idata$6                   10017a9e     U2View:U2View.dll
 0002:000090fc       .idata$6                   100190fc     Qt5Widgets:Qt5Widgets.dll
 0002:000097de       .idata$6                   100197de     Qt5Gui:Qt5Gui.dll
 0002:0000a478       .idata$6                   1001a478     Qt5Core:Qt5Core.dll
 0002:0000a51e       .idata$6                   1001a51e     msvcprt:MSVCP120.dll
 0002:0000a5ac       .idata$6                   1001a5ac     MSVCRT:MSVCR120.dll
 0002:0000a7cc       .idata$6                   1001a7cc     kernel32:KERNEL32.dll
 0003:0000000c       _Service_PluginViewer      1001b00c     ChromaViewPlugin.obj
 0003:00000014       _Service_Project           1001b014     ChromaViewPlugin.obj
 0003:0000001c       _Service_ProjectView       1001b01c     ChromaViewPlugin.obj
 0003:00000024       _Service_DNAGraphPack      1001b024     ChromaViewPlugin.obj
 0003:0000002c       _Service_DNAExport         1001b02c     ChromaViewPlugin.obj
 0003:00000034       _Service_TestRunner        1001b034     ChromaViewPlugin.obj
 0003:0000003c       _Service_ScriptRegistry    1001b03c     ChromaViewPlugin.obj
 0003:00000044       _Service_ExternalToolSupport 1001b044     ChromaViewPlugin.obj
 0003:0000004c       _Service_GUITesting        1001b04c     ChromaViewPlugin.obj
 0003:00000054       _Service_WorkflowDesigner  1001b054     ChromaViewPlugin.obj
 0003:0000005c       _Service_QueryDesigner     1001b05c     ChromaViewPlugin.obj
 0003:00000064       _Service_MinCoreServiceId  1001b064     ChromaViewPlugin.obj
 0003:0000006c       _Service_MaxCoreServiceId  1001b06c     ChromaViewPlugin.obj
 0003:00000074       _Service_PluginViewer      1001b074     ChromatogramView.obj
 0003:0000007c       _Service_Project           1001b07c     ChromatogramView.obj
 0003:00000084       _Service_ProjectView       1001b084     ChromatogramView.obj
 0003:0000008c       _Service_DNAGraphPack      1001b08c     ChromatogramView.obj
 0003:00000094       _Service_DNAExport         1001b094     ChromatogramView.obj
 0003:0000009c       _Service_TestRunner        1001b09c     ChromatogramView.obj
 0003:000000a4       _Service_ScriptRegistry    1001b0a4     ChromatogramView.obj
 0003:000000ac       _Service_ExternalToolSupport 1001b0ac     ChromatogramView.obj
 0003:000000b4       _Service_GUITesting        1001b0b4     ChromatogramView.obj
 0003:000000bc       _Service_WorkflowDesigner  1001b0bc     ChromatogramView.obj
 0003:000000c4       _Service_QueryDesigner     1001b0c4     ChromatogramView.obj
 0003:000000cc       _Service_MinCoreServiceId  1001b0cc     ChromatogramView.obj
 0003:000000d4       _Service_MaxCoreServiceId  1001b0d4     ChromatogramView.obj
 0003:000000dc       _Service_PluginViewer      1001b0dc     moc_ChromaViewPlugin.obj
 0003:000000e4       _Service_Project           1001b0e4     moc_ChromaViewPlugin.obj
 0003:000000ec       _Service_ProjectView       1001b0ec     moc_ChromaViewPlugin.obj
 0003:000000f4       _Service_DNAGraphPack      1001b0f4     moc_ChromaViewPlugin.obj
 0003:000000fc       _Service_DNAExport         1001b0fc     moc_ChromaViewPlugin.obj
 0003:00000104       _Service_TestRunner        1001b104     moc_ChromaViewPlugin.obj
 0003:0000010c       _Service_ScriptRegistry    1001b10c     moc_ChromaViewPlugin.obj
 0003:00000114       _Service_ExternalToolSupport 1001b114     moc_ChromaViewPlugin.obj
 0003:0000011c       _Service_GUITesting        1001b11c     moc_ChromaViewPlugin.obj
 0003:00000124       _Service_WorkflowDesigner  1001b124     moc_ChromaViewPlugin.obj
 0003:0000012c       _Service_QueryDesigner     1001b12c     moc_ChromaViewPlugin.obj
 0003:00000134       _Service_MinCoreServiceId  1001b134     moc_ChromaViewPlugin.obj
 0003:0000013c       _Service_MaxCoreServiceId  1001b13c     moc_ChromaViewPlugin.obj
 0003:00000660       __Tuple_alloc              1001b660     ChromaViewPlugin.obj
 0003:00000661       _ignore                    1001b661     ChromaViewPlugin.obj
 0003:00000662       _allocator_arg             1001b662     ChromaViewPlugin.obj
 0003:00000663       _piecewise_construct       1001b663     ChromaViewPlugin.obj
 0003:00000664       _taskLog                   1001b664     ChromaViewPlugin.obj
 0003:0000066c       _algoLog                   1001b66c     ChromaViewPlugin.obj
 0003:00000674       _userActLog                1001b674     ChromaViewPlugin.obj
 0003:0000067c       _ioLog                     1001b67c     ChromaViewPlugin.obj
 0003:00000684       _coreLog                   1001b684     ChromaViewPlugin.obj
 0003:0000068c       _uiLog                     1001b68c     ChromaViewPlugin.obj
 0003:00000694       _scriptLog                 1001b694     ChromaViewPlugin.obj
 0003:0000069c       _perfLog                   1001b69c     ChromaViewPlugin.obj
 0003:000006a4       _cmdLog                    1001b6a4     ChromaViewPlugin.obj
 0003:000006b4       __Tuple_alloc              1001b6b4     ChromatogramView.obj
 0003:000006b5       _ignore                    1001b6b5     ChromatogramView.obj
 0003:000006b6       _allocator_arg             1001b6b6     ChromatogramView.obj
 0003:000006b7       _piecewise_construct       1001b6b7     ChromatogramView.obj
 0003:000006b8       _taskLog                   1001b6b8     ChromatogramView.obj
 0003:000006c0       _algoLog                   1001b6c0     ChromatogramView.obj
 0003:000006c8       _userActLog                1001b6c8     ChromatogramView.obj
 0003:000006d0       _ioLog                     1001b6d0     ChromatogramView.obj
 0003:000006d8       _coreLog                   1001b6d8     ChromatogramView.obj
 0003:000006e0       _uiLog                     1001b6e0     ChromatogramView.obj
 0003:000006e8       _scriptLog                 1001b6e8     ChromatogramView.obj
 0003:000006f0       _perfLog                   1001b6f0     ChromatogramView.obj
 0003:000006f8       _cmdLog                    1001b6f8     ChromatogramView.obj
 0003:00000700       ?colorForIds@?1??drawAll@ChromatogramViewRenderArea@U2@@MAEXPAVQPaintDevice@@@Z@4QBVQColor@@B 1001b700     ChromatogramView.obj
 0003:00000740       ?$S1@?1??drawAll@ChromatogramViewRenderArea@U2@@MAEXPAVQPaintDevice@@@Z@4IA 1001b740     ChromatogramView.obj
 0003:00000744       ?baseForIds@?1??drawAll@ChromatogramViewRenderArea@U2@@MAEXPAVQPaintDevice@@@Z@4QBVQString@@B 1001b744     ChromatogramView.obj
 0003:00000758       ?colorForIds@?4??drawChromatogramTrace@ChromatogramViewRenderArea@U2@@AAEXNNNNAAVQPainter@@ABVU2Region@3@ABUChromatogramViewSettings@3@@Z@4QBVQColor@@B 1001b758     ChromatogramView.obj
 0003:00000798       ?$S2@?4??drawChromatogramTrace@ChromatogramViewRenderArea@U2@@AAEXNNNNAAVQPainter@@ABVU2Region@3@ABUChromatogramViewSettings@3@@Z@4IA 1001b798     ChromatogramView.obj
 0003:000007a0       ?colorForIds@?1??drawChromatogramBaseCallsLines@ChromatogramViewRenderArea@U2@@AAEXNNNNAAVQPainter@@ABVU2Region@3@ABVQByteArray@@ABUChromatogramViewSettings@3@@Z@4QBVQColor@@B 1001b7a0     ChromatogramView.obj
 0003:000007e0       ?$S3@?1??drawChromatogramBaseCallsLines@ChromatogramViewRenderArea@U2@@AAEXNNNNAAVQPainter@@ABVU2Region@3@ABVQByteArray@@ABUChromatogramViewSettings@3@@Z@4IA 1001b7e0     ChromatogramView.obj
 0003:000007e4       __Tuple_alloc              1001b7e4     moc_ChromaViewPlugin.obj
 0003:000007e5       _ignore                    1001b7e5     moc_ChromaViewPlugin.obj
 0003:000007e6       _allocator_arg             1001b7e6     moc_ChromaViewPlugin.obj
 0003:000007e7       _piecewise_construct       1001b7e7     moc_ChromaViewPlugin.obj
 0003:000007ec       __Tuple_alloc              1001b7ec     moc_ChromatogramView.obj
 0003:000007ed       _ignore                    1001b7ed     moc_ChromatogramView.obj
 0003:000007ee       _allocator_arg             1001b7ee     moc_ChromatogramView.obj
 0003:000007ef       _piecewise_construct       1001b7ef     moc_ChromatogramView.obj
 0003:000007fc       ___proc_attached           1001b7fc     MSVCRT:crtdll.obj
 0003:00000800       _GS_ExceptionRecord        1001b800     MSVCRT:gs_report.obj
 0003:00000850       _GS_ContextRecord          1001b850     MSVCRT:gs_report.obj
 0003:00000b1c       _DebuggerWasPresent        1001bb1c     MSVCRT:gs_report.obj
 0004:00000060       $R000000                   1001c060     * linker generated manifest res *

 Exports

  ordinal    name

        1    _ugene_plugin_init
               exported name: ugene_plugin_init
